 PhysX3CookingPROFILE_x64

 Timestamp is 564e5d75 (Thu Nov 19 18:38:29 2015)

 Preferred load address is 0000000180000000

 Start         Length     Name                   Class
 0001:00000000 00000320H .text$di                CODE
 0001:00000320 00024e36H .text$mn                CODE
 0001:00025160 000000ebH .text$x                 CODE
 0002:00000000 00000168H .idata$5                DATA
 0002:00000168 00000008H .CRT$XCA                DATA
 0002:00000170 000000f0H .CRT$XCU                DATA
 0002:00000260 00000008H .CRT$XCZ                DATA
 0002:00000268 00000008H .CRT$XIA                DATA
 0002:00000270 00000008H .CRT$XIAA               DATA
 0002:00000278 00000008H .CRT$XIC                DATA
 0002:00000280 00000008H .CRT$XIZ                DATA
 0002:00000290 00001a70H .rdata                  DATA
 0002:00001d00 000000a0H .rdata$debug            DATA
 0002:00001da0 00000074H .rdata$r                DATA
 0002:00001e18 00000008H .rtc$IAA                DATA
 0002:00001e20 00000008H .rtc$IZZ                DATA
 0002:00001e28 00000008H .rtc$TAA                DATA
 0002:00001e30 00000008H .rtc$TZZ                DATA
 0002:00001e38 00002c38H .xdata                  DATA
 0002:00004a70 00000020H .didat$2                DATA
 0002:00004a90 00000020H .didat$3                DATA
 0002:00004ab0 00000298H .didat$4                DATA
 0002:00004d48 000010e4H .didat$6                DATA
 0002:00005e30 00000298H .didat$7                DATA
 0002:000060d0 00000088H .edata                  DATA
 0002:00006158 00000028H .idata$2                DATA
 0002:00006180 00000014H .idata$3                DATA
 0002:00006198 00000168H .idata$4                DATA
 0002:00006300 0000031cH .idata$6                DATA
 0003:00000000 000000f8H .data                   DATA
 0003:000000f8 000003a8H .data$r                 DATA
 0003:000004a0 00000298H .didat$5                DATA
 0003:00000740 00000240H .bss                    DATA
 0004:00000000 00001c80H .pdata                  DATA
 0005:00000000 00000058H .rsrc$01                DATA
 0005:00000060 00000180H .rsrc$02                DATA

  Address         Publics by Value              Rva+Base               Lib:Object

 0000:00000000       __guard_fids_table         0000000000000000     <absolute>
 0000:00000000       __guard_fids_count         0000000000000000     <absolute>
 0000:00000000       ___safe_se_handler_table   0000000000000000     <absolute>
 0000:00000000       __guard_flags              0000000000000000     <absolute>
 0000:00000000       ___safe_se_handler_count   0000000000000000     <absolute>
 0000:00000000       __ImageBase                0000000180000000     <linker-defined>
 0001:00000320       PxSetPhysXCookingDelayLoadHook 0000000180001320 f   WindowsCookingDelayLoadHook.obj
 0001:00000330       ?delayHook@@YAP6A_JXZIPEAUDelayLoadInfo@@@Z 0000000180001330 f   WindowsCookingDelayLoadHook.obj
 0001:00000380       ?loadLibrary@shdfnd@physx@@YAPEAUHINSTANCE__@@PEBD@Z 0000000180001380 f i WindowsCookingDelayLoadHook.obj
 0001:00000390       ?physXCommonDliNotePreLoadLibrary@shdfnd@physx@@YAP6A_JXZPEBDPEBVPxDelayLoadHook@2@@Z 0000000180001390 f i WindowsCookingDelayLoadHook.obj
 0001:00000780       ?strstr@@YAPEADPEADPEBD@Z  0000000180001780 f i WindowsCookingDelayLoadHook.obj
 0001:00000790       ?saveHeightField@physx@@YA_NAEBVHeightField@Gu@1@AEAVPxOutputStream@1@_N@Z 0000000180001790 f   HeightFieldCooking.obj
 0001:00000a10       ??B?$PxFlags@W4Enum@PxHeightFieldFlag@physx@@G@physx@@QEBAGXZ 0000000180001a10 f i HeightFieldCooking.obj
 0001:00000a20       ?getData@HeightField@Gu@physx@@QEBAAEBUHeightFieldData@23@XZ 0000000180001a20 f i HeightFieldCooking.obj
 0001:00000a30       ?buildFromTriangles@RTreeCooker@physx@@SAXAEAURTree@Gu@2@PEBVPxVec3@2@IPEBGPEBIIAEAV?$Array@IV?$ReflectionAllocator@I@shdfnd@physx@@@shdfnd@2@PEAURemapCallback@12@MW4Enum@PxMeshCookingHint@2@@Z 0000000180001a30 f   RTreeCooking.obj
 0001:000017b0       ??$PX_UNUSED@I@@YAXAEBI@Z  00000001800027b0 f i RTreeCooking.obj
 0001:000017c0       ??$PX_UNUSED@M@@YAXAEBM@Z  00000001800027c0 f i RTreeCooking.obj
 0001:000017d0       ??$PX_UNUSED@PEAURTreeNodeNQ@physx@@@@YAXAEBQEAURTreeNodeNQ@physx@@@Z 00000001800027d0 f i RTreeCooking.obj
 0001:000017e0       ??$PX_UNUSED@URTreeNodeNQ@physx@@@@YAXAEBURTreeNodeNQ@physx@@@Z 00000001800027e0 f i RTreeCooking.obj
 0001:000017f0       ??$PxMax@H@physx@@YAHHH@Z  00000001800027f0 f i RTreeCooking.obj
 0001:00001800       ??$PxMax@I@physx@@YAIII@Z  0000000180002800 f i RTreeCooking.obj
 0001:00001810       ??$PxMax@M@physx@@YAMMM@Z  0000000180002810 f i RTreeCooking.obj
 0001:00001820       ??$PxMin@I@physx@@YAIII@Z  0000000180002820 f i RTreeCooking.obj
 0001:00001830       ??$PxMin@M@physx@@YAMMM@Z  0000000180002830 f i RTreeCooking.obj
 0001:00001840       ??$median3@I$$CBU?$Less@I@shdfnd@physx@@@internal@shdfnd@physx@@YAXPEAIHHAEBU?$Less@I@12@@Z 0000000180002840 f i RTreeCooking.obj
 0001:000018b0       ??$median3@I$$CBUSortBoundsPredicate@physx@@@internal@shdfnd@physx@@YAXPEAIHHAEBUSortBoundsPredicate@2@@Z 00000001800028b0 f i RTreeCooking.obj
 0001:000019d0       ??$partition@I$$CBU?$Less@I@shdfnd@physx@@@internal@shdfnd@physx@@YAHPEAIHHAEBU?$Less@I@12@@Z 00000001800029d0 f i RTreeCooking.obj
 0001:00001aa0       ??$partition@I$$CBUSortBoundsPredicate@physx@@@internal@shdfnd@physx@@YAHPEAIHHAEBUSortBoundsPredicate@2@@Z 0000000180002aa0 f i RTreeCooking.obj
 0001:00001b90       ??$partition@UBoundsLTE@physx@@@quickSelect@physx@@YAIPEIAIIIIAEBUBoundsLTE@1@@Z 0000000180002b90 f i RTreeCooking.obj
 0001:00001d20       ??$quickSelectFirstK@UBoundsLTE@physx@@@quickSelect@physx@@YAXPEIAIIIIAEBUBoundsLTE@1@@Z 0000000180002d20 f i RTreeCooking.obj
 0001:00001f00       ??$smallSort@I$$CBU?$Less@I@shdfnd@physx@@@internal@shdfnd@physx@@YAXPEAIHHAEBU?$Less@I@12@@Z 0000000180002f00 f i RTreeCooking.obj
 0001:00001fe0       ??$smallSort@I$$CBUSortBoundsPredicate@physx@@@internal@shdfnd@physx@@YAXPEAIHHAEBUSortBoundsPredicate@2@@Z 0000000180002fe0 f i RTreeCooking.obj
 0001:000022d0       ??$sort@I@shdfnd@physx@@YAXPEAII@Z 00000001800032d0 f i RTreeCooking.obj
 0001:000022f0       ??$sort@IU?$Less@I@shdfnd@physx@@V?$ReflectionAllocator@I@23@@shdfnd@physx@@YAXPEAIIAEBU?$Less@I@01@AEBV?$ReflectionAllocator@I@01@I@Z 00000001800032f0 f i RTreeCooking.obj
 0001:00002600       ??$sort@IUSortBoundsPredicate@physx@@@shdfnd@physx@@YAXPEAIIAEBUSortBoundsPredicate@1@@Z 0000000180003600 f i RTreeCooking.obj
 0001:00002620       ??$sort@IUSortBoundsPredicate@physx@@V?$ReflectionAllocator@I@shdfnd@2@@shdfnd@physx@@YAXPEAIIAEBUSortBoundsPredicate@1@AEBV?$ReflectionAllocator@I@01@I@Z 0000000180003620 f i RTreeCooking.obj
 0001:00002930       ??$swap@I@shdfnd@physx@@YAXAEAI0@Z 0000000180003930 f i RTreeCooking.obj
 0001:00002940       ??0?$AlignedAllocator@$0IA@VAllocator@shdfnd@physx@@@shdfnd@physx@@QEAA@AEBVAllocator@12@@Z 0000000180003940 f i RTreeCooking.obj
 0001:00002950       ??0?$Array@IV?$ReflectionAllocator@I@shdfnd@physx@@@shdfnd@physx@@QEAA@IAEBIAEBV?$ReflectionAllocator@I@12@@Z 0000000180003950 f i RTreeCooking.obj
 0001:00002970       ??0?$Array@UInterval@physx@@V?$InlineAllocator@$0CA@V?$ReflectionAllocator@UInterval@physx@@@shdfnd@physx@@@shdfnd@2@@shdfnd@physx@@QEAA@AEBV?$InlineAllocator@$0CA@V?$ReflectionAllocator@UInterval@physx@@@shdfnd@physx@@@12@@Z 0000000180003970 f i RTreeCooking.obj
 0001:00002990       ??0?$Array@UPxBounds3V@physx@@V?$ReflectionAllocator@UPxBounds3V@physx@@@shdfnd@2@@shdfnd@physx@@QEAA@AEBV?$ReflectionAllocator@UPxBounds3V@physx@@@12@@Z 0000000180003990 f i RTreeCooking.obj
 0001:000029a0       ??0?$Array@URTreeNodeNQ@physx@@V?$ReflectionAllocator@URTreeNodeNQ@physx@@@shdfnd@2@@shdfnd@physx@@QEAA@AEBV?$ReflectionAllocator@URTreeNodeNQ@physx@@@12@@Z 00000001800039a0 f i RTreeCooking.obj
 0001:000029b0       ??0?$Array@URTreeNodeQ@Gu@physx@@V?$ReflectionAllocator@URTreeNodeQ@Gu@physx@@@shdfnd@3@@shdfnd@physx@@QEAA@AEBV?$ReflectionAllocator@URTreeNodeQ@Gu@physx@@@12@@Z 00000001800039b0 f i RTreeCooking.obj
 0001:000029c0       ??0?$Array@VPxVec3@physx@@V?$ReflectionAllocator@VPxVec3@physx@@@shdfnd@2@@shdfnd@physx@@QEAA@AEBV?$ReflectionAllocator@VPxVec3@physx@@@12@@Z 00000001800039c0 f i RTreeCooking.obj
 0001:000029d0       ??0?$InlineAllocator@$0CA@V?$ReflectionAllocator@UInterval@physx@@@shdfnd@physx@@@shdfnd@physx@@QEAA@AEBV012@@Z 00000001800039d0 f i RTreeCooking.obj
 0001:000029e0       ??0?$InlineAllocator@$0CA@V?$ReflectionAllocator@UInterval@physx@@@shdfnd@physx@@@shdfnd@physx@@QEAA@AEBV?$ReflectionAllocator@UInterval@physx@@@12@@Z 00000001800039e0 f i RTreeCooking.obj
 0001:000029f0       ??0?$InlineArray@UInterval@physx@@$03V?$ReflectionAllocator@UInterval@physx@@@shdfnd@2@@shdfnd@physx@@QEAA@AEBV?$ReflectionAllocator@UInterval@physx@@@12@@Z 00000001800039f0 f i RTreeCooking.obj
 0001:00002a10       ??0?$ReflectionAllocator@I@shdfnd@physx@@QEAA@AEBV012@@Z 0000000180003a10 f i RTreeCooking.obj
 0001:00002a20       ??0?$ReflectionAllocator@I@shdfnd@physx@@QEAA@PEBD@Z 0000000180003a20 f i RTreeCooking.obj
 0001:00002a30       ??0?$ReflectionAllocator@UInterval@physx@@@shdfnd@physx@@QEAA@AEBV012@@Z 0000000180003a30 f i RTreeCooking.obj
 0001:00002a40       ??0?$ReflectionAllocator@UInterval@physx@@@shdfnd@physx@@QEAA@PEBD@Z 0000000180003a40 f i RTreeCooking.obj
 0001:00002a50       ??0?$ReflectionAllocator@UPxBounds3V@physx@@@shdfnd@physx@@QEAA@AEBV012@@Z 0000000180003a50 f i RTreeCooking.obj
 0001:00002a60       ??0?$ReflectionAllocator@UPxBounds3V@physx@@@shdfnd@physx@@QEAA@PEBD@Z 0000000180003a60 f i RTreeCooking.obj
 0001:00002a70       ??0?$ReflectionAllocator@URTreeNodeNQ@physx@@@shdfnd@physx@@QEAA@AEBV012@@Z 0000000180003a70 f i RTreeCooking.obj
 0001:00002a80       ??0?$ReflectionAllocator@URTreeNodeNQ@physx@@@shdfnd@physx@@QEAA@PEBD@Z 0000000180003a80 f i RTreeCooking.obj
 0001:00002a90       ??0?$ReflectionAllocator@URTreeNodeQ@Gu@physx@@@shdfnd@physx@@QEAA@AEBV012@@Z 0000000180003a90 f i RTreeCooking.obj
 0001:00002aa0       ??0?$ReflectionAllocator@URTreeNodeQ@Gu@physx@@@shdfnd@physx@@QEAA@PEBD@Z 0000000180003aa0 f i RTreeCooking.obj
 0001:00002ab0       ??0?$ReflectionAllocator@VPxVec3@physx@@@shdfnd@physx@@QEAA@AEBV012@@Z 0000000180003ab0 f i RTreeCooking.obj
 0001:00002ac0       ??0?$ReflectionAllocator@VPxVec3@physx@@@shdfnd@physx@@QEAA@PEBD@Z 0000000180003ac0 f i RTreeCooking.obj
 0001:00002ad0       ??0?$ScopedPointer@HVTempAllocator@shdfnd@physx@@@shdfnd@physx@@QEAA@XZ 0000000180003ad0 f i RTreeCooking.obj
 0001:00002ae0       ??0?$Stack@V?$ReflectionAllocator@I@shdfnd@physx@@@internal@shdfnd@physx@@QEAA@PEAHIAEBV?$ReflectionAllocator@I@23@@Z 0000000180003ae0 f i RTreeCooking.obj
 0001:00002b00       ??0BoundsLTE@physx@@QEAA@IPEBVPxVec3@1@@Z 0000000180003b00 f i RTreeCooking.obj
 0001:00002b10       ??0Interval@physx@@QEAA@II@Z 0000000180003b10 f i RTreeCooking.obj
 0001:00002b20       ??0PxBounds3@physx@@QEAA@AEBV01@@Z 0000000180003b20 f i RTreeCooking.obj
 0001:00002b50       ??0PxBounds3@physx@@QEAA@AEBVPxVec3@1@0@Z 0000000180003b50 f i RTreeCooking.obj
 0001:00002b80       ??0PxBounds3V@physx@@QEAA@AEAT__m128@@0@Z 0000000180003b80 f i RTreeCooking.obj
 0001:00002ba0       ??0PxBounds3V@physx@@QEAA@UU@01@@Z 0000000180003ba0 f i RTreeCooking.obj
 0001:00002bb0       ??0PxVec3@physx@@QEAA@AEBV01@@Z 0000000180003bb0 f i RTreeCooking.obj
 0001:00002bd0       ??0PxVec3@physx@@QEAA@M@Z  0000000180003bd0 f i RTreeCooking.obj
 0001:00002bf0       ??0PxVec3@physx@@QEAA@MMM@Z 0000000180003bf0 f i RTreeCooking.obj
 0001:00002c10       ??0PxVec4@physx@@QEAA@AEBVPxVec3@1@M@Z 0000000180003c10 f i RTreeCooking.obj
 0001:00002c30       ??0PxVec4@physx@@QEAA@M@Z  0000000180003c30 f i RTreeCooking.obj
 0001:00002c40       ??0PxVec4@physx@@QEAA@MMMM@Z 0000000180003c40 f i RTreeCooking.obj
 0001:00002c60       ??0RTreeNodeNQ@physx@@QEAA@AEBU01@@Z 0000000180003c60 f i RTreeCooking.obj
 0001:00002ca0       ??0RTreeNodeNQ@physx@@QEAA@XZ 0000000180003ca0 f i RTreeCooking.obj
 0001:00002ce0       ??0SortBoundsPredicate@physx@@QEAA@IPEBUPxBounds3V@1@@Z 0000000180003ce0 f i RTreeCooking.obj
 0001:00002cf0       ??0SubSortQuick@physx@@QEAA@PEAIPEBUPxBounds3V@1@IM@Z 0000000180003cf0 f i RTreeCooking.obj
 0001:00002e30       ??0SubSortSAH@physx@@QEAA@PEAIPEBUPxBounds3V@1@IPEBI22222M@Z 0000000180003e30 f i RTreeCooking.obj
 0001:00002f40       ??1?$Array@IV?$ReflectionAllocator@I@shdfnd@physx@@@shdfnd@physx@@QEAA@XZ 0000000180003f40 f i RTreeCooking.obj
 0001:00002f80       ??1?$Array@UInterval@physx@@V?$InlineAllocator@$0CA@V?$ReflectionAllocator@UInterval@physx@@@shdfnd@physx@@@shdfnd@2@@shdfnd@physx@@QEAA@XZ 0000000180003f80 f i RTreeCooking.obj
 0001:00002fd0       ??1?$Array@UPxBounds3V@physx@@V?$ReflectionAllocator@UPxBounds3V@physx@@@shdfnd@2@@shdfnd@physx@@QEAA@XZ 0000000180003fd0 f i RTreeCooking.obj
 0001:00003010       ??1?$Array@URTreeNodeNQ@physx@@V?$ReflectionAllocator@URTreeNodeNQ@physx@@@shdfnd@2@@shdfnd@physx@@QEAA@XZ 0000000180004010 f i RTreeCooking.obj
 0001:00003050       ??1?$Array@URTreeNodeQ@Gu@physx@@V?$ReflectionAllocator@URTreeNodeQ@Gu@physx@@@shdfnd@3@@shdfnd@physx@@QEAA@XZ 0000000180004050 f i RTreeCooking.obj
 0001:00003090       ??1?$Array@VPxVec3@physx@@V?$ReflectionAllocator@VPxVec3@physx@@@shdfnd@2@@shdfnd@physx@@QEAA@XZ 0000000180004090 f i RTreeCooking.obj
 0001:000030d0       ??1?$InlineArray@UInterval@physx@@$03V?$ReflectionAllocator@UInterval@physx@@@shdfnd@2@@shdfnd@physx@@QEAA@XZ 00000001800040d0 f i RTreeCooking.obj
 0001:00003120       ??1?$ScopedPointer@HVTempAllocator@shdfnd@physx@@@shdfnd@physx@@QEAA@XZ 0000000180004120 f i RTreeCooking.obj
 0001:00003140       ??1?$Stack@V?$ReflectionAllocator@I@shdfnd@physx@@@internal@shdfnd@physx@@QEAA@XZ 0000000180004140 f i RTreeCooking.obj
 0001:00003180       ??1SubSortQuick@physx@@QEAA@XZ 0000000180004180 f i RTreeCooking.obj
 0001:000031c0       ??1SubSortSAH@physx@@QEAA@XZ 00000001800041c0 f i RTreeCooking.obj
 0001:00003210       ??2@YAPEAX_KPEAX@Z         0000000180004210 f i RTreeCooking.obj
 0001:00003220       ??4PxVec3@physx@@QEAAAEAV01@AEBV01@@Z 0000000180004220 f i RTreeCooking.obj
 0001:00003240       ??4PxVec4@physx@@QEAAAEAV01@AEBV01@@Z 0000000180004240 f i RTreeCooking.obj
 0001:00003260       ??A?$Array@IV?$ReflectionAllocator@I@shdfnd@physx@@@shdfnd@physx@@QEAAAEAII@Z 0000000180004260 f i RTreeCooking.obj
 0001:00003270       ??A?$Array@UInterval@physx@@V?$InlineAllocator@$0CA@V?$ReflectionAllocator@UInterval@physx@@@shdfnd@physx@@@shdfnd@2@@shdfnd@physx@@QEAAAEAUInterval@2@I@Z 0000000180004270 f i RTreeCooking.obj
 0001:00003280       ??A?$Array@URTreeNodeNQ@physx@@V?$ReflectionAllocator@URTreeNodeNQ@physx@@@shdfnd@2@@shdfnd@physx@@QEAAAEAURTreeNodeNQ@2@I@Z 0000000180004280 f i RTreeCooking.obj
 0001:00003290       ??A?$Array@URTreeNodeQ@Gu@physx@@V?$ReflectionAllocator@URTreeNodeQ@Gu@physx@@@shdfnd@3@@shdfnd@physx@@QEAAAEAURTreeNodeQ@Gu@2@I@Z 0000000180004290 f i RTreeCooking.obj
 0001:000032a0       ??APxVec3@physx@@QEBAAEBMI@Z 00000001800042a0 f i RTreeCooking.obj
 0001:000032b0       ??B?$ScopedPointer@HVTempAllocator@shdfnd@physx@@@shdfnd@physx@@QEBAPEAHXZ 00000001800042b0 f i RTreeCooking.obj
 0001:000032c0       ??GPxVec4@physx@@QEBA?AV01@AEBV01@@Z 00000001800042c0 f i RTreeCooking.obj
 0001:00003310       ??HPxVec3@physx@@QEBA?AV01@AEBV01@@Z 0000000180004310 f i RTreeCooking.obj
 0001:00003350       ??KPxVec4@physx@@QEBA?AV01@M@Z 0000000180004350 f i RTreeCooking.obj
 0001:00003390       ??R?$Less@I@shdfnd@physx@@QEBA_NAEBI0@Z 0000000180004390 f i RTreeCooking.obj
 0001:000033a0       ??RBoundsLTE@physx@@QEBA_NAEBI0@Z 00000001800043a0 f i RTreeCooking.obj
 0001:000033d0       ??RSortBoundsPredicate@physx@@QEBA_NAEBI0@Z 00000001800043d0 f i RTreeCooking.obj
 0001:00003410       ?FLoad@aos@shdfnd@physx@@YA?AT__m128@@M@Z 0000000180004410 f i RTreeCooking.obj
 0001:00003430       ?FMax@aos@shdfnd@physx@@YA?AT__m128@@XZ 0000000180004430 f i RTreeCooking.obj
 0001:00003450       ?FNegMax@aos@shdfnd@physx@@YA?AT__m128@@XZ 0000000180004450 f i RTreeCooking.obj
 0001:00003470       ?FStore@aos@shdfnd@physx@@YAXT__m128@@PEIAM@Z 0000000180004470 f i RTreeCooking.obj
 0001:00003480       ?PxAbs@physx@@YAHH@Z       0000000180004480 f i RTreeCooking.obj
 0001:00003490       ?PxMemCopy@physx@@YAPEAXPEIAXPEIBXI@Z 0000000180004490 f i RTreeCooking.obj
 0001:000034b0       ?V3Add@aos@shdfnd@physx@@YA?AT__m128@@T4@0@Z 00000001800044b0 f i RTreeCooking.obj
 0001:000034c0       ?V3Dot@aos@shdfnd@physx@@YA?AT__m128@@T4@0@Z 00000001800044c0 f i RTreeCooking.obj
 0001:000034e0       ?V3Load@aos@shdfnd@physx@@YA?AT__m128@@M@Z 00000001800044e0 f i RTreeCooking.obj
 0001:000034f0       ?V3LoadU@aos@shdfnd@physx@@YA?AT__m128@@AEBVPxVec3@3@@Z 00000001800044f0 f i RTreeCooking.obj
 0001:00003510       ?V3Max@aos@shdfnd@physx@@YA?AT__m128@@T4@0@Z 0000000180004510 f i RTreeCooking.obj
 0001:00003520       ?V3Min@aos@shdfnd@physx@@YA?AT__m128@@T4@0@Z 0000000180004520 f i RTreeCooking.obj
 0001:00003530       ?V3PermZXY@aos@shdfnd@physx@@YA?AT__m128@@T4@@Z 0000000180004530 f i RTreeCooking.obj
 0001:00003540       ?V3ReadXYZ@aos@shdfnd@physx@@YAAEBVPxVec3@3@AEBT__m128@@@Z 0000000180004540 f i RTreeCooking.obj
 0001:00003550       ?V3Splat@aos@shdfnd@physx@@YA?AT__m128@@T4@@Z 0000000180004550 f i RTreeCooking.obj
 0001:00003560       ?V3StoreA@aos@shdfnd@physx@@YAXT__m128@@AEAVPxVec3@3@@Z 0000000180004560 f i RTreeCooking.obj
 0001:00003580       ?V3Sub@aos@shdfnd@physx@@YA?AT__m128@@T4@0@Z 0000000180004580 f i RTreeCooking.obj
 0001:00003590       ?V3Zero@aos@shdfnd@physx@@YA?AT__m128@@XZ 0000000180004590 f i RTreeCooking.obj
 0001:000035a0       ?V4ClearW@aos@shdfnd@physx@@YA?AT__m128@@T4@@Z 00000001800045a0 f i RTreeCooking.obj
 0001:000035b0       ?V4Load@aos@shdfnd@physx@@YA?AT__m128@@M@Z 00000001800045b0 f i RTreeCooking.obj
 0001:000035d0       ?Vec3V_From_FloatV@aos@shdfnd@physx@@YA?AT__m128@@T4@@Z 00000001800045d0 f i RTreeCooking.obj
 0001:000035e0       ?Vec3V_From_Vec4V@aos@shdfnd@physx@@YA?AT__m128@@T4@@Z 00000001800045e0 f i RTreeCooking.obj
 0001:000035f0       ?Vec4V_From_FloatV@aos@shdfnd@physx@@YA?AT__m128@@T4@@Z 00000001800045f0 f i RTreeCooking.obj
 0001:00003600       ?allocate@?$AlignedAllocator@$0IA@VAllocator@shdfnd@physx@@@shdfnd@physx@@QEAAPEAX_KPEBDH@Z 0000000180004600 f i RTreeCooking.obj
 0001:00003640       ?allocate@?$Array@IV?$ReflectionAllocator@I@shdfnd@physx@@@shdfnd@physx@@IEAAPEAII@Z 0000000180004640 f i RTreeCooking.obj
 0001:00003660       ?allocate@?$Array@UInterval@physx@@V?$InlineAllocator@$0CA@V?$ReflectionAllocator@UInterval@physx@@@shdfnd@physx@@@shdfnd@2@@shdfnd@physx@@IEAAPEAUInterval@3@I@Z 0000000180004660 f i RTreeCooking.obj
 0001:000036b0       ?allocate@?$Array@UPxBounds3V@physx@@V?$ReflectionAllocator@UPxBounds3V@physx@@@shdfnd@2@@shdfnd@physx@@IEAAPEAUPxBounds3V@3@I@Z 00000001800046b0 f i RTreeCooking.obj
 0001:000036d0       ?allocate@?$Array@URTreeNodeNQ@physx@@V?$ReflectionAllocator@URTreeNodeNQ@physx@@@shdfnd@2@@shdfnd@physx@@IEAAPEAURTreeNodeNQ@3@I@Z 00000001800046d0 f i RTreeCooking.obj
 0001:000036f0       ?allocate@?$Array@URTreeNodeQ@Gu@physx@@V?$ReflectionAllocator@URTreeNodeQ@Gu@physx@@@shdfnd@3@@shdfnd@physx@@IEAAPEAURTreeNodeQ@Gu@3@I@Z 00000001800046f0 f i RTreeCooking.obj
 0001:00003710       ?allocate@?$Array@VPxVec3@physx@@V?$ReflectionAllocator@VPxVec3@physx@@@shdfnd@2@@shdfnd@physx@@IEAAPEAVPxVec3@3@I@Z 0000000180004710 f i RTreeCooking.obj
 0001:00003740       ?allocate@?$InlineAllocator@$0CA@V?$ReflectionAllocator@UInterval@physx@@@shdfnd@physx@@@shdfnd@physx@@QEAAPEAXIPEBDH@Z 0000000180004740 f i RTreeCooking.obj
 0001:00003760       ?allocate@?$ReflectionAllocator@I@shdfnd@physx@@QEAAPEAX_KPEBDH@Z 0000000180004760 f i RTreeCooking.obj
 0001:00003800       ?allocate@?$ReflectionAllocator@UInterval@physx@@@shdfnd@physx@@QEAAPEAX_KPEBDH@Z 0000000180004800 f i RTreeCooking.obj
 0001:000038a0       ?allocate@?$ReflectionAllocator@UPxBounds3V@physx@@@shdfnd@physx@@QEAAPEAX_KPEBDH@Z 00000001800048a0 f i RTreeCooking.obj
 0001:00003940       ?allocate@?$ReflectionAllocator@URTreeNodeNQ@physx@@@shdfnd@physx@@QEAAPEAX_KPEBDH@Z 0000000180004940 f i RTreeCooking.obj
 0001:000039e0       ?allocate@?$ReflectionAllocator@URTreeNodeQ@Gu@physx@@@shdfnd@physx@@QEAAPEAX_KPEBDH@Z 00000001800049e0 f i RTreeCooking.obj
 0001:00003a80       ?allocate@?$ReflectionAllocator@VPxVec3@physx@@@shdfnd@physx@@QEAAPEAX_KPEBDH@Z 0000000180004a80 f i RTreeCooking.obj
 0001:00003b20       ?begin@?$Array@IV?$ReflectionAllocator@I@shdfnd@physx@@@shdfnd@physx@@QEAAPEAIXZ 0000000180004b20 f i RTreeCooking.obj
 0001:00003b30       ?begin@?$Array@UPxBounds3V@physx@@V?$ReflectionAllocator@UPxBounds3V@physx@@@shdfnd@2@@shdfnd@physx@@QEAAPEAUPxBounds3V@3@XZ 0000000180004b30 f i RTreeCooking.obj
 0001:00003b40       ?begin@?$Array@VPxVec3@physx@@V?$ReflectionAllocator@VPxVec3@physx@@@shdfnd@2@@shdfnd@physx@@QEAAPEAVPxVec3@3@XZ 0000000180004b40 f i RTreeCooking.obj
 0001:00003b50       ?capacity@?$Array@IV?$ReflectionAllocator@I@shdfnd@physx@@@shdfnd@physx@@QEBAIXZ 0000000180004b50 f i RTreeCooking.obj
 0001:00003b60       ?capacity@?$Array@UInterval@physx@@V?$InlineAllocator@$0CA@V?$ReflectionAllocator@UInterval@physx@@@shdfnd@physx@@@shdfnd@2@@shdfnd@physx@@QEBAIXZ 0000000180004b60 f i RTreeCooking.obj
 0001:00003b70       ?capacity@?$Array@UPxBounds3V@physx@@V?$ReflectionAllocator@UPxBounds3V@physx@@@shdfnd@2@@shdfnd@physx@@QEBAIXZ 0000000180004b70 f i RTreeCooking.obj
 0001:00003b80       ?capacity@?$Array@URTreeNodeNQ@physx@@V?$ReflectionAllocator@URTreeNodeNQ@physx@@@shdfnd@2@@shdfnd@physx@@QEBAIXZ 0000000180004b80 f i RTreeCooking.obj
 0001:00003b90       ?capacity@?$Array@URTreeNodeQ@Gu@physx@@V?$ReflectionAllocator@URTreeNodeQ@Gu@physx@@@shdfnd@3@@shdfnd@physx@@QEBAIXZ 0000000180004b90 f i RTreeCooking.obj
 0001:00003ba0       ?capacity@?$Array@VPxVec3@physx@@V?$ReflectionAllocator@VPxVec3@physx@@@shdfnd@2@@shdfnd@physx@@QEBAIXZ 0000000180004ba0 f i RTreeCooking.obj
 0001:00003bb0       ?capacityIncrement@?$Array@IV?$ReflectionAllocator@I@shdfnd@physx@@@shdfnd@physx@@IEBAIXZ 0000000180004bb0 f i RTreeCooking.obj
 0001:00003bd0       ?capacityIncrement@?$Array@UInterval@physx@@V?$InlineAllocator@$0CA@V?$ReflectionAllocator@UInterval@physx@@@shdfnd@physx@@@shdfnd@2@@shdfnd@physx@@IEBAIXZ 0000000180004bd0 f i RTreeCooking.obj
 0001:00003bf0       ?capacityIncrement@?$Array@UPxBounds3V@physx@@V?$ReflectionAllocator@UPxBounds3V@physx@@@shdfnd@2@@shdfnd@physx@@IEBAIXZ 0000000180004bf0 f i RTreeCooking.obj
 0001:00003c10       ?capacityIncrement@?$Array@URTreeNodeNQ@physx@@V?$ReflectionAllocator@URTreeNodeNQ@physx@@@shdfnd@2@@shdfnd@physx@@IEBAIXZ 0000000180004c10 f i RTreeCooking.obj
 0001:00003c30       ?capacityIncrement@?$Array@URTreeNodeQ@Gu@physx@@V?$ReflectionAllocator@URTreeNodeQ@Gu@physx@@@shdfnd@3@@shdfnd@physx@@IEBAIXZ 0000000180004c30 f i RTreeCooking.obj
 0001:00003c50       ?capacityIncrement@?$Array@VPxVec3@physx@@V?$ReflectionAllocator@VPxVec3@physx@@@shdfnd@2@@shdfnd@physx@@IEBAIXZ 0000000180004c50 f i RTreeCooking.obj
 0001:00003c70       ?computeSA@SubSortSAH@physx@@QEAAMPEBIAEBUInterval@2@@Z 0000000180004c70 f i RTreeCooking.obj
 0001:00003cf0       ?copy@?$Array@IV?$ReflectionAllocator@I@shdfnd@physx@@@shdfnd@physx@@KAXPEAI0PEBI@Z 0000000180004cf0 f i RTreeCooking.obj
 0001:00003d10       ?copy@?$Array@UInterval@physx@@V?$InlineAllocator@$0CA@V?$ReflectionAllocator@UInterval@physx@@@shdfnd@physx@@@shdfnd@2@@shdfnd@physx@@KAXPEAUInterval@3@0PEBU43@@Z 0000000180004d10 f i RTreeCooking.obj
 0001:00003d30       ?copy@?$Array@UPxBounds3V@physx@@V?$ReflectionAllocator@UPxBounds3V@physx@@@shdfnd@2@@shdfnd@physx@@KAXPEAUPxBounds3V@3@0PEBU43@@Z 0000000180004d30 f i RTreeCooking.obj
 0001:00003d60       ?copy@?$Array@URTreeNodeNQ@physx@@V?$ReflectionAllocator@URTreeNodeNQ@physx@@@shdfnd@2@@shdfnd@physx@@KAXPEAURTreeNodeNQ@3@0PEBU43@@Z 0000000180004d60 f i RTreeCooking.obj
 0001:00003f00       ?copy@?$Array@URTreeNodeQ@Gu@physx@@V?$ReflectionAllocator@URTreeNodeQ@Gu@physx@@@shdfnd@3@@shdfnd@physx@@KAXPEAURTreeNodeQ@Gu@3@0PEBU453@@Z 0000000180004f00 f i RTreeCooking.obj
 0001:00003f40       ?copy@?$Array@VPxVec3@physx@@V?$ReflectionAllocator@VPxVec3@physx@@@shdfnd@2@@shdfnd@physx@@KAXPEAVPxVec3@3@0PEBV43@@Z 0000000180004f40 f i RTreeCooking.obj
 0001:00004040       ?create@?$Array@IV?$ReflectionAllocator@I@shdfnd@physx@@@shdfnd@physx@@KAXPEAI0AEBI@Z 0000000180005040 f i RTreeCooking.obj
 0001:00004060       ?deallocate@?$Array@IV?$ReflectionAllocator@I@shdfnd@physx@@@shdfnd@physx@@IEAAXPEAX@Z 0000000180005060 f i RTreeCooking.obj
 0001:00004090       ?deallocate@?$Array@UInterval@physx@@V?$InlineAllocator@$0CA@V?$ReflectionAllocator@UInterval@physx@@@shdfnd@physx@@@shdfnd@2@@shdfnd@physx@@IEAAXPEAX@Z 0000000180005090 f i RTreeCooking.obj
 0001:000040d0       ?deallocate@?$Array@UPxBounds3V@physx@@V?$ReflectionAllocator@UPxBounds3V@physx@@@shdfnd@2@@shdfnd@physx@@IEAAXPEAX@Z 00000001800050d0 f i RTreeCooking.obj
 0001:00004100       ?deallocate@?$Array@URTreeNodeNQ@physx@@V?$ReflectionAllocator@URTreeNodeNQ@physx@@@shdfnd@2@@shdfnd@physx@@IEAAXPEAX@Z 0000000180005100 f i RTreeCooking.obj
 0001:00004130       ?deallocate@?$Array@URTreeNodeQ@Gu@physx@@V?$ReflectionAllocator@URTreeNodeQ@Gu@physx@@@shdfnd@3@@shdfnd@physx@@IEAAXPEAX@Z 0000000180005130 f i RTreeCooking.obj
 0001:00004160       ?deallocate@?$Array@VPxVec3@physx@@V?$ReflectionAllocator@VPxVec3@physx@@@shdfnd@2@@shdfnd@physx@@IEAAXPEAX@Z 0000000180005160 f i RTreeCooking.obj
 0001:00004190       ?deallocate@?$InlineAllocator@$0CA@V?$ReflectionAllocator@UInterval@physx@@@shdfnd@physx@@@shdfnd@physx@@QEAAXPEAX@Z 0000000180005190 f i RTreeCooking.obj
 0001:000041d0       ?deallocate@?$ReflectionAllocator@I@shdfnd@physx@@QEAAXPEAX@Z 00000001800051d0 f i RTreeCooking.obj
 0001:00004200       ?deallocate@?$ReflectionAllocator@UInterval@physx@@@shdfnd@physx@@QEAAXPEAX@Z 0000000180005200 f i RTreeCooking.obj
 0001:00004230       ?deallocate@?$ReflectionAllocator@UPxBounds3V@physx@@@shdfnd@physx@@QEAAXPEAX@Z 0000000180005230 f i RTreeCooking.obj
 0001:00004260       ?deallocate@?$ReflectionAllocator@URTreeNodeNQ@physx@@@shdfnd@physx@@QEAAXPEAX@Z 0000000180005260 f i RTreeCooking.obj
 0001:00004290       ?deallocate@?$ReflectionAllocator@URTreeNodeQ@Gu@physx@@@shdfnd@physx@@QEAAXPEAX@Z 0000000180005290 f i RTreeCooking.obj
 0001:000042c0       ?deallocate@?$ReflectionAllocator@VPxVec3@physx@@@shdfnd@physx@@QEAAXPEAX@Z 00000001800052c0 f i RTreeCooking.obj
 0001:000042f0       ?destroy@?$Array@IV?$ReflectionAllocator@I@shdfnd@physx@@@shdfnd@physx@@KAXPEAI0@Z 00000001800052f0 f i RTreeCooking.obj
 0001:00004300       ?destroy@?$Array@UInterval@physx@@V?$InlineAllocator@$0CA@V?$ReflectionAllocator@UInterval@physx@@@shdfnd@physx@@@shdfnd@2@@shdfnd@physx@@KAXPEAUInterval@3@0@Z 0000000180005300 f i RTreeCooking.obj
 0001:00004310       ?destroy@?$Array@UPxBounds3V@physx@@V?$ReflectionAllocator@UPxBounds3V@physx@@@shdfnd@2@@shdfnd@physx@@KAXPEAUPxBounds3V@3@0@Z 0000000180005310 f i RTreeCooking.obj
 0001:00004320       ?destroy@?$Array@URTreeNodeNQ@physx@@V?$ReflectionAllocator@URTreeNodeNQ@physx@@@shdfnd@2@@shdfnd@physx@@KAXPEAURTreeNodeNQ@3@0@Z 0000000180005320 f i RTreeCooking.obj
 0001:00004330       ?destroy@?$Array@URTreeNodeQ@Gu@physx@@V?$ReflectionAllocator@URTreeNodeQ@Gu@physx@@@shdfnd@3@@shdfnd@physx@@KAXPEAURTreeNodeQ@Gu@3@0@Z 0000000180005330 f i RTreeCooking.obj
 0001:00004340       ?destroy@?$Array@VPxVec3@physx@@V?$ReflectionAllocator@VPxVec3@physx@@@shdfnd@2@@shdfnd@physx@@KAXPEAVPxVec3@3@0@Z 0000000180005340 f i RTreeCooking.obj
 0001:00004350       ?empty@?$Stack@V?$ReflectionAllocator@I@shdfnd@physx@@@internal@shdfnd@physx@@QEAA_NXZ 0000000180005350 f i RTreeCooking.obj
 0001:00004360       ?empty@PxBounds3@physx@@SA?AV12@XZ 0000000180005360 f i RTreeCooking.obj
 0001:00004390       ?getExtents@PxBounds3V@physx@@QEBA?AT__m128@@XZ 0000000180005390 f i RTreeCooking.obj
 0001:000043a0       ?getMaxVec3@PxBounds3V@physx@@QEBAAEBVPxVec3@2@XZ 00000001800053a0 f i RTreeCooking.obj
 0001:000043b0       ?getMinVec3@PxBounds3V@physx@@QEBAAEBVPxVec3@2@XZ 00000001800053b0 f i RTreeCooking.obj
 0001:000043c0       ?getName@?$ReflectionAllocator@I@shdfnd@physx@@CAPEBDXZ 00000001800053c0 f i RTreeCooking.obj
 0001:00004400       ?getName@?$ReflectionAllocator@UInterval@physx@@@shdfnd@physx@@CAPEBDXZ 0000000180005400 f i RTreeCooking.obj
 0001:00004440       ?getName@?$ReflectionAllocator@UPxBounds3V@physx@@@shdfnd@physx@@CAPEBDXZ 0000000180005440 f i RTreeCooking.obj
 0001:00004480       ?getName@?$ReflectionAllocator@URTreeNodeNQ@physx@@@shdfnd@physx@@CAPEBDXZ 0000000180005480 f i RTreeCooking.obj
 0001:000044c0       ?getName@?$ReflectionAllocator@URTreeNodeQ@Gu@physx@@@shdfnd@physx@@CAPEBDXZ 00000001800054c0 f i RTreeCooking.obj
 0001:00004500       ?getName@?$ReflectionAllocator@VPxVec3@physx@@@shdfnd@physx@@CAPEBDXZ 0000000180005500 f i RTreeCooking.obj
 0001:00004540       ?grow@?$Array@IV?$ReflectionAllocator@I@shdfnd@physx@@@shdfnd@physx@@IEAAXI@Z 0000000180005540 f i RTreeCooking.obj
 0001:00004550       ?grow@?$Array@UPxBounds3V@physx@@V?$ReflectionAllocator@UPxBounds3V@physx@@@shdfnd@2@@shdfnd@physx@@IEAAXI@Z 0000000180005550 f i RTreeCooking.obj
 0001:00004560       ?grow@?$Array@URTreeNodeNQ@physx@@V?$ReflectionAllocator@URTreeNodeNQ@physx@@@shdfnd@2@@shdfnd@physx@@IEAAXI@Z 0000000180005560 f i RTreeCooking.obj
 0001:00004570       ?grow@?$Array@URTreeNodeQ@Gu@physx@@V?$ReflectionAllocator@URTreeNodeQ@Gu@physx@@@shdfnd@3@@shdfnd@physx@@IEAAXI@Z 0000000180005570 f i RTreeCooking.obj
 0001:00004580       ?grow@?$Array@VPxVec3@physx@@V?$ReflectionAllocator@VPxVec3@physx@@@shdfnd@2@@shdfnd@physx@@IEAAXI@Z 0000000180005580 f i RTreeCooking.obj
 0001:00004590       ?grow@?$Stack@V?$ReflectionAllocator@I@shdfnd@physx@@@internal@shdfnd@physx@@QEAAXXZ 0000000180005590 f i RTreeCooking.obj
 0001:00004660       ?growAndPushBack@?$Array@IV?$ReflectionAllocator@I@shdfnd@physx@@@shdfnd@physx@@IEAAAEAIAEBI@Z 0000000180005660 f i RTreeCooking.obj
 0001:00004740       ?growAndPushBack@?$Array@UInterval@physx@@V?$InlineAllocator@$0CA@V?$ReflectionAllocator@UInterval@physx@@@shdfnd@physx@@@shdfnd@2@@shdfnd@physx@@IEAAAEAUInterval@3@AEBU43@@Z 0000000180005740 f i RTreeCooking.obj
 0001:00004850       ?growAndPushBack@?$Array@UPxBounds3V@physx@@V?$ReflectionAllocator@UPxBounds3V@physx@@@shdfnd@2@@shdfnd@physx@@IEAAAEAUPxBounds3V@3@AEBU43@@Z 0000000180005850 f i RTreeCooking.obj
 0001:00004940       ?growAndPushBack@?$Array@URTreeNodeNQ@physx@@V?$ReflectionAllocator@URTreeNodeNQ@physx@@@shdfnd@2@@shdfnd@physx@@IEAAAEAURTreeNodeNQ@3@AEBU43@@Z 0000000180005940 f i RTreeCooking.obj
 0001:00004a50       ?growAndPushBack@?$Array@URTreeNodeQ@Gu@physx@@V?$ReflectionAllocator@URTreeNodeQ@Gu@physx@@@shdfnd@3@@shdfnd@physx@@IEAAAEAURTreeNodeQ@Gu@3@AEBU453@@Z 0000000180005a50 f i RTreeCooking.obj
 0001:00004b50       ?growAndPushBack@?$Array@VPxVec3@physx@@V?$ReflectionAllocator@VPxVec3@physx@@@shdfnd@2@@shdfnd@physx@@IEAAAEAVPxVec3@3@AEBV43@@Z 0000000180005b50 f i RTreeCooking.obj
 0001:00004c40       ?include@PxBounds3V@physx@@QEAAXAEBU12@@Z 0000000180005c40 f i RTreeCooking.obj
 0001:00004c60       ?isInUserMemory@?$Array@IV?$ReflectionAllocator@I@shdfnd@physx@@@shdfnd@physx@@QEBAIXZ 0000000180005c60 f i RTreeCooking.obj
 0001:00004c70       ?isInUserMemory@?$Array@UInterval@physx@@V?$InlineAllocator@$0CA@V?$ReflectionAllocator@UInterval@physx@@@shdfnd@physx@@@shdfnd@2@@shdfnd@physx@@QEBAIXZ 0000000180005c70 f i RTreeCooking.obj
 0001:00004c80       ?isInUserMemory@?$Array@UPxBounds3V@physx@@V?$ReflectionAllocator@UPxBounds3V@physx@@@shdfnd@2@@shdfnd@physx@@QEBAIXZ 0000000180005c80 f i RTreeCooking.obj
 0001:00004c90       ?isInUserMemory@?$Array@URTreeNodeNQ@physx@@V?$ReflectionAllocator@URTreeNodeNQ@physx@@@shdfnd@2@@shdfnd@physx@@QEBAIXZ 0000000180005c90 f i RTreeCooking.obj
 0001:00004ca0       ?isInUserMemory@?$Array@URTreeNodeQ@Gu@physx@@V?$ReflectionAllocator@URTreeNodeQ@Gu@physx@@@shdfnd@3@@shdfnd@physx@@QEBAIXZ 0000000180005ca0 f i RTreeCooking.obj
 0001:00004cb0       ?isInUserMemory@?$Array@VPxVec3@physx@@V?$ReflectionAllocator@VPxVec3@physx@@@shdfnd@2@@shdfnd@physx@@QEBAIXZ 0000000180005cb0 f i RTreeCooking.obj
 0001:00004cc0       ?memCopy@intrinsics@physx@@YAPEAXPEIAXPEIBXI@Z 0000000180005cc0 f i RTreeCooking.obj
 0001:00004ce0       ?pop@?$Stack@V?$ReflectionAllocator@I@shdfnd@physx@@@internal@shdfnd@physx@@QEAAXAEAH0@Z 0000000180005ce0 f i RTreeCooking.obj
 0001:00004d10       ?popBack@?$Array@IV?$ReflectionAllocator@I@shdfnd@physx@@@shdfnd@physx@@QEAAIXZ 0000000180005d10 f i RTreeCooking.obj
 0001:00004d30       ?push@?$Stack@V?$ReflectionAllocator@I@shdfnd@physx@@@internal@shdfnd@physx@@QEAAXHH@Z 0000000180005d30 f i RTreeCooking.obj
 0001:00004d90       ?pushBack@?$Array@IV?$ReflectionAllocator@I@shdfnd@physx@@@shdfnd@physx@@QEAAAEAIAEBI@Z 0000000180005d90 f i RTreeCooking.obj
 0001:00004dd0       ?pushBack@?$Array@UInterval@physx@@V?$InlineAllocator@$0CA@V?$ReflectionAllocator@UInterval@physx@@@shdfnd@physx@@@shdfnd@2@@shdfnd@physx@@QEAAAEAUInterval@3@AEBU43@@Z 0000000180005dd0 f i RTreeCooking.obj
 0001:00004e10       ?pushBack@?$Array@UPxBounds3V@physx@@V?$ReflectionAllocator@UPxBounds3V@physx@@@shdfnd@2@@shdfnd@physx@@QEAAAEAUPxBounds3V@3@AEBU43@@Z 0000000180005e10 f i RTreeCooking.obj
 0001:00004e60       ?pushBack@?$Array@URTreeNodeNQ@physx@@V?$ReflectionAllocator@URTreeNodeNQ@physx@@@shdfnd@2@@shdfnd@physx@@QEAAAEAURTreeNodeNQ@3@AEBU43@@Z 0000000180005e60 f i RTreeCooking.obj
 0001:00004ed0       ?pushBack@?$Array@URTreeNodeQ@Gu@physx@@V?$ReflectionAllocator@URTreeNodeQ@Gu@physx@@@shdfnd@3@@shdfnd@physx@@QEAAAEAURTreeNodeQ@Gu@3@AEBU453@@Z 0000000180005ed0 f i RTreeCooking.obj
 0001:00004f20       ?pushBack@?$Array@VPxVec3@physx@@V?$ReflectionAllocator@VPxVec3@physx@@@shdfnd@2@@shdfnd@physx@@QEAAAEAVPxVec3@3@AEBV43@@Z 0000000180005f20 f i RTreeCooking.obj
 0001:00004f80       ?recreate@?$Array@IV?$ReflectionAllocator@I@shdfnd@physx@@@shdfnd@physx@@IEAAXI@Z 0000000180005f80 f i RTreeCooking.obj
 0001:00005030       ?recreate@?$Array@UPxBounds3V@physx@@V?$ReflectionAllocator@UPxBounds3V@physx@@@shdfnd@2@@shdfnd@physx@@IEAAXI@Z 0000000180006030 f i RTreeCooking.obj
 0001:000050e0       ?recreate@?$Array@URTreeNodeNQ@physx@@V?$ReflectionAllocator@URTreeNodeNQ@physx@@@shdfnd@2@@shdfnd@physx@@IEAAXI@Z 00000001800060e0 f i RTreeCooking.obj
 0001:00005170       ?recreate@?$Array@URTreeNodeQ@Gu@physx@@V?$ReflectionAllocator@URTreeNodeQ@Gu@physx@@@shdfnd@3@@shdfnd@physx@@IEAAXI@Z 0000000180006170 f i RTreeCooking.obj
 0001:00005230       ?recreate@?$Array@VPxVec3@physx@@V?$ReflectionAllocator@VPxVec3@physx@@@shdfnd@2@@shdfnd@physx@@IEAAXI@Z 0000000180006230 f i RTreeCooking.obj
 0001:000052d0       ?replaceWithLast@?$Array@UInterval@physx@@V?$InlineAllocator@$0CA@V?$ReflectionAllocator@UInterval@physx@@@shdfnd@physx@@@shdfnd@2@@shdfnd@physx@@QEAAXI@Z 00000001800062d0 f i RTreeCooking.obj
 0001:000052f0       ?reserve@?$Array@IV?$ReflectionAllocator@I@shdfnd@physx@@@shdfnd@physx@@QEAAXI@Z 00000001800062f0 f i RTreeCooking.obj
 0001:00005300       ?reserve@?$Array@UPxBounds3V@physx@@V?$ReflectionAllocator@UPxBounds3V@physx@@@shdfnd@2@@shdfnd@physx@@QEAAXI@Z 0000000180006300 f i RTreeCooking.obj
 0001:00005310       ?reserve@?$Array@URTreeNodeNQ@physx@@V?$ReflectionAllocator@URTreeNodeNQ@physx@@@shdfnd@2@@shdfnd@physx@@QEAAXI@Z 0000000180006310 f i RTreeCooking.obj
 0001:00005320       ?reserve@?$Array@URTreeNodeQ@Gu@physx@@V?$ReflectionAllocator@URTreeNodeQ@Gu@physx@@@shdfnd@3@@shdfnd@physx@@QEAAXI@Z 0000000180006320 f i RTreeCooking.obj
 0001:00005330       ?reserve@?$Array@VPxVec3@physx@@V?$ReflectionAllocator@VPxVec3@physx@@@shdfnd@2@@shdfnd@physx@@QEAAXI@Z 0000000180006330 f i RTreeCooking.obj
 0001:00005340       ?resize@?$Array@IV?$ReflectionAllocator@I@shdfnd@physx@@@shdfnd@physx@@QEAAXIAEBI@Z 0000000180006340 f i RTreeCooking.obj
 0001:000053b0       ?resizeUninitialized@?$Array@URTreeNodeNQ@physx@@V?$ReflectionAllocator@URTreeNodeNQ@physx@@@shdfnd@2@@shdfnd@physx@@QEAAXI@Z 00000001800063b0 f i RTreeCooking.obj
 0001:000053f0       ?selectMax@intrinsics@physx@@YAMMM@Z 00000001800063f0 f i RTreeCooking.obj
 0001:00005400       ?selectMin@intrinsics@physx@@YAMMM@Z 0000000180006400 f i RTreeCooking.obj
 0001:00005410       ?setEmpty@PxBounds3@physx@@QEAAXXZ 0000000180006410 f i RTreeCooking.obj
 0001:00005440       ?setLeaf@RTreeNodeQ@Gu@physx@@QEAAX_N@Z 0000000180006440 f i RTreeCooking.obj
 0001:00005450       ?size@?$Array@IV?$ReflectionAllocator@I@shdfnd@physx@@@shdfnd@physx@@QEBAIXZ 0000000180006450 f i RTreeCooking.obj
 0001:00005460       ?size@?$Array@UInterval@physx@@V?$InlineAllocator@$0CA@V?$ReflectionAllocator@UInterval@physx@@@shdfnd@physx@@@shdfnd@2@@shdfnd@physx@@QEBAIXZ 0000000180006460 f i RTreeCooking.obj
 0001:00005470       ?size@?$Array@URTreeNodeNQ@physx@@V?$ReflectionAllocator@URTreeNodeNQ@physx@@@shdfnd@2@@shdfnd@physx@@QEBAIXZ 0000000180006470 f i RTreeCooking.obj
 0001:00005480       ?size@?$Array@URTreeNodeQ@Gu@physx@@V?$ReflectionAllocator@URTreeNodeQ@Gu@physx@@@shdfnd@3@@shdfnd@physx@@QEBAIXZ 0000000180006480 f i RTreeCooking.obj
 0001:00005490       ?sort4@SubSortQuick@physx@@QEAAXPEIAIIAEAV?$Array@URTreeNodeNQ@physx@@V?$ReflectionAllocator@URTreeNodeNQ@physx@@@shdfnd@2@@shdfnd@2@AEAIAEAUPxBounds3V@2@I@Z 0000000180006490 f i RTreeCooking.obj
 0001:00005800       ?sort4@SubSortSAH@physx@@QEAAXPEAIIAEAV?$Array@URTreeNodeNQ@physx@@V?$ReflectionAllocator@URTreeNodeNQ@physx@@@shdfnd@2@@shdfnd@2@AEAIIPEAURTreeNodeNQ@2@@Z 0000000180006800 f i RTreeCooking.obj
 0001:00005eb0       ?split@SubSortSAH@physx@@QEAAIPEAII@Z 0000000180006eb0 f i RTreeCooking.obj
 0001:00006690       ?loadFromDesc@TriangleMeshBuilder@physx@@QEAA_NAEBVPxTriangleMeshDesc@2@AEBUPxCookingParams@2@_N@Z 0000000180007690 f   TriangleMeshBuilder.obj
 0001:00006980       ?save@TriangleMeshBuilder@physx@@QEBA_NAEAVPxOutputStream@2@_NAEBUPxCookingParams@2@@Z 0000000180007980 f   TriangleMeshBuilder.obj
 0001:00006ce0       ?computeLocalBounds@TriangleMeshBuilder@physx@@IEAAXXZ 0000000180007ce0 f   TriangleMeshBuilder.obj
 0001:00006db0       ?importMesh@TriangleMeshBuilder@physx@@IEAA_NAEBVPxTriangleMeshDesc@2@AEBUPxCookingParams@2@_N@Z 0000000180007db0 f   TriangleMeshBuilder.obj
 0001:00006fe0       ??$?_UI@@YAPEAX_KV?$ReflectionAllocator@I@shdfnd@physx@@PEBDH@Z 0000000180007fe0 f i TriangleMeshBuilder.obj
 0001:00006ff0       ??0?$PxFlags@W4Enum@PxMeshFlag@physx@@G@physx@@QEAA@AEBV01@@Z 0000000180007ff0 f i TriangleMeshBuilder.obj
 0001:00007000       ??0?$PxFlags@W4Enum@PxMeshFlag@physx@@G@physx@@QEAA@W4Enum@PxMeshFlag@1@@Z 0000000180008000 f i TriangleMeshBuilder.obj
 0001:00007010       ??0?$PxFlags@W4Enum@PxMeshFlag@physx@@G@physx@@QEAA@XZ 0000000180008010 f i TriangleMeshBuilder.obj
 0001:00007020       ??0?$PxFlags@W4Enum@PxMeshPreprocessingFlag@physx@@I@physx@@QEAA@AEBV01@@Z 0000000180008020 f i TriangleMeshBuilder.obj
 0001:00007030       ??0PxSimpleTriangleMesh@physx@@QEAA@AEBV01@@Z 0000000180008030 f i TriangleMeshBuilder.obj
 0001:00007060       ??0PxTriangleMeshDesc@physx@@QEAA@AEBV01@@Z 0000000180008060 f i TriangleMeshBuilder.obj
 0001:000070a0       ??APxVec3@physx@@QEAAAEAMI@Z 00000001800080a0 f i TriangleMeshBuilder.obj
 0001:000070b0       ??B?$PxFlags@W4Enum@PxMeshFlag@physx@@G@physx@@QEBA_NXZ 00000001800080b0 f i TriangleMeshBuilder.obj
 0001:000070c0       ??B?$PxFlags@W4Enum@PxMeshPreprocessingFlag@physx@@I@physx@@QEBA_NXZ 00000001800080c0 f i TriangleMeshBuilder.obj
 0001:000070d0       ??I?$PxFlags@W4Enum@PxMeshFlag@physx@@G@physx@@QEBA?AV01@W4Enum@PxMeshFlag@1@@Z 00000001800080d0 f i TriangleMeshBuilder.obj
 0001:000070e0       ??I?$PxFlags@W4Enum@PxMeshPreprocessingFlag@physx@@I@physx@@QEBA?AV01@W4Enum@PxMeshPreprocessingFlag@1@@Z 00000001800080e0 f i TriangleMeshBuilder.obj
 0001:000070f0       ??S?$PxFlags@W4Enum@PxMeshFlag@physx@@G@physx@@QEBA?AV01@XZ 00000001800080f0 f i TriangleMeshBuilder.obj
 0001:00007100       ??Sphysx@@YA?AV?$PxFlags@W4Enum@PxMeshFlag@physx@@G@0@W4Enum@PxMeshFlag@0@@Z 0000000180008100 f i TriangleMeshBuilder.obj
 0001:00007110       ??_4?$PxFlags@W4Enum@PxMeshFlag@physx@@G@physx@@QEAAAEAV01@AEBV01@@Z 0000000180008110 f i TriangleMeshBuilder.obj
 0001:00007120       ??_H@YAXPEAX_KHP6APEAX0@Z@Z 0000000180008120 f i TriangleMeshBuilder.obj
 0001:00007170       ?PxAbs@physx@@YAMM@Z       0000000180008170 f i TriangleMeshBuilder.obj
 0001:00007180       ?abs@intrinsics@physx@@YAMM@Z 0000000180008180 f i TriangleMeshBuilder.obj
 0001:00007190       ?gatherStrided@shdfnd@physx@@YAXPEBXPEAXIII@Z 0000000180008190 f i TriangleMeshBuilder.obj
 0001:00007200       ?getFoundation@shdfnd@physx@@YAAEAVFoundation@12@XZ 0000000180008200 f i TriangleMeshBuilder.obj
 0001:00007210       ?isValid@PxSimpleTriangleMesh@physx@@QEBA_NXZ 0000000180008210 f i TriangleMeshBuilder.obj
 0001:00007250       ?isValid@PxTriangleMeshDesc@physx@@QEBA_NXZ 0000000180008250 f i TriangleMeshBuilder.obj
 0001:000072d0       ?to16@shdfnd@physx@@YAGI@Z 00000001800082d0 f i TriangleMeshBuilder.obj
 0001:000072e0       ?writeIntBuffer@physx@@YAXPEBII_NAEAVPxOutputStream@1@@Z 00000001800082e0 f i TriangleMeshBuilder.obj
 0001:000072f0       fabsf                      00000001800082f0 f i TriangleMeshBuilder.obj
 0001:00007300       ??0BigConvexDataBuilder@physx@@QEAA@PEBUConvexHullData@Gu@1@PEAVBigConvexData@1@PEBVPxVec3@1@@Z 0000000180008300 f   BigConvexDataBuilder.obj
 0001:00007320       ??1BigConvexDataBuilder@physx@@QEAA@XZ 0000000180008320 f   BigConvexDataBuilder.obj
 0001:00007330       ?Precompute@BigConvexDataBuilder@physx@@QEAA_NI@Z 0000000180008330 f   BigConvexDataBuilder.obj
 0001:00007670       ?Initialize@BigConvexDataBuilder@physx@@QEAA_NXZ 0000000180008670 f   BigConvexDataBuilder.obj
 0001:00007710       ?PrecomputeSample@BigConvexDataBuilder@physx@@QEAA_NIAEBVPxVec3@2@@Z 0000000180008710 f   BigConvexDataBuilder.obj
 0001:00007950       ?Save@BigConvexDataBuilder@physx@@QEBA_NAEAVPxOutputStream@2@_NIPEBUHullTriangleData@2@@Z 0000000180008950 f   BigConvexDataBuilder.obj
 0001:00007a80       ?ComputeValencies@BigConvexDataBuilder@physx@@QEBA_NIPEBUHullTriangleData@2@@Z 0000000180008a80 f   BigConvexDataBuilder.obj
 0001:00007ad0       ?Compute@BigConvexDataBuilder@physx@@QEBA_NAEBUVALENCIESCREATE@2@@Z 0000000180008ad0 f   BigConvexDataBuilder.obj
 0001:00007d90       ?Save@BigConvexDataBuilder@physx@@QEBA_NAEAVPxOutputStream@2@_N@Z 0000000180008d90 f   BigConvexDataBuilder.obj
 0001:00007f30       ??$?_UE@@YAPEAX_KV?$ReflectionAllocator@E@shdfnd@physx@@PEBDH@Z 0000000180008f30 f i BigConvexDataBuilder.obj
 0001:00007f40       ??$?_UG@@YAPEAX_KV?$ReflectionAllocator@G@shdfnd@physx@@PEBDH@Z 0000000180008f40 f i BigConvexDataBuilder.obj
 0001:00007f50       ??$?_UUValency@Gu@physx@@@@YAPEAX_KV?$ReflectionAllocator@UValency@Gu@physx@@@shdfnd@physx@@PEBDH@Z 0000000180008f50 f i BigConvexDataBuilder.obj
 0001:00007f60       ??0?$ReflectionAllocator@E@shdfnd@physx@@QEAA@PEBD@Z 0000000180008f60 f i BigConvexDataBuilder.obj
 0001:00007f70       ??0?$ReflectionAllocator@G@shdfnd@physx@@QEAA@PEBD@Z 0000000180008f70 f i BigConvexDataBuilder.obj
 0001:00007f80       ??0?$ReflectionAllocator@UValency@Gu@physx@@@shdfnd@physx@@QEAA@PEBD@Z 0000000180008f80 f i BigConvexDataBuilder.obj
 0001:00007f90       ??0EDGELISTCREATE@Gu@physx@@QEAA@XZ 0000000180008f90 f i BigConvexDataBuilder.obj
 0001:00007fb0       ??0PxVec3@physx@@QEAA@XZ   0000000180008fb0 f i BigConvexDataBuilder.obj
 0001:00007fc0       ??0VALENCIESCREATE@physx@@QEAA@XZ 0000000180008fc0 f i BigConvexDataBuilder.obj
 0001:00007fe0       ??_0PxVec3@physx@@QEAAAEAV01@M@Z 0000000180008fe0 f i BigConvexDataBuilder.obj
 0001:00008020       ?GetEdge@EdgeList@Gu@physx@@QEBAAEBUEdgeData@23@I@Z 0000000180009020 f i BigConvexDataBuilder.obj
 0001:00008030       ?GetNbEdges@EdgeList@Gu@physx@@QEBAIXZ 0000000180009030 f i BigConvexDataBuilder.obj
 0001:00008040       ?PxMemZero@physx@@YAPEAXPEIAXI@Z 0000000180009040 f i BigConvexDataBuilder.obj
 0001:00008060       ?PxSqrt@physx@@YAMM@Z      0000000180009060 f i BigConvexDataBuilder.obj
 0001:00008070       ?allocate@?$ReflectionAllocator@E@shdfnd@physx@@QEAAPEAX_KPEBDH@Z 0000000180009070 f i BigConvexDataBuilder.obj
 0001:00008110       ?allocate@?$ReflectionAllocator@G@shdfnd@physx@@QEAAPEAX_KPEBDH@Z 0000000180009110 f i BigConvexDataBuilder.obj
 0001:000081b0       ?allocate@?$ReflectionAllocator@UValency@Gu@physx@@@shdfnd@physx@@QEAAPEAX_KPEBDH@Z 00000001800091b0 f i BigConvexDataBuilder.obj
 0001:00008250       ?dot@PxVec3@physx@@QEBAMAEBV12@@Z 0000000180009250 f i BigConvexDataBuilder.obj
 0001:00008280       ?getName@?$ReflectionAllocator@E@shdfnd@physx@@CAPEBDXZ 0000000180009280 f i BigConvexDataBuilder.obj
 0001:000082c0       ?getName@?$ReflectionAllocator@G@shdfnd@physx@@CAPEBDXZ 00000001800092c0 f i BigConvexDataBuilder.obj
 0001:00008300       ?getName@?$ReflectionAllocator@UValency@Gu@physx@@@shdfnd@physx@@CAPEBDXZ 0000000180009300 f i BigConvexDataBuilder.obj
 0001:00008340       ?magnitude@PxVec3@physx@@QEBAMXZ 0000000180009340 f i BigConvexDataBuilder.obj
 0001:00008370       ?magnitudeSquared@PxVec3@physx@@QEBAMXZ 0000000180009370 f i BigConvexDataBuilder.obj
 0001:000083a0       ?memZero@intrinsics@physx@@YAPEAXPEIAXI@Z 00000001800093a0 f i BigConvexDataBuilder.obj
 0001:000083c0       ?normalize@PxVec3@physx@@QEAAMXZ 00000001800093c0 f i BigConvexDataBuilder.obj
 0001:00008430       ?sqrt@intrinsics@physx@@YAMM@Z 0000000180009430 f i BigConvexDataBuilder.obj
 0001:00008470       ??0ConvexHullBuilder@physx@@QEAA@PEAUConvexHullData@Gu@1@@Z 0000000180009470 f   ConvexHullBuilder.obj
 0001:000084b0       ??1ConvexHullBuilder@physx@@QEAA@XZ 00000001800094b0 f   ConvexHullBuilder.obj
 0001:00008560       ?Init@ConvexHullBuilder@physx@@QEAA_NIPEBVPxVec3@2@IPEBIIPEBUPxHullPolygon@2@@Z 0000000180009560 f   ConvexHullBuilder.obj
 0001:00008c10       ?Save@ConvexHullBuilder@physx@@QEBA_NAEAVPxOutputStream@2@_N@Z 0000000180009c10 f   ConvexHullBuilder.obj
 0001:00008f30       ?CreateEdgeList@ConvexHullBuilder@physx@@QEAA_NXZ 0000000180009f30 f   ConvexHullBuilder.obj
 0001:00009970       ?CreatePolygonData@ConvexHullBuilder@physx@@QEAA_NXZ 000000018000a970 f   ConvexHullBuilder.obj
 0001:0000a130       ?CheckHullPolygons@ConvexHullBuilder@physx@@QEBA_NXZ 000000018000b130 f   ConvexHullBuilder.obj
 0001:0000a4f0       ?CreateTrianglesFromPolygons@ConvexHullBuilder@physx@@QEAA_NXZ 000000018000b4f0 f   ConvexHullBuilder.obj
 0001:0000af20       ?ComputeGeomCenter@ConvexHullBuilder@physx@@QEBA_NAEAVPxVec3@2@@Z 000000018000bf20 f   ConvexHullBuilder.obj
 0001:0000b170       ?CalculateVertexMapTable@ConvexHullBuilder@physx@@QEAA_NI_N@Z 000000018000c170 f   ConvexHullBuilder.obj
 0001:0000b370       ?ComputeHullPolygons@ConvexHullBuilder@physx@@QEAA_NAEBIPEBVPxVec3@2@0PEBI@Z 000000018000c370 f   ConvexHullBuilder.obj
 0001:0000d940       ??$?_UUEdgeDescData@Gu@physx@@@@YAPEAX_KV?$ReflectionAllocator@UEdgeDescData@Gu@physx@@@shdfnd@physx@@PEBDH@Z 000000018000e940 f i ConvexHullBuilder.obj
 0001:0000d950       ??$?_UUHullTriangleData@physx@@@@YAPEAX_KV?$ReflectionAllocator@UHullTriangleData@physx@@@shdfnd@physx@@PEBDH@Z 000000018000e950 f i ConvexHullBuilder.obj
 0001:0000d960       ??$PX_UNUSED@H@@YAXAEBH@Z  000000018000e960 f i ConvexHullBuilder.obj
 0001:0000d970       ??$PlaneEquation@U?$TriangleT@I@Gu@physx@@@@YA?AVPxPlane@physx@@AEBU?$TriangleT@I@Gu@1@PEBVPxVec3@1@@Z 000000018000e970 f i ConvexHullBuilder.obj
 0001:0000db00       ??$swap@E@shdfnd@physx@@YAXAEAE0@Z 000000018000eb00 f i ConvexHullBuilder.obj
 0001:0000db10       ??0?$ReflectionAllocator@UEdgeDescData@Gu@physx@@@shdfnd@physx@@QEAA@PEBD@Z 000000018000eb10 f i ConvexHullBuilder.obj
 0001:0000db20       ??0?$ReflectionAllocator@UHullTriangleData@physx@@@shdfnd@physx@@QEAA@PEBD@Z 000000018000eb20 f i ConvexHullBuilder.obj
 0001:0000db30       ??0?$TriangleT@I@Gu@physx@@QEAA@III@Z 000000018000eb30 f i ConvexHullBuilder.obj
 0001:0000db40       ??0ADJACENCIESCREATE@physx@@QEAA@XZ 000000018000eb40 f i ConvexHullBuilder.obj
 0001:0000db60       ??0HullPolygonData@Gu@physx@@QEAA@AEBU012@@Z 000000018000eb60 f i ConvexHullBuilder.obj
 0001:0000db90       ??0PxPlane@physx@@QEAA@AEBV01@@Z 000000018000eb90 f i ConvexHullBuilder.obj
 0001:0000dbb0       ??0PxPlane@physx@@QEAA@AEBVPxVec3@1@00@Z 000000018000ebb0 f i ConvexHullBuilder.obj
 0001:0000dd10       ??0PxPlane@physx@@QEAA@MMMM@Z 000000018000ed10 f i ConvexHullBuilder.obj
 0001:0000dd30       ??4PxPlane@physx@@QEAAAEAV01@AEBV01@@Z 000000018000ed30 f i ConvexHullBuilder.obj
 0001:0000dd50       ??DPxVec3@physx@@QEBA?AV01@M@Z 000000018000ed50 f i ConvexHullBuilder.obj
 0001:0000dd80       ??GPxVec3@physx@@QEBA?AV01@AEBV01@@Z 000000018000ed80 f i ConvexHullBuilder.obj
 0001:0000ddc0       ??GPxVec3@physx@@QEBA?AV01@XZ 000000018000edc0 f i ConvexHullBuilder.obj
 0001:0000de00       ??YPxVec3@physx@@QEAAAEAV01@AEBV01@@Z 000000018000ee00 f i ConvexHullBuilder.obj
 0001:0000de30       ?ComputeNbPolygons@ConvexHullBuilder@physx@@QEBAIXZ 000000018000ee30 f i ConvexHullBuilder.obj
 0001:0000de60       ?Flip@physx@@YAXAEAUHullTriangleData@1@@Z 000000018000ee60 f i ConvexHullBuilder.obj
 0001:0000de70       ?GetAdjTri@AdjTriangle@physx@@QEBAIW4SharedEdgeIndex@2@@Z 000000018000ee70 f i ConvexHullBuilder.obj
 0001:0000de80       ?GetFaces@ConvexHullBuilder@physx@@QEBAPEBUHullTriangleData@2@XZ 000000018000ee80 f i ConvexHullBuilder.obj
 0001:0000de90       ?GetNbFaces@ConvexHullBuilder@physx@@QEBAIXZ 000000018000ee90 f i ConvexHullBuilder.obj
 0001:0000dea0       ?HasActiveEdge01@AdjTriangle@physx@@QEBAHXZ 000000018000eea0 f i ConvexHullBuilder.obj
 0001:0000deb0       ?HasActiveEdge12@AdjTriangle@physx@@QEBAHXZ 000000018000eeb0 f i ConvexHullBuilder.obj
 0001:0000dec0       ?HasActiveEdge20@AdjTriangle@physx@@QEBAHXZ 000000018000eec0 f i ConvexHullBuilder.obj
 0001:0000ded0       ?HasActiveEdge@AdjTriangle@physx@@QEBAHI@Z 000000018000eed0 f i ConvexHullBuilder.obj
 0001:0000dee0       ?PxRecipSqrt@physx@@YAMM@Z 000000018000eee0 f i ConvexHullBuilder.obj
 0001:0000df00       ?allocate@?$ReflectionAllocator@UEdgeDescData@Gu@physx@@@shdfnd@physx@@QEAAPEAX_KPEBDH@Z 000000018000ef00 f i ConvexHullBuilder.obj
 0001:0000dfa0       ?allocate@?$ReflectionAllocator@UHullTriangleData@physx@@@shdfnd@physx@@QEAAPEAX_KPEBDH@Z 000000018000efa0 f i ConvexHullBuilder.obj
 0001:0000e040       ?area@?$TriangleT@I@Gu@physx@@QEBAMPEBVPxVec3@3@@Z 000000018000f040 f i ConvexHullBuilder.obj
 0001:0000e100       ?center@?$TriangleT@I@Gu@physx@@QEBAXPEBVPxVec3@3@AEAV43@@Z 000000018000f100 f i ConvexHullBuilder.obj
 0001:0000e180       ?cross@PxVec3@physx@@QEBA?AV12@AEBV12@@Z 000000018000f180 f i ConvexHullBuilder.obj
 0001:0000e1e0       ?distance@PxPlane@physx@@QEBAMAEBVPxVec3@2@@Z 000000018000f1e0 f i ConvexHullBuilder.obj
 0001:0000e210       ?flip@?$TriangleT@I@Gu@physx@@QEAAXXZ 000000018000f210 f i ConvexHullBuilder.obj
 0001:0000e220       ?flip@physx@@YAXAEAG@Z     000000018000f220 f i ConvexHullBuilder.obj
 0001:0000e230       ?flip@physx@@YAXAEAM@Z     000000018000f230 f i ConvexHullBuilder.obj
 0001:0000e250       ?flipData@Gu@physx@@YAXAEAUHullPolygonData@12@@Z 000000018000f250 f i ConvexHullBuilder.obj
 0001:0000e2f0       ?getName@?$ReflectionAllocator@UEdgeDescData@Gu@physx@@@shdfnd@physx@@CAPEBDXZ 000000018000f2f0 f i ConvexHullBuilder.obj
 0001:0000e330       ?getName@?$ReflectionAllocator@UHullTriangleData@physx@@@shdfnd@physx@@CAPEBDXZ 000000018000f330 f i ConvexHullBuilder.obj
 0001:0000e370       ?getNormalized@PxVec3@physx@@QEBA?AV12@XZ 000000018000f370 f i ConvexHullBuilder.obj
 0001:0000e410       ?recipSqrt@intrinsics@physx@@YAMM@Z 000000018000f410 f i ConvexHullBuilder.obj
 0001:0000e430       ?to8@shdfnd@physx@@YAEI@Z  000000018000f430 f i ConvexHullBuilder.obj
 0001:0000e440       ??0ConvexMeshBuilder@physx@@QEAA@XZ 000000018000f440 f   ConvexMeshBuilder.obj
 0001:0000e490       ??1ConvexMeshBuilder@physx@@UEAA@XZ 000000018000f490 f   ConvexMeshBuilder.obj
 0001:0000e4e0       ?loadFromDesc@ConvexMeshBuilder@physx@@QEAA_NAEBVPxConvexMeshDesc@2@W4Enum@PxPlatform@2@@Z 000000018000f4e0 f   ConvexMeshBuilder.obj
 0001:0000e5c0       ?save@ConvexMeshBuilder@physx@@QEBA_NAEAVPxOutputStream@2@_N@Z 000000018000f5c0 f   ConvexMeshBuilder.obj
 0001:0000e7d0       ?loadConvexHull@ConvexMeshBuilder@physx@@QEAA_NAEBVPxConvexMeshDesc@2@@Z 000000018000f7d0 f   ConvexMeshBuilder.obj
 0001:0000ea90       ?computeHullPolygons@ConvexMeshBuilder@physx@@QEAA_NAEBIPEBVPxVec3@2@0PEBIAEAVPxAllocatorCallback@2@AEAIAEAPEAV32@4AEAPEAI4AEAPEAUPxHullPolygon@2@@Z 000000018000fa90 f   ConvexMeshBuilder.obj
 0001:0000ecc0       ?computeGaussMaps@ConvexMeshBuilder@physx@@QEAA_NXZ 000000018000fcc0 f   ConvexMeshBuilder.obj
 0001:0000eda0       ?computeMassInfo@ConvexMeshBuilder@physx@@QEAAXXZ 000000018000fda0 f   ConvexMeshBuilder.obj
 0001:0000f190       ?computeInternalObjects@ConvexMeshBuilder@physx@@QEAAXXZ 0000000180010190 f   ConvexMeshBuilder.obj
 0001:0000f790       ??$?2V?$ReflectionAllocator@VBigConvexData@physx@@@shdfnd@physx@@@UserAllocated@shdfnd@physx@@SAPEAX_KV?$ReflectionAllocator@VBigConvexData@physx@@@12@PEBDH@Z 0000000180010790 f i ConvexMeshBuilder.obj
 0001:0000f7a0       ??0?$PxFlags@W4Enum@PxBaseFlag@physx@@G@physx@@QEAA@AEBV01@@Z 00000001800107a0 f i ConvexMeshBuilder.obj
 0001:0000f7b0       ??0?$PxFlags@W4Enum@PxConvexFlag@physx@@G@physx@@QEAA@AEBV01@@Z 00000001800107b0 f i ConvexMeshBuilder.obj
 0001:0000f7c0       ??0?$ReflectionAllocator@VBigConvexData@physx@@@shdfnd@physx@@QEAA@PEBD@Z 00000001800107c0 f i ConvexMeshBuilder.obj
 0001:0000f7d0       ??0PxBoundedData@physx@@QEAA@XZ 00000001800107d0 f i ConvexMeshBuilder.obj
 0001:0000f7e0       ??0PxIntegrals@physx@@QEAA@XZ 00000001800107e0 f i ConvexMeshBuilder.obj
 0001:0000f7f0       ??0PxMat33@physx@@QEAA@AEBVPxVec3@1@00@Z 00000001800107f0 f i ConvexMeshBuilder.obj
 0001:0000f830       ??0PxSimpleTriangleMesh@physx@@QEAA@XZ 0000000180010830 f i ConvexMeshBuilder.obj
 0001:0000f850       ??0PxStridedData@physx@@QEAA@XZ 0000000180010850 f i ConvexMeshBuilder.obj
 0001:0000f860       ??3UserAllocated@shdfnd@physx@@SAXPEAX@Z 0000000180010860 f i ConvexMeshBuilder.obj
 0001:0000f880       ??4PxMat33@physx@@QEAAAEAV01@AEBV01@@Z 0000000180010880 f i ConvexMeshBuilder.obj
 0001:0000f8c0       ??APxMat33@physx@@QEAAAEAVPxVec3@1@I@Z 00000001800108c0 f i ConvexMeshBuilder.obj
 0001:0000f8d0       ??B?$PxFlags@W4Enum@PxBaseFlag@physx@@G@physx@@QEBA_NXZ 00000001800108d0 f i ConvexMeshBuilder.obj
 0001:0000f8e0       ??B?$PxFlags@W4Enum@PxConvexFlag@physx@@G@physx@@QEBA_NXZ 00000001800108e0 f i ConvexMeshBuilder.obj
 0001:0000f8f0       ??GPxMat33@physx@@QEBA?AV01@XZ 00000001800108f0 f i ConvexMeshBuilder.obj
 0001:0000f950       ??I?$PxFlags@W4Enum@PxBaseFlag@physx@@G@physx@@QEBA?AV01@W4Enum@PxBaseFlag@1@@Z 0000000180010950 f i ConvexMeshBuilder.obj
 0001:0000f960       ??I?$PxFlags@W4Enum@PxConvexFlag@physx@@G@physx@@QEBA?AV01@W4Enum@PxConvexFlag@1@@Z 0000000180010960 f i ConvexMeshBuilder.obj
 0001:0000f970       ??RPxMat33@physx@@QEAAAEAMII@Z 0000000180010970 f i ConvexMeshBuilder.obj
 0001:0000f990       ??XPxVec3@physx@@QEAAAEAV01@M@Z 0000000180010990 f i ConvexMeshBuilder.obj
 0001:0000f9b8       ??_EConvexMeshBuilder@physx@@WBA@EAAPEAXI@Z 00000001800109b8 f i ConvexMeshBuilder.obj
 0001:0000f9d0       ??_GBigConvexData@physx@@QEAAPEAXI@Z 00000001800109d0 f i ConvexMeshBuilder.obj
 0001:0000fa10       ??_GConvexMeshBuilder@physx@@UEAAPEAXI@Z 0000000180010a10 f i ConvexMeshBuilder.obj
 0001:0000fa10       ??_EConvexMeshBuilder@physx@@UEAAPEAXI@Z 0000000180010a10 f i ConvexMeshBuilder.obj
 0001:0000fa80       ?PxGetGaussMapVertexLimitForPlatform@physx@@YAIW4Enum@PxPlatform@1@@Z 0000000180010a80 f i ConvexMeshBuilder.obj
 0001:0000fab0       ?PxIsFinite@physx@@YA_NM@Z 0000000180010ab0 f i ConvexMeshBuilder.obj
 0001:0000fad0       ?allocate@?$ReflectionAllocator@VBigConvexData@physx@@@shdfnd@physx@@QEAAPEAX_KPEBDH@Z 0000000180010ad0 f i ConvexMeshBuilder.obj
 0001:0000fb70       ?getName@?$ReflectionAllocator@VBigConvexData@physx@@@shdfnd@physx@@CAPEBDXZ 0000000180010b70 f i ConvexMeshBuilder.obj
 0001:0000fbb0       ?getOriginInertia@PxIntegrals@physx@@QEAAXAEAVPxMat33@2@@Z 0000000180010bb0 f i ConvexMeshBuilder.obj
 0001:0000fc30       ?isFinite@PxVec3@physx@@QEBA_NXZ 0000000180010c30 f i ConvexMeshBuilder.obj
 0001:0000fc90       ?isFinite@intrinsics@physx@@YA_NM@Z 0000000180010c90 f i ConvexMeshBuilder.obj
 0001:0000fcb0       ?isReleasable@PxBase@physx@@UEBA_NXZ 0000000180010cb0 f i ConvexMeshBuilder.obj
 0001:0000fcc0       ?isValid@PxConvexMeshDesc@physx@@QEBA_NXZ 0000000180010cc0 f i ConvexMeshBuilder.obj
 0001:0000fd60       ?largestAxis@shdfnd@physx@@YAIAEBVPxVec3@2@@Z 0000000180010d60 f i ConvexMeshBuilder.obj
 0001:0000fd90       ?requires@ConvexMesh@Gu@physx@@UEAAXAEAVPxProcessPxBaseCallback@3@@Z 0000000180010d90 f i ConvexMeshBuilder.obj
 0001:0000fda0       ??0HullLibrary@physx@@QEAA@XZ 0000000180010da0 f   hulllib.obj
 0001:0000fdf0       ??1HullLibrary@physx@@QEAA@XZ 0000000180010df0 f   hulllib.obj
 0001:0000fe50       ?CreateConvexHull@HullLibrary@physx@@QEAA?AW4HullError@2@AEBVHullDesc@2@AEAVHullResult@2@@Z 0000000180010e50 f   hulllib.obj
 0001:000103a0       ?ReleaseResult@HullLibrary@physx@@QEAA?AW4HullError@2@AEAVHullResult@2@@Z 00000001800113a0 f   hulllib.obj
 0001:000103f0       ?CreateTriangleMesh@HullLibrary@physx@@QEAA?AW4HullError@2@AEAVHullResult@2@PEAVConvexHullTriangleInterface@2@@Z 00000001800113f0 f   hulllib.obj
 0001:000106c0       ?b2bfix@HullLibrary@physx@@AEAAXPEAVTri@2@0@Z 00000001800116c0 f   hulllib.obj
 0001:000108e0       ?removeb2b@HullLibrary@physx@@AEAAXPEAVTri@2@0@Z 00000001800118e0 f   hulllib.obj
 0001:00010960       ?checkit@HullLibrary@physx@@AEBAXPEAVTri@2@@Z 0000000180011960 f   hulllib.obj
 0001:00010970       ?extrude@HullLibrary@physx@@AEAAXPEAVTri@2@H@Z 0000000180011970 f   hulllib.obj
 0001:00010ce0       ?extrudable@HullLibrary@physx@@AEBAPEAVTri@2@M@Z 0000000180011ce0 f   hulllib.obj
 0001:00010e00       ?calchullgen@HullLibrary@physx@@AEAA?AW4HullError@2@PEAVfloat3@2@HHM@Z 0000000180011e00 f   hulllib.obj
 0001:00011be0       ?calchull@HullLibrary@physx@@AEAA?AW4HullError@2@PEAVfloat3@2@HAEAPEAHAEAHAEAPEAV42@2HM@Z 0000000180012be0 f   hulllib.obj
 0001:00011fa0       ?expandhull@HullLibrary@physx@@AEAA?AW4HullError@2@PEAVfloat3@2@HAEAPEAV42@AEAHM@Z 0000000180012fa0 f   hulllib.obj
 0001:000128f0       ?calchullpbev@HullLibrary@physx@@AEAA?AW4HullError@2@PEAVfloat3@2@HHAEAV?$Array@VPlane@physx@@@hullLibArray@2@M@Z 00000001800138f0 f   hulllib.obj
 0001:00013440       ?ComputeHull@HullLibrary@physx@@AEAA?AW4HullError@2@IPEBMAEAVPHullResult@2@IMM@Z 0000000180014440 f   hulllib.obj
 0001:00013780       ?overhullv@HullLibrary@physx@@AEAA?AW4HullError@2@PEAVfloat3@2@HHAEAPEAV42@AEAHAEAPEAH2MMHM@Z 0000000180014780 f   hulllib.obj
 0001:00014460       ??0ConvexH@physx@@QEAA@HHH@Z 0000000180015460 f   hulllib.obj
 0001:00016540       ?neib@Tri@physx@@QEAAAEAHHH@Z 0000000180017540 f   hulllib.obj
 0001:00018610       ??$?2V?$ReflectionAllocator@VConvexH@physx@@@shdfnd@physx@@@UserAllocated@shdfnd@physx@@SAPEAX_KV?$ReflectionAllocator@VConvexH@physx@@@12@PEBDH@Z 0000000180019610 f i hulllib.obj
 0001:00018620       ??$?2V?$ReflectionAllocator@VTri@physx@@@shdfnd@physx@@@UserAllocated@shdfnd@physx@@SAPEAX_KV?$ReflectionAllocator@VTri@physx@@@12@PEBDH@Z 0000000180019620 f i hulllib.obj
 0001:00018630       ??$?_UM@@YAPEAX_KV?$ReflectionAllocator@M@shdfnd@physx@@PEBDH@Z 0000000180019630 f i hulllib.obj
 0001:00018640       ??$Max@M@physx@@YAMAEBM0@Z 0000000180019640 f i hulllib.obj
 0001:00018660       ??$Min@H@physx@@YAHAEBH0@Z 0000000180019660 f i hulllib.obj
 0001:00018670       ??$Min@M@physx@@YAMAEBM0@Z 0000000180019670 f i hulllib.obj
 0001:00018690       ??$Swap@H@physx@@YAXAEAH0@Z 0000000180019690 f i hulllib.obj
 0001:000186a0       ??$maxdir@Vfloat3@physx@@@physx@@YAHPEBVfloat3@0@HAEBV10@@Z 00000001800196a0 f i hulllib.obj
 0001:00018940       ??$maxdirfiltered@Vfloat3@physx@@@physx@@YAHPEBVfloat3@0@HAEBV10@PEA_N@Z 0000000180019940 f i hulllib.obj
 0001:00018c30       ??$maxdirsterid@Vfloat3@physx@@@physx@@YAHPEBVfloat3@0@HAEBV10@AEAV?$Array@H@hullLibArray@0@@Z 0000000180019c30 f i hulllib.obj
 0001:00019000       ??0?$Array@H@hullLibArray@physx@@QEAA@H@Z 000000018001a000 f i hulllib.obj
 0001:00019030       ??0?$Array@PEAVTri@physx@@@hullLibArray@physx@@QEAA@H@Z 000000018001a030 f i hulllib.obj
 0001:00019060       ??0?$Array@UExpandPlane@physx@@@hullLibArray@physx@@QEAA@H@Z 000000018001a060 f i hulllib.obj
 0001:00019090       ??0?$Array@VHalfEdge@ConvexH@physx@@@hullLibArray@physx@@QEAA@H@Z 000000018001a090 f i hulllib.obj
 0001:000190c0       ??0?$Array@VPlane@physx@@@hullLibArray@physx@@QEAA@H@Z 000000018001a0c0 f i hulllib.obj
 0001:000190f0       ??0?$Array@Vfloat3@physx@@@hullLibArray@physx@@QEAA@H@Z 000000018001a0f0 f i hulllib.obj
 0001:00019120       ??0?$Array@Vint3@physx@@@hullLibArray@physx@@QEAA@H@Z 000000018001a120 f i hulllib.obj
 0001:00019150       ??0?$ReflectionAllocator@M@shdfnd@physx@@QEAA@PEBD@Z 000000018001a150 f i hulllib.obj
 0001:00019160       ??0?$ReflectionAllocator@VConvexH@physx@@@shdfnd@physx@@QEAA@PEBD@Z 000000018001a160 f i hulllib.obj
 0001:00019170       ??0?$ReflectionAllocator@VTri@physx@@@shdfnd@physx@@QEAA@PEBD@Z 000000018001a170 f i hulllib.obj
 0001:00019180       ??0?$ScopedPointer@_NVTempAllocator@shdfnd@physx@@@shdfnd@physx@@QEAA@XZ 000000018001a180 f i hulllib.obj
 0001:00019190       ??0ExpandPlane@physx@@QEAA@XZ 000000018001a190 f i hulllib.obj
 0001:000191e0       ??0HalfEdge@ConvexH@physx@@QEAA@FEE@Z 000000018001a1e0 f i hulllib.obj
 0001:000191f0       ??0HalfEdge@ConvexH@physx@@QEAA@XZ 000000018001a1f0 f i hulllib.obj
 0001:00019200       ??0PHullResult@physx@@QEAA@XZ 000000018001a200 f i hulllib.obj
 0001:00019220       ??0Plane@physx@@QEAA@AEBVfloat3@1@M@Z 000000018001a220 f i hulllib.obj
 0001:00019240       ??0Plane@physx@@QEAA@XZ    000000018001a240 f i hulllib.obj
 0001:00019250       ??0Tri@physx@@QEAA@HHHPEAV?$Array@PEAVTri@physx@@@hullLibArray@1@@Z 000000018001a250 f i hulllib.obj
 0001:000192d0       ??0float3@physx@@QEAA@MMM@Z 000000018001a2d0 f i hulllib.obj
 0001:000192f0       ??0float3@physx@@QEAA@XZ   000000018001a2f0 f i hulllib.obj
 0001:00019300       ??0float3x3@physx@@QEAA@Vfloat3@1@00@Z 000000018001a300 f i hulllib.obj
 0001:00019340       ??0float3x3@physx@@QEAA@XZ 000000018001a340 f i hulllib.obj
 0001:00019360       ??0int3@physx@@QEAA@HHH@Z  000000018001a360 f i hulllib.obj
 0001:00019370       ??0int4@physx@@QEAA@HHHH@Z 000000018001a370 f i hulllib.obj
 0001:00019390       ??1?$Array@H@hullLibArray@physx@@QEAA@XZ 000000018001a390 f i hulllib.obj
 0001:000193d0       ??1?$Array@PEAVTri@physx@@@hullLibArray@physx@@QEAA@XZ 000000018001a3d0 f i hulllib.obj
 0001:00019410       ??1?$Array@UExpandPlane@physx@@@hullLibArray@physx@@QEAA@XZ 000000018001a410 f i hulllib.obj
 0001:00019450       ??1?$Array@VHalfEdge@ConvexH@physx@@@hullLibArray@physx@@QEAA@XZ 000000018001a450 f i hulllib.obj
 0001:00019490       ??1?$Array@VPlane@physx@@@hullLibArray@physx@@QEAA@XZ 000000018001a490 f i hulllib.obj
 0001:000194d0       ??1?$Array@Vfloat3@physx@@@hullLibArray@physx@@QEAA@XZ 000000018001a4d0 f i hulllib.obj
 0001:00019510       ??1?$Array@Vint3@physx@@@hullLibArray@physx@@QEAA@XZ 000000018001a510 f i hulllib.obj
 0001:00019550       ??1?$ScopedPointer@_NVTempAllocator@shdfnd@physx@@@shdfnd@physx@@QEAA@XZ 000000018001a550 f i hulllib.obj
 0001:00019570       ??1ConvexH@physx@@QEAA@XZ  000000018001a570 f i hulllib.obj
 0001:000195f0       ??1Tri@physx@@IEAA@XZ      000000018001a5f0 f i hulllib.obj
 0001:00019600       ??8physx@@YAHAEBVPlane@0@0@Z 000000018001a600 f i hulllib.obj
 0001:00019640       ??8physx@@YAHAEBVfloat3@0@0@Z 000000018001a640 f i hulllib.obj
 0001:00019670       ??9physx@@YAHAEBVfloat3@0@0@Z 000000018001a670 f i hulllib.obj
 0001:000196a0       ??A?$Array@H@hullLibArray@physx@@QEAAAEAHH@Z 000000018001a6a0 f i hulllib.obj
 0001:000196b0       ??A?$Array@PEAVTri@physx@@@hullLibArray@physx@@QEAAAEAPEAVTri@2@H@Z 000000018001a6b0 f i hulllib.obj
 0001:000196c0       ??A?$Array@UExpandPlane@physx@@@hullLibArray@physx@@QEAAAEAUExpandPlane@2@H@Z 000000018001a6c0 f i hulllib.obj
 0001:000196d0       ??A?$Array@VHalfEdge@ConvexH@physx@@@hullLibArray@physx@@QEAAAEAVHalfEdge@ConvexH@2@H@Z 000000018001a6d0 f i hulllib.obj
 0001:000196e0       ??A?$Array@VPlane@physx@@@hullLibArray@physx@@QEAAAEAVPlane@2@H@Z 000000018001a6e0 f i hulllib.obj
 0001:000196f0       ??A?$Array@Vfloat3@physx@@@hullLibArray@physx@@QEAAAEAVfloat3@2@H@Z 000000018001a6f0 f i hulllib.obj
 0001:00019700       ??Afloat3@physx@@QEAAAEAMH@Z 000000018001a700 f i hulllib.obj
 0001:00019710       ??Afloat3@physx@@QEBAAEBMH@Z 000000018001a710 f i hulllib.obj
 0001:00019720       ??Afloat3x3@physx@@QEAAAEAVfloat3@1@H@Z 000000018001a720 f i hulllib.obj
 0001:00019730       ??Afloat3x3@physx@@QEBAAEBVfloat3@1@H@Z 000000018001a730 f i hulllib.obj
 0001:00019740       ??Aint3@physx@@QEAAAEAHH@Z 000000018001a740 f i hulllib.obj
 0001:00019750       ??Aint3@physx@@QEBAAEBHH@Z 000000018001a750 f i hulllib.obj
 0001:00019760       ??Aint4@physx@@QEAAAEAHH@Z 000000018001a760 f i hulllib.obj
 0001:00019770       ??B?$ScopedPointer@_NVTempAllocator@shdfnd@physx@@@shdfnd@physx@@QEBAPEA_NXZ 000000018001a770 f i hulllib.obj
 0001:00019780       ??_G?$Array@PEAVTri@physx@@@hullLibArray@physx@@QEAAPEAXI@Z 000000018001a780 f i hulllib.obj
 0001:000197e0       ??_GConvexH@physx@@QEAAPEAXI@Z 000000018001a7e0 f i hulllib.obj
 0001:00019820       ??_GTri@physx@@IEAAPEAXI@Z 000000018001a820 f i hulllib.obj
 0001:00019850       ?Add@?$Array@H@hullLibArray@physx@@QEAAAEAHH@Z 000000018001a850 f i hulllib.obj
 0001:000198a0       ?Add@?$Array@PEAVTri@physx@@@hullLibArray@physx@@QEAAAEAPEAVTri@3@PEAV43@@Z 000000018001a8a0 f i hulllib.obj
 0001:00019900       ?Add@?$Array@UExpandPlane@physx@@@hullLibArray@physx@@QEAAAEAUExpandPlane@3@U43@@Z 000000018001a900 f i hulllib.obj
 0001:00019970       ?Add@?$Array@VPlane@physx@@@hullLibArray@physx@@QEAAAEAVPlane@3@V43@@Z 000000018001a970 f i hulllib.obj
 0001:000199d0       ?Add@?$Array@Vfloat3@physx@@@hullLibArray@physx@@QEAAAEAVfloat3@3@V43@@Z 000000018001a9d0 f i hulllib.obj
 0001:00019a40       ?Add@?$Array@Vint3@physx@@@hullLibArray@physx@@QEAAAEAVint3@3@V43@@Z 000000018001aa40 f i hulllib.obj
 0001:00019ab0       ?HasHullFlag@HullDesc@physx@@QEBA_NW4HullFlag@2@@Z 000000018001aab0 f i hulllib.obj
 0001:00019ac0       ?PxMemSet@physx@@YAPEAXPEIAXHI@Z 000000018001aac0 f i hulllib.obj
 0001:00019ae0       ?SetSize@?$Array@PEAVTri@physx@@@hullLibArray@physx@@QEAAXH@Z 000000018001aae0 f i hulllib.obj
 0001:00019b40       ?SetSize@?$Array@Vint3@physx@@@hullLibArray@physx@@QEAAXH@Z 000000018001ab40 f i hulllib.obj
 0001:00019ba0       ?allocate@?$Array@H@hullLibArray@physx@@QEAAXH@Z 000000018001aba0 f i hulllib.obj
 0001:00019c20       ?allocate@?$Array@PEAVTri@physx@@@hullLibArray@physx@@QEAAXH@Z 000000018001ac20 f i hulllib.obj
 0001:00019ca0       ?allocate@?$Array@UExpandPlane@physx@@@hullLibArray@physx@@QEAAXH@Z 000000018001aca0 f i hulllib.obj
 0001:00019d40       ?allocate@?$Array@VHalfEdge@ConvexH@physx@@@hullLibArray@physx@@QEAAXH@Z 000000018001ad40 f i hulllib.obj
 0001:00019dc0       ?allocate@?$Array@VPlane@physx@@@hullLibArray@physx@@QEAAXH@Z 000000018001adc0 f i hulllib.obj
 0001:00019e40       ?allocate@?$Array@Vfloat3@physx@@@hullLibArray@physx@@QEAAXH@Z 000000018001ae40 f i hulllib.obj
 0001:00019ee0       ?allocate@?$Array@Vint3@physx@@@hullLibArray@physx@@QEAAXH@Z 000000018001aee0 f i hulllib.obj
 0001:00019f80       ?allocate@?$ReflectionAllocator@M@shdfnd@physx@@QEAAPEAX_KPEBDH@Z 000000018001af80 f i hulllib.obj
 0001:0001a020       ?allocate@?$ReflectionAllocator@VConvexH@physx@@@shdfnd@physx@@QEAAPEAX_KPEBDH@Z 000000018001b020 f i hulllib.obj
 0001:0001a0c0       ?allocate@?$ReflectionAllocator@VTri@physx@@@shdfnd@physx@@QEAAPEAX_KPEBDH@Z 000000018001b0c0 f i hulllib.obj
 0001:0001a160       ?cos@@YAMM@Z               000000018001b160 f i hulllib.obj
 0001:0001a170       ?distance@Plane@physx@@QEBAMAEBVfloat3@2@@Z 000000018001b170 f i hulllib.obj
 0001:0001a1a0       ?getName@?$ReflectionAllocator@M@shdfnd@physx@@CAPEBDXZ 000000018001b1a0 f i hulllib.obj
 0001:0001a1e0       ?getName@?$ReflectionAllocator@VConvexH@physx@@@shdfnd@physx@@CAPEBDXZ 000000018001b1e0 f i hulllib.obj
 0001:0001a220       ?getName@?$ReflectionAllocator@VTri@physx@@@shdfnd@physx@@CAPEBDXZ 000000018001b220 f i hulllib.obj
 0001:0001a260       ?memSet@intrinsics@physx@@YAPEAXPEIAXHI@Z 000000018001b260 f i hulllib.obj
 0001:0001a280       ?to8@shdfnd@physx@@YAEG@Z  000000018001b280 f i hulllib.obj
 0001:0001a2c0       ?computeVolumeIntegrals@physx@@YA_NAEBVPxSimpleTriangleMesh@1@MAEAUPxIntegrals@1@@Z 000000018001b2c0 f   VolumeIntegration.obj
 0001:0001a330       ?computeVolumeIntegralsEberly@physx@@YA_NAEBVPxSimpleTriangleMesh@1@MAEAUPxIntegrals@1@AEBVPxVec3@1@@Z 000000018001b330 f   VolumeIntegration.obj
 0001:0001a370       ??0VolumeIntegrator@?A0xd2749a4a@physx@@QEAA@VPxSimpleTriangleMesh@2@N@Z 000000018001b370 f   VolumeIntegration.obj
 0001:0001a3d0       ??1VolumeIntegrator@?A0xd2749a4a@physx@@QEAA@XZ 000000018001b3d0 f   VolumeIntegration.obj
 0001:0001a3e0       ?computeVolumeIntegrals@VolumeIntegrator@?A0xd2749a4a@physx@@QEAA_NAEAUPxIntegrals@3@@Z 000000018001b3e0 f   VolumeIntegration.obj
 0001:0001a880       ?computeCenterOfMass@VolumeIntegrator@?A0xd2749a4a@physx@@AEAA?AVPxVec3@3@XZ 000000018001b880 f   VolumeIntegration.obj
 0001:0001a8f0       ?computeInertiaTensor@VolumeIntegrator@?A0xd2749a4a@physx@@AEAAXPEAN@Z 000000018001b8f0 f   VolumeIntegration.obj
 0001:0001a9c0       ?computeCOMInertiaTensor@VolumeIntegrator@?A0xd2749a4a@physx@@AEAAXPEAN@Z 000000018001b9c0 f   VolumeIntegration.obj
 0001:0001ac90       ?computeFaceNormal@VolumeIntegrator@?A0xd2749a4a@physx@@AEAAXAEAUFace@123@PEAI@Z 000000018001bc90 f   VolumeIntegration.obj
 0001:0001ae00       ?computeProjectionIntegrals@VolumeIntegrator@?A0xd2749a4a@physx@@AEAAXAEBUFace@123@@Z 000000018001be00 f   VolumeIntegration.obj
 0001:0001b380       ?computeFaceIntegrals@VolumeIntegrator@?A0xd2749a4a@physx@@AEAAXAEBUFace@123@@Z 000000018001c380 f   VolumeIntegration.obj
 0001:0001b770       ??0VolumeIntegratorEberly@?A0xd2749a4a@physx@@QEAA@AEBVPxSimpleTriangleMesh@2@N@Z 000000018001c770 f   VolumeIntegration.obj
 0001:0001b790       ??1VolumeIntegratorEberly@?A0xd2749a4a@physx@@QEAA@XZ 000000018001c790 f   VolumeIntegration.obj
 0001:0001b7a0       ?computeVolumeIntegrals@VolumeIntegratorEberly@?A0xd2749a4a@physx@@QEAA_NAEAUPxIntegrals@3@AEBVPxVec3@3@@Z 000000018001c7a0 f   VolumeIntegration.obj
 0001:0001c180       ?subexpressions@VolumeIntegratorEberly@?A0xd2749a4a@physx@@AEAAXNNNAEAN00000@Z 000000018001d180 f   VolumeIntegration.obj
 0001:0001c220       ??4?$PxFlags@W4Enum@PxMeshFlag@physx@@G@physx@@QEAAAEAV01@AEBV01@@Z 000000018001d220 f i VolumeIntegration.obj
 0001:0001c230       ??4PxSimpleTriangleMesh@physx@@QEAAAEAV01@AEBV01@@Z 000000018001d230 f i VolumeIntegration.obj
 0001:0001c260       ?isZero@PxVec3@physx@@QEBA_NXZ 000000018001d260 f i VolumeIntegration.obj
 0001:0001c280       ?ComputeNbBoundaryEdges@AdjTriangle@physx@@QEBAIXZ 000000018001d280 f   Adjacencies.obj
 0001:0001c2d0       ?ComputeNbNeighbors@AdjTriangle@physx@@QEBAIXZ 000000018001d2d0 f   Adjacencies.obj
 0001:0001c320       ?HasNeighbor@AdjTriangle@physx@@QEBA_NIPEAI@Z 000000018001d320 f   Adjacencies.obj
 0001:0001c390       ?Flip@AdjTriangle@physx@@QEAAXXZ 000000018001d390 f   Adjacencies.obj
 0001:0001c3b0       ??0Adjacencies@physx@@QEAA@XZ 000000018001d3b0 f   Adjacencies.obj
 0001:0001c3d0       ??1Adjacencies@physx@@QEAA@XZ 000000018001d3d0 f   Adjacencies.obj
 0001:0001c420       ?Load@Adjacencies@physx@@QEAA_NAEAVPxInputStream@2@@Z 000000018001d420 f   Adjacencies.obj
 0001:0001c550       ?Walk@Adjacencies@physx@@QEAA_NP6AXAEBUCommonWalkParams@2@IIII@ZPEAX@Z 000000018001d550 f   Adjacencies.obj
 0001:0001c650       ?Walk2@Adjacencies@physx@@QEAA_NP6AXAEBUCommonWalkParams@2@IIII@ZPEAXPEBVPxVec3@2@PEBU?$TriangleT@I@Gu@2@@Z 000000018001d650 f   Adjacencies.obj
 0001:0001c830       ?ComputeNbBoundaryEdges@Adjacencies@physx@@QEBAIXZ 000000018001d830 f   Adjacencies.obj
 0001:0001c8a0       ?GetBoundaryVertices@Adjacencies@physx@@QEBA_NIPEA_NPEBU?$TriangleT@I@Gu@2@@Z 000000018001d8a0 f   Adjacencies.obj
 0001:0001ca00       ?MakeLastRef@Adjacencies@physx@@QEAA_NAEAVAdjTriangle@2@IPEAU?$TriangleT@I@Gu@2@@Z 000000018001da00 f   Adjacencies.obj
 0001:0001cc40       ?AssignNewEdgeCode@Adjacencies@physx@@AEAAXIE@Z 000000018001dc40 f   Adjacencies.obj
 0001:0001cc90       ??0AdjacenciesBuilder@physx@@QEAA@XZ 000000018001dc90 f   Adjacencies.obj
 0001:0001ccb0       ??1AdjacenciesBuilder@physx@@QEAA@XZ 000000018001dcb0 f   Adjacencies.obj
 0001:0001cd00       ?Init@AdjacenciesBuilder@physx@@QEAA_NAEBUADJACENCIESCREATE@2@@Z 000000018001dd00 f   Adjacencies.obj
 0001:0001dbe0       ??$?_UV?$ReflectionAllocator@VAdjEdge@@@shdfnd@physx@@@UserAllocated@shdfnd@physx@@SAPEAX_KV?$ReflectionAllocator@VAdjEdge@@@12@PEBDH@Z 000000018001ebe0 f i Adjacencies.obj
 0001:0001dbf0       ??$?_UV?$ReflectionAllocator@VAdjTriangle@physx@@@shdfnd@physx@@@UserAllocated@shdfnd@physx@@SAPEAX_KV?$ReflectionAllocator@VAdjTriangle@physx@@@12@PEBDH@Z 000000018001ebf0 f i Adjacencies.obj
 0001:0001dc00       ??$swap@M@shdfnd@physx@@YAXAEAM0@Z 000000018001ec00 f i Adjacencies.obj
 0001:0001dc10       ??0?$ReflectionAllocator@VAdjEdge@@@shdfnd@physx@@QEAA@PEBD@Z 000000018001ec10 f i Adjacencies.obj
 0001:0001dc20       ??0?$ReflectionAllocator@VAdjTriangle@physx@@@shdfnd@physx@@QEAA@PEBD@Z 000000018001ec20 f i Adjacencies.obj
 0001:0001dc30       ??0?$TriangleT@I@Gu@physx@@QEAA@XZ 000000018001ec30 f i Adjacencies.obj
 0001:0001dc40       ??0AdjEdge@@QEAA@XZ        000000018001ec40 f i Adjacencies.obj
 0001:0001dc50       ??0AdjTriangle@physx@@QEAA@XZ 000000018001ec50 f i Adjacencies.obj
 0001:0001dc60       ??0PrivateWalkParams@?1??Walk2@Adjacencies@physx@@QEAA_NP6AXAEBUCommonWalkParams@3@IIII@ZPEAXPEBVPxVec3@3@PEBU?$TriangleT@I@Gu@3@@Z@QEAA@XZ 000000018001ec60 f i Adjacencies.obj
 0001:0001dc70       ??1AdjEdge@@QEAA@XZ        000000018001ec70 f i Adjacencies.obj
 0001:0001dc80       ??1AdjTriangle@physx@@QEAA@XZ 000000018001ec80 f i Adjacencies.obj
 0001:0001dc90       ??_EAdjEdge@@QEAAPEAXI@Z   000000018001ec90 f i Adjacencies.obj
 0001:0001dce0       ??_EAdjTriangle@physx@@QEAAPEAXI@Z 000000018001ece0 f i Adjacencies.obj
 0001:0001dd30       ??_I@YAXPEAX_KHP6AX0@Z@Z   000000018001ed30 f i Adjacencies.obj
 0001:0001dd90       ??_VUserAllocated@shdfnd@physx@@SAXPEAX@Z 000000018001ed90 f i Adjacencies.obj
 0001:0001ddb0       ?GetEdgeTriangle@EdgeList@Gu@physx@@QEBAAEBUEdgeTriangleData@23@I@Z 000000018001edb0 f i Adjacencies.obj
 0001:0001ddc0       ?HasActiveEdge01@EdgeTriangleAC@Gu@physx@@SAHAEBUEdgeTriangleData@23@@Z 000000018001edc0 f i Adjacencies.obj
 0001:0001ddd0       ?HasActiveEdge12@EdgeTriangleAC@Gu@physx@@SAHAEBUEdgeTriangleData@23@@Z 000000018001edd0 f i Adjacencies.obj
 0001:0001dde0       ?HasActiveEdge20@EdgeTriangleAC@Gu@physx@@SAHAEBUEdgeTriangleData@23@@Z 000000018001ede0 f i Adjacencies.obj
 0001:0001ddf0       ?allocate@?$ReflectionAllocator@VAdjEdge@@@shdfnd@physx@@QEAAPEAX_KPEBDH@Z 000000018001edf0 f i Adjacencies.obj
 0001:0001de90       ?allocate@?$ReflectionAllocator@VAdjTriangle@physx@@@shdfnd@physx@@QEAAPEAX_KPEBDH@Z 000000018001ee90 f i Adjacencies.obj
 0001:0001df30       ?findEdge@?$TriangleT@I@Gu@physx@@QEBAEII@Z 000000018001ef30 f i Adjacencies.obj
 0001:0001df80       ?getName@?$ReflectionAllocator@VAdjEdge@@@shdfnd@physx@@CAPEBDXZ 000000018001ef80 f i Adjacencies.obj
 0001:0001dfc0       ?getName@?$ReflectionAllocator@VAdjTriangle@physx@@@shdfnd@physx@@CAPEBDXZ 000000018001efc0 f i Adjacencies.obj
 0001:0001e000       PxCreateCooking            000000018001f000 f   Cooking.obj
 0001:0001e0f0       ?release@Cooking@physx@@UEAAXXZ 000000018001f0f0 f   Cooking.obj
 0001:0001e120       ?setParams@Cooking@physx@@UEAAXAEBUPxCookingParams@2@@Z 000000018001f120 f   Cooking.obj
 0001:0001e170       ?getParams@Cooking@physx@@UEAAAEBUPxCookingParams@2@XZ 000000018001f170 f   Cooking.obj
 0001:0001e180       ?platformMismatch@Cooking@physx@@UEAA_NXZ 000000018001f180 f   Cooking.obj
 0001:0001e1b0       ?cookTriangleMesh@Cooking@physx@@UEAA_NAEBVPxTriangleMeshDesc@2@AEAVPxOutputStream@2@@Z 000000018001f1b0 f   Cooking.obj
 0001:0001e2f0       ?createTriangleMesh@Cooking@physx@@UEAAPEAVPxTriangleMesh@2@AEBVPxTriangleMeshDesc@2@AEAVPxPhysicsInsertionCallback@2@@Z 000000018001f2f0 f   Cooking.obj
 0001:0001e410       ?validateTriangleMesh@Cooking@physx@@UEAA_NAEBVPxTriangleMeshDesc@2@@Z 000000018001f410 f   Cooking.obj
 0001:0001e4d0       ?cookConvexMesh@Cooking@physx@@UEAA_NAEBVPxConvexMeshDesc@2@AEAVPxOutputStream@2@PEAW4Enum@PxConvexMeshCookingResult@2@@Z 000000018001f4d0 f   Cooking.obj
 0001:0001e830       ?computeHullPolygons@Cooking@physx@@UEAA_NAEBVPxSimpleTriangleMesh@2@AEAVPxAllocatorCallback@2@AEAIAEAPEAVPxVec3@2@2AEAPEAI2AEAPEAUPxHullPolygon@2@@Z 000000018001f830 f   Cooking.obj
 0001:0001ea10       ?cookHeightField@Cooking@physx@@UEAA_NAEBVPxHeightFieldDesc@2@AEAVPxOutputStream@2@@Z 000000018001fa10 f   Cooking.obj
 0001:0001ebb0       ?createHeightField@Cooking@physx@@UEAAPEAVPxHeightField@2@AEBVPxHeightFieldDesc@2@AEAVPxPhysicsInsertionCallback@2@@Z 000000018001fbb0 f   Cooking.obj
 0001:0001ed10       ?loadTriangleMeshDesc@Cooking@physx@@AEAA_NAEBVPxTriangleMeshDesc@2@AEAVTriangleMeshBuilder@2@@Z 000000018001fd10 f   Cooking.obj
 0001:0001edf0       ??$?2V?$ReflectionAllocator@VCooking@physx@@@shdfnd@physx@@@UserAllocated@shdfnd@physx@@SAPEAX_KV?$ReflectionAllocator@VCooking@physx@@@12@PEBDH@Z 000000018001fdf0 f i Cooking.obj
 0001:0001ee00       ??$?2V?$ReflectionAllocator@VHeightField@Gu@physx@@@shdfnd@physx@@@UserAllocated@shdfnd@physx@@SAPEAX_KV?$ReflectionAllocator@VHeightField@Gu@physx@@@12@PEBDH@Z 000000018001fe00 f i Cooking.obj
 0001:0001ee10       ??$?2V?$ReflectionAllocator@VTriangleMeshBuilder@physx@@@shdfnd@physx@@@UserAllocated@shdfnd@physx@@SAPEAX_KV?$ReflectionAllocator@VTriangleMeshBuilder@physx@@@12@PEBDH@Z 000000018001fe10 f i Cooking.obj
 0001:0001ee20       ??$PX_UNUSED@VPxFoundation@physx@@@@YAXAEBVPxFoundation@physx@@@Z 000000018001fe20 f i Cooking.obj
 0001:0001ee30       ??0?$PxFlags@W4Enum@PxConvexFlag@physx@@G@physx@@QEAA@W4Enum@PxConvexFlag@1@@Z 000000018001fe30 f i Cooking.obj
 0001:0001ee40       ??0?$PxFlags@W4Enum@PxConvexFlag@physx@@G@physx@@QEAA@XZ 000000018001fe40 f i Cooking.obj
 0001:0001ee50       ??0?$PxFlags@W4Enum@PxHeightFieldFlag@physx@@G@physx@@QEAA@AEBV01@@Z 000000018001fe50 f i Cooking.obj
 0001:0001ee60       ??0?$ReflectionAllocator@VCooking@physx@@@shdfnd@physx@@QEAA@PEBD@Z 000000018001fe60 f i Cooking.obj
 0001:0001ee70       ??0?$ReflectionAllocator@VHeightField@Gu@physx@@@shdfnd@physx@@QEAA@PEBD@Z 000000018001fe70 f i Cooking.obj
 0001:0001ee80       ??0?$ReflectionAllocator@VTriangleMeshBuilder@physx@@@shdfnd@physx@@QEAA@PEBD@Z 000000018001fe80 f i Cooking.obj
 0001:0001ee90       ??0Cooking@physx@@QEAA@AEBUPxCookingParams@1@@Z 000000018001fe90 f i Cooking.obj
 0001:0001eef0       ??0HullDesc@physx@@QEAA@XZ 000000018001fef0 f i Cooking.obj
 0001:0001ef20       ??0HullResult@physx@@QEAA@XZ 000000018001ff20 f i Cooking.obj
 0001:0001ef40       ??0PxConvexMeshDesc@physx@@QEAA@AEBV01@@Z 000000018001ff40 f i Cooking.obj
 0001:0001efa0       ??0PxCooking@physx@@QEAA@XZ 000000018001ffa0 f i Cooking.obj
 0001:0001efb0       ??0PxCookingParams@physx@@QEAA@AEBU01@@Z 000000018001ffb0 f i Cooking.obj
 0001:0001f000       ??0TriangleMeshBuilder@physx@@QEAA@XZ 0000000180020000 f i Cooking.obj
 0001:0001f030       ??1Cooking@physx@@UEAA@XZ  0000000180020030 f i Cooking.obj
 0001:0001f040       ??1PxCooking@physx@@MEAA@XZ 0000000180020040 f i Cooking.obj
 0001:0001f050       ??1TriangleMeshBuilder@physx@@UEAA@XZ 0000000180020050 f i Cooking.obj
 0001:0001f060       ??4?$PxFlags@W4Enum@PxMeshPreprocessingFlag@physx@@I@physx@@QEAAAEAV01@AEBV01@@Z 0000000180020060 f i Cooking.obj
 0001:0001f070       ??4PxCookingParams@physx@@QEAAAEAU01@AEBU01@@Z 0000000180020070 f i Cooking.obj
 0001:0001f0c0       ??9?$PxFlags@W4Enum@PxHeightFieldFlag@physx@@G@physx@@QEBA_NAEBV01@@Z 00000001800200c0 f i Cooking.obj
 0001:0001f0d0       ??I?$PxFlags@W4Enum@PxHeightFieldFlag@physx@@G@physx@@QEBA?AV01@W4Enum@PxHeightFieldFlag@1@@Z 00000001800200d0 f i Cooking.obj
 0001:0001f0e0       ??S?$PxFlags@W4Enum@PxConvexFlag@physx@@G@physx@@QEBA?AV01@XZ 00000001800200e0 f i Cooking.obj
 0001:0001f0f0       ??Sphysx@@YA?AV?$PxFlags@W4Enum@PxConvexFlag@physx@@G@0@W4Enum@PxConvexFlag@0@@Z 00000001800200f0 f i Cooking.obj
 0001:0001f100       ??_4?$PxFlags@W4Enum@PxConvexFlag@physx@@G@physx@@QEAAAEAV01@AEBV01@@Z 0000000180020100 f i Cooking.obj
 0001:0001f10c       ??_ETriangleMeshBuilder@physx@@WBA@EAAPEAXI@Z 000000018002010c f i Cooking.obj
 0001:0001f120       ??_GCooking@physx@@UEAAPEAXI@Z 0000000180020120 f i Cooking.obj
 0001:0001f120       ??_ECooking@physx@@UEAAPEAXI@Z 0000000180020120 f i Cooking.obj
 0001:0001f150       ??_EPxCooking@physx@@MEAAPEAXI@Z 0000000180020150 f i Cooking.obj
 0001:0001f150       ??_GPxCooking@physx@@MEAAPEAXI@Z 0000000180020150 f i Cooking.obj
 0001:0001f180       ??_GTriangleMeshBuilder@physx@@UEAAPEAXI@Z 0000000180020180 f i Cooking.obj
 0001:0001f180       ??_ETriangleMeshBuilder@physx@@UEAAPEAXI@Z 0000000180020180 f i Cooking.obj
 0001:0001f1c0       ?allocate@?$ReflectionAllocator@VCooking@physx@@@shdfnd@physx@@QEAAPEAX_KPEBDH@Z 00000001800201c0 f i Cooking.obj
 0001:0001f260       ?allocate@?$ReflectionAllocator@VHeightField@Gu@physx@@@shdfnd@physx@@QEAAPEAX_KPEBDH@Z 0000000180020260 f i Cooking.obj
 0001:0001f300       ?allocate@?$ReflectionAllocator@VTriangleMeshBuilder@physx@@@shdfnd@physx@@QEAAPEAX_KPEBDH@Z 0000000180020300 f i Cooking.obj
 0001:0001f3a0       ?getName@?$ReflectionAllocator@VCooking@physx@@@shdfnd@physx@@CAPEBDXZ 00000001800203a0 f i Cooking.obj
 0001:0001f3e0       ?getName@?$ReflectionAllocator@VHeightField@Gu@physx@@@shdfnd@physx@@CAPEBDXZ 00000001800203e0 f i Cooking.obj
 0001:0001f420       ?getName@?$ReflectionAllocator@VTriangleMeshBuilder@physx@@@shdfnd@physx@@CAPEBDXZ 0000000180020420 f i Cooking.obj
 0001:0001f460       ?isValid@PxHeightFieldDesc@physx@@QEBA_NXZ 0000000180020460 f i Cooking.obj
 0001:0001f4b0       ?littleEndian@shdfnd@physx@@YADXZ 00000001800204b0 f i Cooking.obj
 0001:0001f4c0       ?requires@TriangleMesh@Gu@physx@@UEAAXAEAVPxProcessPxBaseCallback@3@@Z 00000001800204c0 f i Cooking.obj
 0001:0001f4d0       ??0ReducedVertexCloud@physx@@QEAA@PEBVPxVec3@1@I@Z 00000001800204d0 f   CookingUtils.obj
 0001:0001f4f0       ??1ReducedVertexCloud@physx@@QEAA@XZ 00000001800204f0 f   CookingUtils.obj
 0001:0001f540       ?Clean@ReducedVertexCloud@physx@@QEAAAEAV12@XZ 0000000180020540 f   CookingUtils.obj
 0001:0001f590       ?Reduce@ReducedVertexCloud@physx@@QEAA_NPEAUREDUCEDCLOUD@2@@Z 0000000180020590 f   CookingUtils.obj
 0001:0001f8e0       ??0EdgeList@Gu@physx@@QEAA@XZ 00000001800208e0 f   EdgeList.obj
 0001:0001f900       ??1EdgeList@Gu@physx@@QEAA@XZ 0000000180020900 f   EdgeList.obj
 0001:0001f970       ?Load@EdgeList@Gu@physx@@QEAA_NAEAVPxInputStream@3@@Z 0000000180020970 f   EdgeList.obj
 0001:0001faf0       ??0EdgeListBuilder@Gu@physx@@QEAA@XZ 0000000180020af0 f   EdgeList.obj
 0001:0001fb10       ??1EdgeListBuilder@Gu@physx@@QEAA@XZ 0000000180020b10 f   EdgeList.obj
 0001:0001fb20       ?Init@EdgeListBuilder@Gu@physx@@QEAA_NAEBUEDGELISTCREATE@23@@Z 0000000180020b20 f   EdgeList.obj
 0001:0001fc30       ?CreateFacesToEdges@EdgeListBuilder@Gu@physx@@AEAA_NIPEBIPEBG@Z 0000000180020c30 f   EdgeList.obj
 0001:00020110       ?CreateEdgesToFaces@EdgeListBuilder@Gu@physx@@AEAA_NIPEBIPEBG@Z 0000000180021110 f   EdgeList.obj
 0001:00020320       ?ComputeActiveEdges@EdgeListBuilder@Gu@physx@@AEAA_NIPEBIPEBGPEBVPxVec3@3@M@Z 0000000180021320 f   EdgeList.obj
 0001:000219e0       ??$?_UUEdgeData@Gu@physx@@@@YAPEAX_KV?$ReflectionAllocator@UEdgeData@Gu@physx@@@shdfnd@physx@@PEBDH@Z 00000001800229e0 f i EdgeList.obj
 0001:000219f0       ??$?_UUEdgeTriangleData@Gu@physx@@@@YAPEAX_KV?$ReflectionAllocator@UEdgeTriangleData@Gu@physx@@@shdfnd@physx@@PEBDH@Z 00000001800229f0 f i EdgeList.obj
 0001:00021a00       ??0?$ReflectionAllocator@UEdgeData@Gu@physx@@@shdfnd@physx@@QEAA@PEBD@Z 0000000180022a00 f i EdgeList.obj
 0001:00021a10       ??0?$ReflectionAllocator@UEdgeTriangleData@Gu@physx@@@shdfnd@physx@@QEAA@PEBD@Z 0000000180022a10 f i EdgeList.obj
 0001:00021a20       ??0PxTriangle@physx@@QEAA@AEBVPxVec3@1@00@Z 0000000180022a20 f i EdgeList.obj
 0001:00021a60       ??1PxTriangle@physx@@QEAA@XZ 0000000180022a60 f i EdgeList.obj
 0001:00021a70       ?GetEdgeToTriangles@EdgeList@Gu@physx@@QEBAPEBUEdgeDescData@23@XZ 0000000180022a70 f i EdgeList.obj
 0001:00021a80       ?GetEdges@EdgeList@Gu@physx@@QEBAPEBUEdgeData@23@XZ 0000000180022a80 f i EdgeList.obj
 0001:00021a90       ?GetFacesByEdges@EdgeList@Gu@physx@@QEBAPEBIXZ 0000000180022a90 f i EdgeList.obj
 0001:00021aa0       ?OppositeVertex@@YAIIIIII@Z 0000000180022aa0 f i EdgeList.obj
 0001:00021af0       ?PxAtan2@physx@@YAMMM@Z    0000000180022af0 f i EdgeList.obj
 0001:00021b00       ?allocate@?$ReflectionAllocator@UEdgeData@Gu@physx@@@shdfnd@physx@@QEAAPEAX_KPEBDH@Z 0000000180022b00 f i EdgeList.obj
 0001:00021ba0       ?allocate@?$ReflectionAllocator@UEdgeTriangleData@Gu@physx@@@shdfnd@physx@@QEAAPEAX_KPEBDH@Z 0000000180022ba0 f i EdgeList.obj
 0001:00021c40       ?angle@shdfnd@physx@@YAMAEBVPxVec3@2@0@Z 0000000180022c40 f i EdgeList.obj
 0001:00021cf0       ?getName@?$ReflectionAllocator@UEdgeData@Gu@physx@@@shdfnd@physx@@CAPEBDXZ 0000000180022cf0 f i EdgeList.obj
 0001:00021d30       ?getName@?$ReflectionAllocator@UEdgeTriangleData@Gu@physx@@@shdfnd@physx@@CAPEBDXZ 0000000180022d30 f i EdgeList.obj
 0001:00021d70       ?normal@PxTriangle@physx@@QEBAXAEAVPxVec3@2@@Z 0000000180022d70 f i EdgeList.obj
 0001:00021e80       ??0InternalTriangleMeshBuilder@physx@@QEAA@PEAVInternalTriangleMesh@1@AEBUPxCookingParams@1@@Z 0000000180022e80 f   InternalTriangleMeshBuilder.obj
 0001:00021ea0       ??1InternalTriangleMeshBuilder@physx@@QEAA@XZ 0000000180022ea0 f   InternalTriangleMeshBuilder.obj
 0001:00021f00       ?cleanMesh@InternalTriangleMeshBuilder@physx@@QEAA_N_N@Z 0000000180022f00 f   InternalTriangleMeshBuilder.obj
 0001:00022400       ?fillRemapTable@InternalTriangleMeshBuilder@physx@@QEAAXXZ 0000000180023400 f   InternalTriangleMeshBuilder.obj
 0001:00022500       ?remapTopology@InternalTriangleMeshBuilder@physx@@QEAAXPEBI@Z 0000000180023500 f   InternalTriangleMeshBuilder.obj
 0001:00022790       ?createRTree@InternalTriangleMeshBuilder@physx@@QEAA_NXZ 0000000180023790 f   InternalTriangleMeshBuilder.obj
 0001:00022880       ?createSharedEdgeData@InternalTriangleMeshBuilder@physx@@QEAAX_N0@Z 0000000180023880 f   InternalTriangleMeshBuilder.obj
 0001:00022c90       ?releaseEdgeList@InternalTriangleMeshBuilder@physx@@AEAAXXZ 0000000180023c90 f   InternalTriangleMeshBuilder.obj
 0001:00022cf0       ?createEdgeList@InternalTriangleMeshBuilder@physx@@AEAAXXZ 0000000180023cf0 f   InternalTriangleMeshBuilder.obj
 0001:00022e20       ??$?2V?$ReflectionAllocator@VEdgeListBuilder@Gu@physx@@@shdfnd@physx@@@UserAllocated@shdfnd@physx@@SAPEAX_KV?$ReflectionAllocator@VEdgeListBuilder@Gu@physx@@@12@PEBDH@Z 0000000180023e20 f i InternalTriangleMeshBuilder.obj
 0001:00022e30       ??0?$Array@IV?$ReflectionAllocator@I@shdfnd@physx@@@shdfnd@physx@@QEAA@AEBV?$ReflectionAllocator@I@12@@Z 0000000180023e30 f i InternalTriangleMeshBuilder.obj
 0001:00022e40       ??0?$ReflectionAllocator@VEdgeListBuilder@Gu@physx@@@shdfnd@physx@@QEAA@PEBD@Z 0000000180023e40 f i InternalTriangleMeshBuilder.obj
 0001:00022e50       ??0RTreeCookerRemap@@QEAA@I@Z 0000000180023e50 f i InternalTriangleMeshBuilder.obj
 0001:00022e70       ??0RemapCallback@RTreeCooker@physx@@QEAA@XZ 0000000180023e70 f i InternalTriangleMeshBuilder.obj
 0001:00022e80       ??1RTreeCookerRemap@@UEAA@XZ 0000000180023e80 f i InternalTriangleMeshBuilder.obj
 0001:00022e90       ??1RemapCallback@RTreeCooker@physx@@UEAA@XZ 0000000180023e90 f i InternalTriangleMeshBuilder.obj
 0001:00022ea0       ??_GEdgeListBuilder@Gu@physx@@QEAAPEAXI@Z 0000000180023ea0 f i InternalTriangleMeshBuilder.obj
 0001:00022ee0       ??_ERTreeCookerRemap@@UEAAPEAXI@Z 0000000180023ee0 f i InternalTriangleMeshBuilder.obj
 0001:00022ee0       ??_GRTreeCookerRemap@@UEAAPEAXI@Z 0000000180023ee0 f i InternalTriangleMeshBuilder.obj
 0001:00022f10       ??_ERemapCallback@RTreeCooker@physx@@UEAAPEAXI@Z 0000000180023f10 f i InternalTriangleMeshBuilder.obj
 0001:00022f10       ??_GRemapCallback@RTreeCooker@physx@@UEAAPEAXI@Z 0000000180023f10 f i InternalTriangleMeshBuilder.obj
 0001:00022f40       ?GetNbFaces@EdgeList@Gu@physx@@QEBAIXZ 0000000180023f40 f i InternalTriangleMeshBuilder.obj
 0001:00022f50       ?LeafSetData@Gu@physx@@YAIII@Z 0000000180023f50 f i InternalTriangleMeshBuilder.obj
 0001:00022f70       ?SetData@LeafTriangles@Gu@physx@@QEAAXII@Z 0000000180023f70 f i InternalTriangleMeshBuilder.obj
 0001:00022f90       ?allocate@?$ReflectionAllocator@VEdgeListBuilder@Gu@physx@@@shdfnd@physx@@QEAAPEAX_KPEBDH@Z 0000000180023f90 f i InternalTriangleMeshBuilder.obj
 0001:00023030       ?findEdgeCCW@?$TriangleT@I@Gu@physx@@QEBAEII@Z 0000000180024030 f i InternalTriangleMeshBuilder.obj
 0001:00023080       ?getName@?$ReflectionAllocator@VEdgeListBuilder@Gu@physx@@@shdfnd@physx@@CAPEBDXZ 0000000180024080 f i InternalTriangleMeshBuilder.obj
 0001:000230c0       ?remap@RTreeCookerRemap@@UEAAXPEAIII@Z 00000001800240c0 f i InternalTriangleMeshBuilder.obj
 0001:000230e0       ??0MeshCleaner@physx@@QEAA@IPEBVPxVec3@1@IPEBIM@Z 00000001800240e0 f   MeshCleaner.obj
 0001:000239c0       ??1MeshCleaner@physx@@QEAA@XZ 00000001800249c0 f   MeshCleaner.obj
 0001:00023ae0       ??9Indices@@QEBA_NAEBU0@@Z 0000000180024ae0 f i MeshCleaner.obj
 0001:00023b00       ??9PxVec3@physx@@QEBA_NAEBV01@@Z 0000000180024b00 f i MeshCleaner.obj
 0001:00023b30       ?PxFloor@physx@@YAMM@Z     0000000180024b30 f i MeshCleaner.obj
 0001:00023b60       ?nextPowerOfTwo@shdfnd@physx@@YAII@Z 0000000180024b60 f i MeshCleaner.obj
 0001:00023b86       GetModuleFileNameA         0000000180024b86 f   kernel32:KERNEL32.dll
 0001:00023b8c       LoadLibraryA               0000000180024b8c f   kernel32:KERNEL32.dll
 0001:00023b92       __imp_load_?writeWord@physx@@YAXG_NAEAVPxOutputStream@1@@Z 0000000180024b92 f   PhysX3CommonPROFILE_x64:PhysX3CommonPROFILE_x64.dll
 0001:00023b9e       __tailMerge_PhysX3CommonPROFILE_x64_dll 0000000180024b9e f i PhysX3CommonPROFILE_x64:PhysX3CommonPROFILE_x64.dll
 0001:00023c17       ?writeWord@physx@@YAXG_NAEAVPxOutputStream@1@@Z 0000000180024c17 f   PhysX3CommonPROFILE_x64:PhysX3CommonPROFILE_x64.dll
 0001:00023c1d       __imp_load_?writeDword@physx@@YAXI_NAEAVPxOutputStream@1@@Z 0000000180024c1d f   PhysX3CommonPROFILE_x64:PhysX3CommonPROFILE_x64.dll
 0001:00023c29       ?writeDword@physx@@YAXI_NAEAVPxOutputStream@1@@Z 0000000180024c29 f   PhysX3CommonPROFILE_x64:PhysX3CommonPROFILE_x64.dll
 0001:00023c2f       __imp_load_?writeFloat@physx@@YAXM_NAEAVPxOutputStream@1@@Z 0000000180024c2f f   PhysX3CommonPROFILE_x64:PhysX3CommonPROFILE_x64.dll
 0001:00023c3b       ?writeFloat@physx@@YAXM_NAEAVPxOutputStream@1@@Z 0000000180024c3b f   PhysX3CommonPROFILE_x64:PhysX3CommonPROFILE_x64.dll
 0001:00023c41       __imp_load_?writeHeader@physx@@YA_NCCCCI_NAEAVPxOutputStream@1@@Z 0000000180024c41 f   PhysX3CommonPROFILE_x64:PhysX3CommonPROFILE_x64.dll
 0001:00023c4d       ?writeHeader@physx@@YA_NCCCCI_NAEAVPxOutputStream@1@@Z 0000000180024c4d f   PhysX3CommonPROFILE_x64:PhysX3CommonPROFILE_x64.dll
 0001:00023c53       __imp_load_PxGetFoundation 0000000180024c53 f   PhysX3CommonPROFILE_x64:PhysX3CommonPROFILE_x64.dll
 0001:00023c5f       PxGetFoundation            0000000180024c5f f   PhysX3CommonPROFILE_x64:PhysX3CommonPROFILE_x64.dll
 0001:00023c65       __imp_load_?getAllocator@shdfnd@physx@@YAAEAVPxAllocatorCallback@2@XZ 0000000180024c65 f   PhysX3CommonPROFILE_x64:PhysX3CommonPROFILE_x64.dll
 0001:00023c71       ?getAllocator@shdfnd@physx@@YAAEAVPxAllocatorCallback@2@XZ 0000000180024c71 f   PhysX3CommonPROFILE_x64:PhysX3CommonPROFILE_x64.dll
 0001:00023c77       __imp_load_?allocate@Allocator@shdfnd@physx@@QEAAPEAX_KPEBDH@Z 0000000180024c77 f   PhysX3CommonPROFILE_x64:PhysX3CommonPROFILE_x64.dll
 0001:00023c83       ?allocate@Allocator@shdfnd@physx@@QEAAPEAX_KPEBDH@Z 0000000180024c83 f   PhysX3CommonPROFILE_x64:PhysX3CommonPROFILE_x64.dll
 0001:00023c89       __imp_load_?allocate@TempAllocator@shdfnd@physx@@QEAAPEAX_KPEBDH@Z 0000000180024c89 f   PhysX3CommonPROFILE_x64:PhysX3CommonPROFILE_x64.dll
 0001:00023c95       ?allocate@TempAllocator@shdfnd@physx@@QEAAPEAX_KPEBDH@Z 0000000180024c95 f   PhysX3CommonPROFILE_x64:PhysX3CommonPROFILE_x64.dll
 0001:00023c9b       __imp_load_?deallocate@TempAllocator@shdfnd@physx@@QEAAXPEAX@Z 0000000180024c9b f   PhysX3CommonPROFILE_x64:PhysX3CommonPROFILE_x64.dll
 0001:00023ca7       ?deallocate@TempAllocator@shdfnd@physx@@QEAAXPEAX@Z 0000000180024ca7 f   PhysX3CommonPROFILE_x64:PhysX3CommonPROFILE_x64.dll
 0001:00023cad       __imp_load_?computeBoundsAroundVertices@Gu@physx@@YAXAEAVPxBounds3@2@IPEIBVPxVec3@2@@Z 0000000180024cad f   PhysX3CommonPROFILE_x64:PhysX3CommonPROFILE_x64.dll
 0001:00023cb9       ?computeBoundsAroundVertices@Gu@physx@@YAXAEAVPxBounds3@2@IPEIBVPxVec3@2@@Z 0000000180024cb9 f   PhysX3CommonPROFILE_x64:PhysX3CommonPROFILE_x64.dll
 0001:00023cbf       __imp_load_?deallocate@Allocator@shdfnd@physx@@QEAAXPEAX@Z 0000000180024cbf f   PhysX3CommonPROFILE_x64:PhysX3CommonPROFILE_x64.dll
 0001:00023ccb       ?deallocate@Allocator@shdfnd@physx@@QEAAXPEAX@Z 0000000180024ccb f   PhysX3CommonPROFILE_x64:PhysX3CommonPROFILE_x64.dll
 0001:00023cd1       __imp_load_?getInstance@Foundation@shdfnd@physx@@SAAEAV123@XZ 0000000180024cd1 f   PhysX3CommonPROFILE_x64:PhysX3CommonPROFILE_x64.dll
 0001:00023cdd       ?getInstance@Foundation@shdfnd@physx@@SAAEAV123@XZ 0000000180024cdd f   PhysX3CommonPROFILE_x64:PhysX3CommonPROFILE_x64.dll
 0001:00023ce3       __imp_load_?error@Foundation@shdfnd@physx@@QEAAXW4Enum@PxErrorCode@3@PEBDH1ZZ 0000000180024ce3 f   PhysX3CommonPROFILE_x64:PhysX3CommonPROFILE_x64.dll
 0001:00023cef       ?error@Foundation@shdfnd@physx@@QEAAXW4Enum@PxErrorCode@3@PEBDH1ZZ 0000000180024cef f   PhysX3CommonPROFILE_x64:PhysX3CommonPROFILE_x64.dll
 0001:00023cf5       __imp_load_?save@RTree@Gu@physx@@QEBA_NAEAVPxOutputStream@3@@Z 0000000180024cf5 f   PhysX3CommonPROFILE_x64:PhysX3CommonPROFILE_x64.dll
 0001:00023d01       ?save@RTree@Gu@physx@@QEBA_NAEAVPxOutputStream@3@@Z 0000000180024d01 f   PhysX3CommonPROFILE_x64:PhysX3CommonPROFILE_x64.dll
 0001:00023d07       __imp_load_?release@InternalTriangleMesh@physx@@QEAAXXZ 0000000180024d07 f   PhysX3CommonPROFILE_x64:PhysX3CommonPROFILE_x64.dll
 0001:00023d13       ?release@InternalTriangleMesh@physx@@QEAAXXZ 0000000180024d13 f   PhysX3CommonPROFILE_x64:PhysX3CommonPROFILE_x64.dll
 0001:00023d19       __imp_load_?allocateVertices@InternalTriangleMesh@physx@@QEAAPEAVPxVec3@2@I@Z 0000000180024d19 f   PhysX3CommonPROFILE_x64:PhysX3CommonPROFILE_x64.dll
 0001:00023d25       ?allocateVertices@InternalTriangleMesh@physx@@QEAAPEAVPxVec3@2@I@Z 0000000180024d25 f   PhysX3CommonPROFILE_x64:PhysX3CommonPROFILE_x64.dll
 0001:00023d2b       __imp_load_?allocateTriangles@InternalTriangleMesh@physx@@QEAAPEAXI_N@Z 0000000180024d2b f   PhysX3CommonPROFILE_x64:PhysX3CommonPROFILE_x64.dll
 0001:00023d37       ?allocateTriangles@InternalTriangleMesh@physx@@QEAAPEAXI_N@Z 0000000180024d37 f   PhysX3CommonPROFILE_x64:PhysX3CommonPROFILE_x64.dll
 0001:00023d3d       __imp_load_?allocateMaterials@InternalTriangleMesh@physx@@QEAAPEAGXZ 0000000180024d3d f   PhysX3CommonPROFILE_x64:PhysX3CommonPROFILE_x64.dll
 0001:00023d49       ?allocateMaterials@InternalTriangleMesh@physx@@QEAAPEAGXZ 0000000180024d49 f   PhysX3CommonPROFILE_x64:PhysX3CommonPROFILE_x64.dll
 0001:00023d4f       __imp_load_?writeWordBuffer@physx@@YAXPEBGI_NAEAVPxOutputStream@1@@Z 0000000180024d4f f   PhysX3CommonPROFILE_x64:PhysX3CommonPROFILE_x64.dll
 0001:00023d5b       ?writeWordBuffer@physx@@YAXPEBGI_NAEAVPxOutputStream@1@@Z 0000000180024d5b f   PhysX3CommonPROFILE_x64:PhysX3CommonPROFILE_x64.dll
 0001:00023d61       __imp_load_?writeFloatBuffer@physx@@YAXPEBMI_NAEAVPxOutputStream@1@@Z 0000000180024d61 f   PhysX3CommonPROFILE_x64:PhysX3CommonPROFILE_x64.dll
 0001:00023d6d       ?writeFloatBuffer@physx@@YAXPEBMI_NAEAVPxOutputStream@1@@Z 0000000180024d6d f   PhysX3CommonPROFILE_x64:PhysX3CommonPROFILE_x64.dll
 0001:00023d73       __imp_load_?computeMaxIndex@physx@@YAIPEBII@Z 0000000180024d73 f   PhysX3CommonPROFILE_x64:PhysX3CommonPROFILE_x64.dll
 0001:00023d7f       ?computeMaxIndex@physx@@YAIPEBII@Z 0000000180024d7f f   PhysX3CommonPROFILE_x64:PhysX3CommonPROFILE_x64.dll
 0001:00023d85       __imp_load_?storeIndices@physx@@YAXIIPEBIAEAVPxOutputStream@1@_N@Z 0000000180024d85 f   PhysX3CommonPROFILE_x64:PhysX3CommonPROFILE_x64.dll
 0001:00023d91       ?storeIndices@physx@@YAXIIPEBIAEAVPxOutputStream@1@_N@Z 0000000180024d91 f   PhysX3CommonPROFILE_x64:PhysX3CommonPROFILE_x64.dll
 0001:00023d97       __imp_load_?computeMaxIndex@physx@@YAGPEBGI@Z 0000000180024d97 f   PhysX3CommonPROFILE_x64:PhysX3CommonPROFILE_x64.dll
 0001:00023da3       ?computeMaxIndex@physx@@YAGPEBGI@Z 0000000180024da3 f   PhysX3CommonPROFILE_x64:PhysX3CommonPROFILE_x64.dll
 0001:00023da9       __imp_load_?WriteHeader@Gu@physx@@YA_NEEEEI_NAEAVPxOutputStream@2@@Z 0000000180024da9 f   PhysX3CommonPROFILE_x64:PhysX3CommonPROFILE_x64.dll
 0001:00023db5       ?WriteHeader@Gu@physx@@YA_NEEEEI_NAEAVPxOutputStream@2@@Z 0000000180024db5 f   PhysX3CommonPROFILE_x64:PhysX3CommonPROFILE_x64.dll
 0001:00023dbb       __imp_load_?StoreIndices@Gu@physx@@YAXGIPEBGAEAVPxOutputStream@2@_N@Z 0000000180024dbb f   PhysX3CommonPROFILE_x64:PhysX3CommonPROFILE_x64.dll
 0001:00023dc7       ?StoreIndices@Gu@physx@@YAXGIPEBGAEAVPxOutputStream@2@_N@Z 0000000180024dc7 f   PhysX3CommonPROFILE_x64:PhysX3CommonPROFILE_x64.dll
 0001:00023dcd       __imp_load_?CreateOffsets@BigConvexData@physx@@IEAAXXZ 0000000180024dcd f   PhysX3CommonPROFILE_x64:PhysX3CommonPROFILE_x64.dll
 0001:00023dd9       ?CreateOffsets@BigConvexData@physx@@IEAAXXZ 0000000180024dd9 f   PhysX3CommonPROFILE_x64:PhysX3CommonPROFILE_x64.dll
 0001:00023ddf       __imp_load_??0RadixSortBuffered@Gu@physx@@QEAA@XZ 0000000180024ddf f   PhysX3CommonPROFILE_x64:PhysX3CommonPROFILE_x64.dll
 0001:00023deb       ??0RadixSortBuffered@Gu@physx@@QEAA@XZ 0000000180024deb f   PhysX3CommonPROFILE_x64:PhysX3CommonPROFILE_x64.dll
 0001:00023df1       __imp_load_??1RadixSortBuffered@Gu@physx@@UEAA@XZ 0000000180024df1 f   PhysX3CommonPROFILE_x64:PhysX3CommonPROFILE_x64.dll
 0001:00023dfd       ??1RadixSortBuffered@Gu@physx@@UEAA@XZ 0000000180024dfd f   PhysX3CommonPROFILE_x64:PhysX3CommonPROFILE_x64.dll
 0001:00023e03       __imp_load_?Sort@RadixSortBuffered@Gu@physx@@QEAAAEAV123@PEBIIW4RadixHint@23@@Z 0000000180024e03 f   PhysX3CommonPROFILE_x64:PhysX3CommonPROFILE_x64.dll
 0001:00023e0f       ?Sort@RadixSortBuffered@Gu@physx@@QEAAAEAV123@PEBIIW4RadixHint@23@@Z 0000000180024e0f f   PhysX3CommonPROFILE_x64:PhysX3CommonPROFILE_x64.dll
 0001:00023e15       __imp_load_??0Container@Gu@physx@@QEAA@XZ 0000000180024e15 f   PhysX3CommonPROFILE_x64:PhysX3CommonPROFILE_x64.dll
 0001:00023e21       ??0Container@Gu@physx@@QEAA@XZ 0000000180024e21 f   PhysX3CommonPROFILE_x64:PhysX3CommonPROFILE_x64.dll
 0001:00023e27       __imp_load_??0Container@Gu@physx@@QEAA@AEBV012@@Z 0000000180024e27 f   PhysX3CommonPROFILE_x64:PhysX3CommonPROFILE_x64.dll
 0001:00023e33       ??0Container@Gu@physx@@QEAA@AEBV012@@Z 0000000180024e33 f   PhysX3CommonPROFILE_x64:PhysX3CommonPROFILE_x64.dll
 0001:00023e39       __imp_load_??1Container@Gu@physx@@QEAA@XZ 0000000180024e39 f   PhysX3CommonPROFILE_x64:PhysX3CommonPROFILE_x64.dll
 0001:00023e45       ??1Container@Gu@physx@@QEAA@XZ 0000000180024e45 f   PhysX3CommonPROFILE_x64:PhysX3CommonPROFILE_x64.dll
 0001:00023e4b       __imp_load_?Empty@Container@Gu@physx@@QEAAAEAV123@XZ 0000000180024e4b f   PhysX3CommonPROFILE_x64:PhysX3CommonPROFILE_x64.dll
 0001:00023e57       ?Empty@Container@Gu@physx@@QEAAAEAV123@XZ 0000000180024e57 f   PhysX3CommonPROFILE_x64:PhysX3CommonPROFILE_x64.dll
 0001:00023e5d       __imp_load_?Contains@Container@Gu@physx@@QEBA_NIPEAI@Z 0000000180024e5d f   PhysX3CommonPROFILE_x64:PhysX3CommonPROFILE_x64.dll
 0001:00023e69       ?Contains@Container@Gu@physx@@QEBA_NIPEAI@Z 0000000180024e69 f   PhysX3CommonPROFILE_x64:PhysX3CommonPROFILE_x64.dll
 0001:00023e6f       __imp_load_??4Container@Gu@physx@@QEAAXAEBV012@@Z 0000000180024e6f f   PhysX3CommonPROFILE_x64:PhysX3CommonPROFILE_x64.dll
 0001:00023e7b       ??4Container@Gu@physx@@QEAAXAEBV012@@Z 0000000180024e7b f   PhysX3CommonPROFILE_x64:PhysX3CommonPROFILE_x64.dll
 0001:00023e81       __imp_load_?Resize@Container@Gu@physx@@AEAA_NI@Z 0000000180024e81 f   PhysX3CommonPROFILE_x64:PhysX3CommonPROFILE_x64.dll
 0001:00023e8d       ?Resize@Container@Gu@physx@@AEAA_NI@Z 0000000180024e8d f   PhysX3CommonPROFILE_x64:PhysX3CommonPROFILE_x64.dll
 0001:00023e93       __imp_load_??0ConvexMesh@Gu@physx@@QEAA@XZ 0000000180024e93 f   PhysX3CommonPROFILE_x64:PhysX3CommonPROFILE_x64.dll
 0001:00023e9f       ??0ConvexMesh@Gu@physx@@QEAA@XZ 0000000180024e9f f   PhysX3CommonPROFILE_x64:PhysX3CommonPROFILE_x64.dll
 0001:00023ea5       __imp_load_??1ConvexMesh@Gu@physx@@UEAA@XZ 0000000180024ea5 f   PhysX3CommonPROFILE_x64:PhysX3CommonPROFILE_x64.dll
 0001:00023eb1       ??1ConvexMesh@Gu@physx@@UEAA@XZ 0000000180024eb1 f   PhysX3CommonPROFILE_x64:PhysX3CommonPROFILE_x64.dll
 0001:00023eb7       __imp_load_??0BigConvexData@physx@@QEAA@XZ 0000000180024eb7 f   PhysX3CommonPROFILE_x64:PhysX3CommonPROFILE_x64.dll
 0001:00023ec3       ??0BigConvexData@physx@@QEAA@XZ 0000000180024ec3 f   PhysX3CommonPROFILE_x64:PhysX3CommonPROFILE_x64.dll
 0001:00023ec9       __imp_load_??1BigConvexData@physx@@QEAA@XZ 0000000180024ec9 f   PhysX3CommonPROFILE_x64:PhysX3CommonPROFILE_x64.dll
 0001:00023ed5       ??1BigConvexData@physx@@QEAA@XZ 0000000180024ed5 f   PhysX3CommonPROFILE_x64:PhysX3CommonPROFILE_x64.dll
 0001:00023edb       __imp_load_?exportExtraData@ConvexMesh@Gu@physx@@UEAAXAEAVPxSerializationContext@3@@Z 0000000180024edb f   PhysX3CommonPROFILE_x64:PhysX3CommonPROFILE_x64.dll
 0001:00023ee7       ?exportExtraData@ConvexMesh@Gu@physx@@UEAAXAEAVPxSerializationContext@3@@Z 0000000180024ee7 f   PhysX3CommonPROFILE_x64:PhysX3CommonPROFILE_x64.dll
 0001:00023eed       __imp_load_?getConcreteTypeName@PxConvexMesh@physx@@UEBAPEBDXZ 0000000180024eed f   PhysX3CommonPROFILE_x64:PhysX3CommonPROFILE_x64.dll
 0001:00023ef9       ?getConcreteTypeName@PxConvexMesh@physx@@UEBAPEBDXZ 0000000180024ef9 f   PhysX3CommonPROFILE_x64:PhysX3CommonPROFILE_x64.dll
 0001:00023eff       __imp_load_?getIndexBuffer@ConvexMesh@Gu@physx@@UEBAPEBEXZ 0000000180024eff f   PhysX3CommonPROFILE_x64:PhysX3CommonPROFILE_x64.dll
 0001:00023f0b       ?getIndexBuffer@ConvexMesh@Gu@physx@@UEBAPEBEXZ 0000000180024f0b f   PhysX3CommonPROFILE_x64:PhysX3CommonPROFILE_x64.dll
 0001:00023f11       __imp_load_?getLocalBounds@ConvexMesh@Gu@physx@@UEBA?AVPxBounds3@3@XZ 0000000180024f11 f   PhysX3CommonPROFILE_x64:PhysX3CommonPROFILE_x64.dll
 0001:00023f1d       ?getLocalBounds@ConvexMesh@Gu@physx@@UEBA?AVPxBounds3@3@XZ 0000000180024f1d f   PhysX3CommonPROFILE_x64:PhysX3CommonPROFILE_x64.dll
 0001:00023f23       __imp_load_?getMassInformation@ConvexMesh@Gu@physx@@UEBAXAEAMAEAVPxMat33@3@AEAVPxVec3@3@@Z 0000000180024f23 f   PhysX3CommonPROFILE_x64:PhysX3CommonPROFILE_x64.dll
 0001:00023f2f       ?getMassInformation@ConvexMesh@Gu@physx@@UEBAXAEAMAEAVPxMat33@3@AEAVPxVec3@3@@Z 0000000180024f2f f   PhysX3CommonPROFILE_x64:PhysX3CommonPROFILE_x64.dll
 0001:00023f35       __imp_load_?getNbPolygons@ConvexMesh@Gu@physx@@UEBAIXZ 0000000180024f35 f   PhysX3CommonPROFILE_x64:PhysX3CommonPROFILE_x64.dll
 0001:00023f41       ?getNbPolygons@ConvexMesh@Gu@physx@@UEBAIXZ 0000000180024f41 f   PhysX3CommonPROFILE_x64:PhysX3CommonPROFILE_x64.dll
 0001:00023f47       __imp_load_?getNbVertices@ConvexMesh@Gu@physx@@UEBAIXZ 0000000180024f47 f   PhysX3CommonPROFILE_x64:PhysX3CommonPROFILE_x64.dll
 0001:00023f53       ?getNbVertices@ConvexMesh@Gu@physx@@UEBAIXZ 0000000180024f53 f   PhysX3CommonPROFILE_x64:PhysX3CommonPROFILE_x64.dll
 0001:00023f59       __imp_load_?getPolygonData@ConvexMesh@Gu@physx@@UEBA_NIAEAUPxHullPolygon@3@@Z 0000000180024f59 f   PhysX3CommonPROFILE_x64:PhysX3CommonPROFILE_x64.dll
 0001:00023f65       ?getPolygonData@ConvexMesh@Gu@physx@@UEBA_NIAEAUPxHullPolygon@3@@Z 0000000180024f65 f   PhysX3CommonPROFILE_x64:PhysX3CommonPROFILE_x64.dll
 0001:00023f6b       __imp_load_?getReferenceCount@ConvexMesh@Gu@physx@@UEBAIXZ 0000000180024f6b f   PhysX3CommonPROFILE_x64:PhysX3CommonPROFILE_x64.dll
 0001:00023f77       ?getReferenceCount@ConvexMesh@Gu@physx@@UEBAIXZ 0000000180024f77 f   PhysX3CommonPROFILE_x64:PhysX3CommonPROFILE_x64.dll
 0001:00023f7d       __imp_load_?getVertices@ConvexMesh@Gu@physx@@UEBAPEBVPxVec3@3@XZ 0000000180024f7d f   PhysX3CommonPROFILE_x64:PhysX3CommonPROFILE_x64.dll
 0001:00023f89       ?getVertices@ConvexMesh@Gu@physx@@UEBAPEBVPxVec3@3@XZ 0000000180024f89 f   PhysX3CommonPROFILE_x64:PhysX3CommonPROFILE_x64.dll
 0001:00023f8f       __imp_load_?isKindOf@PxConvexMesh@physx@@MEBA_NPEBD@Z 0000000180024f8f f   PhysX3CommonPROFILE_x64:PhysX3CommonPROFILE_x64.dll
 0001:00023f9b       ?isKindOf@PxConvexMesh@physx@@MEBA_NPEBD@Z 0000000180024f9b f   PhysX3CommonPROFILE_x64:PhysX3CommonPROFILE_x64.dll
 0001:00023fa1       __imp_load_?onRefCountZero@ConvexMesh@Gu@physx@@UEAAXXZ 0000000180024fa1 f   PhysX3CommonPROFILE_x64:PhysX3CommonPROFILE_x64.dll
 0001:00023fad       ?onRefCountZero@ConvexMesh@Gu@physx@@UEAAXXZ 0000000180024fad f   PhysX3CommonPROFILE_x64:PhysX3CommonPROFILE_x64.dll
 0001:00023fb3       __imp_load_?release@ConvexMesh@Gu@physx@@UEAAXXZ 0000000180024fb3 f   PhysX3CommonPROFILE_x64:PhysX3CommonPROFILE_x64.dll
 0001:00023fbf       ?release@ConvexMesh@Gu@physx@@UEAAXXZ 0000000180024fbf f   PhysX3CommonPROFILE_x64:PhysX3CommonPROFILE_x64.dll
 0001:00023fc5       __imp_load_?readDword@physx@@YAI_NAEAVPxInputStream@1@@Z 0000000180024fc5 f   PhysX3CommonPROFILE_x64:PhysX3CommonPROFILE_x64.dll
 0001:00023fd1       ?readDword@physx@@YAI_NAEAVPxInputStream@1@@Z 0000000180024fd1 f   PhysX3CommonPROFILE_x64:PhysX3CommonPROFILE_x64.dll
 0001:00023fd7       __imp_load_?ReadHeader@Gu@physx@@YA_NEEEEAEAIAEA_NAEAVPxInputStream@2@@Z 0000000180024fd7 f   PhysX3CommonPROFILE_x64:PhysX3CommonPROFILE_x64.dll
 0001:00023fe3       ?ReadHeader@Gu@physx@@YA_NEEEEAEAIAEA_NAEAVPxInputStream@2@@Z 0000000180024fe3 f   PhysX3CommonPROFILE_x64:PhysX3CommonPROFILE_x64.dll
 0001:00023fe9       __imp_load_??0FPUGuard@shdfnd@physx@@QEAA@XZ 0000000180024fe9 f   PhysX3CommonPROFILE_x64:PhysX3CommonPROFILE_x64.dll
 0001:00023ff5       ??0FPUGuard@shdfnd@physx@@QEAA@XZ 0000000180024ff5 f   PhysX3CommonPROFILE_x64:PhysX3CommonPROFILE_x64.dll
 0001:00023ffb       __imp_load_??1FPUGuard@shdfnd@physx@@QEAA@XZ 0000000180024ffb f   PhysX3CommonPROFILE_x64:PhysX3CommonPROFILE_x64.dll
 0001:00024007       ??1FPUGuard@shdfnd@physx@@QEAA@XZ 0000000180025007 f   PhysX3CommonPROFILE_x64:PhysX3CommonPROFILE_x64.dll
 0001:0002400d       __imp_load_?incRefCount@Foundation@shdfnd@physx@@SAXXZ 000000018002500d f   PhysX3CommonPROFILE_x64:PhysX3CommonPROFILE_x64.dll
 0001:00024019       ?incRefCount@Foundation@shdfnd@physx@@SAXXZ 0000000180025019 f   PhysX3CommonPROFILE_x64:PhysX3CommonPROFILE_x64.dll
 0001:0002401f       __imp_load_?decRefCount@Foundation@shdfnd@physx@@SAXXZ 000000018002501f f   PhysX3CommonPROFILE_x64:PhysX3CommonPROFILE_x64.dll
 0001:0002402b       ?decRefCount@Foundation@shdfnd@physx@@SAXXZ 000000018002502b f   PhysX3CommonPROFILE_x64:PhysX3CommonPROFILE_x64.dll
 0001:00024031       __imp_load_??0TriangleMesh@Gu@physx@@QEAA@XZ 0000000180025031 f   PhysX3CommonPROFILE_x64:PhysX3CommonPROFILE_x64.dll
 0001:0002403d       ??0TriangleMesh@Gu@physx@@QEAA@XZ 000000018002503d f   PhysX3CommonPROFILE_x64:PhysX3CommonPROFILE_x64.dll
 0001:00024043       __imp_load_?checkMeshIndicesSize@TriangleMesh@Gu@physx@@QEAAXXZ 0000000180025043 f   PhysX3CommonPROFILE_x64:PhysX3CommonPROFILE_x64.dll
 0001:0002404f       ?checkMeshIndicesSize@TriangleMesh@Gu@physx@@QEAAXXZ 000000018002504f f   PhysX3CommonPROFILE_x64:PhysX3CommonPROFILE_x64.dll
 0001:00024055       __imp_load_??1TriangleMesh@Gu@physx@@UEAA@XZ 0000000180025055 f   PhysX3CommonPROFILE_x64:PhysX3CommonPROFILE_x64.dll
 0001:00024061       ??1TriangleMesh@Gu@physx@@UEAA@XZ 0000000180025061 f   PhysX3CommonPROFILE_x64:PhysX3CommonPROFILE_x64.dll
 0001:00024067       __imp_load_??0HeightField@Gu@physx@@QEAA@PEAVGuMeshFactory@2@@Z 0000000180025067 f   PhysX3CommonPROFILE_x64:PhysX3CommonPROFILE_x64.dll
 0001:00024073       ??0HeightField@Gu@physx@@QEAA@PEAVGuMeshFactory@2@@Z 0000000180025073 f   PhysX3CommonPROFILE_x64:PhysX3CommonPROFILE_x64.dll
 0001:00024079       __imp_load_?loadFromDesc@HeightField@Gu@physx@@QEAA_NAEBVPxHeightFieldDesc@3@_N@Z 0000000180025079 f   PhysX3CommonPROFILE_x64:PhysX3CommonPROFILE_x64.dll
 0001:00024085       ?loadFromDesc@HeightField@Gu@physx@@QEAA_NAEBVPxHeightFieldDesc@3@_N@Z 0000000180025085 f   PhysX3CommonPROFILE_x64:PhysX3CommonPROFILE_x64.dll
 0001:0002408b       __imp_load_?releaseMemory@HeightField@Gu@physx@@QEAAX_N@Z 000000018002508b f   PhysX3CommonPROFILE_x64:PhysX3CommonPROFILE_x64.dll
 0001:00024097       ?releaseMemory@HeightField@Gu@physx@@QEAAX_N@Z 0000000180025097 f   PhysX3CommonPROFILE_x64:PhysX3CommonPROFILE_x64.dll
 0001:0002409d       __imp_load_?exportExtraData@TriangleMesh@Gu@physx@@UEAAXAEAVPxSerializationContext@3@@Z 000000018002509d f   PhysX3CommonPROFILE_x64:PhysX3CommonPROFILE_x64.dll
 0001:000240a9       ?exportExtraData@TriangleMesh@Gu@physx@@UEAAXAEAVPxSerializationContext@3@@Z 00000001800250a9 f   PhysX3CommonPROFILE_x64:PhysX3CommonPROFILE_x64.dll
 0001:000240af       __imp_load_?getConcreteTypeName@PxTriangleMesh@physx@@UEBAPEBDXZ 00000001800250af f   PhysX3CommonPROFILE_x64:PhysX3CommonPROFILE_x64.dll
 0001:000240bb       ?getConcreteTypeName@PxTriangleMesh@physx@@UEBAPEBDXZ 00000001800250bb f   PhysX3CommonPROFILE_x64:PhysX3CommonPROFILE_x64.dll
 0001:000240c1       __imp_load_?getLocalBounds@TriangleMesh@Gu@physx@@UEBA?AVPxBounds3@3@XZ 00000001800250c1 f   PhysX3CommonPROFILE_x64:PhysX3CommonPROFILE_x64.dll
 0001:000240cd       ?getLocalBounds@TriangleMesh@Gu@physx@@UEBA?AVPxBounds3@3@XZ 00000001800250cd f   PhysX3CommonPROFILE_x64:PhysX3CommonPROFILE_x64.dll
 0001:000240d3       __imp_load_?getNbTriangles@TriangleMesh@Gu@physx@@UEBAIXZ 00000001800250d3 f   PhysX3CommonPROFILE_x64:PhysX3CommonPROFILE_x64.dll
 0001:000240df       ?getNbTriangles@TriangleMesh@Gu@physx@@UEBAIXZ 00000001800250df f   PhysX3CommonPROFILE_x64:PhysX3CommonPROFILE_x64.dll
 0001:000240e5       __imp_load_?getNbVertices@TriangleMesh@Gu@physx@@UEBAIXZ 00000001800250e5 f   PhysX3CommonPROFILE_x64:PhysX3CommonPROFILE_x64.dll
 0001:000240f1       ?getNbVertices@TriangleMesh@Gu@physx@@UEBAIXZ 00000001800250f1 f   PhysX3CommonPROFILE_x64:PhysX3CommonPROFILE_x64.dll
 0001:000240f7       __imp_load_?getReferenceCount@TriangleMesh@Gu@physx@@UEBAIXZ 00000001800250f7 f   PhysX3CommonPROFILE_x64:PhysX3CommonPROFILE_x64.dll
 0001:00024103       ?getReferenceCount@TriangleMesh@Gu@physx@@UEBAIXZ 0000000180025103 f   PhysX3CommonPROFILE_x64:PhysX3CommonPROFILE_x64.dll
 0001:00024109       __imp_load_?getTriangleMaterialIndex@TriangleMesh@Gu@physx@@UEBAGI@Z 0000000180025109 f   PhysX3CommonPROFILE_x64:PhysX3CommonPROFILE_x64.dll
 0001:00024115       ?getTriangleMaterialIndex@TriangleMesh@Gu@physx@@UEBAGI@Z 0000000180025115 f   PhysX3CommonPROFILE_x64:PhysX3CommonPROFILE_x64.dll
 0001:0002411b       __imp_load_?getTriangleMeshFlags@TriangleMesh@Gu@physx@@UEBA?AV?$PxFlags@W4Enum@PxTriangleMeshFlag@physx@@E@3@XZ 000000018002511b f   PhysX3CommonPROFILE_x64:PhysX3CommonPROFILE_x64.dll
 0001:00024127       ?getTriangleMeshFlags@TriangleMesh@Gu@physx@@UEBA?AV?$PxFlags@W4Enum@PxTriangleMeshFlag@physx@@E@3@XZ 0000000180025127 f   PhysX3CommonPROFILE_x64:PhysX3CommonPROFILE_x64.dll
 0001:0002412d       __imp_load_?getTriangles@TriangleMesh@Gu@physx@@UEBAPEBXXZ 000000018002512d f   PhysX3CommonPROFILE_x64:PhysX3CommonPROFILE_x64.dll
 0001:00024139       ?getTriangles@TriangleMesh@Gu@physx@@UEBAPEBXXZ 0000000180025139 f   PhysX3CommonPROFILE_x64:PhysX3CommonPROFILE_x64.dll
 0001:0002413f       __imp_load_?getTrianglesRemap@TriangleMesh@Gu@physx@@UEBAPEBIXZ 000000018002513f f   PhysX3CommonPROFILE_x64:PhysX3CommonPROFILE_x64.dll
 0001:0002414b       ?getTrianglesRemap@TriangleMesh@Gu@physx@@UEBAPEBIXZ 000000018002514b f   PhysX3CommonPROFILE_x64:PhysX3CommonPROFILE_x64.dll
 0001:00024151       __imp_load_?getVertices@TriangleMesh@Gu@physx@@UEBAPEBVPxVec3@3@XZ 0000000180025151 f   PhysX3CommonPROFILE_x64:PhysX3CommonPROFILE_x64.dll
 0001:0002415d       ?getVertices@TriangleMesh@Gu@physx@@UEBAPEBVPxVec3@3@XZ 000000018002515d f   PhysX3CommonPROFILE_x64:PhysX3CommonPROFILE_x64.dll
 0001:00024163       __imp_load_?getVerticesForModification@TriangleMesh@Gu@physx@@UEAAPEAVPxVec3@3@XZ 0000000180025163 f   PhysX3CommonPROFILE_x64:PhysX3CommonPROFILE_x64.dll
 0001:0002416f       ?getVerticesForModification@TriangleMesh@Gu@physx@@UEAAPEAVPxVec3@3@XZ 000000018002516f f   PhysX3CommonPROFILE_x64:PhysX3CommonPROFILE_x64.dll
 0001:00024175       __imp_load_?isKindOf@PxTriangleMesh@physx@@MEBA_NPEBD@Z 0000000180025175 f   PhysX3CommonPROFILE_x64:PhysX3CommonPROFILE_x64.dll
 0001:00024181       ?isKindOf@PxTriangleMesh@physx@@MEBA_NPEBD@Z 0000000180025181 f   PhysX3CommonPROFILE_x64:PhysX3CommonPROFILE_x64.dll
 0001:00024187       __imp_load_?onRefCountZero@TriangleMesh@Gu@physx@@UEAAXXZ 0000000180025187 f   PhysX3CommonPROFILE_x64:PhysX3CommonPROFILE_x64.dll
 0001:00024193       ?onRefCountZero@TriangleMesh@Gu@physx@@UEAAXXZ 0000000180025193 f   PhysX3CommonPROFILE_x64:PhysX3CommonPROFILE_x64.dll
 0001:00024199       __imp_load_?refitBVH@TriangleMesh@Gu@physx@@UEAA?AVPxBounds3@3@XZ 0000000180025199 f   PhysX3CommonPROFILE_x64:PhysX3CommonPROFILE_x64.dll
 0001:000241a5       ?refitBVH@TriangleMesh@Gu@physx@@UEAA?AVPxBounds3@3@XZ 00000001800251a5 f   PhysX3CommonPROFILE_x64:PhysX3CommonPROFILE_x64.dll
 0001:000241ab       __imp_load_?release@TriangleMesh@Gu@physx@@UEAAXXZ 00000001800251ab f   PhysX3CommonPROFILE_x64:PhysX3CommonPROFILE_x64.dll
 0001:000241b7       ?release@TriangleMesh@Gu@physx@@UEAAXXZ 00000001800251b7 f   PhysX3CommonPROFILE_x64:PhysX3CommonPROFILE_x64.dll
 0001:000241bd       __imp_load_?setupMeshInterface@InternalTriangleMesh@physx@@QEAAXXZ 00000001800251bd f   PhysX3CommonPROFILE_x64:PhysX3CommonPROFILE_x64.dll
 0001:000241c9       ?setupMeshInterface@InternalTriangleMesh@physx@@QEAAXXZ 00000001800251c9 f   PhysX3CommonPROFILE_x64:PhysX3CommonPROFILE_x64.dll
 0001:000241d0       ??$PFromRva@PEAP6A_JXZ@@YAPEAP6A_JXZK@Z 00000001800251d0 f i delayimp:delayhlp.obj
 0001:000241e0       ??$PFromRva@PEAPEAUHINSTANCE__@@@@YAPEAPEAUHINSTANCE__@@K@Z 00000001800251e0 f i delayimp:delayhlp.obj
 0001:000241f0       ??$PFromRva@PEAU_IMAGE_IMPORT_BY_NAME@@@@YAPEAU_IMAGE_IMPORT_BY_NAME@@K@Z 00000001800251f0 f i delayimp:delayhlp.obj
 0001:00024200       ??$PFromRva@PEAU_IMAGE_THUNK_DATA64@@@@YAPEAU_IMAGE_THUNK_DATA64@@K@Z 0000000180025200 f i delayimp:delayhlp.obj
 0001:00024210       ??$PFromRva@PEBD@@YAPEBDK@Z 0000000180025210 f i delayimp:delayhlp.obj
 0001:00024220       ??$PFromRva@PEBUImgDelayDescr@@@@YAPEBUImgDelayDescr@@K@Z 0000000180025220 f i delayimp:delayhlp.obj
 0001:00024230       ??$PFromRva@PEBU_IMAGE_THUNK_DATA64@@@@YAPEBU_IMAGE_THUNK_DATA64@@K@Z 0000000180025230 f i delayimp:delayhlp.obj
 0001:00024240       ?CountOfImports@@YAIPEBU_IMAGE_THUNK_DATA64@@@Z 0000000180025240 f i delayimp:delayhlp.obj
 0001:0002425c       ?IndexFromPImgThunkData@@YAIPEBU_IMAGE_THUNK_DATA64@@0@Z 000000018002525c f i delayimp:delayhlp.obj
 0001:000243a0       HRESULT_FROM_WIN32         00000001800253a0 f i delayimp:delayhlp.obj
 0001:000243b0       __FUnloadDelayLoadedDLL2   00000001800253b0 f   delayimp:delayhlp.obj
 0001:00024440       __HrLoadAllImportsForDll   0000000180025440 f   delayimp:delayhlp.obj
 0001:000244b4       __delayLoadHelper2         00000001800254b4 f   delayimp:delayhlp.obj
 0001:0002474c       strstr                     000000018002574c f   MSVCRT:MSVCR120.dll
 0001:00024752       memset                     0000000180025752 f   MSVCRT:MSVCR120.dll
 0001:00024758       ??_V@YAXPEAX@Z             0000000180025758 f   MSVCRT:MSVCR120.dll
 0001:0002475e       ??_U@YAPEAX_K@Z            000000018002575e f   MSVCRT:MSVCR120.dll
 0001:00024780       __chkstk                   0000000180025780 f   MSVCRT:chkstk.obj
 0001:00024780       _alloca_probe              0000000180025780 f   MSVCRT:chkstk.obj
 0001:000247ce       memcpy                     00000001800257ce f   MSVCRT:MSVCR120.dll
 0001:000247d4       __clean_type_info_names    00000001800257d4 f   MSVCRT:tncleanup.obj
 0001:000247e0       ??0type_info@@AEAA@AEBV0@@Z 00000001800257e0 f   MSVCRT:ti_inst.obj
 0001:000247f0       ??4type_info@@AEAAAEAV0@AEBV0@@Z 00000001800257f0 f   MSVCRT:ti_inst.obj
 0001:000247f4       ??_Etype_info@@UEAAPEAXI@Z 00000001800257f4 f i MSVCRT:ti_inst.obj
 0001:0002485e       powf                       000000018002585e f   MSVCRT:MSVCR120.dll
 0001:00024864       _fpclass                   0000000180025864 f   MSVCRT:MSVCR120.dll
 0001:0002486a       ??3@YAXPEAX@Z              000000018002586a f   MSVCRT:MSVCR120.dll
 0001:00024870       printf                     0000000180025870 f   MSVCRT:MSVCR120.dll
 0001:00024876       cosf                       0000000180025876 f   MSVCRT:MSVCR120.dll
 0001:0002487c       sinf                       000000018002587c f   MSVCRT:MSVCR120.dll
 0001:00024882       _purecall                  0000000180025882 f   MSVCRT:MSVCR120.dll
 0001:00024888       atan2f                     0000000180025888 f   MSVCRT:MSVCR120.dll
 0001:000248f0       NtCurrentTeb               00000001800258f0 f i MSVCRT:crtdll.obj
 0001:000248fc       _CRT_INIT                  00000001800258fc f   MSVCRT:crtdll.obj
 0001:00024b48       _DllMainCRTStartup         0000000180025b48 f   MSVCRT:crtdll.obj
 0001:00024cbe       ?_name_internal_method@type_info@@QEBAPEBDPEAU__type_info_node@@@Z 0000000180025cbe f   MSVCRT:MSVCR120.dll
 0001:00024cc4       __clean_type_info_names_internal 0000000180025cc4 f   MSVCRT:MSVCR120.dll
 0001:00024ccc       ??_M@YAXPEAX_KHP6AX0@Z@Z   0000000180025ccc f   MSVCRT:ehvecdtr.obj
 0001:00024d48       ?__ArrayUnwind@@YAXPEAX_KHP6AX0@Z@Z 0000000180025d48 f   MSVCRT:ehvecdtr.obj
 0001:00024d92       __CppXcptFilter            0000000180025d92 f   MSVCRT:MSVCR120.dll
 0001:00024d98       _amsg_exit                 0000000180025d98 f   MSVCRT:MSVCR120.dll
 0001:00024da0       _FindPESection             0000000180025da0 f   MSVCRT:pesect.obj
 0001:00024df0       _IsNonwritableInCurrentImage 0000000180025df0 f   MSVCRT:pesect.obj
 0001:00024e40       _ValidateImageBase         0000000180025e40 f   MSVCRT:pesect.obj
 0001:00024e70       __atonexitinit             0000000180025e70 f   MSVCRT:atonexit.obj
 0001:00024ec0       _onexit                    0000000180025ec0 f   MSVCRT:atonexit.obj
 0001:00024f70       atexit                     0000000180025f70 f   MSVCRT:atonexit.obj
 0001:00024f88       free                       0000000180025f88 f   MSVCRT:MSVCR120.dll
 0001:00024f90       __security_init_cookie     0000000180025f90 f   MSVCRT:gs_support.obj
 0001:0002503c       DllMain                    000000018002603c f   MSVCRT:dllmain.obj
 0001:00025060       _malloc_crt                0000000180026060 f   MSVCRT:MSVCR120.dll
 0001:00025068       _RTC_Initialize            0000000180026068 f   MSVCRT:initsect.obj
 0001:000250a0       _RTC_Terminate             00000001800260a0 f   MSVCRT:initsect.obj
 0001:000250d8       _initterm                  00000001800260d8 f   MSVCRT:MSVCR120.dll
 0001:000250de       _initterm_e                00000001800260de f   MSVCRT:MSVCR120.dll
 0001:000250e4       __C_specific_handler       00000001800260e4 f   MSVCRT:MSVCR120.dll
 0001:000250ea       ?terminate@@YAXXZ          00000001800260ea f   MSVCRT:MSVCR120.dll
 0001:000250f0       ?_type_info_dtor_internal_method@type_info@@QEAAXXZ 00000001800260f0 f   MSVCRT:MSVCR120.dll
 0001:000250f0       ??1type_info@@UEAA@XZ      00000001800260f0 f   MSVCRT:MSVCR120.dll
 0001:000250f6       _lock                      00000001800260f6 f   MSVCRT:MSVCR120.dll
 0001:000250fc       _unlock                    00000001800260fc f   MSVCRT:MSVCR120.dll
 0001:00025102       _calloc_crt                0000000180026102 f   MSVCRT:MSVCR120.dll
 0001:00025108       __dllonexit                0000000180026108 f   MSVCRT:MSVCR120.dll
 0001:0002510e       RaiseException             000000018002610e f   kernel32:KERNEL32.dll
 0001:00025114       GetLastError               0000000180026114 f   kernel32:KERNEL32.dll
 0001:0002511a       FreeLibrary                000000018002611a f   kernel32:KERNEL32.dll
 0001:00025120       GetProcAddress             0000000180026120 f   kernel32:KERNEL32.dll
 0001:00025126       LoadLibraryExA             0000000180026126 f   kernel32:KERNEL32.dll
 0001:0002512c       EncodePointer              000000018002612c f   kernel32:KERNEL32.dll
 0001:00025132       DecodePointer              0000000180026132 f   kernel32:KERNEL32.dll
 0001:00025138       QueryPerformanceCounter    0000000180026138 f   kernel32:KERNEL32.dll
 0001:0002513e       GetCurrentProcessId        000000018002613e f   kernel32:KERNEL32.dll
 0001:00025144       GetCurrentThreadId         0000000180026144 f   kernel32:KERNEL32.dll
 0001:0002514a       GetSystemTimeAsFileTime    000000018002614a f   kernel32:KERNEL32.dll
 0001:00025150       DisableThreadLibraryCalls  0000000180026150 f   kernel32:KERNEL32.dll
 0002:00000000       __imp_GetModuleFileNameA   0000000180027000     kernel32:KERNEL32.dll
 0002:00000008       __imp_LoadLibraryA         0000000180027008     kernel32:KERNEL32.dll
 0002:00000010       __imp_GetSystemTimeAsFileTime 0000000180027010     kernel32:KERNEL32.dll
 0002:00000018       __imp_GetCurrentThreadId   0000000180027018     kernel32:KERNEL32.dll
 0002:00000020       __imp_GetCurrentProcessId  0000000180027020     kernel32:KERNEL32.dll
 0002:00000028       __imp_QueryPerformanceCounter 0000000180027028     kernel32:KERNEL32.dll
 0002:00000030       __imp_DecodePointer        0000000180027030     kernel32:KERNEL32.dll
 0002:00000038       __imp_EncodePointer        0000000180027038     kernel32:KERNEL32.dll
 0002:00000040       __imp_LoadLibraryExA       0000000180027040     kernel32:KERNEL32.dll
 0002:00000048       __imp_GetProcAddress       0000000180027048     kernel32:KERNEL32.dll
 0002:00000050       __imp_FreeLibrary          0000000180027050     kernel32:KERNEL32.dll
 0002:00000058       __imp_GetLastError         0000000180027058     kernel32:KERNEL32.dll
 0002:00000060       __imp_RaiseException       0000000180027060     kernel32:KERNEL32.dll
 0002:00000068       __imp_DisableThreadLibraryCalls 0000000180027068     kernel32:KERNEL32.dll
 0002:00000070       \177KERNEL32_NULL_THUNK_DATA 0000000180027070     kernel32:KERNEL32.dll
 0002:00000078       __imp_atan2f               0000000180027078     MSVCRT:MSVCR120.dll
 0002:00000080       __imp_?name@type_info@@QEBAPEBDPEAU__type_info_node@@@Z 0000000180027080     MSVCRT:MSVCR120.dll
 0002:00000080       __imp_?_name_internal_method@type_info@@QEBAPEBDPEAU__type_info_node@@@Z 0000000180027080     MSVCRT:MSVCR120.dll
 0002:00000088       __imp___clean_type_info_names_internal 0000000180027088     MSVCRT:MSVCR120.dll
 0002:00000090       __imp___CppXcptFilter      0000000180027090     MSVCRT:MSVCR120.dll
 0002:00000098       __imp__amsg_exit           0000000180027098     MSVCRT:MSVCR120.dll
 0002:000000a0       __imp_free                 00000001800270a0     MSVCRT:MSVCR120.dll
 0002:000000a8       __imp__malloc_crt          00000001800270a8     MSVCRT:MSVCR120.dll
 0002:000000b0       __imp__purecall            00000001800270b0     MSVCRT:MSVCR120.dll
 0002:000000b8       __imp__initterm_e          00000001800270b8     MSVCRT:MSVCR120.dll
 0002:000000c0       __imp___C_specific_handler 00000001800270c0     MSVCRT:MSVCR120.dll
 0002:000000c8       __imp_?terminate@@YAXXZ    00000001800270c8     MSVCRT:MSVCR120.dll
 0002:000000d0       __imp_?_type_info_dtor_internal_method@type_info@@QEAAXXZ 00000001800270d0     MSVCRT:MSVCR120.dll
 0002:000000d8       __imp__lock                00000001800270d8     MSVCRT:MSVCR120.dll
 0002:000000e0       __imp__unlock              00000001800270e0     MSVCRT:MSVCR120.dll
 0002:000000e8       __imp__calloc_crt          00000001800270e8     MSVCRT:MSVCR120.dll
 0002:000000f0       __imp___dllonexit          00000001800270f0     MSVCRT:MSVCR120.dll
 0002:000000f8       __imp__onexit              00000001800270f8     MSVCRT:MSVCR120.dll
 0002:00000100       __imp_sinf                 0000000180027100     MSVCRT:MSVCR120.dll
 0002:00000108       __imp_cosf                 0000000180027108     MSVCRT:MSVCR120.dll
 0002:00000110       __imp_printf               0000000180027110     MSVCRT:MSVCR120.dll
 0002:00000118       __imp_??3@YAXPEAX@Z        0000000180027118     MSVCRT:MSVCR120.dll
 0002:00000120       __imp__fpclass             0000000180027120     MSVCRT:MSVCR120.dll
 0002:00000128       __imp_powf                 0000000180027128     MSVCRT:MSVCR120.dll
 0002:00000130       __imp_memcpy               0000000180027130     MSVCRT:MSVCR120.dll
 0002:00000138       __imp_??_U@YAPEAX_K@Z      0000000180027138     MSVCRT:MSVCR120.dll
 0002:00000140       __imp_??_V@YAXPEAX@Z       0000000180027140     MSVCRT:MSVCR120.dll
 0002:00000148       __imp_memset               0000000180027148     MSVCRT:MSVCR120.dll
 0002:00000150       __imp_strstr               0000000180027150     MSVCRT:MSVCR120.dll
 0002:00000158       __imp__initterm            0000000180027158     MSVCRT:MSVCR120.dll
 0002:00000160       \177MSVCR120_NULL_THUNK_DATA 0000000180027160     MSVCRT:MSVCR120.dll
 0002:00000168       __xc_a                     0000000180027168     MSVCRT:cinitexe.obj
 0002:00000260       __xc_z                     0000000180027260     MSVCRT:cinitexe.obj
 0002:00000268       __xi_a                     0000000180027268     MSVCRT:cinitexe.obj
 0002:00000280       __xi_z                     0000000180027280     MSVCRT:cinitexe.obj
 0002:000002c8       ??_C@_0BK@KKGDMEEI@PhysX3CommonDEBUG_x64?4dll?$AA@ 00000001800272c8     WindowsCookingDelayLoadHook.obj
 0002:000002e8       ??_C@_0BM@FGKCIMCL@PhysX3CommonCHECKED_x64?4dll?$AA@ 00000001800272e8     WindowsCookingDelayLoadHook.obj
 0002:00000308       ??_C@_0BM@NIMEGLC@PhysX3CommonPROFILE_x64?4dll?$AA@ 0000000180027308     WindowsCookingDelayLoadHook.obj
 0002:00000328       ??_C@_0BF@HEEMOJKO@PhysX3Common_x64?4dll?$AA@ 0000000180027328     WindowsCookingDelayLoadHook.obj
 0002:00000340       ??_C@_0BK@LHJEBOBO@PhysX3CommonDEBUG_x86?4dll?$AA@ 0000000180027340     WindowsCookingDelayLoadHook.obj
 0002:00000360       ??_C@_0BM@ELFFFGHN@PhysX3CommonCHECKED_x86?4dll?$AA@ 0000000180027360     WindowsCookingDelayLoadHook.obj
 0002:00000380       ??_C@_0BM@BAHLJMOE@PhysX3CommonPROFILE_x86?4dll?$AA@ 0000000180027380     WindowsCookingDelayLoadHook.obj
 0002:000003a0       ??_C@_0BF@GJLLDDPI@PhysX3Common_x86?4dll?$AA@ 00000001800273a0     WindowsCookingDelayLoadHook.obj
 0002:000003b8       ??_C@_0BK@FCFCOGBN@PhysX3CommonDEBUG_arm?4dll?$AA@ 00000001800273b8     WindowsCookingDelayLoadHook.obj
 0002:000003d8       ??_C@_0BM@KOJDKOHO@PhysX3CommonCHECKED_arm?4dll?$AA@ 00000001800273d8     WindowsCookingDelayLoadHook.obj
 0002:000003f8       ??_C@_0BM@PFLNGEOH@PhysX3CommonPROFILE_arm?4dll?$AA@ 00000001800273f8     WindowsCookingDelayLoadHook.obj
 0002:00000418       ??_C@_0BF@IMHNMLPL@PhysX3Common_arm?4dll?$AA@ 0000000180027418     WindowsCookingDelayLoadHook.obj
 0002:00000430       ??_C@_08NNMANNNO@_x64?4dll?$AA@ 0000000180027430     WindowsCookingDelayLoadHook.obj
 0002:00000440       ??_C@_0O@LLBCKODF@DEBUG_x64?4dll?$AA@ 0000000180027440     WindowsCookingDelayLoadHook.obj
 0002:00000450       ??_C@_0BA@GBFEBCKH@CHECKED_x64?4dll?$AA@ 0000000180027450     WindowsCookingDelayLoadHook.obj
 0002:00000460       ??_C@_0BA@DKHKNIDO@PROFILE_x64?4dll?$AA@ 0000000180027460     WindowsCookingDelayLoadHook.obj
 0002:00000470       ??_C@_08MADHAHII@_x86?4dll?$AA@ 0000000180027470     WindowsCookingDelayLoadHook.obj
 0002:00000480       ??_C@_0O@KGOFHEGD@DEBUG_x86?4dll?$AA@ 0000000180027480     WindowsCookingDelayLoadHook.obj
 0002:00000490       ??_C@_0BA@HMKDMIPB@CHECKED_x86?4dll?$AA@ 0000000180027490     WindowsCookingDelayLoadHook.obj
 0002:000004a0       ??_C@_0BA@CHINACGI@PROFILE_x86?4dll?$AA@ 00000001800274a0     WindowsCookingDelayLoadHook.obj
 0002:000004b0       ?value@?$LogTwo@$00@shdfnd@physx@@2IB 00000001800274b0     HeightFieldCooking.obj
 0002:000004b4       ?value@?$integral_constant@_N$0A@@std@@2_NB 00000001800274b4     HeightFieldCooking.obj
 0002:000004b5       ?value@?$integral_constant@_N$00@std@@2_NB 00000001800274b5     HeightFieldCooking.obj
 0002:000004bc       ?MAX_LISTENER_COUNT@AlignCheckAllocator@Foundation@shdfnd@physx@@0IB 00000001800274bc     HeightFieldCooking.obj
 0002:000004c0       ?EOL@?$HashBase@V?$Pair@QEBVNamedAllocator@shdfnd@physx@@PEBD@shdfnd@physx@@PEBVNamedAllocator@23@U?$Hash@PEBVNamedAllocator@shdfnd@physx@@@23@UGetKey@?$HashMapBase@PEBVNamedAllocator@shdfnd@physx@@PEBDU?$Hash@PEBVNamedAllocator@shdfnd@physx@@@23@VNonTrackingAllocator@23@@internal@23@VNonTrackingAllocator@23@$00@internal@shdfnd@physx@@2IB 00000001800274c0     HeightFieldCooking.obj
 0002:000004d0       ?g_PXSinCoefficients0@aos@shdfnd@physx@@3UPX_VECTORF32@123@B 00000001800274d0     RTreeCooking.obj
 0002:000004e0       ?g_PXSinCoefficients1@aos@shdfnd@physx@@3UPX_VECTORF32@123@B 00000001800274e0     RTreeCooking.obj
 0002:000004f0       ?g_PXSinCoefficients2@aos@shdfnd@physx@@3UPX_VECTORF32@123@B 00000001800274f0     RTreeCooking.obj
 0002:00000500       ?g_PXCosCoefficients0@aos@shdfnd@physx@@3UPX_VECTORF32@123@B 0000000180027500     RTreeCooking.obj
 0002:00000510       ?g_PXCosCoefficients1@aos@shdfnd@physx@@3UPX_VECTORF32@123@B 0000000180027510     RTreeCooking.obj
 0002:00000520       ?g_PXCosCoefficients2@aos@shdfnd@physx@@3UPX_VECTORF32@123@B 0000000180027520     RTreeCooking.obj
 0002:00000530       ?g_PXTanCoefficients0@aos@shdfnd@physx@@3UPX_VECTORF32@123@B 0000000180027530     RTreeCooking.obj
 0002:00000540       ?g_PXTanCoefficients1@aos@shdfnd@physx@@3UPX_VECTORF32@123@B 0000000180027540     RTreeCooking.obj
 0002:00000550       ?g_PXTanCoefficients2@aos@shdfnd@physx@@3UPX_VECTORF32@123@B 0000000180027550     RTreeCooking.obj
 0002:00000560       ?g_PXASinCoefficients0@aos@shdfnd@physx@@3UPX_VECTORF32@123@B 0000000180027560     RTreeCooking.obj
 0002:00000570       ?g_PXASinCoefficients1@aos@shdfnd@physx@@3UPX_VECTORF32@123@B 0000000180027570     RTreeCooking.obj
 0002:00000580       ?g_PXASinCoefficients2@aos@shdfnd@physx@@3UPX_VECTORF32@123@B 0000000180027580     RTreeCooking.obj
 0002:00000590       ?g_PXATanCoefficients0@aos@shdfnd@physx@@3UPX_VECTORF32@123@B 0000000180027590     RTreeCooking.obj
 0002:000005a0       ?g_PXATanCoefficients1@aos@shdfnd@physx@@3UPX_VECTORF32@123@B 00000001800275a0     RTreeCooking.obj
 0002:000005b0       ?g_PXATanCoefficients2@aos@shdfnd@physx@@3UPX_VECTORF32@123@B 00000001800275b0     RTreeCooking.obj
 0002:000005c0       ?g_PXSinEstCoefficients@aos@shdfnd@physx@@3UPX_VECTORF32@123@B 00000001800275c0     RTreeCooking.obj
 0002:000005d0       ?g_PXCosEstCoefficients@aos@shdfnd@physx@@3UPX_VECTORF32@123@B 00000001800275d0     RTreeCooking.obj
 0002:000005e0       ?g_PXASinEstCoefficients@aos@shdfnd@physx@@3UPX_VECTORF32@123@B 00000001800275e0     RTreeCooking.obj
 0002:000005f0       ?reductionFactors@SubSortQuick@physx@@2QBMB 00000001800275f0     RTreeCooking.obj
 0002:00000600       ?stopAtTrisPerLeaf1@SubSortQuick@physx@@2QBIB 0000000180027600     RTreeCooking.obj
 0002:000006c8       ??_C@_0CN@HEFMNGKD@?4?4?2?4?4?2PhysXCooking?2src?2mesh?2RTre@ 00000001800276c8     RTreeCooking.obj
 0002:00000700       ??_C@_0GK@DGBEAAIF@d?3?2ori?4cohen_g6217_framework?2eng@ 0000000180027700     RTreeCooking.obj
 0002:00000770       ??_C@_0BM@OIFKLHDN@?$DMallocation?5names?5disabled?$DO?$AA@ 0000000180027770     RTreeCooking.obj
 0002:00000790       ??_C@_0GJ@DLLPAIJG@D?3?2Ori?4Cohen_G6217_Framework?2Eng@ 0000000180027790     RTreeCooking.obj
 0002:00000800       ??_C@_0HC@HINCINNF@d?3?2ori?4cohen_g6217_framework?2eng@ 0000000180027800     RTreeCooking.obj
 0002:00000874       __real@37800080            0000000180027874     RTreeCooking.obj
 0002:00000878       __real@3a03126f            0000000180027878     RTreeCooking.obj
 0002:0000087c       __real@3a83126f            000000018002787c     RTreeCooking.obj
 0002:00000880       __real@3f800000            0000000180027880     RTreeCooking.obj
 0002:00000884       __real@41100000            0000000180027884     RTreeCooking.obj
 0002:00000888       __real@41700000            0000000180027888     RTreeCooking.obj
 0002:0000088c       __real@42200000            000000018002788c     RTreeCooking.obj
 0002:00000890       __real@7f7fffff            0000000180027890     RTreeCooking.obj
 0002:00000894       __real@ba83126f            0000000180027894     RTreeCooking.obj
 0002:00000898       __real@fe7fffff            0000000180027898     RTreeCooking.obj
 0002:0000089c       __real@ff7fffff            000000018002789c     RTreeCooking.obj
 0002:000008a0       __xmm@000000003a83126f3a83126f3a83126f 00000001800278a0     RTreeCooking.obj
 0002:000008b0       __xmm@00000000ba83126fba83126fba83126f 00000001800278b0     RTreeCooking.obj
 0002:000008c0       __xmm@00000001000000010000000100000001 00000001800278c0     RTreeCooking.obj
 0002:000008d0       __xmm@00000003000000020000000100000000 00000001800278d0     RTreeCooking.obj
 0002:000008e0       __xmm@fe7fffff7e7fffff7e7fffff7e7fffff 00000001800278e0     RTreeCooking.obj
 0002:00000918       ??_C@_0DD@CMJGDCNN@TriangleMesh?3?3loadFromDesc?3?5desc@ 0000000180027918     TriangleMeshBuilder.obj
 0002:00000950       ??_C@_0DE@NHIHKD@?4?4?2?4?4?2PhysXCooking?2src?2mesh?2Tria@ 0000000180027950     TriangleMeshBuilder.obj
 0002:00000990       ??_C@_0FB@HKCCNMI@PxCookingParams?3?3meshSizePerform@ 0000000180027990     TriangleMeshBuilder.obj
 0002:000009e8       ??_C@_0BJ@BKHDBBHO@cleaning?5the?5mesh?5failed?$AA@ 00000001800279e8     TriangleMeshBuilder.obj
 0002:00000a04       __real@40000000            0000000180027a04     TriangleMeshBuilder.obj
 0002:00000a08       __real@c1b00000            0000000180027a08     TriangleMeshBuilder.obj
 0002:00000a10       __xmm@7fffffff7fffffff7fffffff7fffffff 0000000180027a10     TriangleMeshBuilder.obj
 0002:00000a28       ??_C@_0DH@IKCMPFPC@?4?4?2?4?4?2PhysXCooking?2src?2convex?2Bi@ 0000000180027a28     BigConvexDataBuilder.obj
 0002:00000a60       __real@3dcccccd            0000000180027a60     BigConvexDataBuilder.obj
 0002:00000a64       __real@3f000000            0000000180027a64     BigConvexDataBuilder.obj
 0002:00000a68       __real@bf800000            0000000180027a68     BigConvexDataBuilder.obj
 0002:00000a70       __xmm@80000000800000008000000080000000 0000000180027a70     BigConvexDataBuilder.obj
 0002:00000a88       ??_C@_0DP@KFEAHANP@Meshmerizer?3?3ExtractHullPolygons@ 0000000180027a88     ConvexHullBuilder.obj
 0002:00000ac8       ??_C@_0DE@JCGJGFMG@?4?4?2?4?4?2PhysXCooking?2src?2convex?2Co@ 0000000180027ac8     ConvexHullBuilder.obj
 0002:00000b00       ??_C@_0EB@MLICBFEL@ConvexHullBuilder?3?3Init?3?5convex?5@ 0000000180027b00     ConvexHullBuilder.obj
 0002:00000b50       ??_C@_0GF@OJLJHAMH@ConvexHullBuilder?3?3CreateTriangl@ 0000000180027b50     ConvexHullBuilder.obj
 0002:00000bb8       ??_C@_0DL@IAFKOCCK@ConvexHullBuilder?3?5convex?5hull?5h@ 0000000180027bb8     ConvexHullBuilder.obj
 0002:00000c00       ??_C@_0HF@OLJFBIEL@ConvexHullBuilder?3?5convex?5hull?5d@ 0000000180027c00     ConvexHullBuilder.obj
 0002:00000c80       ??_C@_0OG@JNHFOIL@ConvexHullBuilder?3?5convex?5hull?5d@ 0000000180027c80     ConvexHullBuilder.obj
 0002:00000d70       ??_C@_0EJ@NIOIBAKH@Cooking?3?3cookConvexMesh?3?5non?9man@ 0000000180027d70     ConvexHullBuilder.obj
 0002:00000dbc       __real@3ba3d70a            0000000180027dbc     ConvexHullBuilder.obj
 0002:00000dc0       __real@3ca3d70a            0000000180027dc0     ConvexHullBuilder.obj
 0002:00000dc4       __real@3eaaaaab            0000000180027dc4     ConvexHullBuilder.obj
 0002:00000df8       ??_7ConvexMeshBuilder@physx@@6BPxConvexMesh@1@@ 0000000180027df8     ConvexMeshBuilder.obj
 0002:00000e70       ??_7ConvexMeshBuilder@physx@@6BRefCountable@Cm@1@@ 0000000180027e70     ConvexMeshBuilder.obj
 0002:00000e80       ??_C@_0DF@LLFJIJGM@Gu?3?3ConvexMesh?3?3loadFromDesc?3?5de@ 0000000180027e80     ConvexMeshBuilder.obj
 0002:00000eb8       ??_C@_0DE@FMMNMFJD@?4?4?2?4?4?2PhysXCooking?2src?2convex?2Co@ 0000000180027eb8     ConvexMeshBuilder.obj
 0002:00000ef0       ??_C@_0HK@JOGKIEAA@Gu?3?3ConvexMesh?3?5Mesh?5has?5a?5negat@ 0000000180027ef0     ConvexMeshBuilder.obj
 0002:00000f70       ??_C@_0DH@NJPPHFFD@Gu?3?3ConvexMesh?3?5Error?5computing?5@ 0000000180027f70     ConvexMeshBuilder.obj
 0002:00000fa8       ??_C@_0DJ@LJDLGLDJ@Gu?3?3ConvexMesh?3?3loadConvexHull?3?5@ 0000000180027fa8     ConvexMeshBuilder.obj
 0002:00000ff0       ??_C@_0JC@IEAFEIFE@Gu?3?3ConvexMesh?3?3loadConvexHull?3?5@ 0000000180027ff0     ConvexMeshBuilder.obj
 0002:00001090       ??_C@_0HJ@KJANPPOE@ConvexMeshBuilder?3?3computeHullPo@ 0000000180028090     ConvexMeshBuilder.obj
 0002:0000110c       ??_C@_06KDGGGLIJ@PxVec3?$AA@ 000000018002810c     ConvexMeshBuilder.obj
 0002:00001114       ??_C@_05LMJPANIN@PxU32?$AA@ 0000000180028114     ConvexMeshBuilder.obj
 0002:00001120       ??_C@_0O@JMAGMMGG@PxHullPolygon?$AA@ 0000000180028120     ConvexMeshBuilder.obj
 0002:00001130       __real@3a800000            0000000180028130     ConvexMeshBuilder.obj
 0002:00001134       __real@40400000            0000000180028134     ConvexMeshBuilder.obj
 0002:00001140       __xmm@80000000000000008000000000000000 0000000180028140     ConvexMeshBuilder.obj
 0002:00001158       ??_C@_0BM@FNPIOFJJ@Cant?5normalize?5ZERO?5vector?6?$AA@ 0000000180028158     hulllib.obj
 0002:00001178       ??_C@_0CK@LEJAGBKE@?4?4?2?4?4?2PhysXCooking?2src?2convex?2hu@ 0000000180028178     hulllib.obj
 0002:000011b0       ??_C@_0HE@HIPAJHIK@d?3?2ori?4cohen_g6217_framework?2eng@ 00000001800281b0     hulllib.obj
 0002:00001224       __real@1e3ce508            0000000180028224     hulllib.obj
 0002:00001228       __real@358637bd            0000000180028228     hulllib.obj
 0002:0000122c       __real@3c23d70a            000000018002822c     hulllib.obj
 0002:00001230       __real@3c8efa35            0000000180028230     hulllib.obj
 0002:00001234       __real@3ccccccd            0000000180028234     hulllib.obj
 0002:00001238       __real@3d4ccccd            0000000180028238     hulllib.obj
 0002:0000123c       __real@3d567750            000000018002823c     hulllib.obj
 0002:00001240       __real@3e800000            0000000180028240     hulllib.obj
 0002:00001244       __real@40a00000            0000000180028244     hulllib.obj
 0002:00001248       __real@42340000            0000000180028248     hulllib.obj
 0002:0000124c       __real@42f00000            000000018002824c     hulllib.obj
 0002:00001250       __real@43b40000            0000000180028250     hulllib.obj
 0002:00001254       __real@9e3ce508            0000000180028254     hulllib.obj
 0002:00001258       __real@bc23d70a            0000000180028258     hulllib.obj
 0002:0000125c       __real@bca3d70a            000000018002825c     hulllib.obj
 0002:00001268       __real@3f91111111111111    0000000180028268     VolumeIntegration.obj
 0002:00001270       __real@3fa5555555555555    0000000180028270     VolumeIntegration.obj
 0002:00001278       __real@3fa999999999999a    0000000180028278     VolumeIntegration.obj
 0002:00001280       __real@3fb5555555555555    0000000180028280     VolumeIntegration.obj
 0002:00001288       __real@3fc5555555555555    0000000180028288     VolumeIntegration.obj
 0002:00001290       __real@3fe0000000000000    0000000180028290     VolumeIntegration.obj
 0002:00001298       __real@3ff0000000000000    0000000180028298     VolumeIntegration.obj
 0002:000012a0       __real@4000000000000000    00000001800282a0     VolumeIntegration.obj
 0002:000012a8       __real@4008000000000000    00000001800282a8     VolumeIntegration.obj
 0002:000012b0       __real@4010000000000000    00000001800282b0     VolumeIntegration.obj
 0002:000012b8       __real@bf91111111111111    00000001800282b8     VolumeIntegration.obj
 0002:000012c0       __real@bfa999999999999a    00000001800282c0     VolumeIntegration.obj
 0002:000012c8       __real@bfb5555555555555    00000001800282c8     VolumeIntegration.obj
 0002:000012d0       __real@bfc5555555555555    00000001800282d0     VolumeIntegration.obj
 0002:000012e0       __xmm@3f811111111111113f81111111111111 00000001800282e0     VolumeIntegration.obj
 0002:000012f0       __xmm@3f811111111111113f91111111111111 00000001800282f0     VolumeIntegration.obj
 0002:00001300       __xmm@3f911111111111113f91111111111111 0000000180028300     VolumeIntegration.obj
 0002:00001310       __xmm@3fa55555555555553fa5555555555555 0000000180028310     VolumeIntegration.obj
 0002:00001320       __xmm@3fa55555555555553fc5555555555555 0000000180028320     VolumeIntegration.obj
 0002:00001330       __xmm@3fd55555555555553fd5555555555555 0000000180028330     VolumeIntegration.obj
 0002:00001340       __xmm@3fe00000000000003fe0000000000000 0000000180028340     VolumeIntegration.obj
 0002:00001350       __xmm@7fffffffffffffff7fffffffffffffff 0000000180028350     VolumeIntegration.obj
 0002:00001360       ??_C@_0DC@DMHHONHL@Adjacencies?3?3GetBoundaryVertices@ 0000000180028360     Adjacencies.obj
 0002:00001398       ??_C@_0CH@EOBHIJNK@?4?4?2?4?4?2PhysXCooking?2src?2Adjacenci@ 0000000180028398     Adjacencies.obj
 0002:000013c0       ??_C@_0CK@KKNAOLHI@Adjacencies?3?3MakeLastRef?3?5NULL?5p@ 00000001800283c0     Adjacencies.obj
 0002:000013f0       ??_C@_0DA@FMEHLBKI@Adjacencies?3?3UpdateLink?3?5invalid@ 00000001800283f0     Adjacencies.obj
 0002:00001420       ??_C@_0JJ@BJLNDJKO@Adjacencies?3?3CreateDatabase?3?5can@ 0000000180028420     Adjacencies.obj
 0002:000014f0       ??_7PxCooking@physx@@6B@   00000001800284f0     Cooking.obj
 0002:00001550       ??_7Cooking@physx@@6B@     0000000180028550     Cooking.obj
 0002:000015b0       ??_7TriangleMeshBuilder@physx@@6BPxTriangleMesh@1@@ 00000001800285b0     Cooking.obj
 0002:00001640       ??_7TriangleMeshBuilder@physx@@6BRefCountable@Cm@1@@ 0000000180028640     Cooking.obj
 0002:00001650       ??_C@_0FC@PJIHAFK@Cooking?3?3validateTriangleMesh?3?5u@ 0000000180028650     Cooking.obj
 0002:000016a8       ??_C@_0CD@HPMFPCAJ@?4?4?2?4?4?2PhysXCooking?2src?2Cooking?4c@ 00000001800286a8     Cooking.obj
 0002:000016d0       ??_C@_0GF@KBACGOEB@PxTriangleMeshDesc?3?3convexEdgeTh@ 00000001800286d0     Cooking.obj
 0002:00001740       ??_C@_0FF@FCKBBOBA@Cooking?3?3cook?1createTriangleMesh@ 0000000180028740     Cooking.obj
 0002:000017a0       ??_C@_0EK@EKAIJEBL@Cooking?3?3cookConvexMesh?3?5user?9pr@ 00000001800287a0     Cooking.obj
 0002:000017f0       ??_C@_0EJ@EIMOEGKB@Cooking?3?3cookConvexMesh?3?5user?9pr@ 00000001800287f0     Cooking.obj
 0002:00001840       ??_C@_0EP@CKACPLJK@Cooking?3?3cookConvexMesh?3?5user?9pr@ 0000000180028840     Cooking.obj
 0002:00001890       ??_C@_0EO@LKFMMDE@Cooking?3?3cookConvexMesh?3?5user?9pr@ 0000000180028890     Cooking.obj
 0002:000018e0       __real@7e7fffff            00000001800288e0     Cooking.obj
 0002:000018e8       ??_C@_0CI@LKCEKHOD@?4?4?2?4?4?2PhysXCooking?2src?2CookingUt@ 00000001800288e8     CookingUtils.obj
 0002:00001918       ??_C@_0CE@DNAJJHLF@?4?4?2?4?4?2PhysXCooking?2src?2EdgeList?4@ 0000000180028918     EdgeList.obj
 0002:00001940       ??_C@_0CO@GBNJFPN@EdgeList?3?3CreateFacesToEdges?3?5NU@ 0000000180028940     EdgeList.obj
 0002:00001970       ??_C@_0CO@EHJBBMNK@EdgeList?3?3ComputeActiveEdges?3?5NU@ 0000000180028970     EdgeList.obj
 0002:000019a0       ??_C@_0DI@GBHLFOFP@ActiveEdges?3?3ComputeConvexEdges?3@ 00000001800289a0     EdgeList.obj
 0002:000019d8       ??_C@_0DM@JOGBLHDI@ActiveEdges?3?3ComputeConvexEdges?3@ 00000001800289d8     EdgeList.obj
 0002:00001a20       ??_C@_0ED@FEMJKPEL@ActiveEdges?3?3ComputeConvexEdges?3@ 0000000180028a20     EdgeList.obj
 0002:00001a70       ??_C@_0EB@BFDPMFCD@ActiveEdges?3?3ComputeConvexEdges?3@ 0000000180028a70     EdgeList.obj
 0002:00001ab4       __real@bf7fbe77            0000000180028ab4     EdgeList.obj
 0002:00001ae8       ??_7RemapCallback@RTreeCooker@physx@@6B@ 0000000180028ae8     InternalTriangleMeshBuilder.obj
 0002:00001af8       ??_C@_0DH@KAAPMABG@?4?4?2?4?4?2PhysXCooking?2src?2InternalT@ 0000000180028af8     InternalTriangleMeshBuilder.obj
 0002:00001b30       ??_7RTreeCookerRemap@@6B@  0000000180028b30     InternalTriangleMeshBuilder.obj
 0002:00001b40       ??_C@_0DJ@IGODLHLP@TriangleMesh?3?5Enable?5mesh?5weldin@ 0000000180028b40     InternalTriangleMeshBuilder.obj
 0002:00001b80       ??_C@_0FJ@HHJLKGDF@TriangleMesh?3?5triangles?5are?5too?5@ 0000000180028b80     InternalTriangleMeshBuilder.obj
 0002:00001be0       ??_C@_0CN@KGPHHHLK@TriangleMesh?3?5mesh?5is?5too?5big?5fo@ 0000000180028be0     InternalTriangleMeshBuilder.obj
 0002:00001c10       __real@48742400            0000000180028c10     InternalTriangleMeshBuilder.obj
 0002:00001c18       ??_C@_0CH@GLEMKEIO@?4?4?2?4?4?2PhysXCooking?2src?2MeshClean@ 0000000180028c18     MeshCleaner.obj
 0002:00001c40       __sz_PhysX3CommonPROFILE_x64_dll 0000000180028c40     PhysX3CommonPROFILE_x64:PhysX3CommonPROFILE_x64.dll
 0002:00001c5c       ?ProcessDetach@NativeDll@<CrtImplementationDetails>@@0IB 0000000180028c5c     MSVCRT:tncleanup.obj
 0002:00001c60       ?ProcessAttach@NativeDll@<CrtImplementationDetails>@@0IB 0000000180028c60     MSVCRT:tncleanup.obj
 0002:00001c64       ?ThreadAttach@NativeDll@<CrtImplementationDetails>@@0IB 0000000180028c64     MSVCRT:tncleanup.obj
 0002:00001c68       ?ThreadDetach@NativeDll@<CrtImplementationDetails>@@0IB 0000000180028c68     MSVCRT:tncleanup.obj
 0002:00001c6c       ?ProcessVerifier@NativeDll@<CrtImplementationDetails>@@0IB 0000000180028c6c     MSVCRT:tncleanup.obj
 0002:00001c78       ??_7type_info@@6B@         0000000180028c78     MSVCRT:ti_inst.obj
 0002:00001c80       _pRawDllMain               0000000180028c80     MSVCRT:crtdll.obj
 0002:00001c80       _pDefaultRawDllMain        0000000180028c80     MSVCRT:crtdll.obj
 0002:00001c90       _load_config_used          0000000180028c90     MSVCRT:loadcfg.obj
 0002:00001da0       ??_R4type_info@@6B@        0000000180028da0     MSVCRT:ti_inst.obj
 0002:00001dc8       ??_R3type_info@@8          0000000180028dc8     MSVCRT:ti_inst.obj
 0002:00001de0       ??_R2type_info@@8          0000000180028de0     MSVCRT:ti_inst.obj
 0002:00001df0       ??_R1A@?0A@EA@type_info@@8 0000000180028df0     MSVCRT:ti_inst.obj
 0002:00001e18       __rtc_iaa                  0000000180028e18     MSVCRT:initsect.obj
 0002:00001e20       __rtc_izz                  0000000180028e20     MSVCRT:initsect.obj
 0002:00001e28       __rtc_taa                  0000000180028e28     MSVCRT:initsect.obj
 0002:00001e30       __rtc_tzz                  0000000180028e30     MSVCRT:initsect.obj
 0002:00004a70       __DELAY_IMPORT_DESCRIPTOR_PhysX3CommonPROFILE_x64_dll 000000018002ba70     PhysX3CommonPROFILE_x64:PhysX3CommonPROFILE_x64.dll
 0002:00004a90       __NULL_DELAY_IMPORT_DESCRIPTOR 000000018002ba90     PhysX3CommonPROFILE_x64:PhysX3CommonPROFILE_x64.dll
 0002:00004d40       \177PhysX3CommonPROFILE_x64_NULL_THUNK_DATA_DLN 000000018002bd40     PhysX3CommonPROFILE_x64:PhysX3CommonPROFILE_x64.dll
 0002:00005e38       \177PhysX3CommonPROFILE_x64_NULL_THUNK_DATA_DLB 000000018002ce38     PhysX3CommonPROFILE_x64:PhysX3CommonPROFILE_x64.dll
 0002:00006158       __IMPORT_DESCRIPTOR_KERNEL32 000000018002d158     kernel32:KERNEL32.dll
 0002:0000616c       __IMPORT_DESCRIPTOR_MSVCR120 000000018002d16c     MSVCRT:MSVCR120.dll
 0002:00006180       __NULL_IMPORT_DESCRIPTOR   000000018002d180     kernel32:KERNEL32.dll
 0003:00000060       __pfnDliNotifyHook2        000000018002e060     WindowsCookingDelayLoadHook.obj
 0003:00000070       ?g_PXTanEstCoefficients@aos@shdfnd@physx@@3UPX_VECTORF32@123@B 000000018002e070     RTreeCooking.obj
 0003:00000080       ?g_PXATanEstCoefficients@aos@shdfnd@physx@@3UPX_VECTORF32@123@B 000000018002e080     RTreeCooking.obj
 0003:00000090       ?g_PXASinEstConstants@aos@shdfnd@physx@@3UPX_VECTORF32@123@B 000000018002e090     RTreeCooking.obj
 0003:000000a0       ?g_PXPiConstants0@aos@shdfnd@physx@@3UPX_VECTORF32@123@B 000000018002e0a0     RTreeCooking.obj
 0003:000000b0       ?g_PXReciprocalTwoPi@aos@shdfnd@physx@@3UPX_VECTORF32@123@B 000000018002e0b0     RTreeCooking.obj
 0003:000000c0       ?g_PXTwoPi@aos@shdfnd@physx@@3UPX_VECTORF32@123@B 000000018002e0c0     RTreeCooking.obj
 0003:000000d0       ?planetestepsilon@physx@@3MA 000000018002e0d0     hulllib.obj
 0003:000000d8       _fltused                   000000018002e0d8     MSVCRT:dllsupp.obj
 0003:000000e0       __native_dllmain_reason    000000018002e0e0     MSVCRT:natstart.obj
 0003:000000e8       __security_cookie          000000018002e0e8     MSVCRT:gs_cookie.obj
 0003:000000f0       __security_cookie_complement 000000018002e0f0     MSVCRT:gs_cookie.obj
 0003:000000f8       ??_R0?AUInterval@physx@@@8 000000018002e0f8     RTreeCooking.obj
 0003:00000120       ??_R0?AUPxBounds3V@physx@@@8 000000018002e120     RTreeCooking.obj
 0003:00000148       ??_R0I@8                   000000018002e148     RTreeCooking.obj
 0003:00000160       ??_R0?AVPxVec3@physx@@@8   000000018002e160     RTreeCooking.obj
 0003:00000188       ??_R0?AURTreeNodeNQ@physx@@@8 000000018002e188     RTreeCooking.obj
 0003:000001b0       ??_R0?AURTreeNodeQ@Gu@physx@@@8 000000018002e1b0     RTreeCooking.obj
 0003:000001e0       ??_R0E@8                   000000018002e1e0     BigConvexDataBuilder.obj
 0003:000001f8       ??_R0?AUValency@Gu@physx@@@8 000000018002e1f8     BigConvexDataBuilder.obj
 0003:00000220       ??_R0G@8                   000000018002e220     BigConvexDataBuilder.obj
 0003:00000238       ??_R0?AUHullTriangleData@physx@@@8 000000018002e238     ConvexHullBuilder.obj
 0003:00000268       ??_R0?AUEdgeDescData@Gu@physx@@@8 000000018002e268     ConvexHullBuilder.obj
 0003:00000298       ??_R0?AVBigConvexData@physx@@@8 000000018002e298     ConvexMeshBuilder.obj
 0003:000002c8       ??_R0?AVConvexH@physx@@@8  000000018002e2c8     hulllib.obj
 0003:000002f0       ??_R0?AVTri@physx@@@8      000000018002e2f0     hulllib.obj
 0003:00000310       ??_R0M@8                   000000018002e310     hulllib.obj
 0003:00000328       ??_R0?AVAdjTriangle@physx@@@8 000000018002e328     Adjacencies.obj
 0003:00000350       ??_R0?AVAdjEdge@@@8        000000018002e350     Adjacencies.obj
 0003:00000370       ??_R0?AVTriangleMeshBuilder@physx@@@8 000000018002e370     Cooking.obj
 0003:000003a0       ??_R0?AVHeightField@Gu@physx@@@8 000000018002e3a0     Cooking.obj
 0003:000003d0       ??_R0?AVCooking@physx@@@8  000000018002e3d0     Cooking.obj
 0003:000003f8       ??_R0?AUEdgeTriangleData@Gu@physx@@@8 000000018002e3f8     EdgeList.obj
 0003:00000428       ??_R0?AUEdgeData@Gu@physx@@@8 000000018002e428     EdgeList.obj
 0003:00000450       ??_R0?AVEdgeListBuilder@Gu@physx@@@8 000000018002e450     InternalTriangleMeshBuilder.obj
 0003:00000480       ??_R0?AVtype_info@@@8      000000018002e480     MSVCRT:ti_inst.obj
 0003:000004a0       __imp_?writeWord@physx@@YAXG_NAEAVPxOutputStream@1@@Z 000000018002e4a0     PhysX3CommonPROFILE_x64:PhysX3CommonPROFILE_x64.dll
 0003:000004a8       __imp_?writeDword@physx@@YAXI_NAEAVPxOutputStream@1@@Z 000000018002e4a8     PhysX3CommonPROFILE_x64:PhysX3CommonPROFILE_x64.dll
 0003:000004b0       __imp_?writeFloat@physx@@YAXM_NAEAVPxOutputStream@1@@Z 000000018002e4b0     PhysX3CommonPROFILE_x64:PhysX3CommonPROFILE_x64.dll
 0003:000004b8       __imp_?writeHeader@physx@@YA_NCCCCI_NAEAVPxOutputStream@1@@Z 000000018002e4b8     PhysX3CommonPROFILE_x64:PhysX3CommonPROFILE_x64.dll
 0003:000004c0       __imp_PxGetFoundation      000000018002e4c0     PhysX3CommonPROFILE_x64:PhysX3CommonPROFILE_x64.dll
 0003:000004c8       __imp_?getAllocator@shdfnd@physx@@YAAEAVPxAllocatorCallback@2@XZ 000000018002e4c8     PhysX3CommonPROFILE_x64:PhysX3CommonPROFILE_x64.dll
 0003:000004d0       __imp_?allocate@Allocator@shdfnd@physx@@QEAAPEAX_KPEBDH@Z 000000018002e4d0     PhysX3CommonPROFILE_x64:PhysX3CommonPROFILE_x64.dll
 0003:000004d8       __imp_?allocate@TempAllocator@shdfnd@physx@@QEAAPEAX_KPEBDH@Z 000000018002e4d8     PhysX3CommonPROFILE_x64:PhysX3CommonPROFILE_x64.dll
 0003:000004e0       __imp_?deallocate@TempAllocator@shdfnd@physx@@QEAAXPEAX@Z 000000018002e4e0     PhysX3CommonPROFILE_x64:PhysX3CommonPROFILE_x64.dll
 0003:000004e8       __imp_?computeBoundsAroundVertices@Gu@physx@@YAXAEAVPxBounds3@2@IPEIBVPxVec3@2@@Z 000000018002e4e8     PhysX3CommonPROFILE_x64:PhysX3CommonPROFILE_x64.dll
 0003:000004f0       __imp_?deallocate@Allocator@shdfnd@physx@@QEAAXPEAX@Z 000000018002e4f0     PhysX3CommonPROFILE_x64:PhysX3CommonPROFILE_x64.dll
 0003:000004f8       __imp_?getInstance@Foundation@shdfnd@physx@@SAAEAV123@XZ 000000018002e4f8     PhysX3CommonPROFILE_x64:PhysX3CommonPROFILE_x64.dll
 0003:00000500       __imp_?error@Foundation@shdfnd@physx@@QEAAXW4Enum@PxErrorCode@3@PEBDH1ZZ 000000018002e500     PhysX3CommonPROFILE_x64:PhysX3CommonPROFILE_x64.dll
 0003:00000508       __imp_?save@RTree@Gu@physx@@QEBA_NAEAVPxOutputStream@3@@Z 000000018002e508     PhysX3CommonPROFILE_x64:PhysX3CommonPROFILE_x64.dll
 0003:00000510       __imp_?release@InternalTriangleMesh@physx@@QEAAXXZ 000000018002e510     PhysX3CommonPROFILE_x64:PhysX3CommonPROFILE_x64.dll
 0003:00000518       __imp_?allocateVertices@InternalTriangleMesh@physx@@QEAAPEAVPxVec3@2@I@Z 000000018002e518     PhysX3CommonPROFILE_x64:PhysX3CommonPROFILE_x64.dll
 0003:00000520       __imp_?allocateTriangles@InternalTriangleMesh@physx@@QEAAPEAXI_N@Z 000000018002e520     PhysX3CommonPROFILE_x64:PhysX3CommonPROFILE_x64.dll
 0003:00000528       __imp_?allocateMaterials@InternalTriangleMesh@physx@@QEAAPEAGXZ 000000018002e528     PhysX3CommonPROFILE_x64:PhysX3CommonPROFILE_x64.dll
 0003:00000530       __imp_?writeWordBuffer@physx@@YAXPEBGI_NAEAVPxOutputStream@1@@Z 000000018002e530     PhysX3CommonPROFILE_x64:PhysX3CommonPROFILE_x64.dll
 0003:00000538       __imp_?writeFloatBuffer@physx@@YAXPEBMI_NAEAVPxOutputStream@1@@Z 000000018002e538     PhysX3CommonPROFILE_x64:PhysX3CommonPROFILE_x64.dll
 0003:00000540       __imp_?computeMaxIndex@physx@@YAIPEBII@Z 000000018002e540     PhysX3CommonPROFILE_x64:PhysX3CommonPROFILE_x64.dll
 0003:00000548       __imp_?storeIndices@physx@@YAXIIPEBIAEAVPxOutputStream@1@_N@Z 000000018002e548     PhysX3CommonPROFILE_x64:PhysX3CommonPROFILE_x64.dll
 0003:00000550       __imp_?computeMaxIndex@physx@@YAGPEBGI@Z 000000018002e550     PhysX3CommonPROFILE_x64:PhysX3CommonPROFILE_x64.dll
 0003:00000558       __imp_?WriteHeader@Gu@physx@@YA_NEEEEI_NAEAVPxOutputStream@2@@Z 000000018002e558     PhysX3CommonPROFILE_x64:PhysX3CommonPROFILE_x64.dll
 0003:00000560       __imp_?StoreIndices@Gu@physx@@YAXGIPEBGAEAVPxOutputStream@2@_N@Z 000000018002e560     PhysX3CommonPROFILE_x64:PhysX3CommonPROFILE_x64.dll
 0003:00000568       __imp_?CreateOffsets@BigConvexData@physx@@IEAAXXZ 000000018002e568     PhysX3CommonPROFILE_x64:PhysX3CommonPROFILE_x64.dll
 0003:00000570       __imp_??0RadixSortBuffered@Gu@physx@@QEAA@XZ 000000018002e570     PhysX3CommonPROFILE_x64:PhysX3CommonPROFILE_x64.dll
 0003:00000578       __imp_??1RadixSortBuffered@Gu@physx@@UEAA@XZ 000000018002e578     PhysX3CommonPROFILE_x64:PhysX3CommonPROFILE_x64.dll
 0003:00000580       __imp_?Sort@RadixSortBuffered@Gu@physx@@QEAAAEAV123@PEBIIW4RadixHint@23@@Z 000000018002e580     PhysX3CommonPROFILE_x64:PhysX3CommonPROFILE_x64.dll
 0003:00000588       __imp_??0Container@Gu@physx@@QEAA@XZ 000000018002e588     PhysX3CommonPROFILE_x64:PhysX3CommonPROFILE_x64.dll
 0003:00000590       __imp_??0Container@Gu@physx@@QEAA@AEBV012@@Z 000000018002e590     PhysX3CommonPROFILE_x64:PhysX3CommonPROFILE_x64.dll
 0003:00000598       __imp_??1Container@Gu@physx@@QEAA@XZ 000000018002e598     PhysX3CommonPROFILE_x64:PhysX3CommonPROFILE_x64.dll
 0003:000005a0       __imp_?Empty@Container@Gu@physx@@QEAAAEAV123@XZ 000000018002e5a0     PhysX3CommonPROFILE_x64:PhysX3CommonPROFILE_x64.dll
 0003:000005a8       __imp_?Contains@Container@Gu@physx@@QEBA_NIPEAI@Z 000000018002e5a8     PhysX3CommonPROFILE_x64:PhysX3CommonPROFILE_x64.dll
 0003:000005b0       __imp_??4Container@Gu@physx@@QEAAXAEBV012@@Z 000000018002e5b0     PhysX3CommonPROFILE_x64:PhysX3CommonPROFILE_x64.dll
 0003:000005b8       __imp_?Resize@Container@Gu@physx@@AEAA_NI@Z 000000018002e5b8     PhysX3CommonPROFILE_x64:PhysX3CommonPROFILE_x64.dll
 0003:000005c0       __imp_??0ConvexMesh@Gu@physx@@QEAA@XZ 000000018002e5c0     PhysX3CommonPROFILE_x64:PhysX3CommonPROFILE_x64.dll
 0003:000005c8       __imp_??1ConvexMesh@Gu@physx@@UEAA@XZ 000000018002e5c8     PhysX3CommonPROFILE_x64:PhysX3CommonPROFILE_x64.dll
 0003:000005d0       __imp_??0BigConvexData@physx@@QEAA@XZ 000000018002e5d0     PhysX3CommonPROFILE_x64:PhysX3CommonPROFILE_x64.dll
 0003:000005d8       __imp_??1BigConvexData@physx@@QEAA@XZ 000000018002e5d8     PhysX3CommonPROFILE_x64:PhysX3CommonPROFILE_x64.dll
 0003:000005e0       __imp_?exportExtraData@ConvexMesh@Gu@physx@@UEAAXAEAVPxSerializationContext@3@@Z 000000018002e5e0     PhysX3CommonPROFILE_x64:PhysX3CommonPROFILE_x64.dll
 0003:000005e8       __imp_?getConcreteTypeName@PxConvexMesh@physx@@UEBAPEBDXZ 000000018002e5e8     PhysX3CommonPROFILE_x64:PhysX3CommonPROFILE_x64.dll
 0003:000005f0       __imp_?getIndexBuffer@ConvexMesh@Gu@physx@@UEBAPEBEXZ 000000018002e5f0     PhysX3CommonPROFILE_x64:PhysX3CommonPROFILE_x64.dll
 0003:000005f8       __imp_?getLocalBounds@ConvexMesh@Gu@physx@@UEBA?AVPxBounds3@3@XZ 000000018002e5f8     PhysX3CommonPROFILE_x64:PhysX3CommonPROFILE_x64.dll
 0003:00000600       __imp_?getMassInformation@ConvexMesh@Gu@physx@@UEBAXAEAMAEAVPxMat33@3@AEAVPxVec3@3@@Z 000000018002e600     PhysX3CommonPROFILE_x64:PhysX3CommonPROFILE_x64.dll
 0003:00000608       __imp_?getNbPolygons@ConvexMesh@Gu@physx@@UEBAIXZ 000000018002e608     PhysX3CommonPROFILE_x64:PhysX3CommonPROFILE_x64.dll
 0003:00000610       __imp_?getNbVertices@ConvexMesh@Gu@physx@@UEBAIXZ 000000018002e610     PhysX3CommonPROFILE_x64:PhysX3CommonPROFILE_x64.dll
 0003:00000618       __imp_?getPolygonData@ConvexMesh@Gu@physx@@UEBA_NIAEAUPxHullPolygon@3@@Z 000000018002e618     PhysX3CommonPROFILE_x64:PhysX3CommonPROFILE_x64.dll
 0003:00000620       __imp_?getReferenceCount@ConvexMesh@Gu@physx@@UEBAIXZ 000000018002e620     PhysX3CommonPROFILE_x64:PhysX3CommonPROFILE_x64.dll
 0003:00000628       __imp_?getVertices@ConvexMesh@Gu@physx@@UEBAPEBVPxVec3@3@XZ 000000018002e628     PhysX3CommonPROFILE_x64:PhysX3CommonPROFILE_x64.dll
 0003:00000630       __imp_?isKindOf@PxConvexMesh@physx@@MEBA_NPEBD@Z 000000018002e630     PhysX3CommonPROFILE_x64:PhysX3CommonPROFILE_x64.dll
 0003:00000638       __imp_?onRefCountZero@ConvexMesh@Gu@physx@@UEAAXXZ 000000018002e638     PhysX3CommonPROFILE_x64:PhysX3CommonPROFILE_x64.dll
 0003:00000640       __imp_?release@ConvexMesh@Gu@physx@@UEAAXXZ 000000018002e640     PhysX3CommonPROFILE_x64:PhysX3CommonPROFILE_x64.dll
 0003:00000648       __imp_?readDword@physx@@YAI_NAEAVPxInputStream@1@@Z 000000018002e648     PhysX3CommonPROFILE_x64:PhysX3CommonPROFILE_x64.dll
 0003:00000650       __imp_?ReadHeader@Gu@physx@@YA_NEEEEAEAIAEA_NAEAVPxInputStream@2@@Z 000000018002e650     PhysX3CommonPROFILE_x64:PhysX3CommonPROFILE_x64.dll
 0003:00000658       __imp_??0FPUGuard@shdfnd@physx@@QEAA@XZ 000000018002e658     PhysX3CommonPROFILE_x64:PhysX3CommonPROFILE_x64.dll
 0003:00000660       __imp_??1FPUGuard@shdfnd@physx@@QEAA@XZ 000000018002e660     PhysX3CommonPROFILE_x64:PhysX3CommonPROFILE_x64.dll
 0003:00000668       __imp_?incRefCount@Foundation@shdfnd@physx@@SAXXZ 000000018002e668     PhysX3CommonPROFILE_x64:PhysX3CommonPROFILE_x64.dll
 0003:00000670       __imp_?decRefCount@Foundation@shdfnd@physx@@SAXXZ 000000018002e670     PhysX3CommonPROFILE_x64:PhysX3CommonPROFILE_x64.dll
 0003:00000678       __imp_??0TriangleMesh@Gu@physx@@QEAA@XZ 000000018002e678     PhysX3CommonPROFILE_x64:PhysX3CommonPROFILE_x64.dll
 0003:00000680       __imp_?checkMeshIndicesSize@TriangleMesh@Gu@physx@@QEAAXXZ 000000018002e680     PhysX3CommonPROFILE_x64:PhysX3CommonPROFILE_x64.dll
 0003:00000688       __imp_??1TriangleMesh@Gu@physx@@UEAA@XZ 000000018002e688     PhysX3CommonPROFILE_x64:PhysX3CommonPROFILE_x64.dll
 0003:00000690       __imp_??0HeightField@Gu@physx@@QEAA@PEAVGuMeshFactory@2@@Z 000000018002e690     PhysX3CommonPROFILE_x64:PhysX3CommonPROFILE_x64.dll
 0003:00000698       __imp_?loadFromDesc@HeightField@Gu@physx@@QEAA_NAEBVPxHeightFieldDesc@3@_N@Z 000000018002e698     PhysX3CommonPROFILE_x64:PhysX3CommonPROFILE_x64.dll
 0003:000006a0       __imp_?releaseMemory@HeightField@Gu@physx@@QEAAX_N@Z 000000018002e6a0     PhysX3CommonPROFILE_x64:PhysX3CommonPROFILE_x64.dll
 0003:000006a8       __imp_?exportExtraData@TriangleMesh@Gu@physx@@UEAAXAEAVPxSerializationContext@3@@Z 000000018002e6a8     PhysX3CommonPROFILE_x64:PhysX3CommonPROFILE_x64.dll
 0003:000006b0       __imp_?getConcreteTypeName@PxTriangleMesh@physx@@UEBAPEBDXZ 000000018002e6b0     PhysX3CommonPROFILE_x64:PhysX3CommonPROFILE_x64.dll
 0003:000006b8       __imp_?getLocalBounds@TriangleMesh@Gu@physx@@UEBA?AVPxBounds3@3@XZ 000000018002e6b8     PhysX3CommonPROFILE_x64:PhysX3CommonPROFILE_x64.dll
 0003:000006c0       __imp_?getNbTriangles@TriangleMesh@Gu@physx@@UEBAIXZ 000000018002e6c0     PhysX3CommonPROFILE_x64:PhysX3CommonPROFILE_x64.dll
 0003:000006c8       __imp_?getNbVertices@TriangleMesh@Gu@physx@@UEBAIXZ 000000018002e6c8     PhysX3CommonPROFILE_x64:PhysX3CommonPROFILE_x64.dll
 0003:000006d0       __imp_?getReferenceCount@TriangleMesh@Gu@physx@@UEBAIXZ 000000018002e6d0     PhysX3CommonPROFILE_x64:PhysX3CommonPROFILE_x64.dll
 0003:000006d8       __imp_?getTriangleMaterialIndex@TriangleMesh@Gu@physx@@UEBAGI@Z 000000018002e6d8     PhysX3CommonPROFILE_x64:PhysX3CommonPROFILE_x64.dll
 0003:000006e0       __imp_?getTriangleMeshFlags@TriangleMesh@Gu@physx@@UEBA?AV?$PxFlags@W4Enum@PxTriangleMeshFlag@physx@@E@3@XZ 000000018002e6e0     PhysX3CommonPROFILE_x64:PhysX3CommonPROFILE_x64.dll
 0003:000006e8       __imp_?getTriangles@TriangleMesh@Gu@physx@@UEBAPEBXXZ 000000018002e6e8     PhysX3CommonPROFILE_x64:PhysX3CommonPROFILE_x64.dll
 0003:000006f0       __imp_?getTrianglesRemap@TriangleMesh@Gu@physx@@UEBAPEBIXZ 000000018002e6f0     PhysX3CommonPROFILE_x64:PhysX3CommonPROFILE_x64.dll
 0003:000006f8       __imp_?getVertices@TriangleMesh@Gu@physx@@UEBAPEBVPxVec3@3@XZ 000000018002e6f8     PhysX3CommonPROFILE_x64:PhysX3CommonPROFILE_x64.dll
 0003:00000700       __imp_?getVerticesForModification@TriangleMesh@Gu@physx@@UEAAPEAVPxVec3@3@XZ 000000018002e700     PhysX3CommonPROFILE_x64:PhysX3CommonPROFILE_x64.dll
 0003:00000708       __imp_?isKindOf@PxTriangleMesh@physx@@MEBA_NPEBD@Z 000000018002e708     PhysX3CommonPROFILE_x64:PhysX3CommonPROFILE_x64.dll
 0003:00000710       __imp_?onRefCountZero@TriangleMesh@Gu@physx@@UEAAXXZ 000000018002e710     PhysX3CommonPROFILE_x64:PhysX3CommonPROFILE_x64.dll
 0003:00000718       __imp_?refitBVH@TriangleMesh@Gu@physx@@UEAA?AVPxBounds3@3@XZ 000000018002e718     PhysX3CommonPROFILE_x64:PhysX3CommonPROFILE_x64.dll
 0003:00000720       __imp_?release@TriangleMesh@Gu@physx@@UEAAXXZ 000000018002e720     PhysX3CommonPROFILE_x64:PhysX3CommonPROFILE_x64.dll
 0003:00000728       __imp_?setupMeshInterface@InternalTriangleMesh@physx@@QEAAXXZ 000000018002e728     PhysX3CommonPROFILE_x64:PhysX3CommonPROFILE_x64.dll
 0003:00000730       \177PhysX3CommonPROFILE_x64_NULL_THUNK_DATA_DLA 000000018002e730     PhysX3CommonPROFILE_x64:PhysX3CommonPROFILE_x64.dll
 0003:00000930       __hmod__PhysX3CommonPROFILE_x64_dll 000000018002e930     PhysX3CommonPROFILE_x64:PhysX3CommonPROFILE_x64.dll
 0003:00000938       __pfnDliFailureHook2       000000018002e938     delayimp:delayhk1.obj
 0003:00000940       ?__type_info_root_node@@3U__type_info_node@@A 000000018002e940     MSVCRT:tncleanup.obj
 0003:00000958       __native_startup_lock      000000018002e958     <common>
 0003:00000960       __native_startup_state     000000018002e960     <common>
 0003:00000968       __onexitend                000000018002e968     <common>
 0003:00000970       __onexitbegin              000000018002e970     <common>
 0003:00000978       __dyn_tls_init_callback    000000018002e978     <common>

 entry point at        0001:00024b48

 Static symbols

 0000:fffcd000       .debug$S                   0000000180000000     MSVCRT:MSVCR120.dll
 0000:fffcd000       .debug$S                   0000000180000000     MSVCRT:MSVCR120.dll
 0000:fffcd000       .debug$S                   0000000180000000     MSVCRT:MSVCR120.dll
 0000:fffcd000       .debug$S                   0000000180000000     MSVCRT:MSVCR120.dll
 0000:fffcd000       .debug$S                   0000000180000000     MSVCRT:MSVCR120.dll
 0000:fffcd000       .debug$S                   0000000180000000     MSVCRT:MSVCR120.dll
 0000:fffcd000       .debug$S                   0000000180000000     MSVCRT:MSVCR120.dll
 0000:fffcd000       .debug$S                   0000000180000000     MSVCRT:MSVCR120.dll
 0004:fffd1000       $pdata$?memCopy@intrinsics@physx@@YAPEAXPEIAXPEIBXI@Z 0000000180000000     VolumeIntegration.obj
 0002:fffd9000       $unwind$?normalize@PxVec3@physx@@QEAAMXZ 0000000180000000     VolumeIntegration.obj
 0000:fffcd000       .debug$S                   0000000180000000     MSVCRT:MSVCR120.dll
 0000:fffcd000       .debug$S                   0000000180000000     MSVCRT:MSVCR120.dll
 0000:fffcd000       .debug$S                   0000000180000000     MSVCRT:MSVCR120.dll
 0000:fffcd000       .debug$S                   0000000180000000     MSVCRT:MSVCR120.dll
 0000:fffcd000       .debug$S                   0000000180000000     MSVCRT:MSVCR120.dll
 0000:fffcd000       .debug$S                   0000000180000000     MSVCRT:MSVCR120.dll
 0000:fffcd000       .debug$S                   0000000180000000     MSVCRT:MSVCR120.dll
 0000:fffcd000       .debug$S                   0000000180000000     MSVCRT:MSVCR120.dll
 0000:fffcd000       .debug$S                   0000000180000000     MSVCRT:MSVCR120.dll
 0000:fffcd000       .debug$S                   0000000180000000     MSVCRT:MSVCR120.dll
 0000:fffcd000       .debug$S                   0000000180000000     MSVCRT:MSVCR120.dll
 0000:fffcd000       .debug$S                   0000000180000000     MSVCRT:MSVCR120.dll
 0000:fffcd000       .debug$S                   0000000180000000     MSVCRT:MSVCR120.dll
 0000:fffcd000       .debug$S                   0000000180000000     MSVCRT:MSVCR120.dll
 0000:fffcd000       .debug$S                   0000000180000000     MSVCRT:MSVCR120.dll
 0000:fffcd000       .debug$S                   0000000180000000     MSVCRT:MSVCR120.dll
 0000:fffcd000       .debug$S                   0000000180000000     MSVCRT:MSVCR120.dll
 0000:fffcd000       .debug$S                   0000000180000000     MSVCRT:MSVCR120.dll
 0000:fffcd000       .debug$S                   0000000180000000     MSVCRT:MSVCR120.dll
 0000:fffcd000       .debug$S                   0000000180000000     MSVCRT:MSVCR120.dll
 0000:fffcd000       .debug$S                   0000000180000000     MSVCRT:MSVCR120.dll
 0004:fffd1000       $pdata$?normalize@PxVec3@physx@@QEAAMXZ 0000000180000000     VolumeIntegration.obj
 0002:fffd9000       $unwind$?PxMemCopy@physx@@YAPEAXPEIAXPEIBXI@Z 0000000180000000     VolumeIntegration.obj
 0004:fffd1000       $pdata$?PxMemCopy@physx@@YAPEAXPEIAXPEIBXI@Z 0000000180000000     VolumeIntegration.obj
 0004:fffd1000       $pdata$1$?allocate@?$ReflectionAllocator@I@shdfnd@physx@@QEAAPEAX_KPEBDH@Z 0000000180000000     Adjacencies.obj
 0002:fffd9000       $chain$1$?allocate@?$ReflectionAllocator@I@shdfnd@physx@@QEAAPEAX_KPEBDH@Z 0000000180000000     Adjacencies.obj
 0004:fffd1000       $pdata$0$?allocate@?$ReflectionAllocator@I@shdfnd@physx@@QEAAPEAX_KPEBDH@Z 0000000180000000     Adjacencies.obj
 0002:fffd9000       $chain$0$?allocate@?$ReflectionAllocator@I@shdfnd@physx@@QEAAPEAX_KPEBDH@Z 0000000180000000     Adjacencies.obj
 0004:fffd1000       $pdata$?allocate@?$ReflectionAllocator@I@shdfnd@physx@@QEAAPEAX_KPEBDH@Z 0000000180000000     Adjacencies.obj
 0002:fffd9000       $unwind$?allocate@?$ReflectionAllocator@I@shdfnd@physx@@QEAAPEAX_KPEBDH@Z 0000000180000000     Adjacencies.obj
 0004:fffd1000       $pdata$?getName@?$ReflectionAllocator@I@shdfnd@physx@@CAPEBDXZ 0000000180000000     Adjacencies.obj
 0002:fffd9000       $unwind$?getName@?$ReflectionAllocator@I@shdfnd@physx@@CAPEBDXZ 0000000180000000     Adjacencies.obj
 0002:fffd9000       $unwind$??_H@YAXPEAX_KHP6APEAX0@Z@Z 0000000180000000     hulllib.obj
 0004:fffd1000       $pdata$??_H@YAXPEAX_KHP6APEAX0@Z@Z 0000000180000000     hulllib.obj
 0002:fffd9000       $unwind$?memCopy@intrinsics@physx@@YAPEAXPEIAXPEIBXI@Z 0000000180000000     hulllib.obj
 0004:fffd1000       $pdata$?memCopy@intrinsics@physx@@YAPEAXPEIAXPEIBXI@Z 0000000180000000     hulllib.obj
 0002:fffd9000       $unwind$?memCopy@intrinsics@physx@@YAPEAXPEIAXPEIBXI@Z 0000000180000000     InternalTriangleMeshBuilder.obj
 0004:fffd1000       $pdata$?memCopy@intrinsics@physx@@YAPEAXPEIAXPEIBXI@Z 0000000180000000     InternalTriangleMeshBuilder.obj
 0002:fffd9000       $unwind$?PxMemCopy@physx@@YAPEAXPEIAXPEIBXI@Z 0000000180000000     InternalTriangleMeshBuilder.obj
 0004:fffd1000       $pdata$?PxMemCopy@physx@@YAPEAXPEIAXPEIBXI@Z 0000000180000000     InternalTriangleMeshBuilder.obj
 0002:fffd9000       $unwind$??3UserAllocated@shdfnd@physx@@SAXPEAX@Z 0000000180000000     InternalTriangleMeshBuilder.obj
 0004:fffd1000       $pdata$??3UserAllocated@shdfnd@physx@@SAXPEAX@Z 0000000180000000     InternalTriangleMeshBuilder.obj
 0002:fffd9000       $unwind$?PxMemCopy@physx@@YAPEAXPEIAXPEIBXI@Z 0000000180000000     hulllib.obj
 0004:fffd1000       $pdata$?PxMemCopy@physx@@YAPEAXPEIAXPEIBXI@Z 0000000180000000     hulllib.obj
 0002:fffd9000       $unwind$??3UserAllocated@shdfnd@physx@@SAXPEAX@Z 0000000180000000     hulllib.obj
 0004:fffd1000       $pdata$??3UserAllocated@shdfnd@physx@@SAXPEAX@Z 0000000180000000     hulllib.obj
 0002:fffd9000       $unwind$?getName@?$ReflectionAllocator@I@shdfnd@physx@@CAPEBDXZ 0000000180000000     hulllib.obj
 0004:fffd1000       $pdata$?getName@?$ReflectionAllocator@I@shdfnd@physx@@CAPEBDXZ 0000000180000000     hulllib.obj
 0002:fffd9000       $unwind$?allocate@?$ReflectionAllocator@I@shdfnd@physx@@QEAAPEAX_KPEBDH@Z 0000000180000000     hulllib.obj
 0004:fffd1000       $pdata$?allocate@?$ReflectionAllocator@I@shdfnd@physx@@QEAAPEAX_KPEBDH@Z 0000000180000000     hulllib.obj
 0002:fffd9000       $chain$0$?allocate@?$ReflectionAllocator@I@shdfnd@physx@@QEAAPEAX_KPEBDH@Z 0000000180000000     hulllib.obj
 0004:fffd1000       $pdata$0$?allocate@?$ReflectionAllocator@I@shdfnd@physx@@QEAAPEAX_KPEBDH@Z 0000000180000000     hulllib.obj
 0002:fffd9000       $chain$1$?allocate@?$ReflectionAllocator@I@shdfnd@physx@@QEAAPEAX_KPEBDH@Z 0000000180000000     hulllib.obj
 0000:fffcd000       .debug$S                   0000000180000000     PhysX3CommonPROFILE_x64:PhysX3CommonPROFILE_x64.dll
 0000:fffcd000       .debug$S                   0000000180000000     PhysX3CommonPROFILE_x64:PhysX3CommonPROFILE_x64.dll
 0000:fffcd000       .debug$S                   0000000180000000     PhysX3CommonPROFILE_x64:PhysX3CommonPROFILE_x64.dll
 0000:fffcd000       .debug$S                   0000000180000000     PhysX3CommonPROFILE_x64:PhysX3CommonPROFILE_x64.dll
 0000:fffcd000       .debug$S                   0000000180000000     PhysX3CommonPROFILE_x64:PhysX3CommonPROFILE_x64.dll
 0000:fffcd000       .debug$S                   0000000180000000     PhysX3CommonPROFILE_x64:PhysX3CommonPROFILE_x64.dll
 0000:fffcd000       .debug$S                   0000000180000000     PhysX3CommonPROFILE_x64:PhysX3CommonPROFILE_x64.dll
 0000:fffcd000       .debug$S                   0000000180000000     PhysX3CommonPROFILE_x64:PhysX3CommonPROFILE_x64.dll
 0000:fffcd000       .debug$S                   0000000180000000     PhysX3CommonPROFILE_x64:PhysX3CommonPROFILE_x64.dll
 0000:fffcd000       .debug$S                   0000000180000000     PhysX3CommonPROFILE_x64:PhysX3CommonPROFILE_x64.dll
 0000:fffcd000       .debug$S                   0000000180000000     PhysX3CommonPROFILE_x64:PhysX3CommonPROFILE_x64.dll
 0000:fffcd000       .debug$S                   0000000180000000     PhysX3CommonPROFILE_x64:PhysX3CommonPROFILE_x64.dll
 0000:fffcd000       .debug$S                   0000000180000000     PhysX3CommonPROFILE_x64:PhysX3CommonPROFILE_x64.dll
 0000:fffcd000       .debug$S                   0000000180000000     PhysX3CommonPROFILE_x64:PhysX3CommonPROFILE_x64.dll
 0000:fffcd000       .debug$S                   0000000180000000     PhysX3CommonPROFILE_x64:PhysX3CommonPROFILE_x64.dll
 0000:fffcd000       .debug$S                   0000000180000000     PhysX3CommonPROFILE_x64:PhysX3CommonPROFILE_x64.dll
 0000:fffcd000       .debug$S                   0000000180000000     PhysX3CommonPROFILE_x64:PhysX3CommonPROFILE_x64.dll
 0000:fffcd000       .debug$S                   0000000180000000     PhysX3CommonPROFILE_x64:PhysX3CommonPROFILE_x64.dll
 0000:fffcd000       .debug$S                   0000000180000000     PhysX3CommonPROFILE_x64:PhysX3CommonPROFILE_x64.dll
 0000:fffcd000       .debug$S                   0000000180000000     PhysX3CommonPROFILE_x64:PhysX3CommonPROFILE_x64.dll
 0000:fffcd000       .debug$S                   0000000180000000     PhysX3CommonPROFILE_x64:PhysX3CommonPROFILE_x64.dll
 0000:fffcd000       .debug$S                   0000000180000000     PhysX3CommonPROFILE_x64:PhysX3CommonPROFILE_x64.dll
 0000:fffcd000       .debug$S                   0000000180000000     PhysX3CommonPROFILE_x64:PhysX3CommonPROFILE_x64.dll
 0000:fffcd000       .debug$S                   0000000180000000     PhysX3CommonPROFILE_x64:PhysX3CommonPROFILE_x64.dll
 0000:fffcd000       .debug$S                   0000000180000000     PhysX3CommonPROFILE_x64:PhysX3CommonPROFILE_x64.dll
 0000:fffcd000       .debug$S                   0000000180000000     PhysX3CommonPROFILE_x64:PhysX3CommonPROFILE_x64.dll
 0000:fffcd000       .debug$S                   0000000180000000     PhysX3CommonPROFILE_x64:PhysX3CommonPROFILE_x64.dll
 0000:fffcd000       .debug$S                   0000000180000000     PhysX3CommonPROFILE_x64:PhysX3CommonPROFILE_x64.dll
 0000:fffcd000       .debug$S                   0000000180000000     PhysX3CommonPROFILE_x64:PhysX3CommonPROFILE_x64.dll
 0000:fffcd000       .debug$S                   0000000180000000     PhysX3CommonPROFILE_x64:PhysX3CommonPROFILE_x64.dll
 0000:fffcd000       .debug$S                   0000000180000000     PhysX3CommonPROFILE_x64:PhysX3CommonPROFILE_x64.dll
 0000:fffcd000       .debug$S                   0000000180000000     PhysX3CommonPROFILE_x64:PhysX3CommonPROFILE_x64.dll
 0000:fffcd000       .debug$S                   0000000180000000     PhysX3CommonPROFILE_x64:PhysX3CommonPROFILE_x64.dll
 0000:fffcd000       .debug$S                   0000000180000000     PhysX3CommonPROFILE_x64:PhysX3CommonPROFILE_x64.dll
 0000:fffcd000       .debug$S                   0000000180000000     PhysX3CommonPROFILE_x64:PhysX3CommonPROFILE_x64.dll
 0000:fffcd000       .debug$S                   0000000180000000     PhysX3CommonPROFILE_x64:PhysX3CommonPROFILE_x64.dll
 0000:fffcd000       .debug$S                   0000000180000000     PhysX3CommonPROFILE_x64:PhysX3CommonPROFILE_x64.dll
 0002:fffd9000       $unwind$?getName@?$ReflectionAllocator@G@shdfnd@physx@@CAPEBDXZ 0000000180000000     InternalTriangleMeshBuilder.obj
 0004:fffd1000       $pdata$?getName@?$ReflectionAllocator@G@shdfnd@physx@@CAPEBDXZ 0000000180000000     InternalTriangleMeshBuilder.obj
 0002:fffd9000       $unwind$?allocate@?$ReflectionAllocator@G@shdfnd@physx@@QEAAPEAX_KPEBDH@Z 0000000180000000     InternalTriangleMeshBuilder.obj
 0004:fffd1000       $pdata$?allocate@?$ReflectionAllocator@G@shdfnd@physx@@QEAAPEAX_KPEBDH@Z 0000000180000000     InternalTriangleMeshBuilder.obj
 0002:fffd9000       $chain$0$?allocate@?$ReflectionAllocator@G@shdfnd@physx@@QEAAPEAX_KPEBDH@Z 0000000180000000     InternalTriangleMeshBuilder.obj
 0004:fffd1000       $pdata$0$?allocate@?$ReflectionAllocator@G@shdfnd@physx@@QEAAPEAX_KPEBDH@Z 0000000180000000     InternalTriangleMeshBuilder.obj
 0002:fffd9000       $chain$1$?allocate@?$ReflectionAllocator@G@shdfnd@physx@@QEAAPEAX_KPEBDH@Z 0000000180000000     InternalTriangleMeshBuilder.obj
 0004:fffd1000       $pdata$1$?allocate@?$ReflectionAllocator@G@shdfnd@physx@@QEAAPEAX_KPEBDH@Z 0000000180000000     InternalTriangleMeshBuilder.obj
 0002:fffd9000       $unwind$?getName@?$ReflectionAllocator@I@shdfnd@physx@@CAPEBDXZ 0000000180000000     InternalTriangleMeshBuilder.obj
 0004:fffd1000       $pdata$?getName@?$ReflectionAllocator@I@shdfnd@physx@@CAPEBDXZ 0000000180000000     InternalTriangleMeshBuilder.obj
 0002:fffd9000       $unwind$?allocate@?$ReflectionAllocator@I@shdfnd@physx@@QEAAPEAX_KPEBDH@Z 0000000180000000     InternalTriangleMeshBuilder.obj
 0004:fffd1000       $pdata$?allocate@?$ReflectionAllocator@I@shdfnd@physx@@QEAAPEAX_KPEBDH@Z 0000000180000000     InternalTriangleMeshBuilder.obj
 0002:fffd9000       $chain$0$?allocate@?$ReflectionAllocator@I@shdfnd@physx@@QEAAPEAX_KPEBDH@Z 0000000180000000     InternalTriangleMeshBuilder.obj
 0004:fffd1000       $pdata$0$?allocate@?$ReflectionAllocator@I@shdfnd@physx@@QEAAPEAX_KPEBDH@Z 0000000180000000     InternalTriangleMeshBuilder.obj
 0002:fffd9000       $chain$1$?allocate@?$ReflectionAllocator@I@shdfnd@physx@@QEAAPEAX_KPEBDH@Z 0000000180000000     InternalTriangleMeshBuilder.obj
 0004:fffd1000       $pdata$1$?allocate@?$ReflectionAllocator@I@shdfnd@physx@@QEAAPEAX_KPEBDH@Z 0000000180000000     InternalTriangleMeshBuilder.obj
 0002:fffd9000       $unwind$?deallocate@?$ReflectionAllocator@I@shdfnd@physx@@QEAAXPEAX@Z 0000000180000000     InternalTriangleMeshBuilder.obj
 0004:fffd1000       $pdata$?deallocate@?$ReflectionAllocator@I@shdfnd@physx@@QEAAXPEAX@Z 0000000180000000     InternalTriangleMeshBuilder.obj
 0000:fffcd000       .debug$S                   0000000180000000     PhysX3CommonPROFILE_x64:PhysX3CommonPROFILE_x64.dll
 0000:fffcd000       .debug$S                   0000000180000000     PhysX3CommonPROFILE_x64:PhysX3CommonPROFILE_x64.dll
 0002:fffd9000       $unwind$??1?$Array@IV?$ReflectionAllocator@I@shdfnd@physx@@@shdfnd@physx@@QEAA@XZ 0000000180000000     InternalTriangleMeshBuilder.obj
 0004:fffd1000       $pdata$??1?$Array@IV?$ReflectionAllocator@I@shdfnd@physx@@@shdfnd@physx@@QEAA@XZ 0000000180000000     InternalTriangleMeshBuilder.obj
 0002:fffd9000       $unwind$?deallocate@?$Array@IV?$ReflectionAllocator@I@shdfnd@physx@@@shdfnd@physx@@IEAAXPEAX@Z 0000000180000000     InternalTriangleMeshBuilder.obj
 0004:fffd1000       $pdata$?deallocate@?$Array@IV?$ReflectionAllocator@I@shdfnd@physx@@@shdfnd@physx@@IEAAXPEAX@Z 0000000180000000     InternalTriangleMeshBuilder.obj
 0002:fffd9000       $unwind$?getName@?$ReflectionAllocator@E@shdfnd@physx@@CAPEBDXZ 0000000180000000     InternalTriangleMeshBuilder.obj
 0004:fffd1000       $pdata$?getName@?$ReflectionAllocator@E@shdfnd@physx@@CAPEBDXZ 0000000180000000     InternalTriangleMeshBuilder.obj
 0002:fffd9000       $unwind$?allocate@?$ReflectionAllocator@E@shdfnd@physx@@QEAAPEAX_KPEBDH@Z 0000000180000000     InternalTriangleMeshBuilder.obj
 0004:fffd1000       $pdata$?allocate@?$ReflectionAllocator@E@shdfnd@physx@@QEAAPEAX_KPEBDH@Z 0000000180000000     InternalTriangleMeshBuilder.obj
 0002:fffd9000       $chain$0$?allocate@?$ReflectionAllocator@E@shdfnd@physx@@QEAAPEAX_KPEBDH@Z 0000000180000000     InternalTriangleMeshBuilder.obj
 0004:fffd1000       $pdata$0$?allocate@?$ReflectionAllocator@E@shdfnd@physx@@QEAAPEAX_KPEBDH@Z 0000000180000000     InternalTriangleMeshBuilder.obj
 0002:fffd9000       $chain$1$?allocate@?$ReflectionAllocator@E@shdfnd@physx@@QEAAPEAX_KPEBDH@Z 0000000180000000     InternalTriangleMeshBuilder.obj
 0004:fffd1000       $pdata$1$?allocate@?$ReflectionAllocator@E@shdfnd@physx@@QEAAPEAX_KPEBDH@Z 0000000180000000     InternalTriangleMeshBuilder.obj
 0000:fffcd000       .debug$S                   0000000180000000     PhysX3CommonPROFILE_x64:PhysX3CommonPROFILE_x64.dll
 0000:fffcd000       .debug$S                   0000000180000000     PhysX3CommonPROFILE_x64:PhysX3CommonPROFILE_x64.dll
 0000:fffcd000       .debug$S                   0000000180000000     PhysX3CommonPROFILE_x64:PhysX3CommonPROFILE_x64.dll
 0000:fffcd000       .debug$S                   0000000180000000     PhysX3CommonPROFILE_x64:PhysX3CommonPROFILE_x64.dll
 0000:fffcd000       .debug$S                   0000000180000000     PhysX3CommonPROFILE_x64:PhysX3CommonPROFILE_x64.dll
 0000:fffcd000       .debug$S                   0000000180000000     PhysX3CommonPROFILE_x64:PhysX3CommonPROFILE_x64.dll
 0000:fffcd000       .debug$S                   0000000180000000     PhysX3CommonPROFILE_x64:PhysX3CommonPROFILE_x64.dll
 0000:fffcd000       .debug$S                   0000000180000000     PhysX3CommonPROFILE_x64:PhysX3CommonPROFILE_x64.dll
 0000:fffcd000       .debug$S                   0000000180000000     PhysX3CommonPROFILE_x64:PhysX3CommonPROFILE_x64.dll
 0000:fffcd000       .debug$S                   0000000180000000     PhysX3CommonPROFILE_x64:PhysX3CommonPROFILE_x64.dll
 0000:fffcd000       .debug$S                   0000000180000000     PhysX3CommonPROFILE_x64:PhysX3CommonPROFILE_x64.dll
 0000:fffcd000       .debug$S                   0000000180000000     PhysX3CommonPROFILE_x64:PhysX3CommonPROFILE_x64.dll
 0000:fffcd000       .debug$S                   0000000180000000     PhysX3CommonPROFILE_x64:PhysX3CommonPROFILE_x64.dll
 0000:fffcd000       .debug$S                   0000000180000000     PhysX3CommonPROFILE_x64:PhysX3CommonPROFILE_x64.dll
 0004:fffd1000       $pdata$1$?allocate@?$ReflectionAllocator@I@shdfnd@physx@@QEAAPEAX_KPEBDH@Z 0000000180000000     hulllib.obj
 0002:fffd9000       $unwind$?memCopy@intrinsics@physx@@YAPEAXPEIAXPEIBXI@Z 0000000180000000     ConvexMeshBuilder.obj
 0004:fffd1000       $pdata$?memCopy@intrinsics@physx@@YAPEAXPEIAXPEIBXI@Z 0000000180000000     ConvexMeshBuilder.obj
 0002:fffd9000       $unwind$?PxMemCopy@physx@@YAPEAXPEIAXPEIBXI@Z 0000000180000000     ConvexMeshBuilder.obj
 0004:fffd1000       $pdata$?PxMemCopy@physx@@YAPEAXPEIAXPEIBXI@Z 0000000180000000     ConvexMeshBuilder.obj
 0002:fffd9000       $unwind$?gatherStrided@shdfnd@physx@@YAXPEBXPEAXIII@Z 0000000180000000     ConvexMeshBuilder.obj
 0000:fffcd000       .debug$S                   0000000180000000     PhysX3CommonPROFILE_x64:PhysX3CommonPROFILE_x64.dll
 0002:fffd9000       $unwind$??_H@YAXPEAX_KHP6APEAX0@Z@Z 0000000180000000     EdgeList.obj
 0004:fffd1000       $pdata$??_H@YAXPEAX_KHP6APEAX0@Z@Z 0000000180000000     EdgeList.obj
 0002:fffd9000       $unwind$?memZero@intrinsics@physx@@YAPEAXPEIAXI@Z 0000000180000000     EdgeList.obj
 0004:fffd1000       $pdata$?memZero@intrinsics@physx@@YAPEAXPEIAXI@Z 0000000180000000     EdgeList.obj
 0002:fffd9000       $unwind$?memCopy@intrinsics@physx@@YAPEAXPEIAXPEIBXI@Z 0000000180000000     EdgeList.obj
 0004:fffd1000       $pdata$?memCopy@intrinsics@physx@@YAPEAXPEIAXPEIBXI@Z 0000000180000000     EdgeList.obj
 0002:fffd9000       $unwind$?PxMemZero@physx@@YAPEAXPEIAXI@Z 0000000180000000     EdgeList.obj
 0004:fffd1000       $pdata$?PxMemZero@physx@@YAPEAXPEIAXI@Z 0000000180000000     EdgeList.obj
 0002:fffd9000       $unwind$?PxMemCopy@physx@@YAPEAXPEIAXPEIBXI@Z 0000000180000000     EdgeList.obj
 0004:fffd1000       $pdata$?PxMemCopy@physx@@YAPEAXPEIAXPEIBXI@Z 0000000180000000     EdgeList.obj
 0002:fffd9000       $unwind$?getNormalized@PxVec3@physx@@QEBA?AV12@XZ 0000000180000000     EdgeList.obj
 0004:fffd1000       $pdata$?getNormalized@PxVec3@physx@@QEBA?AV12@XZ 0000000180000000     EdgeList.obj
 0002:fffd9000       $unwind$?normalize@PxVec3@physx@@QEAAMXZ 0000000180000000     EdgeList.obj
 0004:fffd1000       $pdata$?normalize@PxVec3@physx@@QEAAMXZ 0000000180000000     EdgeList.obj
 0000:fffcd000       .debug$S                   0000000180000000     PhysX3CommonPROFILE_x64:PhysX3CommonPROFILE_x64.dll
 0000:fffcd000       .debug$S                   0000000180000000     PhysX3CommonPROFILE_x64:PhysX3CommonPROFILE_x64.dll
 0000:fffcd000       .debug$S                   0000000180000000     PhysX3CommonPROFILE_x64:PhysX3CommonPROFILE_x64.dll
 0000:fffcd000       .debug$S                   0000000180000000     PhysX3CommonPROFILE_x64:PhysX3CommonPROFILE_x64.dll
 0000:fffcd000       .debug$S                   0000000180000000     PhysX3CommonPROFILE_x64:PhysX3CommonPROFILE_x64.dll
 0000:fffcd000       .debug$S                   0000000180000000     PhysX3CommonPROFILE_x64:PhysX3CommonPROFILE_x64.dll
 0000:fffcd000       .debug$S                   0000000180000000     PhysX3CommonPROFILE_x64:PhysX3CommonPROFILE_x64.dll
 0000:fffcd000       .debug$S                   0000000180000000     PhysX3CommonPROFILE_x64:PhysX3CommonPROFILE_x64.dll
 0000:fffcd000       .debug$S                   0000000180000000     PhysX3CommonPROFILE_x64:PhysX3CommonPROFILE_x64.dll
 0000:fffcd000       .debug$S                   0000000180000000     PhysX3CommonPROFILE_x64:PhysX3CommonPROFILE_x64.dll
 0000:fffcd000       .debug$S                   0000000180000000     PhysX3CommonPROFILE_x64:PhysX3CommonPROFILE_x64.dll
 0000:fffcd000       .debug$S                   0000000180000000     PhysX3CommonPROFILE_x64:PhysX3CommonPROFILE_x64.dll
 0000:fffcd000       .debug$S                   0000000180000000     PhysX3CommonPROFILE_x64:PhysX3CommonPROFILE_x64.dll
 0000:fffcd000       .debug$S                   0000000180000000     PhysX3CommonPROFILE_x64:PhysX3CommonPROFILE_x64.dll
 0000:fffcd000       .debug$S                   0000000180000000     PhysX3CommonPROFILE_x64:PhysX3CommonPROFILE_x64.dll
 0000:fffcd000       .debug$S                   0000000180000000     PhysX3CommonPROFILE_x64:PhysX3CommonPROFILE_x64.dll
 0000:fffcd000       .debug$S                   0000000180000000     PhysX3CommonPROFILE_x64:PhysX3CommonPROFILE_x64.dll
 0000:fffcd000       .debug$S                   0000000180000000     PhysX3CommonPROFILE_x64:PhysX3CommonPROFILE_x64.dll
 0000:fffcd000       .debug$S                   0000000180000000     PhysX3CommonPROFILE_x64:PhysX3CommonPROFILE_x64.dll
 0000:fffcd000       .debug$S                   0000000180000000     PhysX3CommonPROFILE_x64:PhysX3CommonPROFILE_x64.dll
 0000:fffcd000       .debug$S                   0000000180000000     PhysX3CommonPROFILE_x64:PhysX3CommonPROFILE_x64.dll
 0000:fffcd000       .debug$S                   0000000180000000     PhysX3CommonPROFILE_x64:PhysX3CommonPROFILE_x64.dll
 0000:fffcd000       .debug$S                   0000000180000000     PhysX3CommonPROFILE_x64:PhysX3CommonPROFILE_x64.dll
 0000:fffcd000       .debug$S                   0000000180000000     PhysX3CommonPROFILE_x64:PhysX3CommonPROFILE_x64.dll
 0000:fffcd000       .debug$S                   0000000180000000     PhysX3CommonPROFILE_x64:PhysX3CommonPROFILE_x64.dll
 0000:fffcd000       .debug$S                   0000000180000000     PhysX3CommonPROFILE_x64:PhysX3CommonPROFILE_x64.dll
 0000:fffcd000       .debug$S                   0000000180000000     PhysX3CommonPROFILE_x64:PhysX3CommonPROFILE_x64.dll
 0000:fffcd000       .debug$S                   0000000180000000     PhysX3CommonPROFILE_x64:PhysX3CommonPROFILE_x64.dll
 0000:fffcd000       .debug$S                   0000000180000000     kernel32:KERNEL32.dll
 0000:fffcd000       .debug$S                   0000000180000000     kernel32:KERNEL32.dll
 0000:fffcd000       .debug$S                   0000000180000000     kernel32:KERNEL32.dll
 0000:fffcd000       .debug$S                   0000000180000000     kernel32:KERNEL32.dll
 0002:fffd9000       $unwind$??0PxPlane@physx@@QEAA@AEBVPxVec3@1@00@Z 0000000180000000     EdgeList.obj
 0004:fffd1000       $pdata$??0PxPlane@physx@@QEAA@AEBVPxVec3@1@00@Z 0000000180000000     EdgeList.obj
 0000:fffcd000       .debug$S                   0000000180000000     kernel32:KERNEL32.dll
 0000:fffcd000       .debug$S                   0000000180000000     kernel32:KERNEL32.dll
 0000:fffcd000       .debug$S                   0000000180000000     kernel32:KERNEL32.dll
 0000:fffcd000       .debug$S                   0000000180000000     kernel32:KERNEL32.dll
 0000:fffcd000       .debug$S                   0000000180000000     kernel32:KERNEL32.dll
 0000:fffcd000       .debug$S                   0000000180000000     kernel32:KERNEL32.dll
 0000:fffcd000       .debug$S                   0000000180000000     kernel32:KERNEL32.dll
 0000:fffcd000       .debug$S                   0000000180000000     kernel32:KERNEL32.dll
 0000:fffcd000       .debug$S                   0000000180000000     kernel32:KERNEL32.dll
 0000:fffcd000       .debug$S                   0000000180000000     kernel32:KERNEL32.dll
 0002:fffd9000       $unwind$?getName@?$ReflectionAllocator@I@shdfnd@physx@@CAPEBDXZ 0000000180000000     EdgeList.obj
 0004:fffd1000       $pdata$?getName@?$ReflectionAllocator@I@shdfnd@physx@@CAPEBDXZ 0000000180000000     EdgeList.obj
 0002:fffd9000       $unwind$?allocate@?$ReflectionAllocator@I@shdfnd@physx@@QEAAPEAX_KPEBDH@Z 0000000180000000     EdgeList.obj
 0004:fffd1000       $pdata$?allocate@?$ReflectionAllocator@I@shdfnd@physx@@QEAAPEAX_KPEBDH@Z 0000000180000000     EdgeList.obj
 0002:fffd9000       $chain$0$?allocate@?$ReflectionAllocator@I@shdfnd@physx@@QEAAPEAX_KPEBDH@Z 0000000180000000     EdgeList.obj
 0004:fffd1000       $pdata$0$?allocate@?$ReflectionAllocator@I@shdfnd@physx@@QEAAPEAX_KPEBDH@Z 0000000180000000     EdgeList.obj
 0002:fffd9000       $chain$1$?allocate@?$ReflectionAllocator@I@shdfnd@physx@@QEAAPEAX_KPEBDH@Z 0000000180000000     EdgeList.obj
 0004:fffd1000       $pdata$1$?allocate@?$ReflectionAllocator@I@shdfnd@physx@@QEAAPEAX_KPEBDH@Z 0000000180000000     EdgeList.obj
 0004:fffd1000       $pdata$?gatherStrided@shdfnd@physx@@YAXPEBXPEAXIII@Z 0000000180000000     ConvexMeshBuilder.obj
 0002:fffd9000       $chain$1$?gatherStrided@shdfnd@physx@@YAXPEBXPEAXIII@Z 0000000180000000     ConvexMeshBuilder.obj
 0004:fffd1000       $pdata$1$?gatherStrided@shdfnd@physx@@YAXPEBXPEAXIII@Z 0000000180000000     ConvexMeshBuilder.obj
 0002:fffd9000       $chain$2$?gatherStrided@shdfnd@physx@@YAXPEBXPEAXIII@Z 0000000180000000     ConvexMeshBuilder.obj
 0004:fffd1000       $pdata$2$?gatherStrided@shdfnd@physx@@YAXPEBXPEAXIII@Z 0000000180000000     ConvexMeshBuilder.obj
 0004:fffd1000       $pdata$??3UserAllocated@shdfnd@physx@@SAXPEAX@Z 0000000180000000     Adjacencies.obj
 0002:fffd9000       $unwind$??3UserAllocated@shdfnd@physx@@SAXPEAX@Z 0000000180000000     Adjacencies.obj
 0004:fffd1000       $pdata$?PxMemZero@physx@@YAPEAXPEIAXI@Z 0000000180000000     Adjacencies.obj
 0002:fffd9000       $unwind$?PxMemZero@physx@@YAPEAXPEIAXI@Z 0000000180000000     Adjacencies.obj
 0004:fffd1000       $pdata$?memZero@intrinsics@physx@@YAPEAXPEIAXI@Z 0000000180000000     Adjacencies.obj
 0002:fffd9000       $unwind$?memZero@intrinsics@physx@@YAPEAXPEIAXI@Z 0000000180000000     Adjacencies.obj
 0004:fffd1000       $pdata$??_H@YAXPEAX_KHP6APEAX0@Z@Z 0000000180000000     Adjacencies.obj
 0002:fffd9000       $unwind$??_H@YAXPEAX_KHP6APEAX0@Z@Z 0000000180000000     Adjacencies.obj
 0002:fffd9000       $unwind$??_H@YAXPEAX_KHP6APEAX0@Z@Z 0000000180000000     ConvexHullBuilder.obj
 0004:fffd1000       $pdata$??_H@YAXPEAX_KHP6APEAX0@Z@Z 0000000180000000     ConvexHullBuilder.obj
 0002:fffd9000       $unwind$?memZero@intrinsics@physx@@YAPEAXPEIAXI@Z 0000000180000000     ConvexHullBuilder.obj
 0004:fffd1000       $pdata$?memZero@intrinsics@physx@@YAPEAXPEIAXI@Z 0000000180000000     ConvexHullBuilder.obj
 0002:fffd9000       $unwind$?memCopy@intrinsics@physx@@YAPEAXPEIAXPEIBXI@Z 0000000180000000     ConvexHullBuilder.obj
 0004:fffd1000       $pdata$?memCopy@intrinsics@physx@@YAPEAXPEIAXPEIBXI@Z 0000000180000000     ConvexHullBuilder.obj
 0002:fffd9000       $unwind$?normalize@PxVec3@physx@@QEAAMXZ 0000000180000000     ConvexHullBuilder.obj
 0002:fffd9000       $unwind$?memCopy@intrinsics@physx@@YAPEAXPEIAXPEIBXI@Z 0000000180000000     VolumeIntegration.obj
 0004:fffd1000       $pdata$?normalize@PxVec3@physx@@QEAAMXZ 0000000180000000     ConvexHullBuilder.obj
 0002:fffd9000       $unwind$?PxMemZero@physx@@YAPEAXPEIAXI@Z 0000000180000000     ConvexHullBuilder.obj
 0004:fffd1000       $pdata$?PxMemZero@physx@@YAPEAXPEIAXI@Z 0000000180000000     ConvexHullBuilder.obj
 0002:fffd9000       $unwind$?getName@?$ReflectionAllocator@I@shdfnd@physx@@CAPEBDXZ 0000000180000000     CookingUtils.obj
 0004:fffd1000       $pdata$?getName@?$ReflectionAllocator@I@shdfnd@physx@@CAPEBDXZ 0000000180000000     CookingUtils.obj
 0002:fffd9000       $unwind$?allocate@?$ReflectionAllocator@I@shdfnd@physx@@QEAAPEAX_KPEBDH@Z 0000000180000000     CookingUtils.obj
 0004:fffd1000       $pdata$?allocate@?$ReflectionAllocator@I@shdfnd@physx@@QEAAPEAX_KPEBDH@Z 0000000180000000     CookingUtils.obj
 0002:fffd9000       $chain$0$?allocate@?$ReflectionAllocator@I@shdfnd@physx@@QEAAPEAX_KPEBDH@Z 0000000180000000     CookingUtils.obj
 0004:fffd1000       $pdata$0$?allocate@?$ReflectionAllocator@I@shdfnd@physx@@QEAAPEAX_KPEBDH@Z 0000000180000000     CookingUtils.obj
 0002:fffd9000       $chain$1$?allocate@?$ReflectionAllocator@I@shdfnd@physx@@QEAAPEAX_KPEBDH@Z 0000000180000000     CookingUtils.obj
 0004:fffd1000       $pdata$1$?allocate@?$ReflectionAllocator@I@shdfnd@physx@@QEAAPEAX_KPEBDH@Z 0000000180000000     CookingUtils.obj
 0002:fffd9000       $unwind$?getName@?$ReflectionAllocator@M@shdfnd@physx@@CAPEBDXZ 0000000180000000     CookingUtils.obj
 0004:fffd1000       $pdata$?getName@?$ReflectionAllocator@M@shdfnd@physx@@CAPEBDXZ 0000000180000000     CookingUtils.obj
 0002:fffd9000       $unwind$?allocate@?$ReflectionAllocator@M@shdfnd@physx@@QEAAPEAX_KPEBDH@Z 0000000180000000     CookingUtils.obj
 0004:fffd1000       $pdata$?allocate@?$ReflectionAllocator@M@shdfnd@physx@@QEAAPEAX_KPEBDH@Z 0000000180000000     CookingUtils.obj
 0002:fffd9000       $chain$0$?allocate@?$ReflectionAllocator@M@shdfnd@physx@@QEAAPEAX_KPEBDH@Z 0000000180000000     CookingUtils.obj
 0004:fffd1000       $pdata$0$?allocate@?$ReflectionAllocator@M@shdfnd@physx@@QEAAPEAX_KPEBDH@Z 0000000180000000     CookingUtils.obj
 0002:fffd9000       $chain$1$?allocate@?$ReflectionAllocator@M@shdfnd@physx@@QEAAPEAX_KPEBDH@Z 0000000180000000     CookingUtils.obj
 0004:fffd1000       $pdata$1$?allocate@?$ReflectionAllocator@M@shdfnd@physx@@QEAAPEAX_KPEBDH@Z 0000000180000000     CookingUtils.obj
 0002:fffd9000       $unwind$?PxMemCopy@physx@@YAPEAXPEIAXPEIBXI@Z 0000000180000000     ConvexHullBuilder.obj
 0004:fffd1000       $pdata$?PxMemCopy@physx@@YAPEAXPEIAXPEIBXI@Z 0000000180000000     ConvexHullBuilder.obj
 0002:fffd9000       $unwind$?getName@?$ReflectionAllocator@E@shdfnd@physx@@CAPEBDXZ 0000000180000000     ConvexHullBuilder.obj
 0004:fffd1000       $pdata$?getName@?$ReflectionAllocator@E@shdfnd@physx@@CAPEBDXZ 0000000180000000     ConvexHullBuilder.obj
 0002:fffd9000       $unwind$?allocate@?$ReflectionAllocator@E@shdfnd@physx@@QEAAPEAX_KPEBDH@Z 0000000180000000     ConvexHullBuilder.obj
 0004:fffd1000       $pdata$?allocate@?$ReflectionAllocator@E@shdfnd@physx@@QEAAPEAX_KPEBDH@Z 0000000180000000     ConvexHullBuilder.obj
 0002:fffd9000       $chain$0$?allocate@?$ReflectionAllocator@E@shdfnd@physx@@QEAAPEAX_KPEBDH@Z 0000000180000000     ConvexHullBuilder.obj
 0004:fffd1000       $pdata$0$?allocate@?$ReflectionAllocator@E@shdfnd@physx@@QEAAPEAX_KPEBDH@Z 0000000180000000     ConvexHullBuilder.obj
 0002:fffd9000       $chain$1$?allocate@?$ReflectionAllocator@E@shdfnd@physx@@QEAAPEAX_KPEBDH@Z 0000000180000000     ConvexHullBuilder.obj
 0004:fffd1000       $pdata$1$?allocate@?$ReflectionAllocator@E@shdfnd@physx@@QEAAPEAX_KPEBDH@Z 0000000180000000     ConvexHullBuilder.obj
 0002:fffd9000       $unwind$?getName@?$ReflectionAllocator@I@shdfnd@physx@@CAPEBDXZ 0000000180000000     ConvexHullBuilder.obj
 0004:fffd1000       $pdata$?getName@?$ReflectionAllocator@I@shdfnd@physx@@CAPEBDXZ 0000000180000000     ConvexHullBuilder.obj
 0002:fffd9000       $unwind$??_H@YAXPEAX_KHP6APEAX0@Z@Z 0000000180000000     Cooking.obj
 0004:fffd1000       $pdata$??_H@YAXPEAX_KHP6APEAX0@Z@Z 0000000180000000     Cooking.obj
 0002:fffd9000       $unwind$??3UserAllocated@shdfnd@physx@@SAXPEAX@Z 0000000180000000     Cooking.obj
 0004:fffd1000       $pdata$??3UserAllocated@shdfnd@physx@@SAXPEAX@Z 0000000180000000     Cooking.obj
 0002:fffd9000       $unwind$?gatherStrided@shdfnd@physx@@YAXPEBXPEAXIII@Z 0000000180000000     Cooking.obj
 0004:fffd1000       $pdata$?gatherStrided@shdfnd@physx@@YAXPEBXPEAXIII@Z 0000000180000000     Cooking.obj
 0002:fffd9000       $chain$1$?gatherStrided@shdfnd@physx@@YAXPEBXPEAXIII@Z 0000000180000000     Cooking.obj
 0004:fffd1000       $pdata$1$?gatherStrided@shdfnd@physx@@YAXPEBXPEAXIII@Z 0000000180000000     Cooking.obj
 0002:fffd9000       $chain$2$?gatherStrided@shdfnd@physx@@YAXPEBXPEAXIII@Z 0000000180000000     Cooking.obj
 0004:fffd1000       $pdata$2$?gatherStrided@shdfnd@physx@@YAXPEBXPEAXIII@Z 0000000180000000     Cooking.obj
 0004:fffd1000       $pdata$1$?allocate@?$ReflectionAllocator@I@shdfnd@physx@@QEAAPEAX_KPEBDH@Z 0000000180000000     TriangleMeshBuilder.obj
 0002:fffd9000       $chain$1$?allocate@?$ReflectionAllocator@I@shdfnd@physx@@QEAAPEAX_KPEBDH@Z 0000000180000000     TriangleMeshBuilder.obj
 0004:fffd1000       $pdata$0$?allocate@?$ReflectionAllocator@I@shdfnd@physx@@QEAAPEAX_KPEBDH@Z 0000000180000000     TriangleMeshBuilder.obj
 0002:fffd9000       $chain$0$?allocate@?$ReflectionAllocator@I@shdfnd@physx@@QEAAPEAX_KPEBDH@Z 0000000180000000     TriangleMeshBuilder.obj
 0004:fffd1000       $pdata$?allocate@?$ReflectionAllocator@I@shdfnd@physx@@QEAAPEAX_KPEBDH@Z 0000000180000000     TriangleMeshBuilder.obj
 0002:fffd9000       $unwind$?allocate@?$ReflectionAllocator@I@shdfnd@physx@@QEAAPEAX_KPEBDH@Z 0000000180000000     TriangleMeshBuilder.obj
 0004:fffd1000       $pdata$?getName@?$ReflectionAllocator@I@shdfnd@physx@@CAPEBDXZ 0000000180000000     TriangleMeshBuilder.obj
 0002:fffd9000       $unwind$?getName@?$ReflectionAllocator@I@shdfnd@physx@@CAPEBDXZ 0000000180000000     TriangleMeshBuilder.obj
 0002:fffd9000       $unwind$?allocate@?$ReflectionAllocator@I@shdfnd@physx@@QEAAPEAX_KPEBDH@Z 0000000180000000     ConvexHullBuilder.obj
 0004:fffd1000       $pdata$?allocate@?$ReflectionAllocator@I@shdfnd@physx@@QEAAPEAX_KPEBDH@Z 0000000180000000     ConvexHullBuilder.obj
 0002:fffd9000       $chain$0$?allocate@?$ReflectionAllocator@I@shdfnd@physx@@QEAAPEAX_KPEBDH@Z 0000000180000000     ConvexHullBuilder.obj
 0004:fffd1000       $pdata$0$?allocate@?$ReflectionAllocator@I@shdfnd@physx@@QEAAPEAX_KPEBDH@Z 0000000180000000     ConvexHullBuilder.obj
 0002:fffd9000       $chain$1$?allocate@?$ReflectionAllocator@I@shdfnd@physx@@QEAAPEAX_KPEBDH@Z 0000000180000000     ConvexHullBuilder.obj
 0004:fffd1000       $pdata$1$?allocate@?$ReflectionAllocator@I@shdfnd@physx@@QEAAPEAX_KPEBDH@Z 0000000180000000     ConvexHullBuilder.obj
 0002:fffd9000       $unwind$?getName@?$ReflectionAllocator@G@shdfnd@physx@@CAPEBDXZ 0000000180000000     ConvexHullBuilder.obj
 0004:fffd1000       $pdata$?getName@?$ReflectionAllocator@G@shdfnd@physx@@CAPEBDXZ 0000000180000000     ConvexHullBuilder.obj
 0002:fffd9000       $unwind$?allocate@?$ReflectionAllocator@G@shdfnd@physx@@QEAAPEAX_KPEBDH@Z 0000000180000000     ConvexHullBuilder.obj
 0004:fffd1000       $pdata$?allocate@?$ReflectionAllocator@G@shdfnd@physx@@QEAAPEAX_KPEBDH@Z 0000000180000000     ConvexHullBuilder.obj
 0002:fffd9000       $chain$0$?allocate@?$ReflectionAllocator@G@shdfnd@physx@@QEAAPEAX_KPEBDH@Z 0000000180000000     ConvexHullBuilder.obj
 0004:fffd1000       $pdata$0$?allocate@?$ReflectionAllocator@G@shdfnd@physx@@QEAAPEAX_KPEBDH@Z 0000000180000000     ConvexHullBuilder.obj
 0002:fffd9000       $chain$1$?allocate@?$ReflectionAllocator@G@shdfnd@physx@@QEAAPEAX_KPEBDH@Z 0000000180000000     ConvexHullBuilder.obj
 0004:fffd1000       $pdata$1$?allocate@?$ReflectionAllocator@G@shdfnd@physx@@QEAAPEAX_KPEBDH@Z 0000000180000000     ConvexHullBuilder.obj
 0001:00000000       ??__EmaxFError@_VecMathTests@aos@shdfnd@physx@@YAXXZ 0000000180001000 f   RTreeCooking.obj
 0001:00000020       ??__EmaxV3Error@_VecMathTests@aos@shdfnd@physx@@YAXXZ 0000000180001020 f   RTreeCooking.obj
 0001:00000030       ??__EmaxV4Error@_VecMathTests@aos@shdfnd@physx@@YAXXZ 0000000180001030 f   RTreeCooking.obj
 0001:00000050       ??__EminFError@_VecMathTests@aos@shdfnd@physx@@YAXXZ 0000000180001050 f   RTreeCooking.obj
 0001:00000070       ??__EminV3Error@_VecMathTests@aos@shdfnd@physx@@YAXXZ 0000000180001070 f   RTreeCooking.obj
 0001:00000080       ??__EminV4Error@_VecMathTests@aos@shdfnd@physx@@YAXXZ 0000000180001080 f   RTreeCooking.obj
 0001:000000a0       ??__EmaxFError@_VecMathTests@aos@shdfnd@physx@@YAXXZ 00000001800010a0 f   TriangleMeshBuilder.obj
 0001:000000c0       ??__EmaxV3Error@_VecMathTests@aos@shdfnd@physx@@YAXXZ 00000001800010c0 f   TriangleMeshBuilder.obj
 0001:000000d0       ??__EmaxV4Error@_VecMathTests@aos@shdfnd@physx@@YAXXZ 00000001800010d0 f   TriangleMeshBuilder.obj
 0001:000000f0       ??__EminFError@_VecMathTests@aos@shdfnd@physx@@YAXXZ 00000001800010f0 f   TriangleMeshBuilder.obj
 0001:00000110       ??__EminV3Error@_VecMathTests@aos@shdfnd@physx@@YAXXZ 0000000180001110 f   TriangleMeshBuilder.obj
 0001:00000120       ??__EminV4Error@_VecMathTests@aos@shdfnd@physx@@YAXXZ 0000000180001120 f   TriangleMeshBuilder.obj
 0001:00000140       ??__EmaxFError@_VecMathTests@aos@shdfnd@physx@@YAXXZ 0000000180001140 f   ConvexMeshBuilder.obj
 0001:00000160       ??__EmaxV3Error@_VecMathTests@aos@shdfnd@physx@@YAXXZ 0000000180001160 f   ConvexMeshBuilder.obj
 0001:00000170       ??__EmaxV4Error@_VecMathTests@aos@shdfnd@physx@@YAXXZ 0000000180001170 f   ConvexMeshBuilder.obj
 0001:00000190       ??__EminFError@_VecMathTests@aos@shdfnd@physx@@YAXXZ 0000000180001190 f   ConvexMeshBuilder.obj
 0001:000001b0       ??__EminV3Error@_VecMathTests@aos@shdfnd@physx@@YAXXZ 00000001800011b0 f   ConvexMeshBuilder.obj
 0001:000001c0       ??__EminV4Error@_VecMathTests@aos@shdfnd@physx@@YAXXZ 00000001800011c0 f   ConvexMeshBuilder.obj
 0001:000001e0       ??__EmaxFError@_VecMathTests@aos@shdfnd@physx@@YAXXZ 00000001800011e0 f   Cooking.obj
 0001:00000200       ??__EmaxV3Error@_VecMathTests@aos@shdfnd@physx@@YAXXZ 0000000180001200 f   Cooking.obj
 0001:00000210       ??__EmaxV4Error@_VecMathTests@aos@shdfnd@physx@@YAXXZ 0000000180001210 f   Cooking.obj
 0001:00000230       ??__EminFError@_VecMathTests@aos@shdfnd@physx@@YAXXZ 0000000180001230 f   Cooking.obj
 0001:00000250       ??__EminV3Error@_VecMathTests@aos@shdfnd@physx@@YAXXZ 0000000180001250 f   Cooking.obj
 0001:00000260       ??__EminV4Error@_VecMathTests@aos@shdfnd@physx@@YAXXZ 0000000180001260 f   Cooking.obj
 0001:00000280       ??__EmaxFError@_VecMathTests@aos@shdfnd@physx@@YAXXZ 0000000180001280 f   InternalTriangleMeshBuilder.obj
 0001:000002a0       ??__EmaxV3Error@_VecMathTests@aos@shdfnd@physx@@YAXXZ 00000001800012a0 f   InternalTriangleMeshBuilder.obj
 0001:000002b0       ??__EmaxV4Error@_VecMathTests@aos@shdfnd@physx@@YAXXZ 00000001800012b0 f   InternalTriangleMeshBuilder.obj
 0001:000002d0       ??__EminFError@_VecMathTests@aos@shdfnd@physx@@YAXXZ 00000001800012d0 f   InternalTriangleMeshBuilder.obj
 0001:000002f0       ??__EminV3Error@_VecMathTests@aos@shdfnd@physx@@YAXXZ 00000001800012f0 f   InternalTriangleMeshBuilder.obj
 0001:00000300       ??__EminV4Error@_VecMathTests@aos@shdfnd@physx@@YAXXZ 0000000180001300 f   InternalTriangleMeshBuilder.obj
 0001:00000360       $LN12                      0000000180001360     WindowsCookingDelayLoadHook.obj
 0001:00000d00       ?buildFromBounds@physx@@YAXAEAURTree@Gu@1@PEBUPxBounds3V@1@IAEAV?$Array@IV?$ReflectionAllocator@I@shdfnd@physx@@@shdfnd@1@PEAURemapCallback@RTreeCooker@1@AEAT__m128@@4MW4Enum@PxMeshCookingHint@1@@Z 0000000180001d00 f   RTreeCooking.obj
 0001:00001780       ?PxSAH@physx@@YAXAEBT__m128@@AEAM@Z 0000000180002780 f   RTreeCooking.obj
 0001:00007644       $LN58                      0000000180008644     BigConvexDataBuilder.obj
 0001:00008440       ??Dphysx@@YA?AVPxVec3@0@MAEBV10@@Z 0000000180009440 f   ConvexHullBuilder.obj
 0001:0000b650       ?inverseBuffer@@YA_NIPEAE@Z 000000018000c650 f   ConvexHullBuilder.obj
 0001:0000b6c0       ?negatePlane@@YAXAEAUHullPolygonData@Gu@physx@@@Z 000000018000c6c0 f   ConvexHullBuilder.obj
 0001:0000b6e0       ?findLineStrip@@YA_NAEAVContainer@Gu@physx@@AEBV123@@Z 000000018000c6e0 f   ConvexHullBuilder.obj
 0001:0000b970       ?CheckRedundantVertices@@YAXAEAIAEAVContainer@Gu@physx@@AEBVConvexHullBuilder@3@11@Z 000000018000c970 f   ConvexHullBuilder.obj
 0001:0000bef0       ?ExtractHullPolygons@@YA_NAEAIAEAVContainer@Gu@physx@@AEBVConvexHullBuilder@3@PEAV123@1@Z 000000018000cef0 f   ConvexHullBuilder.obj
 0001:0000c640       ?FloodFill@Local@?8??ExtractHullPolygons@@YA_NAEAIAEAVContainer@Gu@physx@@AEBVConvexHullBuilder@5@PEAV345@1@Z@SAX1PEBVAdjTriangle@5@IPEA_N@Z 000000018000d640 f   ConvexHullBuilder.obj
 0001:0000c730       ?GetNeighborFace@Local@?8??ExtractHullPolygons@@YA_NAEAIAEAVContainer@Gu@physx@@AEBVConvexHullBuilder@5@PEAV345@1@Z@SA_NIIPEBVAdjTriangle@5@PEBI00@Z 000000018000d730 f   ConvexHullBuilder.obj
 0001:0000c8b0       ?CheckFloodFillFace@Local@?8??ExtractHullPolygons@@YA_NAEAIAEAVContainer@Gu@physx@@AEBVConvexHullBuilder@5@PEAV345@1@Z@SA_NIPEBVAdjTriangle@5@PEBI@Z 000000018000d8b0 f   ConvexHullBuilder.obj
 0001:0000cb00       ?CheckFloodFill@Local@?8??ExtractHullPolygons@@YA_NAEAIAEAVContainer@Gu@physx@@AEBVConvexHullBuilder@5@PEAV345@1@Z@SA_N1PEAVAdjTriangle@5@PEA_NPEBI@Z 000000018000db00 f   ConvexHullBuilder.obj
 0001:0000cc80       ?TestDuplicateTriangles@@YA_NAEAIPEAU?$TriangleT@I@Gu@physx@@_N@Z 000000018000dc80 f   ConvexHullBuilder.obj
 0001:0000cdb0       ?testCulling@@YA_NAEBU?$TriangleT@I@Gu@physx@@PEBVPxVec3@3@AEBV43@@Z 000000018000ddb0 f   ConvexHullBuilder.obj
 0001:0000cf60       ?TestUnifiedNormals@@YA_NIPEBVPxVec3@physx@@IPEAU?$TriangleT@I@Gu@2@_N@Z 000000018000df60 f   ConvexHullBuilder.obj
 0001:0000d530       ?cleanMesh@@YA_NAEAI0PEAVPxVec3@physx@@PEAU?$TriangleT@I@Gu@2@@Z 000000018000e530 f   ConvexHullBuilder.obj
 0001:0000d600       ?CleanHull@@YA_NAEAIPEAU?$TriangleT@I@Gu@physx@@0PEAVPxVec3@3@@Z 000000018000e600 f   ConvexHullBuilder.obj
 0001:0000d6a0       ?CheckHull@@YA_NIPEBU?$TriangleT@I@Gu@physx@@IPEBVPxVec3@3@@Z 000000018000e6a0 f   ConvexHullBuilder.obj
 0001:0000d710       ?computeNewellPlane@@YA_NAEAVPxPlane@physx@@IPEBEPEBVPxVec3@2@@Z 000000018000e710 f   ConvexHullBuilder.obj
 0001:0000f3e0       ?ComputeAABBNoTransform@@YAXAEAVPxVec3@physx@@0IPEBV12@@Z 00000001800103e0 f   ConvexMeshBuilder.obj
 0001:0000f610       ?TestContainment@@YA_NAEBVPxVec3@physx@@QEBMIPEBUHullPolygonData@Gu@2@@Z 0000000180010610 f   ConvexMeshBuilder.obj
 0001:00013ac0       ?sqr@physx@@YAMM@Z         0000000180014ac0 f   hulllib.obj
 0001:00013ad0       ??Hphysx@@YA?AVfloat3@0@AEBV10@0@Z 0000000180014ad0 f   hulllib.obj
 0001:00013b10       ??Gphysx@@YA?AVfloat3@0@AEBV10@0@Z 0000000180014b10 f   hulllib.obj
 0001:00013b50       ??Gphysx@@YA?AVfloat3@0@AEBV10@@Z 0000000180014b50 f   hulllib.obj
 0001:00013b90       ??Dphysx@@YA?AVfloat3@0@AEBV10@M@Z 0000000180014b90 f   hulllib.obj
 0001:00013bc0       ??Kphysx@@YA?AVfloat3@0@AEBV10@M@Z 0000000180014bc0 f   hulllib.obj
 0001:00013c00       ?dot@physx@@YAMAEBVfloat3@1@0@Z 0000000180014c00 f   hulllib.obj
 0001:00013c30       ?cross@physx@@YA?AVfloat3@1@AEBV21@0@Z 0000000180014c30 f   hulllib.obj
 0001:00013c90       ??Yphysx@@YAAEAVfloat3@0@AEAV10@AEBV10@@Z 0000000180014c90 f   hulllib.obj
 0001:00013cd0       ?magnitude@physx@@YAMAEBVfloat3@1@@Z 0000000180014cd0 f   hulllib.obj
 0001:00013d00       ?normalize@physx@@YA?AVfloat3@1@AEBV21@@Z 0000000180014d00 f   hulllib.obj
 0001:00013da0       ?VectorMin@physx@@YA?AVfloat3@1@AEBV21@0@Z 0000000180014da0 f   hulllib.obj
 0001:00013df0       ?VectorMax@physx@@YA?AVfloat3@1@AEBV21@0@Z 0000000180014df0 f   hulllib.obj
 0001:00013e40       ?Determinant@physx@@YAMAEBVfloat3x3@1@@Z 0000000180014e40 f   hulllib.obj
 0001:00013ef0       ?Inverse@physx@@YA?AVfloat3x3@1@AEBV21@@Z 0000000180014ef0 f   hulllib.obj
 0001:000140b0       ?Transpose@physx@@YA?AVfloat3x3@1@AEBV21@@Z 00000001800150b0 f   hulllib.obj
 0001:00014130       ??Dphysx@@YA?AVfloat3@0@AEBV10@AEBVfloat3x3@0@@Z 0000000180015130 f   hulllib.obj
 0001:000141d0       ?ThreePlaneIntersection@physx@@YA?AVfloat3@1@AEBVPlane@1@00@Z 00000001800151d0 f   hulllib.obj
 0001:00014360       ?TriNormal@physx@@YA?AVfloat3@1@AEBV21@00@Z 0000000180015360 f   hulllib.obj
 0001:00014500       ?ConvexHDup@physx@@YAPEAVConvexH@1@PEAV21@@Z 0000000180015500 f   hulllib.obj
 0001:000145e0       ?PlaneTest@physx@@YAHAEBVPlane@1@AEBVfloat3@1@@Z 00000001800155e0 f   hulllib.obj
 0001:00014640       ?AssertIntact@physx@@YAHAEAVConvexH@1@@Z 0000000180015640 f   hulllib.obj
 0001:00014910       ?test_cube@physx@@YAPEAVConvexH@1@XZ 0000000180015910 f   hulllib.obj
 0001:00014d90       ?ConvexHMakeCube@physx@@YAPEAVConvexH@1@AEBVfloat3@1@0@Z 0000000180015d90 f   hulllib.obj
 0001:00015030       ?ConvexHCrop@physx@@YAPEAVConvexH@1@AEAV21@AEBVPlane@1@@Z 0000000180016030 f   hulllib.obj
 0001:00015e10       ?candidateplane@physx@@YAHPEAVPlane@1@HPEAVConvexH@1@M@Z 0000000180016e10 f   hulllib.obj
 0001:000162e0       ?orth@physx@@YA?AVfloat3@1@AEBV21@@Z 00000001800172e0 f   hulllib.obj
 0001:00016450       ?above@physx@@YAHPEAVfloat3@1@AEBVint3@1@AEBV21@M@Z 0000000180017450 f   hulllib.obj
 0001:000164f0       ?hasvert@physx@@YAHAEBVint3@1@H@Z 00000001800174f0 f   hulllib.obj
 0001:00016510       ?deleteTri@physx@@YAXPEAVTri@1@PEAV?$Array@PEAVTri@physx@@@hullLibArray@1@@Z 0000000180017510 f   hulllib.obj
 0001:000165f0       ?hasVolume@physx@@YA_NPEAVfloat3@1@HHHH@Z 00000001800175f0 f   hulllib.obj
 0001:000167c0       ?FindSimplex@physx@@YA?AVint4@1@PEAVfloat3@1@HAEAV?$Array@H@hullLibArray@1@AEBV31@@Z 00000001800177c0 f   hulllib.obj
 0001:00016f20       ?PlaneCheck@LocalTests@?1??expandhull@HullLibrary@physx@@AEAA?AW4HullError@4@PEAVfloat3@4@HAEAPEAV64@AEAHM@Z@SA_NPEBV64@HAEAV?$Array@UExpandPlane@physx@@@hullLibArray@4@@Z 0000000180017f20 f   hulllib.obj
 0001:00016ff0       ?area2@physx@@YAMAEBVfloat3@1@00@Z 0000000180017ff0 f   hulllib.obj
 0001:00017090       ?overhull@physx@@YA?AW4HullError@1@PEAVPlane@1@HPEAVfloat3@1@HHAEAPEAV41@AEAHAEAPEAH3M@Z 0000000180018090 f   hulllib.obj
 0001:00017780       ?ReleaseHull@physx@@YAXAEAVPHullResult@1@@Z 0000000180018780 f   hulllib.obj
 0001:000177d0       ?BringOutYourDead@physx@@YAXPEBMIPEAMAEAIPEAII@Z 00000001800187d0 f   hulllib.obj
 0001:00017b00       ?AddPoint@physx@@YAXAEAIPEAMMMM@Z 0000000180018b00 f   hulllib.obj
 0001:00017b30       ?GetDist@physx@@YAMMMMPEBM@Z 0000000180018b30 f   hulllib.obj
 0001:00017b60       ?CleanupVertices@physx@@YA_NIPEBMIAEAIPEAMM2@Z 0000000180018b60 f   hulllib.obj
 0001:00018320       ?ComputeNormal@physx@@YAMPEAMPEBM11@Z 0000000180019320 f   hulllib.obj
 0001:00018440       ?AddConvexTriangle@physx@@YAXPEAVConvexHullTriangleInterface@1@PEBM11@Z 0000000180019440 f   hulllib.obj
 0001:0001a290       ??Dphysx@@YA?AVPxVec3@0@MAEBV10@@Z 000000018001b290 f   VolumeIntegration.obj
 0001:0001d090       ?_WalkFace@Local@?1??Walk@Adjacencies@physx@@QEAA_NP6AXAEBUCommonWalkParams@4@IIII@ZPEAX@Z@SAXAEAUPrivateWalkParams@?1??234@QEAA_N12@Z@IIII@Z 000000018001e090 f   Adjacencies.obj
 0001:0001d1b0       ?_WalkFace@Local@?1??Walk2@Adjacencies@physx@@QEAA_NP6AXAEBUCommonWalkParams@4@IIII@ZPEAXPEBVPxVec3@4@PEBU?$TriangleT@I@Gu@4@@Z@SAXAEAUPrivateWalkParams@?1??234@QEAA_N1234@Z@IIII@Z 000000018001e1b0 f   Adjacencies.obj
 0001:0001d600       ?AddEdge@@YAXIIIAEAIPEAVAdjEdge@@@Z 000000018001e600 f   Adjacencies.obj
 0001:0001d640       ?AddTriangle@@YAXIIIIPEAVAdjTriangle@physx@@AEAIPEAVAdjEdge@@@Z 000000018001e640 f   Adjacencies.obj
 0001:0001d740       ?UpdateLink@@YA_NIIIIPEAVAdjTriangle@physx@@AEBUADJACENCIESCREATE@2@@Z 000000018001e740 f   Adjacencies.obj
 0001:0001d980       ?CreateDatabase@@YA_NPEAVAdjTriangle@physx@@IPEBVAdjEdge@@AEBUADJACENCIESCREATE@2@@Z 000000018001e980 f   Adjacencies.obj
 0001:00023a20       ?getHashValue@@YAIAEBVPxVec3@physx@@@Z 0000000180024a20 f   MeshCleaner.obj
 0001:00023a50       ?getHashValue@@YAIAEBUIndices@@@Z 0000000180024a50 f   MeshCleaner.obj
 0001:00024254       ?FLoadedAtPreferredAddress@@YA_NPEAU_IMAGE_NT_HEADERS64@@PEAUHINSTANCE__@@@Z 0000000180025254 f   delayimp:delayhlp.obj
 0001:00024268       ?OverlayIAT@@YAXPEAU_IMAGE_THUNK_DATA64@@PEBU1@@Z 0000000180025268 f   delayimp:delayhlp.obj
 0001:0002429c       ?PiddFromDllName@@YAPEBUImgDelayDescr@@PEBD@Z 000000018002529c f   delayimp:delayhlp.obj
 0001:0002433c       ?PinhFromImageBase@@YAPEAU_IMAGE_NT_HEADERS64@@PEAUHINSTANCE__@@@Z 000000018002533c f   delayimp:delayhlp.obj
 0001:00024344       ?TimeStampOfImage@@YAKPEAU_IMAGE_NT_HEADERS64@@@Z 0000000180025344 f   delayimp:delayhlp.obj
 0001:00024348       ?__memcmp@@YAHPEBX0_K@Z    0000000180025348 f   delayimp:delayhlp.obj
 0001:0002436c       ?__memcpy@@YAPEAXPEAXPEBX_K@Z 000000018002536c f   delayimp:delayhlp.obj
 0001:0002438c       ?__strlen@@YA_KPEBD@Z      000000018002538c f   delayimp:delayhlp.obj
 0001:00024770       $$000000                   0000000180025770     MSVCRT:chkstk.obj
 0001:00024890       pre_c_init                 0000000180025890 f   MSVCRT:crtdll.obj
 0001:00024b88       __DllMainCRTStartup        0000000180025b88 f   MSVCRT:crtdll.obj
 0001:00024d2c       ?ArrayUnwindFilter@@YAHPEAU_EXCEPTION_POINTERS@@@Z 0000000180025d2c f   MSVCRT:ehvecdtr.obj
 0001:00025160       __DllMainCRTStartup$filt$0 0000000180026160 f   MSVCRT:crtdll.obj
 0001:00025185       __DllMainCRTStartup$fin$1  0000000180026185 f   MSVCRT:crtdll.obj
 0001:0002519f       ?fin$0@?0???_M@YAXPEAX_KHP6AX0@Z@Z@4HA 000000018002619f f   MSVCRT:ehvecdtr.obj
 0001:000251cb       ?filt$0@?0??__ArrayUnwind@@YAXPEAX_KHP6AX0@Z@Z@4HA 00000001800261cb f   MSVCRT:ehvecdtr.obj
 0001:00025210       _IsNonwritableInCurrentImage$filt$0 0000000180026210 f   MSVCRT:pesect.obj
 0001:00025230       _onexit$fin$0              0000000180026230 f   MSVCRT:atonexit.obj
 0002:00000170       minFError$initializer$     0000000180027170     RTreeCooking.obj
 0002:00000178       maxFError$initializer$     0000000180027178     RTreeCooking.obj
 0002:00000180       minV3Error$initializer$    0000000180027180     RTreeCooking.obj
 0002:00000188       maxV3Error$initializer$    0000000180027188     RTreeCooking.obj
 0002:00000190       minV4Error$initializer$    0000000180027190     RTreeCooking.obj
 0002:00000198       maxV4Error$initializer$    0000000180027198     RTreeCooking.obj
 0002:000001a0       minFError$initializer$     00000001800271a0     TriangleMeshBuilder.obj
 0002:000001a8       maxFError$initializer$     00000001800271a8     TriangleMeshBuilder.obj
 0002:000001b0       minV3Error$initializer$    00000001800271b0     TriangleMeshBuilder.obj
 0002:000001b8       maxV3Error$initializer$    00000001800271b8     TriangleMeshBuilder.obj
 0002:000001c0       minV4Error$initializer$    00000001800271c0     TriangleMeshBuilder.obj
 0002:000001c8       maxV4Error$initializer$    00000001800271c8     TriangleMeshBuilder.obj
 0002:000001d0       minFError$initializer$     00000001800271d0     ConvexMeshBuilder.obj
 0002:000001d8       maxFError$initializer$     00000001800271d8     ConvexMeshBuilder.obj
 0002:000001e0       minV3Error$initializer$    00000001800271e0     ConvexMeshBuilder.obj
 0002:000001e8       maxV3Error$initializer$    00000001800271e8     ConvexMeshBuilder.obj
 0002:000001f0       minV4Error$initializer$    00000001800271f0     ConvexMeshBuilder.obj
 0002:000001f8       maxV4Error$initializer$    00000001800271f8     ConvexMeshBuilder.obj
 0002:00000200       minFError$initializer$     0000000180027200     Cooking.obj
 0002:00000208       maxFError$initializer$     0000000180027208     Cooking.obj
 0002:00000210       minV3Error$initializer$    0000000180027210     Cooking.obj
 0002:00000218       maxV3Error$initializer$    0000000180027218     Cooking.obj
 0002:00000220       minV4Error$initializer$    0000000180027220     Cooking.obj
 0002:00000228       maxV4Error$initializer$    0000000180027228     Cooking.obj
 0002:00000230       minFError$initializer$     0000000180027230     InternalTriangleMeshBuilder.obj
 0002:00000238       maxFError$initializer$     0000000180027238     InternalTriangleMeshBuilder.obj
 0002:00000240       minV3Error$initializer$    0000000180027240     InternalTriangleMeshBuilder.obj
 0002:00000248       maxV3Error$initializer$    0000000180027248     InternalTriangleMeshBuilder.obj
 0002:00000250       minV4Error$initializer$    0000000180027250     InternalTriangleMeshBuilder.obj
 0002:00000258       maxV4Error$initializer$    0000000180027258     InternalTriangleMeshBuilder.obj
 0002:00000270       pcinit                     0000000180027270     MSVCRT:crtdll.obj
 0002:00000278       pinit                      0000000180027278     MSVCRT:atonexit.obj
 0002:000004b8       PxPi                       00000001800274b8     HeightFieldCooking.obj
 0002:000005fc       PxPi                       00000001800275fc     RTreeCooking.obj
 0002:00000624       PxTwoPi                    0000000180027624     RTreeCooking.obj
 0002:00000628       PxInvPi                    0000000180027628     RTreeCooking.obj
 0002:0000062c       PxInvTwoPi                 000000018002762c     RTreeCooking.obj
 0002:00000630       gMaskXYZ                   0000000180027630     RTreeCooking.obj
 0002:00000640       PxPiDivTwo                 0000000180027640     RTreeCooking.obj
 0002:00000648       stopAtTrisPerPage          0000000180027648     RTreeCooking.obj
 0002:00000688       stopAtTrisPerLeaf          0000000180027688     RTreeCooking.obj
 0002:000008f0       gMaskXYZ                   00000001800278f0     TriangleMeshBuilder.obj
 0002:00000900       PxPi                       0000000180027900     TriangleMeshBuilder.obj
 0002:00000904       PxTwoPi                    0000000180027904     TriangleMeshBuilder.obj
 0002:00000908       PxInvPi                    0000000180027908     TriangleMeshBuilder.obj
 0002:0000090c       PxInvTwoPi                 000000018002790c     TriangleMeshBuilder.obj
 0002:00000910       PxPiDivTwo                 0000000180027910     TriangleMeshBuilder.obj
 0002:00000a20       PxPi                       0000000180027a20     BigConvexDataBuilder.obj
 0002:00000a80       PxPi                       0000000180027a80     ConvexHullBuilder.obj
 0002:00000dd0       gMaskXYZ                   0000000180027dd0     ConvexMeshBuilder.obj
 0002:00000de0       PxPi                       0000000180027de0     ConvexMeshBuilder.obj
 0002:00000de4       PxTwoPi                    0000000180027de4     ConvexMeshBuilder.obj
 0002:00000de8       PxInvPi                    0000000180027de8     ConvexMeshBuilder.obj
 0002:00000dec       PxInvTwoPi                 0000000180027dec     ConvexMeshBuilder.obj
 0002:00000df0       PxPiDivTwo                 0000000180027df0     ConvexMeshBuilder.obj
 0002:00001150       minadjangle                0000000180028150     hulllib.obj
 0002:00001260       PxPi                       0000000180028260     VolumeIntegration.obj
 0002:000014c0       PxPi                       00000001800284c0     Cooking.obj
 0002:000014c4       PxTwoPi                    00000001800284c4     Cooking.obj
 0002:000014c8       PxInvPi                    00000001800284c8     Cooking.obj
 0002:000014cc       PxInvTwoPi                 00000001800284cc     Cooking.obj
 0002:000014d0       PxPiDivTwo                 00000001800284d0     Cooking.obj
 0002:000014e0       gMaskXYZ                   00000001800284e0     Cooking.obj
 0002:00001910       PxPi                       0000000180028910     EdgeList.obj
 0002:00001ac0       gMaskXYZ                   0000000180028ac0     InternalTriangleMeshBuilder.obj
 0002:00001ad0       PxPi                       0000000180028ad0     InternalTriangleMeshBuilder.obj
 0002:00001ad4       PxTwoPi                    0000000180028ad4     InternalTriangleMeshBuilder.obj
 0002:00001ad8       PxInvPi                    0000000180028ad8     InternalTriangleMeshBuilder.obj
 0002:00001adc       PxInvTwoPi                 0000000180028adc     InternalTriangleMeshBuilder.obj
 0002:00001ae0       PxPiDivTwo                 0000000180028ae0     InternalTriangleMeshBuilder.obj
 0002:00001e38       $unwind$?physXCommonDliNotePreLoadLibrary@shdfnd@physx@@YAP6A_JXZPEBDPEBVPxDelayLoadHook@2@@Z 0000000180028e38     WindowsCookingDelayLoadHook.obj
 0002:00001e44       $unwind$?saveHeightField@physx@@YA_NAEBVHeightField@Gu@1@AEAVPxOutputStream@1@_N@Z 0000000180028e44     HeightFieldCooking.obj
 0002:00001e54       $chain$1$?saveHeightField@physx@@YA_NAEBVHeightField@Gu@1@AEAVPxOutputStream@1@_N@Z 0000000180028e54     HeightFieldCooking.obj
 0002:00001e6c       $chain$2$?saveHeightField@physx@@YA_NAEBVHeightField@Gu@1@AEAVPxOutputStream@1@_N@Z 0000000180028e6c     HeightFieldCooking.obj
 0002:00001e7c       $unwind$?memCopy@intrinsics@physx@@YAPEAXPEIAXPEIBXI@Z 0000000180028e7c     RTreeCooking.obj
 0002:00001e84       $unwind$?PxMemCopy@physx@@YAPEAXPEIAXPEIBXI@Z 0000000180028e84     RTreeCooking.obj
 0002:00001e8c       $unwind$?buildFromTriangles@RTreeCooker@physx@@SAXAEAURTree@Gu@2@PEBVPxVec3@2@IPEBGPEBIIAEAV?$Array@IV?$ReflectionAllocator@I@shdfnd@physx@@@shdfnd@2@PEAURemapCallback@12@MW4Enum@PxMeshCookingHint@2@@Z 0000000180028e8c     RTreeCooking.obj
 0002:00001e9c       $chain$4$?buildFromTriangles@RTreeCooker@physx@@SAXAEAURTree@Gu@2@PEBVPxVec3@2@IPEBGPEBIIAEAV?$Array@IV?$ReflectionAllocator@I@shdfnd@physx@@@shdfnd@2@PEAURemapCallback@12@MW4Enum@PxMeshCookingHint@2@@Z 0000000180028e9c     RTreeCooking.obj
 0002:00001ec0       $chain$7$?buildFromTriangles@RTreeCooker@physx@@SAXAEAURTree@Gu@2@PEBVPxVec3@2@IPEBGPEBIIAEAV?$Array@IV?$ReflectionAllocator@I@shdfnd@physx@@@shdfnd@2@PEAURemapCallback@12@MW4Enum@PxMeshCookingHint@2@@Z 0000000180028ec0     RTreeCooking.obj
 0002:00001edc       $chain$8$?buildFromTriangles@RTreeCooker@physx@@SAXAEAURTree@Gu@2@PEBVPxVec3@2@IPEBGPEBIIAEAV?$Array@IV?$ReflectionAllocator@I@shdfnd@physx@@@shdfnd@2@PEAURemapCallback@12@MW4Enum@PxMeshCookingHint@2@@Z 0000000180028edc     RTreeCooking.obj
 0002:00001eec       $chain$9$?buildFromTriangles@RTreeCooker@physx@@SAXAEAURTree@Gu@2@PEBVPxVec3@2@IPEBGPEBIIAEAV?$Array@IV?$ReflectionAllocator@I@shdfnd@physx@@@shdfnd@2@PEAURemapCallback@12@MW4Enum@PxMeshCookingHint@2@@Z 0000000180028eec     RTreeCooking.obj
 0002:00001efc       $unwind$?buildFromBounds@physx@@YAXAEAURTree@Gu@1@PEBUPxBounds3V@1@IAEAV?$Array@IV?$ReflectionAllocator@I@shdfnd@physx@@@shdfnd@1@PEAURemapCallback@RTreeCooker@1@AEAT__m128@@4MW4Enum@PxMeshCookingHint@1@@Z 0000000180028efc     RTreeCooking.obj
 0002:00001f18       $unwind$?getName@?$ReflectionAllocator@UPxBounds3V@physx@@@shdfnd@physx@@CAPEBDXZ 0000000180028f18     RTreeCooking.obj
 0002:00001f20       $unwind$?allocate@?$ReflectionAllocator@UPxBounds3V@physx@@@shdfnd@physx@@QEAAPEAX_KPEBDH@Z 0000000180028f20     RTreeCooking.obj
 0002:00001f30       $chain$0$?allocate@?$ReflectionAllocator@UPxBounds3V@physx@@@shdfnd@physx@@QEAAPEAX_KPEBDH@Z 0000000180028f30     RTreeCooking.obj
 0002:00001f44       $chain$1$?allocate@?$ReflectionAllocator@UPxBounds3V@physx@@@shdfnd@physx@@QEAAPEAX_KPEBDH@Z 0000000180028f44     RTreeCooking.obj
 0002:00001f54       $unwind$?deallocate@?$ReflectionAllocator@UPxBounds3V@physx@@@shdfnd@physx@@QEAAXPEAX@Z 0000000180028f54     RTreeCooking.obj
 0002:00001f5c       $unwind$??1?$Array@UPxBounds3V@physx@@V?$ReflectionAllocator@UPxBounds3V@physx@@@shdfnd@2@@shdfnd@physx@@QEAA@XZ 0000000180028f5c     RTreeCooking.obj
 0002:00001f64       $unwind$?deallocate@?$Array@UPxBounds3V@physx@@V?$ReflectionAllocator@UPxBounds3V@physx@@@shdfnd@2@@shdfnd@physx@@IEAAXPEAX@Z 0000000180028f64     RTreeCooking.obj
 0002:00001f6c       $unwind$?growAndPushBack@?$Array@UPxBounds3V@physx@@V?$ReflectionAllocator@UPxBounds3V@physx@@@shdfnd@2@@shdfnd@physx@@IEAAAEAUPxBounds3V@3@AEBU43@@Z 0000000180028f6c     RTreeCooking.obj
 0002:00001f80       $unwind$?recreate@?$Array@UPxBounds3V@physx@@V?$ReflectionAllocator@UPxBounds3V@physx@@@shdfnd@2@@shdfnd@physx@@IEAAXI@Z 0000000180028f80     RTreeCooking.obj
 0002:00001f94       $unwind$?getName@?$ReflectionAllocator@I@shdfnd@physx@@CAPEBDXZ 0000000180028f94     RTreeCooking.obj
 0002:00001f9c       $unwind$?allocate@?$ReflectionAllocator@I@shdfnd@physx@@QEAAPEAX_KPEBDH@Z 0000000180028f9c     RTreeCooking.obj
 0002:00001fac       $chain$0$?allocate@?$ReflectionAllocator@I@shdfnd@physx@@QEAAPEAX_KPEBDH@Z 0000000180028fac     RTreeCooking.obj
 0002:00001fc0       $chain$1$?allocate@?$ReflectionAllocator@I@shdfnd@physx@@QEAAPEAX_KPEBDH@Z 0000000180028fc0     RTreeCooking.obj
 0002:00001fd0       $unwind$?deallocate@?$ReflectionAllocator@I@shdfnd@physx@@QEAAXPEAX@Z 0000000180028fd0     RTreeCooking.obj
 0002:00001fd8       $unwind$??0?$Array@IV?$ReflectionAllocator@I@shdfnd@physx@@@shdfnd@physx@@QEAA@IAEBIAEBV?$ReflectionAllocator@I@12@@Z 0000000180028fd8     RTreeCooking.obj
 0002:00001fe0       $unwind$??1?$Array@IV?$ReflectionAllocator@I@shdfnd@physx@@@shdfnd@physx@@QEAA@XZ 0000000180028fe0     RTreeCooking.obj
 0002:00001fe8       $unwind$?resize@?$Array@IV?$ReflectionAllocator@I@shdfnd@physx@@@shdfnd@physx@@QEAAXIAEBI@Z 0000000180028fe8     RTreeCooking.obj
 0002:00001ff8       $unwind$?deallocate@?$Array@IV?$ReflectionAllocator@I@shdfnd@physx@@@shdfnd@physx@@IEAAXPEAX@Z 0000000180028ff8     RTreeCooking.obj
 0002:00002000       $unwind$?growAndPushBack@?$Array@IV?$ReflectionAllocator@I@shdfnd@physx@@@shdfnd@physx@@IEAAAEAIAEBI@Z 0000000180029000     RTreeCooking.obj
 0002:00002014       $unwind$?recreate@?$Array@IV?$ReflectionAllocator@I@shdfnd@physx@@@shdfnd@physx@@IEAAXI@Z 0000000180029014     RTreeCooking.obj
 0002:00002028       $unwind$?getName@?$ReflectionAllocator@VPxVec3@physx@@@shdfnd@physx@@CAPEBDXZ 0000000180029028     RTreeCooking.obj
 0002:00002030       $unwind$?allocate@?$ReflectionAllocator@VPxVec3@physx@@@shdfnd@physx@@QEAAPEAX_KPEBDH@Z 0000000180029030     RTreeCooking.obj
 0002:00002040       $chain$0$?allocate@?$ReflectionAllocator@VPxVec3@physx@@@shdfnd@physx@@QEAAPEAX_KPEBDH@Z 0000000180029040     RTreeCooking.obj
 0002:00002054       $chain$1$?allocate@?$ReflectionAllocator@VPxVec3@physx@@@shdfnd@physx@@QEAAPEAX_KPEBDH@Z 0000000180029054     RTreeCooking.obj
 0002:00002064       $unwind$?deallocate@?$ReflectionAllocator@VPxVec3@physx@@@shdfnd@physx@@QEAAXPEAX@Z 0000000180029064     RTreeCooking.obj
 0002:0000206c       $unwind$??1?$Array@VPxVec3@physx@@V?$ReflectionAllocator@VPxVec3@physx@@@shdfnd@2@@shdfnd@physx@@QEAA@XZ 000000018002906c     RTreeCooking.obj
 0002:00002074       $unwind$?deallocate@?$Array@VPxVec3@physx@@V?$ReflectionAllocator@VPxVec3@physx@@@shdfnd@2@@shdfnd@physx@@IEAAXPEAX@Z 0000000180029074     RTreeCooking.obj
 0002:0000207c       $unwind$?growAndPushBack@?$Array@VPxVec3@physx@@V?$ReflectionAllocator@VPxVec3@physx@@@shdfnd@2@@shdfnd@physx@@IEAAAEAVPxVec3@3@AEBV43@@Z 000000018002907c     RTreeCooking.obj
 0002:00002094       $unwind$?recreate@?$Array@VPxVec3@physx@@V?$ReflectionAllocator@VPxVec3@physx@@@shdfnd@2@@shdfnd@physx@@IEAAXI@Z 0000000180029094     RTreeCooking.obj
 0002:000020a8       $unwind$??0SubSortQuick@physx@@QEAA@PEAIPEBUPxBounds3V@1@IM@Z 00000001800290a8     RTreeCooking.obj
 0002:000020c0       $unwind$?sort4@SubSortQuick@physx@@QEAAXPEIAIIAEAV?$Array@URTreeNodeNQ@physx@@V?$ReflectionAllocator@URTreeNodeNQ@physx@@@shdfnd@2@@shdfnd@2@AEAIAEAUPxBounds3V@2@I@Z 00000001800290c0     RTreeCooking.obj
 0002:000020d0       $unwind$??1SubSortQuick@physx@@QEAA@XZ 00000001800290d0     RTreeCooking.obj
 0002:000020d8       $unwind$?getName@?$ReflectionAllocator@URTreeNodeNQ@physx@@@shdfnd@physx@@CAPEBDXZ 00000001800290d8     RTreeCooking.obj
 0002:000020e0       $unwind$?allocate@?$ReflectionAllocator@URTreeNodeNQ@physx@@@shdfnd@physx@@QEAAPEAX_KPEBDH@Z 00000001800290e0     RTreeCooking.obj
 0002:000020f0       $chain$0$?allocate@?$ReflectionAllocator@URTreeNodeNQ@physx@@@shdfnd@physx@@QEAAPEAX_KPEBDH@Z 00000001800290f0     RTreeCooking.obj
 0002:00002104       $chain$1$?allocate@?$ReflectionAllocator@URTreeNodeNQ@physx@@@shdfnd@physx@@QEAAPEAX_KPEBDH@Z 0000000180029104     RTreeCooking.obj
 0002:00002114       $unwind$?deallocate@?$ReflectionAllocator@URTreeNodeNQ@physx@@@shdfnd@physx@@QEAAXPEAX@Z 0000000180029114     RTreeCooking.obj
 0002:0000211c       $unwind$??1?$Array@URTreeNodeNQ@physx@@V?$ReflectionAllocator@URTreeNodeNQ@physx@@@shdfnd@2@@shdfnd@physx@@QEAA@XZ 000000018002911c     RTreeCooking.obj
 0002:00002124       $unwind$?resizeUninitialized@?$Array@URTreeNodeNQ@physx@@V?$ReflectionAllocator@URTreeNodeNQ@physx@@@shdfnd@2@@shdfnd@physx@@QEAAXI@Z 0000000180029124     RTreeCooking.obj
 0002:00002130       $unwind$?deallocate@?$Array@URTreeNodeNQ@physx@@V?$ReflectionAllocator@URTreeNodeNQ@physx@@@shdfnd@2@@shdfnd@physx@@IEAAXPEAX@Z 0000000180029130     RTreeCooking.obj
 0002:00002138       $unwind$?copy@?$Array@URTreeNodeNQ@physx@@V?$ReflectionAllocator@URTreeNodeNQ@physx@@@shdfnd@2@@shdfnd@physx@@KAXPEAURTreeNodeNQ@3@0PEBU43@@Z 0000000180029138     RTreeCooking.obj
 0002:00002140       $chain$0$?copy@?$Array@URTreeNodeNQ@physx@@V?$ReflectionAllocator@URTreeNodeNQ@physx@@@shdfnd@2@@shdfnd@physx@@KAXPEAURTreeNodeNQ@3@0PEBU43@@Z 0000000180029140     RTreeCooking.obj
 0002:00002154       $chain$1$?copy@?$Array@URTreeNodeNQ@physx@@V?$ReflectionAllocator@URTreeNodeNQ@physx@@@shdfnd@2@@shdfnd@physx@@KAXPEAURTreeNodeNQ@3@0PEBU43@@Z 0000000180029154     RTreeCooking.obj
 0002:00002164       $unwind$?growAndPushBack@?$Array@URTreeNodeNQ@physx@@V?$ReflectionAllocator@URTreeNodeNQ@physx@@@shdfnd@2@@shdfnd@physx@@IEAAAEAURTreeNodeNQ@3@AEBU43@@Z 0000000180029164     RTreeCooking.obj
 0002:0000217c       $unwind$?recreate@?$Array@URTreeNodeNQ@physx@@V?$ReflectionAllocator@URTreeNodeNQ@physx@@@shdfnd@2@@shdfnd@physx@@IEAAXI@Z 000000018002917c     RTreeCooking.obj
 0002:00002190       $unwind$??$quickSelectFirstK@UBoundsLTE@physx@@@quickSelect@physx@@YAXPEIAIIIIAEBUBoundsLTE@1@@Z 0000000180029190     RTreeCooking.obj
 0002:000021ac       $unwind$??0SubSortSAH@physx@@QEAA@PEAIPEBUPxBounds3V@1@IPEBI22222M@Z 00000001800291ac     RTreeCooking.obj
 0002:000021c0       $unwind$??1SubSortSAH@physx@@QEAA@XZ 00000001800291c0     RTreeCooking.obj
 0002:000021cc       $unwind$?split@SubSortSAH@physx@@QEAAIPEAII@Z 00000001800291cc     RTreeCooking.obj
 0002:000021dc       $chain$4$?split@SubSortSAH@physx@@QEAAIPEAII@Z 00000001800291dc     RTreeCooking.obj
 0002:00002200       $chain$5$?split@SubSortSAH@physx@@QEAAIPEAII@Z 0000000180029200     RTreeCooking.obj
 0002:00002214       $chain$6$?split@SubSortSAH@physx@@QEAAIPEAII@Z 0000000180029214     RTreeCooking.obj
 0002:00002224       $chain$7$?split@SubSortSAH@physx@@QEAAIPEAII@Z 0000000180029224     RTreeCooking.obj
 0002:00002238       $unwind$?sort4@SubSortSAH@physx@@QEAAXPEAIIAEAV?$Array@URTreeNodeNQ@physx@@V?$ReflectionAllocator@URTreeNodeNQ@physx@@@shdfnd@2@@shdfnd@2@AEAIIPEAURTreeNodeNQ@2@@Z 0000000180029238     RTreeCooking.obj
 0002:00002260       $unwind$??$sort@I@shdfnd@physx@@YAXPEAII@Z 0000000180029260     RTreeCooking.obj
 0002:00002268       $unwind$?getName@?$ReflectionAllocator@UInterval@physx@@@shdfnd@physx@@CAPEBDXZ 0000000180029268     RTreeCooking.obj
 0002:00002270       $unwind$?allocate@?$ReflectionAllocator@UInterval@physx@@@shdfnd@physx@@QEAAPEAX_KPEBDH@Z 0000000180029270     RTreeCooking.obj
 0002:00002280       $chain$0$?allocate@?$ReflectionAllocator@UInterval@physx@@@shdfnd@physx@@QEAAPEAX_KPEBDH@Z 0000000180029280     RTreeCooking.obj
 0002:00002294       $chain$1$?allocate@?$ReflectionAllocator@UInterval@physx@@@shdfnd@physx@@QEAAPEAX_KPEBDH@Z 0000000180029294     RTreeCooking.obj
 0002:000022a4       $unwind$?deallocate@?$ReflectionAllocator@UInterval@physx@@@shdfnd@physx@@QEAAXPEAX@Z 00000001800292a4     RTreeCooking.obj
 0002:000022ac       $unwind$?deallocate@?$InlineAllocator@$0CA@V?$ReflectionAllocator@UInterval@physx@@@shdfnd@physx@@@shdfnd@physx@@QEAAXPEAX@Z 00000001800292ac     RTreeCooking.obj
 0002:000022b4       $unwind$??1?$Array@UInterval@physx@@V?$InlineAllocator@$0CA@V?$ReflectionAllocator@UInterval@physx@@@shdfnd@physx@@@shdfnd@2@@shdfnd@physx@@QEAA@XZ 00000001800292b4     RTreeCooking.obj
 0002:000022bc       $unwind$?allocate@?$Array@UInterval@physx@@V?$InlineAllocator@$0CA@V?$ReflectionAllocator@UInterval@physx@@@shdfnd@physx@@@shdfnd@2@@shdfnd@physx@@IEAAPEAUInterval@3@I@Z 00000001800292bc     RTreeCooking.obj
 0002:000022c4       $unwind$?deallocate@?$Array@UInterval@physx@@V?$InlineAllocator@$0CA@V?$ReflectionAllocator@UInterval@physx@@@shdfnd@physx@@@shdfnd@2@@shdfnd@physx@@IEAAXPEAX@Z 00000001800292c4     RTreeCooking.obj
 0002:000022cc       $unwind$?growAndPushBack@?$Array@UInterval@physx@@V?$InlineAllocator@$0CA@V?$ReflectionAllocator@UInterval@physx@@@shdfnd@physx@@@shdfnd@2@@shdfnd@physx@@IEAAAEAUInterval@3@AEBU43@@Z 00000001800292cc     RTreeCooking.obj
 0002:000022e0       $unwind$??1?$InlineArray@UInterval@physx@@$03V?$ReflectionAllocator@UInterval@physx@@@shdfnd@2@@shdfnd@physx@@QEAA@XZ 00000001800292e0     RTreeCooking.obj
 0002:000022e8       $unwind$??$sort@IUSortBoundsPredicate@physx@@@shdfnd@physx@@YAXPEAIIAEBUSortBoundsPredicate@1@@Z 00000001800292e8     RTreeCooking.obj
 0002:000022f0       $unwind$?getName@?$ReflectionAllocator@URTreeNodeQ@Gu@physx@@@shdfnd@physx@@CAPEBDXZ 00000001800292f0     RTreeCooking.obj
 0002:000022f8       $unwind$?allocate@?$ReflectionAllocator@URTreeNodeQ@Gu@physx@@@shdfnd@physx@@QEAAPEAX_KPEBDH@Z 00000001800292f8     RTreeCooking.obj
 0002:00002308       $chain$0$?allocate@?$ReflectionAllocator@URTreeNodeQ@Gu@physx@@@shdfnd@physx@@QEAAPEAX_KPEBDH@Z 0000000180029308     RTreeCooking.obj
 0002:0000231c       $chain$1$?allocate@?$ReflectionAllocator@URTreeNodeQ@Gu@physx@@@shdfnd@physx@@QEAAPEAX_KPEBDH@Z 000000018002931c     RTreeCooking.obj
 0002:0000232c       $unwind$?deallocate@?$ReflectionAllocator@URTreeNodeQ@Gu@physx@@@shdfnd@physx@@QEAAXPEAX@Z 000000018002932c     RTreeCooking.obj
 0002:00002334       $unwind$??1?$Array@URTreeNodeQ@Gu@physx@@V?$ReflectionAllocator@URTreeNodeQ@Gu@physx@@@shdfnd@3@@shdfnd@physx@@QEAA@XZ 0000000180029334     RTreeCooking.obj
 0002:0000233c       $unwind$?deallocate@?$Array@URTreeNodeQ@Gu@physx@@V?$ReflectionAllocator@URTreeNodeQ@Gu@physx@@@shdfnd@3@@shdfnd@physx@@IEAAXPEAX@Z 000000018002933c     RTreeCooking.obj
 0002:00002344       $unwind$?growAndPushBack@?$Array@URTreeNodeQ@Gu@physx@@V?$ReflectionAllocator@URTreeNodeQ@Gu@physx@@@shdfnd@3@@shdfnd@physx@@IEAAAEAURTreeNodeQ@Gu@3@AEBU453@@Z 0000000180029344     RTreeCooking.obj
 0002:00002358       $unwind$?recreate@?$Array@URTreeNodeQ@Gu@physx@@V?$ReflectionAllocator@URTreeNodeQ@Gu@physx@@@shdfnd@3@@shdfnd@physx@@IEAAXI@Z 0000000180029358     RTreeCooking.obj
 0002:0000236c       $unwind$?allocate@?$AlignedAllocator@$0IA@VAllocator@shdfnd@physx@@@shdfnd@physx@@QEAAPEAX_KPEBDH@Z 000000018002936c     RTreeCooking.obj
 0002:00002374       $unwind$??$partition@UBoundsLTE@physx@@@quickSelect@physx@@YAIPEIAIIIIAEBUBoundsLTE@1@@Z 0000000180029374     RTreeCooking.obj
 0002:00002384       $chain$2$??$partition@UBoundsLTE@physx@@@quickSelect@physx@@YAIPEIAIIIIAEBUBoundsLTE@1@@Z 0000000180029384     RTreeCooking.obj
 0002:000023a0       $chain$3$??$partition@UBoundsLTE@physx@@@quickSelect@physx@@YAIPEIAIIIIAEBUBoundsLTE@1@@Z 00000001800293a0     RTreeCooking.obj
 0002:000023b0       $unwind$??$sort@IU?$Less@I@shdfnd@physx@@V?$ReflectionAllocator@I@23@@shdfnd@physx@@YAXPEAIIAEBU?$Less@I@01@AEBV?$ReflectionAllocator@I@01@I@Z 00000001800293b0     RTreeCooking.obj
 0002:000023cc       $unwind$??$sort@IUSortBoundsPredicate@physx@@V?$ReflectionAllocator@I@shdfnd@2@@shdfnd@physx@@YAXPEAIIAEBUSortBoundsPredicate@1@AEBV?$ReflectionAllocator@I@01@I@Z 00000001800293cc     RTreeCooking.obj
 0002:000023e8       $unwind$??1?$Stack@V?$ReflectionAllocator@I@shdfnd@physx@@@internal@shdfnd@physx@@QEAA@XZ 00000001800293e8     RTreeCooking.obj
 0002:000023f0       $chain$0$??1?$Stack@V?$ReflectionAllocator@I@shdfnd@physx@@@internal@shdfnd@physx@@QEAA@XZ 00000001800293f0     RTreeCooking.obj
 0002:00002404       $chain$2$??1?$Stack@V?$ReflectionAllocator@I@shdfnd@physx@@@internal@shdfnd@physx@@QEAA@XZ 0000000180029404     RTreeCooking.obj
 0002:00002418       $chain$3$??1?$Stack@V?$ReflectionAllocator@I@shdfnd@physx@@@internal@shdfnd@physx@@QEAA@XZ 0000000180029418     RTreeCooking.obj
 0002:00002428       $unwind$?grow@?$Stack@V?$ReflectionAllocator@I@shdfnd@physx@@@internal@shdfnd@physx@@QEAAXXZ 0000000180029428     RTreeCooking.obj
 0002:00002438       $unwind$?push@?$Stack@V?$ReflectionAllocator@I@shdfnd@physx@@@internal@shdfnd@physx@@QEAAXHH@Z 0000000180029438     RTreeCooking.obj
 0002:00002448       $unwind$??$smallSort@I$$CBU?$Less@I@shdfnd@physx@@@internal@shdfnd@physx@@YAXPEAIHHAEBU?$Less@I@12@@Z 0000000180029448     RTreeCooking.obj
 0002:00002450       $chain$5$??$smallSort@I$$CBU?$Less@I@shdfnd@physx@@@internal@shdfnd@physx@@YAXPEAIHHAEBU?$Less@I@12@@Z 0000000180029450     RTreeCooking.obj
 0002:00002478       $chain$6$??$smallSort@I$$CBU?$Less@I@shdfnd@physx@@@internal@shdfnd@physx@@YAXPEAIHHAEBU?$Less@I@12@@Z 0000000180029478     RTreeCooking.obj
 0002:00002488       $unwind$??$partition@I$$CBU?$Less@I@shdfnd@physx@@@internal@shdfnd@physx@@YAHPEAIHHAEBU?$Less@I@12@@Z 0000000180029488     RTreeCooking.obj
 0002:00002494       $unwind$??$smallSort@I$$CBUSortBoundsPredicate@physx@@@internal@shdfnd@physx@@YAXPEAIHHAEBUSortBoundsPredicate@2@@Z 0000000180029494     RTreeCooking.obj
 0002:0000249c       $chain$6$??$smallSort@I$$CBUSortBoundsPredicate@physx@@@internal@shdfnd@physx@@YAXPEAIHHAEBUSortBoundsPredicate@2@@Z 000000018002949c     RTreeCooking.obj
 0002:000024c8       $chain$7$??$smallSort@I$$CBUSortBoundsPredicate@physx@@@internal@shdfnd@physx@@YAXPEAIHHAEBUSortBoundsPredicate@2@@Z 00000001800294c8     RTreeCooking.obj
 0002:000024d8       $unwind$??$partition@I$$CBUSortBoundsPredicate@physx@@@internal@shdfnd@physx@@YAHPEAIHHAEBUSortBoundsPredicate@2@@Z 00000001800294d8     RTreeCooking.obj
 0002:000024ec       $unwind$??$median3@I$$CBUSortBoundsPredicate@physx@@@internal@shdfnd@physx@@YAXPEAIHHAEBUSortBoundsPredicate@2@@Z 00000001800294ec     RTreeCooking.obj
 0002:000024fc       $unwind$??_H@YAXPEAX_KHP6APEAX0@Z@Z 00000001800294fc     TriangleMeshBuilder.obj
 0002:00002510       $unwind$?loadFromDesc@TriangleMeshBuilder@physx@@QEAA_NAEBVPxTriangleMeshDesc@2@AEBUPxCookingParams@2@_N@Z 0000000180029510     TriangleMeshBuilder.obj
 0002:00002524       $chain$0$?loadFromDesc@TriangleMeshBuilder@physx@@QEAA_NAEBVPxTriangleMeshDesc@2@AEBUPxCookingParams@2@_N@Z 0000000180029524     TriangleMeshBuilder.obj
 0002:00002538       $chain$1$?loadFromDesc@TriangleMeshBuilder@physx@@QEAA_NAEBVPxTriangleMeshDesc@2@AEBUPxCookingParams@2@_N@Z 0000000180029538     TriangleMeshBuilder.obj
 0002:0000254c       $chain$2$?loadFromDesc@TriangleMeshBuilder@physx@@QEAA_NAEBVPxTriangleMeshDesc@2@AEBUPxCookingParams@2@_N@Z 000000018002954c     TriangleMeshBuilder.obj
 0002:00002560       $chain$3$?loadFromDesc@TriangleMeshBuilder@physx@@QEAA_NAEBVPxTriangleMeshDesc@2@AEBUPxCookingParams@2@_N@Z 0000000180029560     TriangleMeshBuilder.obj
 0002:00002570       $chain$4$?loadFromDesc@TriangleMeshBuilder@physx@@QEAA_NAEBVPxTriangleMeshDesc@2@AEBUPxCookingParams@2@_N@Z 0000000180029570     TriangleMeshBuilder.obj
 0002:00002580       $chain$5$?loadFromDesc@TriangleMeshBuilder@physx@@QEAA_NAEBVPxTriangleMeshDesc@2@AEBUPxCookingParams@2@_N@Z 0000000180029580     TriangleMeshBuilder.obj
 0002:00002590       $unwind$?save@TriangleMeshBuilder@physx@@QEBA_NAEAVPxOutputStream@2@_NAEBUPxCookingParams@2@@Z 0000000180029590     TriangleMeshBuilder.obj
 0002:000025a0       $chain$0$?save@TriangleMeshBuilder@physx@@QEBA_NAEAVPxOutputStream@2@_NAEBUPxCookingParams@2@@Z 00000001800295a0     TriangleMeshBuilder.obj
 0002:000025b4       $chain$3$?save@TriangleMeshBuilder@physx@@QEBA_NAEAVPxOutputStream@2@_NAEBUPxCookingParams@2@@Z 00000001800295b4     TriangleMeshBuilder.obj
 0002:000025d0       $chain$4$?save@TriangleMeshBuilder@physx@@QEBA_NAEAVPxOutputStream@2@_NAEBUPxCookingParams@2@@Z 00000001800295d0     TriangleMeshBuilder.obj
 0002:000025e0       $chain$5$?save@TriangleMeshBuilder@physx@@QEBA_NAEAVPxOutputStream@2@_NAEBUPxCookingParams@2@@Z 00000001800295e0     TriangleMeshBuilder.obj
 0002:000025f0       $unwind$?computeLocalBounds@TriangleMeshBuilder@physx@@IEAAXXZ 00000001800295f0     TriangleMeshBuilder.obj
 0002:00002600       $unwind$?importMesh@TriangleMeshBuilder@physx@@IEAA_NAEBVPxTriangleMeshDesc@2@AEBUPxCookingParams@2@_N@Z 0000000180029600     TriangleMeshBuilder.obj
 0002:00002618       $unwind$?gatherStrided@shdfnd@physx@@YAXPEBXPEAXIII@Z 0000000180029618     TriangleMeshBuilder.obj
 0002:00002628       $chain$1$?gatherStrided@shdfnd@physx@@YAXPEBXPEAXIII@Z 0000000180029628     TriangleMeshBuilder.obj
 0002:00002640       $chain$2$?gatherStrided@shdfnd@physx@@YAXPEBXPEAXIII@Z 0000000180029640     TriangleMeshBuilder.obj
 0002:00002650       $unwind$?memZero@intrinsics@physx@@YAPEAXPEIAXI@Z 0000000180029650     BigConvexDataBuilder.obj
 0002:00002658       $unwind$?normalize@PxVec3@physx@@QEAAMXZ 0000000180029658     BigConvexDataBuilder.obj
 0002:00002664       $unwind$?PxMemZero@physx@@YAPEAXPEIAXI@Z 0000000180029664     BigConvexDataBuilder.obj
 0002:0000266c       $unwind$?Precompute@BigConvexDataBuilder@physx@@QEAA_NI@Z 000000018002966c     BigConvexDataBuilder.obj
 0002:00002678       $chain$12$?Precompute@BigConvexDataBuilder@physx@@QEAA_NI@Z 0000000180029678     BigConvexDataBuilder.obj
 0002:000026bc       $chain$14$?Precompute@BigConvexDataBuilder@physx@@QEAA_NI@Z 00000001800296bc     BigConvexDataBuilder.obj
 0002:00002700       $chain$15$?Precompute@BigConvexDataBuilder@physx@@QEAA_NI@Z 0000000180029700     BigConvexDataBuilder.obj
 0002:00002710       $unwind$?Initialize@BigConvexDataBuilder@physx@@QEAA_NXZ 0000000180029710     BigConvexDataBuilder.obj
 0002:0000271c       $chain$0$?Initialize@BigConvexDataBuilder@physx@@QEAA_NXZ 000000018002971c     BigConvexDataBuilder.obj
 0002:00002730       $chain$1$?Initialize@BigConvexDataBuilder@physx@@QEAA_NXZ 0000000180029730     BigConvexDataBuilder.obj
 0002:00002740       $unwind$?PrecomputeSample@BigConvexDataBuilder@physx@@QEAA_NIAEBVPxVec3@2@@Z 0000000180029740     BigConvexDataBuilder.obj
 0002:00002760       $unwind$?Save@BigConvexDataBuilder@physx@@QEBA_NAEAVPxOutputStream@2@_NIPEBUHullTriangleData@2@@Z 0000000180029760     BigConvexDataBuilder.obj
 0002:00002774       $unwind$?ComputeValencies@BigConvexDataBuilder@physx@@QEBA_NIPEBUHullTriangleData@2@@Z 0000000180029774     BigConvexDataBuilder.obj
 0002:0000277c       $unwind$?Compute@BigConvexDataBuilder@physx@@QEBA_NAEBUVALENCIESCREATE@2@@Z 000000018002977c     BigConvexDataBuilder.obj
 0002:00002798       $unwind$?Save@BigConvexDataBuilder@physx@@QEBA_NAEAVPxOutputStream@2@_N@Z 0000000180029798     BigConvexDataBuilder.obj
 0002:000027ac       $chain$2$?Save@BigConvexDataBuilder@physx@@QEBA_NAEAVPxOutputStream@2@_N@Z 00000001800297ac     BigConvexDataBuilder.obj
 0002:000027c0       $chain$3$?Save@BigConvexDataBuilder@physx@@QEBA_NAEAVPxOutputStream@2@_N@Z 00000001800297c0     BigConvexDataBuilder.obj
 0002:000027d0       $unwind$?getName@?$ReflectionAllocator@E@shdfnd@physx@@CAPEBDXZ 00000001800297d0     BigConvexDataBuilder.obj
 0002:000027d8       $unwind$?allocate@?$ReflectionAllocator@E@shdfnd@physx@@QEAAPEAX_KPEBDH@Z 00000001800297d8     BigConvexDataBuilder.obj
 0002:000027e8       $chain$0$?allocate@?$ReflectionAllocator@E@shdfnd@physx@@QEAAPEAX_KPEBDH@Z 00000001800297e8     BigConvexDataBuilder.obj
 0002:000027fc       $chain$1$?allocate@?$ReflectionAllocator@E@shdfnd@physx@@QEAAPEAX_KPEBDH@Z 00000001800297fc     BigConvexDataBuilder.obj
 0002:0000280c       $unwind$?getName@?$ReflectionAllocator@UValency@Gu@physx@@@shdfnd@physx@@CAPEBDXZ 000000018002980c     BigConvexDataBuilder.obj
 0002:00002814       $unwind$?allocate@?$ReflectionAllocator@UValency@Gu@physx@@@shdfnd@physx@@QEAAPEAX_KPEBDH@Z 0000000180029814     BigConvexDataBuilder.obj
 0002:00002824       $chain$0$?allocate@?$ReflectionAllocator@UValency@Gu@physx@@@shdfnd@physx@@QEAAPEAX_KPEBDH@Z 0000000180029824     BigConvexDataBuilder.obj
 0002:00002838       $chain$1$?allocate@?$ReflectionAllocator@UValency@Gu@physx@@@shdfnd@physx@@QEAAPEAX_KPEBDH@Z 0000000180029838     BigConvexDataBuilder.obj
 0002:00002848       $unwind$?getName@?$ReflectionAllocator@G@shdfnd@physx@@CAPEBDXZ 0000000180029848     BigConvexDataBuilder.obj
 0002:00002850       $unwind$?allocate@?$ReflectionAllocator@G@shdfnd@physx@@QEAAPEAX_KPEBDH@Z 0000000180029850     BigConvexDataBuilder.obj
 0002:00002860       $chain$0$?allocate@?$ReflectionAllocator@G@shdfnd@physx@@QEAAPEAX_KPEBDH@Z 0000000180029860     BigConvexDataBuilder.obj
 0002:00002874       $chain$1$?allocate@?$ReflectionAllocator@G@shdfnd@physx@@QEAAPEAX_KPEBDH@Z 0000000180029874     BigConvexDataBuilder.obj
 0002:00002884       $unwind$?getNormalized@PxVec3@physx@@QEBA?AV12@XZ 0000000180029884     ConvexHullBuilder.obj
 0002:0000288c       $unwind$??0PxPlane@physx@@QEAA@AEBVPxVec3@1@00@Z 000000018002988c     ConvexHullBuilder.obj
 0002:000028a4       $unwind$??1ConvexHullBuilder@physx@@QEAA@XZ 00000001800298a4     ConvexHullBuilder.obj
 0002:000028b0       $unwind$?Init@ConvexHullBuilder@physx@@QEAA_NIPEBVPxVec3@2@IPEBIIPEBUPxHullPolygon@2@@Z 00000001800298b0     ConvexHullBuilder.obj
 0002:000028d0       $chain$1$?Init@ConvexHullBuilder@physx@@QEAA_NIPEBVPxVec3@2@IPEBIIPEBUPxHullPolygon@2@@Z 00000001800298d0     ConvexHullBuilder.obj
 0002:000028e8       $chain$2$?Init@ConvexHullBuilder@physx@@QEAA_NIPEBVPxVec3@2@IPEBIIPEBUPxHullPolygon@2@@Z 00000001800298e8     ConvexHullBuilder.obj
 0002:000028f8       $unwind$?Save@ConvexHullBuilder@physx@@QEBA_NAEAVPxOutputStream@2@_N@Z 00000001800298f8     ConvexHullBuilder.obj
 0002:00002914       $chain$3$?Save@ConvexHullBuilder@physx@@QEBA_NAEAVPxOutputStream@2@_N@Z 0000000180029914     ConvexHullBuilder.obj
 0002:00002928       $chain$4$?Save@ConvexHullBuilder@physx@@QEBA_NAEAVPxOutputStream@2@_N@Z 0000000180029928     ConvexHullBuilder.obj
 0002:00002938       $unwind$?CreateEdgeList@ConvexHullBuilder@physx@@QEAA_NXZ 0000000180029938     ConvexHullBuilder.obj
 0002:00002950       $unwind$?CreatePolygonData@ConvexHullBuilder@physx@@QEAA_NXZ 0000000180029950     ConvexHullBuilder.obj
 0002:00002970       $chain$2$?CreatePolygonData@ConvexHullBuilder@physx@@QEAA_NXZ 0000000180029970     ConvexHullBuilder.obj
 0002:0000298c       $chain$3$?CreatePolygonData@ConvexHullBuilder@physx@@QEAA_NXZ 000000018002998c     ConvexHullBuilder.obj
 0002:0000299c       $unwind$?CheckHullPolygons@ConvexHullBuilder@physx@@QEBA_NXZ 000000018002999c     ConvexHullBuilder.obj
 0002:000029bc       $unwind$?CreateTrianglesFromPolygons@ConvexHullBuilder@physx@@QEAA_NXZ 00000001800299bc     ConvexHullBuilder.obj
 0002:000029c8       $chain$0$?CreateTrianglesFromPolygons@ConvexHullBuilder@physx@@QEAA_NXZ 00000001800299c8     ConvexHullBuilder.obj
 0002:000029dc       $chain$6$?CreateTrianglesFromPolygons@ConvexHullBuilder@physx@@QEAA_NXZ 00000001800299dc     ConvexHullBuilder.obj
 0002:00002a04       $chain$7$?CreateTrianglesFromPolygons@ConvexHullBuilder@physx@@QEAA_NXZ 0000000180029a04     ConvexHullBuilder.obj
 0002:00002a14       $chain$12$?CreateTrianglesFromPolygons@ConvexHullBuilder@physx@@QEAA_NXZ 0000000180029a14     ConvexHullBuilder.obj
 0002:00002a4c       $chain$14$?CreateTrianglesFromPolygons@ConvexHullBuilder@physx@@QEAA_NXZ 0000000180029a4c     ConvexHullBuilder.obj
 0002:00002a84       $chain$21$?CreateTrianglesFromPolygons@ConvexHullBuilder@physx@@QEAA_NXZ 0000000180029a84     ConvexHullBuilder.obj
 0002:00002ab0       $chain$22$?CreateTrianglesFromPolygons@ConvexHullBuilder@physx@@QEAA_NXZ 0000000180029ab0     ConvexHullBuilder.obj
 0002:00002ac0       $chain$23$?CreateTrianglesFromPolygons@ConvexHullBuilder@physx@@QEAA_NXZ 0000000180029ac0     ConvexHullBuilder.obj
 0002:00002ad0       $unwind$?ComputeGeomCenter@ConvexHullBuilder@physx@@QEBA_NAEAVPxVec3@2@@Z 0000000180029ad0     ConvexHullBuilder.obj
 0002:00002ad8       $chain$1$?ComputeGeomCenter@ConvexHullBuilder@physx@@QEBA_NAEAVPxVec3@2@@Z 0000000180029ad8     ConvexHullBuilder.obj
 0002:00002af0       $chain$7$?ComputeGeomCenter@ConvexHullBuilder@physx@@QEBA_NAEAVPxVec3@2@@Z 0000000180029af0     ConvexHullBuilder.obj
 0002:00002b18       $chain$8$?ComputeGeomCenter@ConvexHullBuilder@physx@@QEBA_NAEAVPxVec3@2@@Z 0000000180029b18     ConvexHullBuilder.obj
 0002:00002b28       $chain$9$?ComputeGeomCenter@ConvexHullBuilder@physx@@QEBA_NAEAVPxVec3@2@@Z 0000000180029b28     ConvexHullBuilder.obj
 0002:00002b38       $unwind$?CalculateVertexMapTable@ConvexHullBuilder@physx@@QEAA_NI_N@Z 0000000180029b38     ConvexHullBuilder.obj
 0002:00002b54       $unwind$?ComputeHullPolygons@ConvexHullBuilder@physx@@QEAA_NAEBIPEBVPxVec3@2@0PEBI@Z 0000000180029b54     ConvexHullBuilder.obj
 0002:00002b6c       $unwind$?inverseBuffer@@YA_NIPEAE@Z 0000000180029b6c     ConvexHullBuilder.obj
 0002:00002b74       $chain$0$?inverseBuffer@@YA_NIPEAE@Z 0000000180029b74     ConvexHullBuilder.obj
 0002:00002b88       $chain$1$?inverseBuffer@@YA_NIPEAE@Z 0000000180029b88     ConvexHullBuilder.obj
 0002:00002b98       $unwind$?findLineStrip@@YA_NAEAVContainer@Gu@physx@@AEBV123@@Z 0000000180029b98     ConvexHullBuilder.obj
 0002:00002bac       $chain$1$?findLineStrip@@YA_NAEAVContainer@Gu@physx@@AEBV123@@Z 0000000180029bac     ConvexHullBuilder.obj
 0002:00002bc4       $unwind$?CheckRedundantVertices@@YAXAEAIAEAVContainer@Gu@physx@@AEBVConvexHullBuilder@3@11@Z 0000000180029bc4     ConvexHullBuilder.obj
 0002:00002be0       $unwind$?ExtractHullPolygons@@YA_NAEAIAEAVContainer@Gu@physx@@AEBVConvexHullBuilder@3@PEAV123@1@Z 0000000180029be0     ConvexHullBuilder.obj
 0002:00002bfc       $unwind$?FloodFill@Local@?8??ExtractHullPolygons@@YA_NAEAIAEAVContainer@Gu@physx@@AEBVConvexHullBuilder@5@PEAV345@1@Z@SAX1PEBVAdjTriangle@5@IPEA_N@Z 0000000180029bfc     ConvexHullBuilder.obj
 0002:00002c10       $unwind$?GetNeighborFace@Local@?8??ExtractHullPolygons@@YA_NAEAIAEAVContainer@Gu@physx@@AEBVConvexHullBuilder@5@PEAV345@1@Z@SA_NIIPEBVAdjTriangle@5@PEBI00@Z 0000000180029c10     ConvexHullBuilder.obj
 0002:00002c28       $unwind$?CheckFloodFillFace@Local@?8??ExtractHullPolygons@@YA_NAEAIAEAVContainer@Gu@physx@@AEBVConvexHullBuilder@5@PEAV345@1@Z@SA_NIPEBVAdjTriangle@5@PEBI@Z 0000000180029c28     ConvexHullBuilder.obj
 0002:00002c34       $chain$6$?CheckFloodFillFace@Local@?8??ExtractHullPolygons@@YA_NAEAIAEAVContainer@Gu@physx@@AEBVConvexHullBuilder@5@PEAV345@1@Z@SA_NIPEBVAdjTriangle@5@PEBI@Z 0000000180029c34     ConvexHullBuilder.obj
 0002:00002c60       $chain$8$?CheckFloodFillFace@Local@?8??ExtractHullPolygons@@YA_NAEAIAEAVContainer@Gu@physx@@AEBVConvexHullBuilder@5@PEAV345@1@Z@SA_NIPEBVAdjTriangle@5@PEBI@Z 0000000180029c60     ConvexHullBuilder.obj
 0002:00002c8c       $unwind$?CheckFloodFill@Local@?8??ExtractHullPolygons@@YA_NAEAIAEAVContainer@Gu@physx@@AEBVConvexHullBuilder@5@PEAV345@1@Z@SA_N1PEAVAdjTriangle@5@PEA_NPEBI@Z 0000000180029c8c     ConvexHullBuilder.obj
 0002:00002ca8       $unwind$?TestDuplicateTriangles@@YA_NAEAIPEAU?$TriangleT@I@Gu@physx@@_N@Z 0000000180029ca8     ConvexHullBuilder.obj
 0002:00002cc4       $unwind$?testCulling@@YA_NAEBU?$TriangleT@I@Gu@physx@@PEBVPxVec3@3@AEBV43@@Z 0000000180029cc4     ConvexHullBuilder.obj
 0002:00002ce0       $unwind$?TestUnifiedNormals@@YA_NIPEBVPxVec3@physx@@IPEAU?$TriangleT@I@Gu@2@_N@Z 0000000180029ce0     ConvexHullBuilder.obj
 0002:00002cf0       $chain$8$?TestUnifiedNormals@@YA_NIPEBVPxVec3@physx@@IPEAU?$TriangleT@I@Gu@2@_N@Z 0000000180029cf0     ConvexHullBuilder.obj
 0002:00002d24       $chain$12$?TestUnifiedNormals@@YA_NIPEBVPxVec3@physx@@IPEAU?$TriangleT@I@Gu@2@_N@Z 0000000180029d24     ConvexHullBuilder.obj
 0002:00002d44       $chain$13$?TestUnifiedNormals@@YA_NIPEBVPxVec3@physx@@IPEAU?$TriangleT@I@Gu@2@_N@Z 0000000180029d44     ConvexHullBuilder.obj
 0002:00002d54       $chain$14$?TestUnifiedNormals@@YA_NIPEBVPxVec3@physx@@IPEAU?$TriangleT@I@Gu@2@_N@Z 0000000180029d54     ConvexHullBuilder.obj
 0002:00002d64       $unwind$?cleanMesh@@YA_NAEAI0PEAVPxVec3@physx@@PEAU?$TriangleT@I@Gu@2@@Z 0000000180029d64     ConvexHullBuilder.obj
 0002:00002d7c       $unwind$?CleanHull@@YA_NAEAIPEAU?$TriangleT@I@Gu@physx@@0PEAVPxVec3@3@@Z 0000000180029d7c     ConvexHullBuilder.obj
 0002:00002d90       $unwind$?CheckHull@@YA_NIPEBU?$TriangleT@I@Gu@physx@@IPEBVPxVec3@3@@Z 0000000180029d90     ConvexHullBuilder.obj
 0002:00002da0       $unwind$?computeNewellPlane@@YA_NAEAVPxPlane@physx@@IPEBEPEBVPxVec3@2@@Z 0000000180029da0     ConvexHullBuilder.obj
 0002:00002da8       $chain$7$?computeNewellPlane@@YA_NAEAVPxPlane@physx@@IPEBEPEBVPxVec3@2@@Z 0000000180029da8     ConvexHullBuilder.obj
 0002:00002dd8       $chain$10$?computeNewellPlane@@YA_NAEAVPxPlane@physx@@IPEBEPEBVPxVec3@2@@Z 0000000180029dd8     ConvexHullBuilder.obj
 0002:00002df4       $chain$11$?computeNewellPlane@@YA_NAEAVPxPlane@physx@@IPEBEPEBVPxVec3@2@@Z 0000000180029df4     ConvexHullBuilder.obj
 0002:00002e04       $chain$12$?computeNewellPlane@@YA_NAEAVPxPlane@physx@@IPEBEPEBVPxVec3@2@@Z 0000000180029e04     ConvexHullBuilder.obj
 0002:00002e2c       $chain$13$?computeNewellPlane@@YA_NAEAVPxPlane@physx@@IPEBEPEBVPxVec3@2@@Z 0000000180029e2c     ConvexHullBuilder.obj
 0002:00002e3c       $unwind$?ComputeNbPolygons@ConvexHullBuilder@physx@@QEBAIXZ 0000000180029e3c     ConvexHullBuilder.obj
 0002:00002e44       $unwind$?area@?$TriangleT@I@Gu@physx@@QEBAMPEBVPxVec3@3@@Z 0000000180029e44     ConvexHullBuilder.obj
 0002:00002e54       $unwind$?getName@?$ReflectionAllocator@UHullTriangleData@physx@@@shdfnd@physx@@CAPEBDXZ 0000000180029e54     ConvexHullBuilder.obj
 0002:00002e5c       $unwind$?allocate@?$ReflectionAllocator@UHullTriangleData@physx@@@shdfnd@physx@@QEAAPEAX_KPEBDH@Z 0000000180029e5c     ConvexHullBuilder.obj
 0002:00002e6c       $chain$0$?allocate@?$ReflectionAllocator@UHullTriangleData@physx@@@shdfnd@physx@@QEAAPEAX_KPEBDH@Z 0000000180029e6c     ConvexHullBuilder.obj
 0002:00002e80       $chain$1$?allocate@?$ReflectionAllocator@UHullTriangleData@physx@@@shdfnd@physx@@QEAAPEAX_KPEBDH@Z 0000000180029e80     ConvexHullBuilder.obj
 0002:00002e90       $unwind$??$PlaneEquation@U?$TriangleT@I@Gu@physx@@@@YA?AVPxPlane@physx@@AEBU?$TriangleT@I@Gu@1@PEBVPxVec3@1@@Z 0000000180029e90     ConvexHullBuilder.obj
 0002:00002ea8       $unwind$?getName@?$ReflectionAllocator@UEdgeDescData@Gu@physx@@@shdfnd@physx@@CAPEBDXZ 0000000180029ea8     ConvexHullBuilder.obj
 0002:00002eb0       $unwind$?allocate@?$ReflectionAllocator@UEdgeDescData@Gu@physx@@@shdfnd@physx@@QEAAPEAX_KPEBDH@Z 0000000180029eb0     ConvexHullBuilder.obj
 0002:00002ec0       $chain$0$?allocate@?$ReflectionAllocator@UEdgeDescData@Gu@physx@@@shdfnd@physx@@QEAAPEAX_KPEBDH@Z 0000000180029ec0     ConvexHullBuilder.obj
 0002:00002ed4       $chain$1$?allocate@?$ReflectionAllocator@UEdgeDescData@Gu@physx@@@shdfnd@physx@@QEAAPEAX_KPEBDH@Z 0000000180029ed4     ConvexHullBuilder.obj
 0002:00002ee4       $unwind$?isFinite@intrinsics@physx@@YA_NM@Z 0000000180029ee4     ConvexMeshBuilder.obj
 0002:00002eec       $unwind$?PxIsFinite@physx@@YA_NM@Z 0000000180029eec     ConvexMeshBuilder.obj
 0002:00002ef4       $unwind$?isFinite@PxVec3@physx@@QEBA_NXZ 0000000180029ef4     ConvexMeshBuilder.obj
 0002:00002efc       $unwind$??3UserAllocated@shdfnd@physx@@SAXPEAX@Z 0000000180029efc     ConvexMeshBuilder.obj
 0002:00002f04       $unwind$??GPxMat33@physx@@QEBA?AV01@XZ 0000000180029f04     ConvexMeshBuilder.obj
 0002:00002f1c       $unwind$??_GBigConvexData@physx@@QEAAPEAXI@Z 0000000180029f1c     ConvexMeshBuilder.obj
 0002:00002f28       $unwind$??0ConvexMeshBuilder@physx@@QEAA@XZ 0000000180029f28     ConvexMeshBuilder.obj
 0002:00002f30       $unwind$??1ConvexMeshBuilder@physx@@UEAA@XZ 0000000180029f30     ConvexMeshBuilder.obj
 0002:00002f38       $unwind$?loadFromDesc@ConvexMeshBuilder@physx@@QEAA_NAEBVPxConvexMeshDesc@2@W4Enum@PxPlatform@2@@Z 0000000180029f38     ConvexMeshBuilder.obj
 0002:00002f48       $unwind$?save@ConvexMeshBuilder@physx@@QEBA_NAEAVPxOutputStream@2@_N@Z 0000000180029f48     ConvexMeshBuilder.obj
 0002:00002f5c       $chain$1$?save@ConvexMeshBuilder@physx@@QEBA_NAEAVPxOutputStream@2@_N@Z 0000000180029f5c     ConvexMeshBuilder.obj
 0002:00002f70       $chain$2$?save@ConvexMeshBuilder@physx@@QEBA_NAEAVPxOutputStream@2@_N@Z 0000000180029f70     ConvexMeshBuilder.obj
 0002:00002f80       $unwind$?loadConvexHull@ConvexMeshBuilder@physx@@QEAA_NAEBVPxConvexMeshDesc@2@@Z 0000000180029f80     ConvexMeshBuilder.obj
 0002:00002fa0       $unwind$?computeHullPolygons@ConvexMeshBuilder@physx@@QEAA_NAEBIPEBVPxVec3@2@0PEBIAEAVPxAllocatorCallback@2@AEAIAEAPEAV32@4AEAPEAI4AEAPEAUPxHullPolygon@2@@Z 0000000180029fa0     ConvexMeshBuilder.obj
 0002:00002fac       $chain$2$?computeHullPolygons@ConvexMeshBuilder@physx@@QEAA_NAEBIPEBVPxVec3@2@0PEBIAEAVPxAllocatorCallback@2@AEAIAEAPEAV32@4AEAPEAI4AEAPEAUPxHullPolygon@2@@Z 0000000180029fac     ConvexMeshBuilder.obj
 0002:00002fc8       $chain$3$?computeHullPolygons@ConvexMeshBuilder@physx@@QEAA_NAEBIPEBVPxVec3@2@0PEBIAEAVPxAllocatorCallback@2@AEAIAEAPEAV32@4AEAPEAI4AEAPEAUPxHullPolygon@2@@Z 0000000180029fc8     ConvexMeshBuilder.obj
 0002:00002fdc       $unwind$?computeGaussMaps@ConvexMeshBuilder@physx@@QEAA_NXZ 0000000180029fdc     ConvexMeshBuilder.obj
 0002:00002fe8       $unwind$?computeMassInfo@ConvexMeshBuilder@physx@@QEAAXXZ 0000000180029fe8     ConvexMeshBuilder.obj
 0002:00002ff8       $chain$1$?computeMassInfo@ConvexMeshBuilder@physx@@QEAAXXZ 0000000180029ff8     ConvexMeshBuilder.obj
 0002:00003010       $chain$2$?computeMassInfo@ConvexMeshBuilder@physx@@QEAAXXZ 000000018002a010     ConvexMeshBuilder.obj
 0002:00003024       $chain$6$?computeMassInfo@ConvexMeshBuilder@physx@@QEAAXXZ 000000018002a024     ConvexMeshBuilder.obj
 0002:00003044       $chain$7$?computeMassInfo@ConvexMeshBuilder@physx@@QEAAXXZ 000000018002a044     ConvexMeshBuilder.obj
 0002:00003054       $chain$8$?computeMassInfo@ConvexMeshBuilder@physx@@QEAAXXZ 000000018002a054     ConvexMeshBuilder.obj
 0002:00003064       $chain$9$?computeMassInfo@ConvexMeshBuilder@physx@@QEAAXXZ 000000018002a064     ConvexMeshBuilder.obj
 0002:00003074       $unwind$?computeInternalObjects@ConvexMeshBuilder@physx@@QEAAXXZ 000000018002a074     ConvexMeshBuilder.obj
 0002:0000309c       $unwind$?ComputeAABBNoTransform@@YAXAEAVPxVec3@physx@@0IPEBV12@@Z 000000018002a09c     ConvexMeshBuilder.obj
 0002:000030b0       $unwind$?TestContainment@@YA_NAEBVPxVec3@physx@@QEBMIPEBUHullPolygonData@Gu@2@@Z 000000018002a0b0     ConvexMeshBuilder.obj
 0002:000030c0       $unwind$??_GConvexMeshBuilder@physx@@UEAAPEAXI@Z 000000018002a0c0     ConvexMeshBuilder.obj
 0002:000030cc       $unwind$?getName@?$ReflectionAllocator@VBigConvexData@physx@@@shdfnd@physx@@CAPEBDXZ 000000018002a0cc     ConvexMeshBuilder.obj
 0002:000030d4       $unwind$?allocate@?$ReflectionAllocator@VBigConvexData@physx@@@shdfnd@physx@@QEAAPEAX_KPEBDH@Z 000000018002a0d4     ConvexMeshBuilder.obj
 0002:000030e4       $chain$0$?allocate@?$ReflectionAllocator@VBigConvexData@physx@@@shdfnd@physx@@QEAAPEAX_KPEBDH@Z 000000018002a0e4     ConvexMeshBuilder.obj
 0002:000030f8       $chain$1$?allocate@?$ReflectionAllocator@VBigConvexData@physx@@@shdfnd@physx@@QEAAPEAX_KPEBDH@Z 000000018002a0f8     ConvexMeshBuilder.obj
 0002:00003108       $unwind$?memSet@intrinsics@physx@@YAPEAXPEIAXHI@Z 000000018002a108     hulllib.obj
 0002:00003110       $unwind$?PxMemSet@physx@@YAPEAXPEIAXHI@Z 000000018002a110     hulllib.obj
 0002:00003118       $unwind$??0HullLibrary@physx@@QEAA@XZ 000000018002a118     hulllib.obj
 0002:00003120       $unwind$??1HullLibrary@physx@@QEAA@XZ 000000018002a120     hulllib.obj
 0002:00003130       $unwind$?CreateConvexHull@HullLibrary@physx@@QEAA?AW4HullError@2@AEBVHullDesc@2@AEAVHullResult@2@@Z 000000018002a130     hulllib.obj
 0002:00003140       $chain$3$?CreateConvexHull@HullLibrary@physx@@QEAA?AW4HullError@2@AEBVHullDesc@2@AEAVHullResult@2@@Z 000000018002a140     hulllib.obj
 0002:00003160       $chain$4$?CreateConvexHull@HullLibrary@physx@@QEAA?AW4HullError@2@AEBVHullDesc@2@AEAVHullResult@2@@Z 000000018002a160     hulllib.obj
 0002:00003174       $chain$5$?CreateConvexHull@HullLibrary@physx@@QEAA?AW4HullError@2@AEBVHullDesc@2@AEAVHullResult@2@@Z 000000018002a174     hulllib.obj
 0002:00003184       $chain$6$?CreateConvexHull@HullLibrary@physx@@QEAA?AW4HullError@2@AEBVHullDesc@2@AEAVHullResult@2@@Z 000000018002a184     hulllib.obj
 0002:00003194       $unwind$?ReleaseResult@HullLibrary@physx@@QEAA?AW4HullError@2@AEAVHullResult@2@@Z 000000018002a194     hulllib.obj
 0002:0000319c       $unwind$?CreateTriangleMesh@HullLibrary@physx@@QEAA?AW4HullError@2@AEAVHullResult@2@PEAVConvexHullTriangleInterface@2@@Z 000000018002a19c     hulllib.obj
 0002:000031ac       $chain$5$?CreateTriangleMesh@HullLibrary@physx@@QEAA?AW4HullError@2@AEAVHullResult@2@PEAVConvexHullTriangleInterface@2@@Z 000000018002a1ac     hulllib.obj
 0002:000031d4       $chain$6$?CreateTriangleMesh@HullLibrary@physx@@QEAA?AW4HullError@2@AEAVHullResult@2@PEAVConvexHullTriangleInterface@2@@Z 000000018002a1d4     hulllib.obj
 0002:000031e4       $unwind$?b2bfix@HullLibrary@physx@@AEAAXPEAVTri@2@0@Z 000000018002a1e4     hulllib.obj
 0002:00003200       $unwind$?removeb2b@HullLibrary@physx@@AEAAXPEAVTri@2@0@Z 000000018002a200     hulllib.obj
 0002:00003210       $unwind$?extrude@HullLibrary@physx@@AEAAXPEAVTri@2@H@Z 000000018002a210     hulllib.obj
 0002:00003228       $unwind$?extrudable@HullLibrary@physx@@AEBAPEAVTri@2@M@Z 000000018002a228     hulllib.obj
 0002:00003230       $unwind$?calchullgen@HullLibrary@physx@@AEAA?AW4HullError@2@PEAVfloat3@2@HHM@Z 000000018002a230     hulllib.obj
 0002:00003240       $chain$6$?calchullgen@HullLibrary@physx@@AEAA?AW4HullError@2@PEAVfloat3@2@HHM@Z 000000018002a240     hulllib.obj
 0002:0000326c       $chain$11$?calchullgen@HullLibrary@physx@@AEAA?AW4HullError@2@PEAVfloat3@2@HHM@Z 000000018002a26c     hulllib.obj
 0002:00003290       $chain$12$?calchullgen@HullLibrary@physx@@AEAA?AW4HullError@2@PEAVfloat3@2@HHM@Z 000000018002a290     hulllib.obj
 0002:000032a4       $chain$13$?calchullgen@HullLibrary@physx@@AEAA?AW4HullError@2@PEAVfloat3@2@HHM@Z 000000018002a2a4     hulllib.obj
 0002:000032b4       $chain$14$?calchullgen@HullLibrary@physx@@AEAA?AW4HullError@2@PEAVfloat3@2@HHM@Z 000000018002a2b4     hulllib.obj
 0002:000032c8       $chain$15$?calchullgen@HullLibrary@physx@@AEAA?AW4HullError@2@PEAVfloat3@2@HHM@Z 000000018002a2c8     hulllib.obj
 0002:000032d8       $chain$16$?calchullgen@HullLibrary@physx@@AEAA?AW4HullError@2@PEAVfloat3@2@HHM@Z 000000018002a2d8     hulllib.obj
 0002:000032ec       $unwind$?calchull@HullLibrary@physx@@AEAA?AW4HullError@2@PEAVfloat3@2@HAEAPEAHAEAHAEAPEAV42@2HM@Z 000000018002a2ec     hulllib.obj
 0002:000032fc       $chain$4$?calchull@HullLibrary@physx@@AEAA?AW4HullError@2@PEAVfloat3@2@HAEAPEAHAEAHAEAPEAV42@2HM@Z 000000018002a2fc     hulllib.obj
 0002:00003320       $chain$5$?calchull@HullLibrary@physx@@AEAA?AW4HullError@2@PEAVfloat3@2@HAEAPEAHAEAHAEAPEAV42@2HM@Z 000000018002a320     hulllib.obj
 0002:00003330       $unwind$?expandhull@HullLibrary@physx@@AEAA?AW4HullError@2@PEAVfloat3@2@HAEAPEAV42@AEAHM@Z 000000018002a330     hulllib.obj
 0002:0000333c       $chain$1$?expandhull@HullLibrary@physx@@AEAA?AW4HullError@2@PEAVfloat3@2@HAEAPEAV42@AEAHM@Z 000000018002a33c     hulllib.obj
 0002:00003354       $chain$2$?expandhull@HullLibrary@physx@@AEAA?AW4HullError@2@PEAVfloat3@2@HAEAPEAV42@AEAHM@Z 000000018002a354     hulllib.obj
 0002:00003368       $chain$7$?expandhull@HullLibrary@physx@@AEAA?AW4HullError@2@PEAVfloat3@2@HAEAPEAV42@AEAHM@Z 000000018002a368     hulllib.obj
 0002:0000338c       $chain$8$?expandhull@HullLibrary@physx@@AEAA?AW4HullError@2@PEAVfloat3@2@HAEAPEAV42@AEAHM@Z 000000018002a38c     hulllib.obj
 0002:000033a0       $chain$9$?expandhull@HullLibrary@physx@@AEAA?AW4HullError@2@PEAVfloat3@2@HAEAPEAV42@AEAHM@Z 000000018002a3a0     hulllib.obj
 0002:000033b0       $chain$10$?expandhull@HullLibrary@physx@@AEAA?AW4HullError@2@PEAVfloat3@2@HAEAPEAV42@AEAHM@Z 000000018002a3b0     hulllib.obj
 0002:000033c4       $chain$11$?expandhull@HullLibrary@physx@@AEAA?AW4HullError@2@PEAVfloat3@2@HAEAPEAV42@AEAHM@Z 000000018002a3c4     hulllib.obj
 0002:000033d4       $unwind$?calchullpbev@HullLibrary@physx@@AEAA?AW4HullError@2@PEAVfloat3@2@HHAEAV?$Array@VPlane@physx@@@hullLibArray@2@M@Z 000000018002a3d4     hulllib.obj
 0002:000033e4       $chain$14$?calchullpbev@HullLibrary@physx@@AEAA?AW4HullError@2@PEAVfloat3@2@HHAEAV?$Array@VPlane@physx@@@hullLibArray@2@M@Z 000000018002a3e4     hulllib.obj
 0002:00003430       $chain$15$?calchullpbev@HullLibrary@physx@@AEAA?AW4HullError@2@PEAVfloat3@2@HHAEAV?$Array@VPlane@physx@@@hullLibArray@2@M@Z 000000018002a430     hulllib.obj
 0002:00003440       $unwind$?ComputeHull@HullLibrary@physx@@AEAA?AW4HullError@2@IPEBMAEAVPHullResult@2@IMM@Z 000000018002a440     hulllib.obj
 0002:00003454       $chain$0$?ComputeHull@HullLibrary@physx@@AEAA?AW4HullError@2@IPEBMAEAVPHullResult@2@IMM@Z 000000018002a454     hulllib.obj
 0002:00003468       $chain$2$?ComputeHull@HullLibrary@physx@@AEAA?AW4HullError@2@IPEBMAEAVPHullResult@2@IMM@Z 000000018002a468     hulllib.obj
 0002:00003480       $chain$3$?ComputeHull@HullLibrary@physx@@AEAA?AW4HullError@2@IPEBMAEAVPHullResult@2@IMM@Z 000000018002a480     hulllib.obj
 0002:00003490       $chain$4$?ComputeHull@HullLibrary@physx@@AEAA?AW4HullError@2@IPEBMAEAVPHullResult@2@IMM@Z 000000018002a490     hulllib.obj
 0002:000034a0       $unwind$?overhullv@HullLibrary@physx@@AEAA?AW4HullError@2@PEAVfloat3@2@HHAEAPEAV42@AEAHAEAPEAH2MMHM@Z 000000018002a4a0     hulllib.obj
 0002:000034c0       $chain$3$?overhullv@HullLibrary@physx@@AEAA?AW4HullError@2@PEAVfloat3@2@HHAEAPEAV42@AEAHAEAPEAH2MMHM@Z 000000018002a4c0     hulllib.obj
 0002:000034d4       $chain$4$?overhullv@HullLibrary@physx@@AEAA?AW4HullError@2@PEAVfloat3@2@HHAEAPEAV42@AEAHAEAPEAH2MMHM@Z 000000018002a4d4     hulllib.obj
 0002:000034e4       $unwind$?normalize@physx@@YA?AVfloat3@1@AEBV21@@Z 000000018002a4e4     hulllib.obj
 0002:000034f0       $unwind$?Determinant@physx@@YAMAEBVfloat3x3@1@@Z 000000018002a4f0     hulllib.obj
 0002:00003504       $unwind$?Inverse@physx@@YA?AVfloat3x3@1@AEBV21@@Z 000000018002a504     hulllib.obj
 0002:0000351c       $unwind$?Transpose@physx@@YA?AVfloat3x3@1@AEBV21@@Z 000000018002a51c     hulllib.obj
 0002:00003524       $unwind$??Dphysx@@YA?AVfloat3@0@AEBV10@AEBVfloat3x3@0@@Z 000000018002a524     hulllib.obj
 0002:00003530       $unwind$?ThreePlaneIntersection@physx@@YA?AVfloat3@1@AEBVPlane@1@00@Z 000000018002a530     hulllib.obj
 0002:00003550       $unwind$?TriNormal@physx@@YA?AVfloat3@1@AEBV21@00@Z 000000018002a550     hulllib.obj
 0002:00003560       $unwind$??0ConvexH@physx@@QEAA@HHH@Z 000000018002a560     hulllib.obj
 0002:00003578       $unwind$?ConvexHDup@physx@@YAPEAVConvexH@1@PEAV21@@Z 000000018002a578     hulllib.obj
 0002:00003584       $unwind$?AssertIntact@physx@@YAHAEAVConvexH@1@@Z 000000018002a584     hulllib.obj
 0002:00003594       $chain$6$?AssertIntact@physx@@YAHAEAVConvexH@1@@Z 000000018002a594     hulllib.obj
 0002:000035c0       $chain$7$?AssertIntact@physx@@YAHAEAVConvexH@1@@Z 000000018002a5c0     hulllib.obj
 0002:000035d0       $chain$8$?AssertIntact@physx@@YAHAEAVConvexH@1@@Z 000000018002a5d0     hulllib.obj
 0002:000035fc       $unwind$?test_cube@physx@@YAPEAVConvexH@1@XZ 000000018002a5fc     hulllib.obj
 0002:00003610       $unwind$?ConvexHMakeCube@physx@@YAPEAVConvexH@1@AEBVfloat3@1@0@Z 000000018002a610     hulllib.obj
 0002:00003620       $unwind$?ConvexHCrop@physx@@YAPEAVConvexH@1@AEAV21@AEBVPlane@1@@Z 000000018002a620     hulllib.obj
 0002:00003630       $chain$7$?ConvexHCrop@physx@@YAPEAVConvexH@1@AEAV21@AEBVPlane@1@@Z 000000018002a630     hulllib.obj
 0002:00003660       $chain$8$?ConvexHCrop@physx@@YAPEAVConvexH@1@AEAV21@AEBVPlane@1@@Z 000000018002a660     hulllib.obj
 0002:00003670       $unwind$?candidateplane@physx@@YAHPEAVPlane@1@HPEAVConvexH@1@M@Z 000000018002a670     hulllib.obj
 0002:00003698       $chain$6$?candidateplane@physx@@YAHPEAVPlane@1@HPEAVConvexH@1@M@Z 000000018002a698     hulllib.obj
 0002:000036c4       $chain$7$?candidateplane@physx@@YAHPEAVPlane@1@HPEAVConvexH@1@M@Z 000000018002a6c4     hulllib.obj
 0002:000036d4       $unwind$?orth@physx@@YA?AVfloat3@1@AEBV21@@Z 000000018002a6d4     hulllib.obj
 0002:000036ec       $unwind$?above@physx@@YAHPEAVfloat3@1@AEBVint3@1@AEBV21@M@Z 000000018002a6ec     hulllib.obj
 0002:000036f8       $unwind$?deleteTri@physx@@YAXPEAVTri@1@PEAV?$Array@PEAVTri@physx@@@hullLibArray@1@@Z 000000018002a6f8     hulllib.obj
 0002:00003700       $unwind$?neib@Tri@physx@@QEAAAEAHHH@Z 000000018002a700     hulllib.obj
 0002:0000370c       $unwind$?hasVolume@physx@@YA_NPEAVfloat3@1@HHHH@Z 000000018002a70c     hulllib.obj
 0002:00003720       $chain$2$?hasVolume@physx@@YA_NPEAVfloat3@1@HHHH@Z 000000018002a720     hulllib.obj
 0002:0000373c       $chain$3$?hasVolume@physx@@YA_NPEAVfloat3@1@HHHH@Z 000000018002a73c     hulllib.obj
 0002:0000374c       $unwind$?FindSimplex@physx@@YA?AVint4@1@PEAVfloat3@1@HAEAV?$Array@H@hullLibArray@1@AEBV31@@Z 000000018002a74c     hulllib.obj
 0002:00003780       $chain$2$?FindSimplex@physx@@YA?AVint4@1@PEAVfloat3@1@HAEAV?$Array@H@hullLibArray@1@AEBV31@@Z 000000018002a780     hulllib.obj
 0002:0000379c       $chain$3$?FindSimplex@physx@@YA?AVint4@1@PEAVfloat3@1@HAEAV?$Array@H@hullLibArray@1@AEBV31@@Z 000000018002a79c     hulllib.obj
 0002:000037ac       $chain$4$?FindSimplex@physx@@YA?AVint4@1@PEAVfloat3@1@HAEAV?$Array@H@hullLibArray@1@AEBV31@@Z 000000018002a7ac     hulllib.obj
 0002:000037c8       $chain$5$?FindSimplex@physx@@YA?AVint4@1@PEAVfloat3@1@HAEAV?$Array@H@hullLibArray@1@AEBV31@@Z 000000018002a7c8     hulllib.obj
 0002:000037d8       $unwind$?PlaneCheck@LocalTests@?1??expandhull@HullLibrary@physx@@AEAA?AW4HullError@4@PEAVfloat3@4@HAEAPEAV64@AEAHM@Z@SA_NPEBV64@HAEAV?$Array@UExpandPlane@physx@@@hullLibArray@4@@Z 000000018002a7d8     hulllib.obj
 0002:000037e8       $unwind$?area2@physx@@YAMAEBVfloat3@1@00@Z 000000018002a7e8     hulllib.obj
 0002:000037f8       $unwind$?overhull@physx@@YA?AW4HullError@1@PEAVPlane@1@HPEAVfloat3@1@HHAEAPEAV41@AEAHAEAPEAH3M@Z 000000018002a7f8     hulllib.obj
 0002:0000380c       $chain$3$?overhull@physx@@YA?AW4HullError@1@PEAVPlane@1@HPEAVfloat3@1@HHAEAPEAV41@AEAHAEAPEAH3M@Z 000000018002a80c     hulllib.obj
 0002:00003828       $chain$4$?overhull@physx@@YA?AW4HullError@1@PEAVPlane@1@HPEAVfloat3@1@HHAEAPEAV41@AEAHAEAPEAH3M@Z 000000018002a828     hulllib.obj
 0002:0000383c       $chain$8$?overhull@physx@@YA?AW4HullError@1@PEAVPlane@1@HPEAVfloat3@1@HHAEAPEAV41@AEAHAEAPEAH3M@Z 000000018002a83c     hulllib.obj
 0002:0000385c       $chain$9$?overhull@physx@@YA?AW4HullError@1@PEAVPlane@1@HPEAVfloat3@1@HHAEAPEAV41@AEAHAEAPEAH3M@Z 000000018002a85c     hulllib.obj
 0002:00003870       $chain$10$?overhull@physx@@YA?AW4HullError@1@PEAVPlane@1@HPEAVfloat3@1@HHAEAPEAV41@AEAHAEAPEAH3M@Z 000000018002a870     hulllib.obj
 0002:00003884       $chain$11$?overhull@physx@@YA?AW4HullError@1@PEAVPlane@1@HPEAVfloat3@1@HHAEAPEAV41@AEAHAEAPEAH3M@Z 000000018002a884     hulllib.obj
 0002:00003898       $chain$12$?overhull@physx@@YA?AW4HullError@1@PEAVPlane@1@HPEAVfloat3@1@HHAEAPEAV41@AEAHAEAPEAH3M@Z 000000018002a898     hulllib.obj
 0002:000038ac       $unwind$?ReleaseHull@physx@@YAXAEAVPHullResult@1@@Z 000000018002a8ac     hulllib.obj
 0002:000038b8       $unwind$?BringOutYourDead@physx@@YAXPEBMIPEAMAEAIPEAII@Z 000000018002a8b8     hulllib.obj
 0002:000038d4       $unwind$?CleanupVertices@physx@@YA_NIPEBMIAEAIPEAMM2@Z 000000018002a8d4     hulllib.obj
 0002:000038ec       $chain$5$?CleanupVertices@physx@@YA_NIPEBMIAEAIPEAMM2@Z 000000018002a8ec     hulllib.obj
 0002:0000390c       $chain$9$?CleanupVertices@physx@@YA_NIPEBMIAEAIPEAMM2@Z 000000018002a90c     hulllib.obj
 0002:0000392c       $chain$10$?CleanupVertices@physx@@YA_NIPEBMIAEAIPEAMM2@Z 000000018002a92c     hulllib.obj
 0002:00003940       $chain$11$?CleanupVertices@physx@@YA_NIPEBMIAEAIPEAMM2@Z 000000018002a940     hulllib.obj
 0002:00003950       $chain$12$?CleanupVertices@physx@@YA_NIPEBMIAEAIPEAMM2@Z 000000018002a950     hulllib.obj
 0002:00003964       $chain$13$?CleanupVertices@physx@@YA_NIPEBMIAEAIPEAMM2@Z 000000018002a964     hulllib.obj
 0002:00003974       $chain$15$?CleanupVertices@physx@@YA_NIPEBMIAEAIPEAMM2@Z 000000018002a974     hulllib.obj
 0002:00003994       $unwind$?ComputeNormal@physx@@YAMPEAMPEBM11@Z 000000018002a994     hulllib.obj
 0002:000039ac       $unwind$?AddConvexTriangle@physx@@YAXPEAVConvexHullTriangleInterface@1@PEBM11@Z 000000018002a9ac     hulllib.obj
 0002:000039c0       $unwind$??0?$Array@Vfloat3@physx@@@hullLibArray@physx@@QEAA@H@Z 000000018002a9c0     hulllib.obj
 0002:000039c8       $unwind$??1?$Array@Vfloat3@physx@@@hullLibArray@physx@@QEAA@XZ 000000018002a9c8     hulllib.obj
 0002:000039d4       $unwind$?allocate@?$Array@Vfloat3@physx@@@hullLibArray@physx@@QEAAXH@Z 000000018002a9d4     hulllib.obj
 0002:000039e0       $unwind$?Add@?$Array@Vfloat3@physx@@@hullLibArray@physx@@QEAAAEAVfloat3@3@V43@@Z 000000018002a9e0     hulllib.obj
 0002:000039ec       $unwind$??0?$Array@VHalfEdge@ConvexH@physx@@@hullLibArray@physx@@QEAA@H@Z 000000018002a9ec     hulllib.obj
 0002:000039f4       $unwind$??1?$Array@VHalfEdge@ConvexH@physx@@@hullLibArray@physx@@QEAA@XZ 000000018002a9f4     hulllib.obj
 0002:00003a00       $unwind$?allocate@?$Array@VHalfEdge@ConvexH@physx@@@hullLibArray@physx@@QEAAXH@Z 000000018002aa00     hulllib.obj
 0002:00003a0c       $unwind$??0?$Array@VPlane@physx@@@hullLibArray@physx@@QEAA@H@Z 000000018002aa0c     hulllib.obj
 0002:00003a14       $unwind$??1?$Array@VPlane@physx@@@hullLibArray@physx@@QEAA@XZ 000000018002aa14     hulllib.obj
 0002:00003a20       $unwind$?allocate@?$Array@VPlane@physx@@@hullLibArray@physx@@QEAAXH@Z 000000018002aa20     hulllib.obj
 0002:00003a2c       $unwind$?Add@?$Array@VPlane@physx@@@hullLibArray@physx@@QEAAAEAVPlane@3@V43@@Z 000000018002aa2c     hulllib.obj
 0002:00003a38       $unwind$??1ConvexH@physx@@QEAA@XZ 000000018002aa38     hulllib.obj
 0002:00003a44       $unwind$??_GConvexH@physx@@QEAAPEAXI@Z 000000018002aa44     hulllib.obj
 0002:00003a50       $unwind$?getName@?$ReflectionAllocator@VConvexH@physx@@@shdfnd@physx@@CAPEBDXZ 000000018002aa50     hulllib.obj
 0002:00003a58       $unwind$?allocate@?$ReflectionAllocator@VConvexH@physx@@@shdfnd@physx@@QEAAPEAX_KPEBDH@Z 000000018002aa58     hulllib.obj
 0002:00003a68       $chain$0$?allocate@?$ReflectionAllocator@VConvexH@physx@@@shdfnd@physx@@QEAAPEAX_KPEBDH@Z 000000018002aa68     hulllib.obj
 0002:00003a7c       $chain$1$?allocate@?$ReflectionAllocator@VConvexH@physx@@@shdfnd@physx@@QEAAPEAX_KPEBDH@Z 000000018002aa7c     hulllib.obj
 0002:00003a8c       $unwind$??0Tri@physx@@QEAA@HHHPEAV?$Array@PEAVTri@physx@@@hullLibArray@1@@Z 000000018002aa8c     hulllib.obj
 0002:00003a98       $unwind$??_GTri@physx@@IEAAPEAXI@Z 000000018002aa98     hulllib.obj
 0002:00003aa0       $unwind$??0?$Array@PEAVTri@physx@@@hullLibArray@physx@@QEAA@H@Z 000000018002aaa0     hulllib.obj
 0002:00003aa8       $unwind$??1?$Array@PEAVTri@physx@@@hullLibArray@physx@@QEAA@XZ 000000018002aaa8     hulllib.obj
 0002:00003ab4       $unwind$?allocate@?$Array@PEAVTri@physx@@@hullLibArray@physx@@QEAAXH@Z 000000018002aab4     hulllib.obj
 0002:00003ac0       $unwind$?SetSize@?$Array@PEAVTri@physx@@@hullLibArray@physx@@QEAAXH@Z 000000018002aac0     hulllib.obj
 0002:00003acc       $unwind$?Add@?$Array@PEAVTri@physx@@@hullLibArray@physx@@QEAAAEAPEAVTri@3@PEAV43@@Z 000000018002aacc     hulllib.obj
 0002:00003ad8       $unwind$??_G?$Array@PEAVTri@physx@@@hullLibArray@physx@@QEAAPEAXI@Z 000000018002aad8     hulllib.obj
 0002:00003ae8       $unwind$?getName@?$ReflectionAllocator@VTri@physx@@@shdfnd@physx@@CAPEBDXZ 000000018002aae8     hulllib.obj
 0002:00003af0       $unwind$?allocate@?$ReflectionAllocator@VTri@physx@@@shdfnd@physx@@QEAAPEAX_KPEBDH@Z 000000018002aaf0     hulllib.obj
 0002:00003b00       $chain$0$?allocate@?$ReflectionAllocator@VTri@physx@@@shdfnd@physx@@QEAAPEAX_KPEBDH@Z 000000018002ab00     hulllib.obj
 0002:00003b14       $chain$1$?allocate@?$ReflectionAllocator@VTri@physx@@@shdfnd@physx@@QEAAPEAX_KPEBDH@Z 000000018002ab14     hulllib.obj
 0002:00003b24       $unwind$??0?$Array@H@hullLibArray@physx@@QEAA@H@Z 000000018002ab24     hulllib.obj
 0002:00003b2c       $unwind$??1?$Array@H@hullLibArray@physx@@QEAA@XZ 000000018002ab2c     hulllib.obj
 0002:00003b38       $unwind$?allocate@?$Array@H@hullLibArray@physx@@QEAAXH@Z 000000018002ab38     hulllib.obj
 0002:00003b44       $unwind$?Add@?$Array@H@hullLibArray@physx@@QEAAAEAHH@Z 000000018002ab44     hulllib.obj
 0002:00003b50       $unwind$??$maxdirsterid@Vfloat3@physx@@@physx@@YAHPEBVfloat3@0@HAEBV10@AEAV?$Array@H@hullLibArray@0@@Z 000000018002ab50     hulllib.obj
 0002:00003b94       $unwind$??0?$Array@UExpandPlane@physx@@@hullLibArray@physx@@QEAA@H@Z 000000018002ab94     hulllib.obj
 0002:00003b9c       $unwind$??1?$Array@UExpandPlane@physx@@@hullLibArray@physx@@QEAA@XZ 000000018002ab9c     hulllib.obj
 0002:00003ba8       $unwind$?allocate@?$Array@UExpandPlane@physx@@@hullLibArray@physx@@QEAAXH@Z 000000018002aba8     hulllib.obj
 0002:00003bb4       $unwind$?Add@?$Array@UExpandPlane@physx@@@hullLibArray@physx@@QEAAAEAUExpandPlane@3@U43@@Z 000000018002abb4     hulllib.obj
 0002:00003bc0       $unwind$??$maxdir@Vfloat3@physx@@@physx@@YAHPEBVfloat3@0@HAEBV10@@Z 000000018002abc0     hulllib.obj
 0002:00003bcc       $chain$0$??$maxdir@Vfloat3@physx@@@physx@@YAHPEBVfloat3@0@HAEBV10@@Z 000000018002abcc     hulllib.obj
 0002:00003be0       $chain$2$??$maxdir@Vfloat3@physx@@@physx@@YAHPEBVfloat3@0@HAEBV10@@Z 000000018002abe0     hulllib.obj
 0002:00003bf8       $chain$3$??$maxdir@Vfloat3@physx@@@physx@@YAHPEBVfloat3@0@HAEBV10@@Z 000000018002abf8     hulllib.obj
 0002:00003c08       $chain$4$??$maxdir@Vfloat3@physx@@@physx@@YAHPEBVfloat3@0@HAEBV10@@Z 000000018002ac08     hulllib.obj
 0002:00003c18       $unwind$??0?$Array@Vint3@physx@@@hullLibArray@physx@@QEAA@H@Z 000000018002ac18     hulllib.obj
 0002:00003c20       $unwind$??1?$Array@Vint3@physx@@@hullLibArray@physx@@QEAA@XZ 000000018002ac20     hulllib.obj
 0002:00003c2c       $unwind$?allocate@?$Array@Vint3@physx@@@hullLibArray@physx@@QEAAXH@Z 000000018002ac2c     hulllib.obj
 0002:00003c38       $unwind$?SetSize@?$Array@Vint3@physx@@@hullLibArray@physx@@QEAAXH@Z 000000018002ac38     hulllib.obj
 0002:00003c44       $unwind$?Add@?$Array@Vint3@physx@@@hullLibArray@physx@@QEAAAEAVint3@3@V43@@Z 000000018002ac44     hulllib.obj
 0002:00003c50       $unwind$?getName@?$ReflectionAllocator@M@shdfnd@physx@@CAPEBDXZ 000000018002ac50     hulllib.obj
 0002:00003c58       $unwind$?allocate@?$ReflectionAllocator@M@shdfnd@physx@@QEAAPEAX_KPEBDH@Z 000000018002ac58     hulllib.obj
 0002:00003c68       $chain$0$?allocate@?$ReflectionAllocator@M@shdfnd@physx@@QEAAPEAX_KPEBDH@Z 000000018002ac68     hulllib.obj
 0002:00003c7c       $chain$1$?allocate@?$ReflectionAllocator@M@shdfnd@physx@@QEAAPEAX_KPEBDH@Z 000000018002ac7c     hulllib.obj
 0002:00003c8c       $unwind$??$maxdirfiltered@Vfloat3@physx@@@physx@@YAHPEBVfloat3@0@HAEBV10@PEA_N@Z 000000018002ac8c     hulllib.obj
 0002:00003c9c       $chain$2$??$maxdirfiltered@Vfloat3@physx@@@physx@@YAHPEBVfloat3@0@HAEBV10@PEA_N@Z 000000018002ac9c     hulllib.obj
 0002:00003cb8       $chain$3$??$maxdirfiltered@Vfloat3@physx@@@physx@@YAHPEBVfloat3@0@HAEBV10@PEA_N@Z 000000018002acb8     hulllib.obj
 0002:00003cc8       $unwind$?computeVolumeIntegrals@physx@@YA_NAEBVPxSimpleTriangleMesh@1@MAEAUPxIntegrals@1@@Z 000000018002acc8     VolumeIntegration.obj
 0002:00003cd0       $unwind$?computeVolumeIntegralsEberly@physx@@YA_NAEBVPxSimpleTriangleMesh@1@MAEAUPxIntegrals@1@AEBVPxVec3@1@@Z 000000018002acd0     VolumeIntegration.obj
 0002:00003cd8       $unwind$?computeVolumeIntegrals@VolumeIntegrator@?A0xd2749a4a@physx@@QEAA_NAEAUPxIntegrals@3@@Z 000000018002acd8     VolumeIntegration.obj
 0002:00003cfc       $unwind$?computeInertiaTensor@VolumeIntegrator@?A0xd2749a4a@physx@@AEAAXPEAN@Z 000000018002acfc     VolumeIntegration.obj
 0002:00003d08       $unwind$?computeCOMInertiaTensor@VolumeIntegrator@?A0xd2749a4a@physx@@AEAAXPEAN@Z 000000018002ad08     VolumeIntegration.obj
 0002:00003d38       $unwind$?computeFaceNormal@VolumeIntegrator@?A0xd2749a4a@physx@@AEAAXAEAUFace@123@PEAI@Z 000000018002ad38     VolumeIntegration.obj
 0002:00003d4c       $unwind$?computeProjectionIntegrals@VolumeIntegrator@?A0xd2749a4a@physx@@AEAAXAEBUFace@123@@Z 000000018002ad4c     VolumeIntegration.obj
 0002:00003d88       $unwind$?computeFaceIntegrals@VolumeIntegrator@?A0xd2749a4a@physx@@AEAAXAEBUFace@123@@Z 000000018002ad88     VolumeIntegration.obj
 0002:00003dbc       $unwind$?computeVolumeIntegrals@VolumeIntegratorEberly@?A0xd2749a4a@physx@@QEAA_NAEAUPxIntegrals@3@AEBVPxVec3@3@@Z 000000018002adbc     VolumeIntegration.obj
 0002:00003de8       $chain$7$?computeVolumeIntegrals@VolumeIntegratorEberly@?A0xd2749a4a@physx@@QEAA_NAEAUPxIntegrals@3@AEBVPxVec3@3@@Z 000000018002ade8     VolumeIntegration.obj
 0002:00003e18       $chain$8$?computeVolumeIntegrals@VolumeIntegratorEberly@?A0xd2749a4a@physx@@QEAA_NAEAUPxIntegrals@3@AEBVPxVec3@3@@Z 000000018002ae18     VolumeIntegration.obj
 0002:00003e28       $unwind$??_I@YAXPEAX_KHP6AX0@Z@Z 000000018002ae28     Adjacencies.obj
 0002:00003e3c       $unwind$??_VUserAllocated@shdfnd@physx@@SAXPEAX@Z 000000018002ae3c     Adjacencies.obj
 0002:00003e44       $unwind$??_EAdjTriangle@physx@@QEAAPEAXI@Z 000000018002ae44     Adjacencies.obj
 0002:00003e4c       $unwind$??1Adjacencies@physx@@QEAA@XZ 000000018002ae4c     Adjacencies.obj
 0002:00003e54       $unwind$?Load@Adjacencies@physx@@QEAA_NAEAVPxInputStream@2@@Z 000000018002ae54     Adjacencies.obj
 0002:00003e68       $chain$2$?Load@Adjacencies@physx@@QEAA_NAEAVPxInputStream@2@@Z 000000018002ae68     Adjacencies.obj
 0002:00003e7c       $chain$3$?Load@Adjacencies@physx@@QEAA_NAEAVPxInputStream@2@@Z 000000018002ae7c     Adjacencies.obj
 0002:00003e8c       $unwind$?Walk@Adjacencies@physx@@QEAA_NP6AXAEBUCommonWalkParams@2@IIII@ZPEAX@Z 000000018002ae8c     Adjacencies.obj
 0002:00003e98       $chain$2$?Walk@Adjacencies@physx@@QEAA_NP6AXAEBUCommonWalkParams@2@IIII@ZPEAX@Z 000000018002ae98     Adjacencies.obj
 0002:00003eb4       $chain$3$?Walk@Adjacencies@physx@@QEAA_NP6AXAEBUCommonWalkParams@2@IIII@ZPEAX@Z 000000018002aeb4     Adjacencies.obj
 0002:00003ec4       $unwind$?Walk2@Adjacencies@physx@@QEAA_NP6AXAEBUCommonWalkParams@2@IIII@ZPEAXPEBVPxVec3@2@PEBU?$TriangleT@I@Gu@2@@Z 000000018002aec4     Adjacencies.obj
 0002:00003ed4       $chain$4$?Walk2@Adjacencies@physx@@QEAA_NP6AXAEBUCommonWalkParams@2@IIII@ZPEAXPEBVPxVec3@2@PEBU?$TriangleT@I@Gu@2@@Z 000000018002aed4     Adjacencies.obj
 0002:00003ef8       $chain$5$?Walk2@Adjacencies@physx@@QEAA_NP6AXAEBUCommonWalkParams@2@IIII@ZPEAXPEBVPxVec3@2@PEBU?$TriangleT@I@Gu@2@@Z 000000018002aef8     Adjacencies.obj
 0002:00003f08       $unwind$?GetBoundaryVertices@Adjacencies@physx@@QEBA_NIPEA_NPEBU?$TriangleT@I@Gu@2@@Z 000000018002af08     Adjacencies.obj
 0002:00003f1c       $unwind$?MakeLastRef@Adjacencies@physx@@QEAA_NAEAVAdjTriangle@2@IPEAU?$TriangleT@I@Gu@2@@Z 000000018002af1c     Adjacencies.obj
 0002:00003f24       $chain$1$?MakeLastRef@Adjacencies@physx@@QEAA_NAEAVAdjTriangle@2@IPEAU?$TriangleT@I@Gu@2@@Z 000000018002af24     Adjacencies.obj
 0002:00003f3c       $chain$3$?MakeLastRef@Adjacencies@physx@@QEAA_NAEAVAdjTriangle@2@IPEAU?$TriangleT@I@Gu@2@@Z 000000018002af3c     Adjacencies.obj
 0002:00003f54       $chain$4$?MakeLastRef@Adjacencies@physx@@QEAA_NAEAVAdjTriangle@2@IPEAU?$TriangleT@I@Gu@2@@Z 000000018002af54     Adjacencies.obj
 0002:00003f68       $chain$5$?MakeLastRef@Adjacencies@physx@@QEAA_NAEAVAdjTriangle@2@IPEAU?$TriangleT@I@Gu@2@@Z 000000018002af68     Adjacencies.obj
 0002:00003f78       $chain$7$?MakeLastRef@Adjacencies@physx@@QEAA_NAEAVAdjTriangle@2@IPEAU?$TriangleT@I@Gu@2@@Z 000000018002af78     Adjacencies.obj
 0002:00003f90       $unwind$??1AdjacenciesBuilder@physx@@QEAA@XZ 000000018002af90     Adjacencies.obj
 0002:00003f98       $unwind$?Init@AdjacenciesBuilder@physx@@QEAA_NAEBUADJACENCIESCREATE@2@@Z 000000018002af98     Adjacencies.obj
 0002:00003fa4       $chain$2$?Init@AdjacenciesBuilder@physx@@QEAA_NAEBUADJACENCIESCREATE@2@@Z 000000018002afa4     Adjacencies.obj
 0002:00003fc0       $chain$3$?Init@AdjacenciesBuilder@physx@@QEAA_NAEBUADJACENCIESCREATE@2@@Z 000000018002afc0     Adjacencies.obj
 0002:00003fd4       $chain$5$?Init@AdjacenciesBuilder@physx@@QEAA_NAEBUADJACENCIESCREATE@2@@Z 000000018002afd4     Adjacencies.obj
 0002:00003fec       $chain$6$?Init@AdjacenciesBuilder@physx@@QEAA_NAEBUADJACENCIESCREATE@2@@Z 000000018002afec     Adjacencies.obj
 0002:00004000       $chain$7$?Init@AdjacenciesBuilder@physx@@QEAA_NAEBUADJACENCIESCREATE@2@@Z 000000018002b000     Adjacencies.obj
 0002:00004010       $chain$8$?Init@AdjacenciesBuilder@physx@@QEAA_NAEBUADJACENCIESCREATE@2@@Z 000000018002b010     Adjacencies.obj
 0002:00004028       $unwind$?_WalkFace@Local@?1??Walk@Adjacencies@physx@@QEAA_NP6AXAEBUCommonWalkParams@4@IIII@ZPEAX@Z@SAXAEAUPrivateWalkParams@?1??234@QEAA_N12@Z@IIII@Z 000000018002b028     Adjacencies.obj
 0002:00004034       $chain$1$?_WalkFace@Local@?1??Walk@Adjacencies@physx@@QEAA_NP6AXAEBUCommonWalkParams@4@IIII@ZPEAX@Z@SAXAEAUPrivateWalkParams@?1??234@QEAA_N12@Z@IIII@Z 000000018002b034     Adjacencies.obj
 0002:0000404c       $chain$2$?_WalkFace@Local@?1??Walk@Adjacencies@physx@@QEAA_NP6AXAEBUCommonWalkParams@4@IIII@ZPEAX@Z@SAXAEAUPrivateWalkParams@?1??234@QEAA_N12@Z@IIII@Z 000000018002b04c     Adjacencies.obj
 0002:0000405c       $unwind$?_WalkFace@Local@?1??Walk2@Adjacencies@physx@@QEAA_NP6AXAEBUCommonWalkParams@4@IIII@ZPEAXPEBVPxVec3@4@PEBU?$TriangleT@I@Gu@4@@Z@SAXAEAUPrivateWalkParams@?1??234@QEAA_N1234@Z@IIII@Z 000000018002b05c     Adjacencies.obj
 0002:00004068       $chain$2$?_WalkFace@Local@?1??Walk2@Adjacencies@physx@@QEAA_NP6AXAEBUCommonWalkParams@4@IIII@ZPEAXPEBVPxVec3@4@PEBU?$TriangleT@I@Gu@4@@Z@SAXAEAUPrivateWalkParams@?1??234@QEAA_N1234@Z@IIII@Z 000000018002b068     Adjacencies.obj
 0002:00004084       $chain$3$?_WalkFace@Local@?1??Walk2@Adjacencies@physx@@QEAA_NP6AXAEBUCommonWalkParams@4@IIII@ZPEAXPEBVPxVec3@4@PEBU?$TriangleT@I@Gu@4@@Z@SAXAEAUPrivateWalkParams@?1??234@QEAA_N1234@Z@IIII@Z 000000018002b084     Adjacencies.obj
 0002:00004098       $chain$4$?_WalkFace@Local@?1??Walk2@Adjacencies@physx@@QEAA_NP6AXAEBUCommonWalkParams@4@IIII@ZPEAXPEBVPxVec3@4@PEBU?$TriangleT@I@Gu@4@@Z@SAXAEAUPrivateWalkParams@?1??234@QEAA_N1234@Z@IIII@Z 000000018002b098     Adjacencies.obj
 0002:000040a8       $chain$5$?_WalkFace@Local@?1??Walk2@Adjacencies@physx@@QEAA_NP6AXAEBUCommonWalkParams@4@IIII@ZPEAXPEBVPxVec3@4@PEBU?$TriangleT@I@Gu@4@@Z@SAXAEAUPrivateWalkParams@?1??234@QEAA_N1234@Z@IIII@Z 000000018002b0a8     Adjacencies.obj
 0002:000040bc       $chain$6$?_WalkFace@Local@?1??Walk2@Adjacencies@physx@@QEAA_NP6AXAEBUCommonWalkParams@4@IIII@ZPEAXPEBVPxVec3@4@PEBU?$TriangleT@I@Gu@4@@Z@SAXAEAUPrivateWalkParams@?1??234@QEAA_N1234@Z@IIII@Z 000000018002b0bc     Adjacencies.obj
 0002:000040cc       $unwind$?AddTriangle@@YAXIIIIPEAVAdjTriangle@physx@@AEAIPEAVAdjEdge@@@Z 000000018002b0cc     Adjacencies.obj
 0002:000040d8       $unwind$?UpdateLink@@YA_NIIIIPEAVAdjTriangle@physx@@AEBUADJACENCIESCREATE@2@@Z 000000018002b0d8     Adjacencies.obj
 0002:000040e4       $chain$3$?UpdateLink@@YA_NIIIIPEAVAdjTriangle@physx@@AEBUADJACENCIESCREATE@2@@Z 000000018002b0e4     Adjacencies.obj
 0002:00004104       $chain$5$?UpdateLink@@YA_NIIIIPEAVAdjTriangle@physx@@AEBUADJACENCIESCREATE@2@@Z 000000018002b104     Adjacencies.obj
 0002:0000411c       $chain$6$?UpdateLink@@YA_NIIIIPEAVAdjTriangle@physx@@AEBUADJACENCIESCREATE@2@@Z 000000018002b11c     Adjacencies.obj
 0002:0000412c       $chain$7$?UpdateLink@@YA_NIIIIPEAVAdjTriangle@physx@@AEBUADJACENCIESCREATE@2@@Z 000000018002b12c     Adjacencies.obj
 0002:00004144       $chain$8$?UpdateLink@@YA_NIIIIPEAVAdjTriangle@physx@@AEBUADJACENCIESCREATE@2@@Z 000000018002b144     Adjacencies.obj
 0002:00004154       $unwind$?CreateDatabase@@YA_NPEAVAdjTriangle@physx@@IPEBVAdjEdge@@AEBUADJACENCIESCREATE@2@@Z 000000018002b154     Adjacencies.obj
 0002:0000416c       $unwind$?getName@?$ReflectionAllocator@VAdjTriangle@physx@@@shdfnd@physx@@CAPEBDXZ 000000018002b16c     Adjacencies.obj
 0002:00004174       $unwind$?allocate@?$ReflectionAllocator@VAdjTriangle@physx@@@shdfnd@physx@@QEAAPEAX_KPEBDH@Z 000000018002b174     Adjacencies.obj
 0002:00004184       $chain$0$?allocate@?$ReflectionAllocator@VAdjTriangle@physx@@@shdfnd@physx@@QEAAPEAX_KPEBDH@Z 000000018002b184     Adjacencies.obj
 0002:00004198       $chain$1$?allocate@?$ReflectionAllocator@VAdjTriangle@physx@@@shdfnd@physx@@QEAAPEAX_KPEBDH@Z 000000018002b198     Adjacencies.obj
 0002:000041a8       $unwind$??_EAdjEdge@@QEAAPEAXI@Z 000000018002b1a8     Adjacencies.obj
 0002:000041b0       $unwind$?getName@?$ReflectionAllocator@VAdjEdge@@@shdfnd@physx@@CAPEBDXZ 000000018002b1b0     Adjacencies.obj
 0002:000041b8       $unwind$?allocate@?$ReflectionAllocator@VAdjEdge@@@shdfnd@physx@@QEAAPEAX_KPEBDH@Z 000000018002b1b8     Adjacencies.obj
 0002:000041c8       $chain$0$?allocate@?$ReflectionAllocator@VAdjEdge@@@shdfnd@physx@@QEAAPEAX_KPEBDH@Z 000000018002b1c8     Adjacencies.obj
 0002:000041dc       $chain$1$?allocate@?$ReflectionAllocator@VAdjEdge@@@shdfnd@physx@@QEAAPEAX_KPEBDH@Z 000000018002b1dc     Adjacencies.obj
 0002:000041ec       $unwind$??_GPxCooking@physx@@MEAAPEAXI@Z 000000018002b1ec     Cooking.obj
 0002:000041f4       $unwind$PxCreateCooking    000000018002b1f4     Cooking.obj
 0002:00004200       $unwind$?release@Cooking@physx@@UEAAXXZ 000000018002b200     Cooking.obj
 0002:00004208       $unwind$?cookTriangleMesh@Cooking@physx@@UEAA_NAEBVPxTriangleMeshDesc@2@AEAVPxOutputStream@2@@Z 000000018002b208     Cooking.obj
 0002:00004220       $unwind$?createTriangleMesh@Cooking@physx@@UEAAPEAVPxTriangleMesh@2@AEBVPxTriangleMeshDesc@2@AEAVPxPhysicsInsertionCallback@2@@Z 000000018002b220     Cooking.obj
 0002:00004234       $unwind$?validateTriangleMesh@Cooking@physx@@UEAA_NAEBVPxTriangleMeshDesc@2@@Z 000000018002b234     Cooking.obj
 0002:00004244       $unwind$?cookConvexMesh@Cooking@physx@@UEAA_NAEBVPxConvexMeshDesc@2@AEAVPxOutputStream@2@PEAW4Enum@PxConvexMeshCookingResult@2@@Z 000000018002b244     Cooking.obj
 0002:0000425c       $unwind$?computeHullPolygons@Cooking@physx@@UEAA_NAEBVPxSimpleTriangleMesh@2@AEAVPxAllocatorCallback@2@AEAIAEAPEAVPxVec3@2@2AEAPEAI2AEAPEAUPxHullPolygon@2@@Z 000000018002b25c     Cooking.obj
 0002:0000427c       $unwind$?cookHeightField@Cooking@physx@@UEAA_NAEBVPxHeightFieldDesc@2@AEAVPxOutputStream@2@@Z 000000018002b27c     Cooking.obj
 0002:00004290       $unwind$?createHeightField@Cooking@physx@@UEAAPEAVPxHeightField@2@AEBVPxHeightFieldDesc@2@AEAVPxPhysicsInsertionCallback@2@@Z 000000018002b290     Cooking.obj
 0002:000042a0       $unwind$?loadTriangleMeshDesc@Cooking@physx@@AEAA_NAEBVPxTriangleMeshDesc@2@AEAVTriangleMeshBuilder@2@@Z 000000018002b2a0     Cooking.obj
 0002:000042b0       $unwind$??_GCooking@physx@@UEAAPEAXI@Z 000000018002b2b0     Cooking.obj
 0002:000042b8       $unwind$??0TriangleMeshBuilder@physx@@QEAA@XZ 000000018002b2b8     Cooking.obj
 0002:000042c0       $unwind$??_GTriangleMeshBuilder@physx@@UEAAPEAXI@Z 000000018002b2c0     Cooking.obj
 0002:000042cc       $unwind$?getName@?$ReflectionAllocator@VTriangleMeshBuilder@physx@@@shdfnd@physx@@CAPEBDXZ 000000018002b2cc     Cooking.obj
 0002:000042d4       $unwind$?allocate@?$ReflectionAllocator@VTriangleMeshBuilder@physx@@@shdfnd@physx@@QEAAPEAX_KPEBDH@Z 000000018002b2d4     Cooking.obj
 0002:000042e4       $chain$0$?allocate@?$ReflectionAllocator@VTriangleMeshBuilder@physx@@@shdfnd@physx@@QEAAPEAX_KPEBDH@Z 000000018002b2e4     Cooking.obj
 0002:000042f8       $chain$1$?allocate@?$ReflectionAllocator@VTriangleMeshBuilder@physx@@@shdfnd@physx@@QEAAPEAX_KPEBDH@Z 000000018002b2f8     Cooking.obj
 0002:00004308       $unwind$?getName@?$ReflectionAllocator@VHeightField@Gu@physx@@@shdfnd@physx@@CAPEBDXZ 000000018002b308     Cooking.obj
 0002:00004310       $unwind$?allocate@?$ReflectionAllocator@VHeightField@Gu@physx@@@shdfnd@physx@@QEAAPEAX_KPEBDH@Z 000000018002b310     Cooking.obj
 0002:00004320       $chain$0$?allocate@?$ReflectionAllocator@VHeightField@Gu@physx@@@shdfnd@physx@@QEAAPEAX_KPEBDH@Z 000000018002b320     Cooking.obj
 0002:00004334       $chain$1$?allocate@?$ReflectionAllocator@VHeightField@Gu@physx@@@shdfnd@physx@@QEAAPEAX_KPEBDH@Z 000000018002b334     Cooking.obj
 0002:00004344       $unwind$?getName@?$ReflectionAllocator@VCooking@physx@@@shdfnd@physx@@CAPEBDXZ 000000018002b344     Cooking.obj
 0002:0000434c       $unwind$?allocate@?$ReflectionAllocator@VCooking@physx@@@shdfnd@physx@@QEAAPEAX_KPEBDH@Z 000000018002b34c     Cooking.obj
 0002:0000435c       $chain$0$?allocate@?$ReflectionAllocator@VCooking@physx@@@shdfnd@physx@@QEAAPEAX_KPEBDH@Z 000000018002b35c     Cooking.obj
 0002:00004370       $chain$1$?allocate@?$ReflectionAllocator@VCooking@physx@@@shdfnd@physx@@QEAAPEAX_KPEBDH@Z 000000018002b370     Cooking.obj
 0002:00004380       $unwind$??1ReducedVertexCloud@physx@@QEAA@XZ 000000018002b380     CookingUtils.obj
 0002:00004388       $unwind$?Clean@ReducedVertexCloud@physx@@QEAAAEAV12@XZ 000000018002b388     CookingUtils.obj
 0002:00004390       $unwind$?Reduce@ReducedVertexCloud@physx@@QEAA_NPEAUREDUCEDCLOUD@2@@Z 000000018002b390     CookingUtils.obj
 0002:0000439c       $chain$1$?Reduce@ReducedVertexCloud@physx@@QEAA_NPEAUREDUCEDCLOUD@2@@Z 000000018002b39c     CookingUtils.obj
 0002:000043b4       $chain$3$?Reduce@ReducedVertexCloud@physx@@QEAA_NPEAUREDUCEDCLOUD@2@@Z 000000018002b3b4     CookingUtils.obj
 0002:000043cc       $chain$4$?Reduce@ReducedVertexCloud@physx@@QEAA_NPEAUREDUCEDCLOUD@2@@Z 000000018002b3cc     CookingUtils.obj
 0002:000043e0       $chain$5$?Reduce@ReducedVertexCloud@physx@@QEAA_NPEAUREDUCEDCLOUD@2@@Z 000000018002b3e0     CookingUtils.obj
 0002:000043f0       $chain$6$?Reduce@ReducedVertexCloud@physx@@QEAA_NPEAUREDUCEDCLOUD@2@@Z 000000018002b3f0     CookingUtils.obj
 0002:00004400       $unwind$??1EdgeList@Gu@physx@@QEAA@XZ 000000018002b400     EdgeList.obj
 0002:0000440c       $unwind$?Load@EdgeList@Gu@physx@@QEAA_NAEAVPxInputStream@3@@Z 000000018002b40c     EdgeList.obj
 0002:0000441c       $unwind$?Init@EdgeListBuilder@Gu@physx@@QEAA_NAEBUEDGELISTCREATE@23@@Z 000000018002b41c     EdgeList.obj
 0002:0000442c       $unwind$?CreateFacesToEdges@EdgeListBuilder@Gu@physx@@AEAA_NIPEBIPEBG@Z 000000018002b42c     EdgeList.obj
 0002:0000443c       $chain$4$?CreateFacesToEdges@EdgeListBuilder@Gu@physx@@AEAA_NIPEBIPEBG@Z 000000018002b43c     EdgeList.obj
 0002:00004460       $chain$5$?CreateFacesToEdges@EdgeListBuilder@Gu@physx@@AEAA_NIPEBIPEBG@Z 000000018002b460     EdgeList.obj
 0002:00004470       $unwind$?CreateEdgesToFaces@EdgeListBuilder@Gu@physx@@AEAA_NIPEBIPEBG@Z 000000018002b470     EdgeList.obj
 0002:00004480       $unwind$?ComputeActiveEdges@EdgeListBuilder@Gu@physx@@AEAA_NIPEBIPEBGPEBVPxVec3@3@M@Z 000000018002b480     EdgeList.obj
 0002:00004490       $chain$0$?ComputeActiveEdges@EdgeListBuilder@Gu@physx@@AEAA_NIPEBIPEBGPEBVPxVec3@3@M@Z 000000018002b490     EdgeList.obj
 0002:000044a4       $chain$3$?ComputeActiveEdges@EdgeListBuilder@Gu@physx@@AEAA_NIPEBIPEBGPEBVPxVec3@3@M@Z 000000018002b4a4     EdgeList.obj
 0002:000044bc       $chain$5$?ComputeActiveEdges@EdgeListBuilder@Gu@physx@@AEAA_NIPEBIPEBGPEBVPxVec3@3@M@Z 000000018002b4bc     EdgeList.obj
 0002:000044d4       $chain$15$?ComputeActiveEdges@EdgeListBuilder@Gu@physx@@AEAA_NIPEBIPEBGPEBVPxVec3@3@M@Z 000000018002b4d4     EdgeList.obj
 0002:0000450c       $chain$16$?ComputeActiveEdges@EdgeListBuilder@Gu@physx@@AEAA_NIPEBIPEBGPEBVPxVec3@3@M@Z 000000018002b50c     EdgeList.obj
 0002:0000451c       $chain$17$?ComputeActiveEdges@EdgeListBuilder@Gu@physx@@AEAA_NIPEBIPEBGPEBVPxVec3@3@M@Z 000000018002b51c     EdgeList.obj
 0002:00004530       $chain$18$?ComputeActiveEdges@EdgeListBuilder@Gu@physx@@AEAA_NIPEBIPEBGPEBVPxVec3@3@M@Z 000000018002b530     EdgeList.obj
 0002:00004540       $unwind$?normal@PxTriangle@physx@@QEBAXAEAVPxVec3@2@@Z 000000018002b540     EdgeList.obj
 0002:00004558       $unwind$?angle@shdfnd@physx@@YAMAEBVPxVec3@2@0@Z 000000018002b558     EdgeList.obj
 0002:00004568       $unwind$?getName@?$ReflectionAllocator@UEdgeTriangleData@Gu@physx@@@shdfnd@physx@@CAPEBDXZ 000000018002b568     EdgeList.obj
 0002:00004570       $unwind$?allocate@?$ReflectionAllocator@UEdgeTriangleData@Gu@physx@@@shdfnd@physx@@QEAAPEAX_KPEBDH@Z 000000018002b570     EdgeList.obj
 0002:00004580       $chain$0$?allocate@?$ReflectionAllocator@UEdgeTriangleData@Gu@physx@@@shdfnd@physx@@QEAAPEAX_KPEBDH@Z 000000018002b580     EdgeList.obj
 0002:00004594       $chain$1$?allocate@?$ReflectionAllocator@UEdgeTriangleData@Gu@physx@@@shdfnd@physx@@QEAAPEAX_KPEBDH@Z 000000018002b594     EdgeList.obj
 0002:000045a4       $unwind$?getName@?$ReflectionAllocator@UEdgeData@Gu@physx@@@shdfnd@physx@@CAPEBDXZ 000000018002b5a4     EdgeList.obj
 0002:000045ac       $unwind$?allocate@?$ReflectionAllocator@UEdgeData@Gu@physx@@@shdfnd@physx@@QEAAPEAX_KPEBDH@Z 000000018002b5ac     EdgeList.obj
 0002:000045bc       $chain$0$?allocate@?$ReflectionAllocator@UEdgeData@Gu@physx@@@shdfnd@physx@@QEAAPEAX_KPEBDH@Z 000000018002b5bc     EdgeList.obj
 0002:000045d0       $chain$1$?allocate@?$ReflectionAllocator@UEdgeData@Gu@physx@@@shdfnd@physx@@QEAAPEAX_KPEBDH@Z 000000018002b5d0     EdgeList.obj
 0002:000045e0       $unwind$??_GRemapCallback@RTreeCooker@physx@@UEAAPEAXI@Z 000000018002b5e0     InternalTriangleMeshBuilder.obj
 0002:000045e8       $unwind$??1InternalTriangleMeshBuilder@physx@@QEAA@XZ 000000018002b5e8     InternalTriangleMeshBuilder.obj
 0002:000045f4       $unwind$?cleanMesh@InternalTriangleMeshBuilder@physx@@QEAA_N_N@Z 000000018002b5f4     InternalTriangleMeshBuilder.obj
 0002:00004600       $chain$0$?cleanMesh@InternalTriangleMeshBuilder@physx@@QEAA_N_N@Z 000000018002b600     InternalTriangleMeshBuilder.obj
 0002:00004614       $chain$1$?cleanMesh@InternalTriangleMeshBuilder@physx@@QEAA_N_N@Z 000000018002b614     InternalTriangleMeshBuilder.obj
 0002:00004624       $chain$2$?cleanMesh@InternalTriangleMeshBuilder@physx@@QEAA_N_N@Z 000000018002b624     InternalTriangleMeshBuilder.obj
 0002:00004638       $chain$5$?cleanMesh@InternalTriangleMeshBuilder@physx@@QEAA_N_N@Z 000000018002b638     InternalTriangleMeshBuilder.obj
 0002:00004654       $chain$6$?cleanMesh@InternalTriangleMeshBuilder@physx@@QEAA_N_N@Z 000000018002b654     InternalTriangleMeshBuilder.obj
 0002:00004668       $chain$7$?cleanMesh@InternalTriangleMeshBuilder@physx@@QEAA_N_N@Z 000000018002b668     InternalTriangleMeshBuilder.obj
 0002:00004678       $chain$8$?cleanMesh@InternalTriangleMeshBuilder@physx@@QEAA_N_N@Z 000000018002b678     InternalTriangleMeshBuilder.obj
 0002:00004688       $chain$9$?cleanMesh@InternalTriangleMeshBuilder@physx@@QEAA_N_N@Z 000000018002b688     InternalTriangleMeshBuilder.obj
 0002:00004698       $unwind$?fillRemapTable@InternalTriangleMeshBuilder@physx@@QEAAXXZ 000000018002b698     InternalTriangleMeshBuilder.obj
 0002:000046a4       $chain$0$?fillRemapTable@InternalTriangleMeshBuilder@physx@@QEAAXXZ 000000018002b6a4     InternalTriangleMeshBuilder.obj
 0002:000046b8       $chain$1$?fillRemapTable@InternalTriangleMeshBuilder@physx@@QEAAXXZ 000000018002b6b8     InternalTriangleMeshBuilder.obj
 0002:000046cc       $chain$2$?fillRemapTable@InternalTriangleMeshBuilder@physx@@QEAAXXZ 000000018002b6cc     InternalTriangleMeshBuilder.obj
 0002:000046dc       $chain$3$?fillRemapTable@InternalTriangleMeshBuilder@physx@@QEAAXXZ 000000018002b6dc     InternalTriangleMeshBuilder.obj
 0002:000046ec       $unwind$?remapTopology@InternalTriangleMeshBuilder@physx@@QEAAXPEBI@Z 000000018002b6ec     InternalTriangleMeshBuilder.obj
 0002:000046f8       $chain$3$?remapTopology@InternalTriangleMeshBuilder@physx@@QEAAXPEBI@Z 000000018002b6f8     InternalTriangleMeshBuilder.obj
 0002:00004718       $chain$4$?remapTopology@InternalTriangleMeshBuilder@physx@@QEAAXPEBI@Z 000000018002b718     InternalTriangleMeshBuilder.obj
 0002:00004728       $unwind$?createRTree@InternalTriangleMeshBuilder@physx@@QEAA_NXZ 000000018002b728     InternalTriangleMeshBuilder.obj
 0002:00004730       $unwind$?createSharedEdgeData@InternalTriangleMeshBuilder@physx@@QEAAX_N0@Z 000000018002b730     InternalTriangleMeshBuilder.obj
 0002:00004748       $unwind$?releaseEdgeList@InternalTriangleMeshBuilder@physx@@AEAAXXZ 000000018002b748     InternalTriangleMeshBuilder.obj
 0002:00004754       $unwind$?createEdgeList@InternalTriangleMeshBuilder@physx@@AEAAXXZ 000000018002b754     InternalTriangleMeshBuilder.obj
 0002:00004764       $unwind$??_GEdgeListBuilder@Gu@physx@@QEAAPEAXI@Z 000000018002b764     InternalTriangleMeshBuilder.obj
 0002:00004770       $unwind$??_GRTreeCookerRemap@@UEAAPEAXI@Z 000000018002b770     InternalTriangleMeshBuilder.obj
 0002:00004778       $unwind$?getName@?$ReflectionAllocator@VEdgeListBuilder@Gu@physx@@@shdfnd@physx@@CAPEBDXZ 000000018002b778     InternalTriangleMeshBuilder.obj
 0002:00004780       $unwind$?allocate@?$ReflectionAllocator@VEdgeListBuilder@Gu@physx@@@shdfnd@physx@@QEAAPEAX_KPEBDH@Z 000000018002b780     InternalTriangleMeshBuilder.obj
 0002:00004790       $chain$0$?allocate@?$ReflectionAllocator@VEdgeListBuilder@Gu@physx@@@shdfnd@physx@@QEAAPEAX_KPEBDH@Z 000000018002b790     InternalTriangleMeshBuilder.obj
 0002:000047a4       $chain$1$?allocate@?$ReflectionAllocator@VEdgeListBuilder@Gu@physx@@@shdfnd@physx@@QEAAPEAX_KPEBDH@Z 000000018002b7a4     InternalTriangleMeshBuilder.obj
 0002:000047b4       $unwind$??0MeshCleaner@physx@@QEAA@IPEBVPxVec3@1@IPEBIM@Z 000000018002b7b4     MeshCleaner.obj
 0002:000047c0       $chain$3$??0MeshCleaner@physx@@QEAA@IPEBVPxVec3@1@IPEBIM@Z 000000018002b7c0     MeshCleaner.obj
 0002:000047e0       $chain$5$??0MeshCleaner@physx@@QEAA@IPEBVPxVec3@1@IPEBIM@Z 000000018002b7e0     MeshCleaner.obj
 0002:000047f8       $chain$7$??0MeshCleaner@physx@@QEAA@IPEBVPxVec3@1@IPEBIM@Z 000000018002b7f8     MeshCleaner.obj
 0002:00004810       $chain$8$??0MeshCleaner@physx@@QEAA@IPEBVPxVec3@1@IPEBIM@Z 000000018002b810     MeshCleaner.obj
 0002:00004824       $chain$9$??0MeshCleaner@physx@@QEAA@IPEBVPxVec3@1@IPEBIM@Z 000000018002b824     MeshCleaner.obj
 0002:00004834       $chain$10$??0MeshCleaner@physx@@QEAA@IPEBVPxVec3@1@IPEBIM@Z 000000018002b834     MeshCleaner.obj
 0002:00004844       $chain$11$??0MeshCleaner@physx@@QEAA@IPEBVPxVec3@1@IPEBIM@Z 000000018002b844     MeshCleaner.obj
 0002:0000485c       $chain$12$??0MeshCleaner@physx@@QEAA@IPEBVPxVec3@1@IPEBIM@Z 000000018002b85c     MeshCleaner.obj
 0002:0000486c       $chain$13$??0MeshCleaner@physx@@QEAA@IPEBVPxVec3@1@IPEBIM@Z 000000018002b86c     MeshCleaner.obj
 0002:00004880       $chain$14$??0MeshCleaner@physx@@QEAA@IPEBVPxVec3@1@IPEBIM@Z 000000018002b880     MeshCleaner.obj
 0002:00004890       $unwind$??1MeshCleaner@physx@@QEAA@XZ 000000018002b890     MeshCleaner.obj
 0002:00004898       xdata                      000000018002b898     PhysX3CommonPROFILE_x64:PhysX3CommonPROFILE_x64.dll
 0002:000048a0       $unwind$__FUnloadDelayLoadedDLL2 000000018002b8a0     delayimp:delayhlp.obj
 0002:000048ac       $unwind$__HrLoadAllImportsForDll 000000018002b8ac     delayimp:delayhlp.obj
 0002:000048bc       $unwind$?PiddFromDllName@@YAPEBUImgDelayDescr@@PEBD@Z 000000018002b8bc     delayimp:delayhlp.obj
 0002:000048c4       $unwind$__delayLoadHelper2 000000018002b8c4     delayimp:delayhlp.obj
 0002:000048e0       $xdatasym                  000000018002b8e0     MSVCRT:chkstk.obj
 0002:000048e8       $unwind$??_Etype_info@@UEAAPEAXI@Z 000000018002b8e8     MSVCRT:ti_inst.obj
 0002:000048f8       $unwind$_CRT_INIT          000000018002b8f8     MSVCRT:crtdll.obj
 0002:00004914       $unwind$pre_c_init         000000018002b914     MSVCRT:crtdll.obj
 0002:0000491c       $unwind$__DllMainCRTStartup 000000018002b91c     MSVCRT:crtdll.obj
 0002:00004958       $unwind$__DllMainCRTStartup$filt$0 000000018002b958     MSVCRT:crtdll.obj
 0002:00004960       $unwind$__DllMainCRTStartup$fin$1 000000018002b960     MSVCRT:crtdll.obj
 0002:00004968       $unwind$_DllMainCRTStartup 000000018002b968     MSVCRT:crtdll.obj
 0002:00004978       $unwind$??_M@YAXPEAX_KHP6AX0@Z@Z 000000018002b978     MSVCRT:ehvecdtr.obj
 0002:000049a0       $unwind$?fin$0@?0???_M@YAXPEAX_KHP6AX0@Z@Z@4HA 000000018002b9a0     MSVCRT:ehvecdtr.obj
 0002:000049a8       $unwind$?__ArrayUnwind@@YAXPEAX_KHP6AX0@Z@Z 000000018002b9a8     MSVCRT:ehvecdtr.obj
 0002:000049d0       $unwind$?filt$0@?0??__ArrayUnwind@@YAXPEAX_KHP6AX0@Z@Z@4HA 000000018002b9d0     MSVCRT:ehvecdtr.obj
 0002:000049d8       $unwind$?ArrayUnwindFilter@@YAHPEAU_EXCEPTION_POINTERS@@@Z 000000018002b9d8     MSVCRT:ehvecdtr.obj
 0002:000049e0       $unwind$_IsNonwritableInCurrentImage 000000018002b9e0     MSVCRT:pesect.obj
 0002:00004a04       $unwind$_IsNonwritableInCurrentImage$filt$0 000000018002ba04     MSVCRT:pesect.obj
 0002:00004a0c       $unwind$atexit             000000018002ba0c     MSVCRT:atonexit.obj
 0002:00004a14       $unwind$_onexit            000000018002ba14     MSVCRT:atonexit.obj
 0002:00004a34       $unwind$_onexit$fin$0      000000018002ba34     MSVCRT:atonexit.obj
 0002:00004a3c       $unwind$__atonexitinit     000000018002ba3c     MSVCRT:atonexit.obj
 0002:00004a44       $unwind$__security_init_cookie 000000018002ba44     MSVCRT:gs_support.obj
 0002:00004a50       $unwind$DllMain            000000018002ba50     MSVCRT:dllmain.obj
 0002:00004a58       $unwind$_RTC_Initialize    000000018002ba58     MSVCRT:initsect.obj
 0002:00004a64       $unwind$_RTC_Terminate     000000018002ba64     MSVCRT:initsect.obj
 0002:000060d0       .edata                     000000018002d0d0     PhysX3CookingPROFILE_x64.exp
 0002:000060f8       rgpv                       000000018002d0f8     PhysX3CookingPROFILE_x64.exp
 0002:00006100       rgszName                   000000018002d100     PhysX3CookingPROFILE_x64.exp
 0002:00006108       rgwOrd                     000000018002d108     PhysX3CookingPROFILE_x64.exp
 0002:0000610c       szName                     000000018002d10c     PhysX3CookingPROFILE_x64.exp
 0002:00006129       $N00001                    000000018002d129     PhysX3CookingPROFILE_x64.exp
 0002:00006139       $N00002                    000000018002d139     PhysX3CookingPROFILE_x64.exp
 0002:00006326       .idata$6                   000000018002d326     kernel32:KERNEL32.dll
 0002:000063ca       .idata$6                   000000018002d3ca     MSVCRT:MSVCR120.dll
 0003:00000000       physXCommonDebugx64        000000018002e000     WindowsCookingDelayLoadHook.obj
 0003:00000008       physXCommonCheckedx64      000000018002e008     WindowsCookingDelayLoadHook.obj
 0003:00000010       physXCommonProfilex64      000000018002e010     WindowsCookingDelayLoadHook.obj
 0003:00000018       physXCommonReleasex64      000000018002e018     WindowsCookingDelayLoadHook.obj
 0003:00000020       physXCommonDebugx86        000000018002e020     WindowsCookingDelayLoadHook.obj
 0003:00000028       physXCommonCheckedx86      000000018002e028     WindowsCookingDelayLoadHook.obj
 0003:00000030       physXCommonProfilex86      000000018002e030     WindowsCookingDelayLoadHook.obj
 0003:00000038       physXCommonReleasex86      000000018002e038     WindowsCookingDelayLoadHook.obj
 0003:00000040       physXCommonDebugARM        000000018002e040     WindowsCookingDelayLoadHook.obj
 0003:00000048       physXCommonCheckedARM      000000018002e048     WindowsCookingDelayLoadHook.obj
 0003:00000050       physXCommonProfileARM      000000018002e050     WindowsCookingDelayLoadHook.obj
 0003:00000058       physXCommonReleaseARM      000000018002e058     WindowsCookingDelayLoadHook.obj
 0003:000000d4       ?er@?1??neib@Tri@physx@@QEAAAEAHHH@Z@4HA 000000018002e0d4     hulllib.obj
 0003:00000740       gDelayLoadHook             000000018002e740     WindowsCookingDelayLoadHook.obj
 0003:00000750       minV4Error                 000000018002e750     RTreeCooking.obj
 0003:00000760       maxV4Error                 000000018002e760     RTreeCooking.obj
 0003:00000770       minFError                  000000018002e770     RTreeCooking.obj
 0003:00000780       minV3Error                 000000018002e780     RTreeCooking.obj
 0003:00000790       maxV3Error                 000000018002e790     RTreeCooking.obj
 0003:000007a0       maxFError                  000000018002e7a0     RTreeCooking.obj
 0003:000007b0       minV4Error                 000000018002e7b0     TriangleMeshBuilder.obj
 0003:000007c0       maxV4Error                 000000018002e7c0     TriangleMeshBuilder.obj
 0003:000007d0       minFError                  000000018002e7d0     TriangleMeshBuilder.obj
 0003:000007e0       minV3Error                 000000018002e7e0     TriangleMeshBuilder.obj
 0003:000007f0       maxV3Error                 000000018002e7f0     TriangleMeshBuilder.obj
 0003:00000800       maxFError                  000000018002e800     TriangleMeshBuilder.obj
 0003:00000810       minV4Error                 000000018002e810     ConvexMeshBuilder.obj
 0003:00000820       maxV4Error                 000000018002e820     ConvexMeshBuilder.obj
 0003:00000830       minFError                  000000018002e830     ConvexMeshBuilder.obj
 0003:00000840       minV3Error                 000000018002e840     ConvexMeshBuilder.obj
 0003:00000850       maxV3Error                 000000018002e850     ConvexMeshBuilder.obj
 0003:00000860       maxFError                  000000018002e860     ConvexMeshBuilder.obj
 0003:00000870       minV4Error                 000000018002e870     Cooking.obj
 0003:00000880       maxV4Error                 000000018002e880     Cooking.obj
 0003:00000890       minFError                  000000018002e890     Cooking.obj
 0003:000008a0       minV3Error                 000000018002e8a0     Cooking.obj
 0003:000008b0       maxV3Error                 000000018002e8b0     Cooking.obj
 0003:000008c0       maxFError                  000000018002e8c0     Cooking.obj
 0003:000008d0       minV4Error                 000000018002e8d0     InternalTriangleMeshBuilder.obj
 0003:000008e0       maxV4Error                 000000018002e8e0     InternalTriangleMeshBuilder.obj
 0003:000008f0       minFError                  000000018002e8f0     InternalTriangleMeshBuilder.obj
 0003:00000900       minV3Error                 000000018002e900     InternalTriangleMeshBuilder.obj
 0003:00000910       maxV3Error                 000000018002e910     InternalTriangleMeshBuilder.obj
 0003:00000920       maxFError                  000000018002e920     InternalTriangleMeshBuilder.obj
 0003:00000950       __proc_attached            000000018002e950     MSVCRT:crtdll.obj
 0004:00000000       $pdata$?physXCommonDliNotePreLoadLibrary@shdfnd@physx@@YAP6A_JXZPEBDPEBVPxDelayLoadHook@2@@Z 000000018002f000     WindowsCookingDelayLoadHook.obj
 0004:0000000c       $pdata$?saveHeightField@physx@@YA_NAEBVHeightField@Gu@1@AEAVPxOutputStream@1@_N@Z 000000018002f00c     HeightFieldCooking.obj
 0004:00000018       $pdata$1$?saveHeightField@physx@@YA_NAEBVHeightField@Gu@1@AEAVPxOutputStream@1@_N@Z 000000018002f018     HeightFieldCooking.obj
 0004:00000024       $pdata$2$?saveHeightField@physx@@YA_NAEBVHeightField@Gu@1@AEAVPxOutputStream@1@_N@Z 000000018002f024     HeightFieldCooking.obj
 0004:00000030       $pdata$?buildFromTriangles@RTreeCooker@physx@@SAXAEAURTree@Gu@2@PEBVPxVec3@2@IPEBGPEBIIAEAV?$Array@IV?$ReflectionAllocator@I@shdfnd@physx@@@shdfnd@2@PEAURemapCallback@12@MW4Enum@PxMeshCookingHint@2@@Z 000000018002f030     RTreeCooking.obj
 0004:0000003c       $pdata$4$?buildFromTriangles@RTreeCooker@physx@@SAXAEAURTree@Gu@2@PEBVPxVec3@2@IPEBGPEBIIAEAV?$Array@IV?$ReflectionAllocator@I@shdfnd@physx@@@shdfnd@2@PEAURemapCallback@12@MW4Enum@PxMeshCookingHint@2@@Z 000000018002f03c     RTreeCooking.obj
 0004:00000048       $pdata$7$?buildFromTriangles@RTreeCooker@physx@@SAXAEAURTree@Gu@2@PEBVPxVec3@2@IPEBGPEBIIAEAV?$Array@IV?$ReflectionAllocator@I@shdfnd@physx@@@shdfnd@2@PEAURemapCallback@12@MW4Enum@PxMeshCookingHint@2@@Z 000000018002f048     RTreeCooking.obj
 0004:00000054       $pdata$8$?buildFromTriangles@RTreeCooker@physx@@SAXAEAURTree@Gu@2@PEBVPxVec3@2@IPEBGPEBIIAEAV?$Array@IV?$ReflectionAllocator@I@shdfnd@physx@@@shdfnd@2@PEAURemapCallback@12@MW4Enum@PxMeshCookingHint@2@@Z 000000018002f054     RTreeCooking.obj
 0004:00000060       $pdata$9$?buildFromTriangles@RTreeCooker@physx@@SAXAEAURTree@Gu@2@PEBVPxVec3@2@IPEBGPEBIIAEAV?$Array@IV?$ReflectionAllocator@I@shdfnd@physx@@@shdfnd@2@PEAURemapCallback@12@MW4Enum@PxMeshCookingHint@2@@Z 000000018002f060     RTreeCooking.obj
 0004:0000006c       $pdata$?buildFromBounds@physx@@YAXAEAURTree@Gu@1@PEBUPxBounds3V@1@IAEAV?$Array@IV?$ReflectionAllocator@I@shdfnd@physx@@@shdfnd@1@PEAURemapCallback@RTreeCooker@1@AEAT__m128@@4MW4Enum@PxMeshCookingHint@1@@Z 000000018002f06c     RTreeCooking.obj
 0004:00000078       $pdata$??$median3@I$$CBUSortBoundsPredicate@physx@@@internal@shdfnd@physx@@YAXPEAIHHAEBUSortBoundsPredicate@2@@Z 000000018002f078     RTreeCooking.obj
 0004:00000084       $pdata$??$partition@I$$CBU?$Less@I@shdfnd@physx@@@internal@shdfnd@physx@@YAHPEAIHHAEBU?$Less@I@12@@Z 000000018002f084     RTreeCooking.obj
 0004:00000090       $pdata$??$partition@I$$CBUSortBoundsPredicate@physx@@@internal@shdfnd@physx@@YAHPEAIHHAEBUSortBoundsPredicate@2@@Z 000000018002f090     RTreeCooking.obj
 0004:0000009c       $pdata$??$partition@UBoundsLTE@physx@@@quickSelect@physx@@YAIPEIAIIIIAEBUBoundsLTE@1@@Z 000000018002f09c     RTreeCooking.obj
 0004:000000a8       $pdata$2$??$partition@UBoundsLTE@physx@@@quickSelect@physx@@YAIPEIAIIIIAEBUBoundsLTE@1@@Z 000000018002f0a8     RTreeCooking.obj
 0004:000000b4       $pdata$3$??$partition@UBoundsLTE@physx@@@quickSelect@physx@@YAIPEIAIIIIAEBUBoundsLTE@1@@Z 000000018002f0b4     RTreeCooking.obj
 0004:000000c0       $pdata$??$quickSelectFirstK@UBoundsLTE@physx@@@quickSelect@physx@@YAXPEIAIIIIAEBUBoundsLTE@1@@Z 000000018002f0c0     RTreeCooking.obj
 0004:000000cc       $pdata$??$smallSort@I$$CBU?$Less@I@shdfnd@physx@@@internal@shdfnd@physx@@YAXPEAIHHAEBU?$Less@I@12@@Z 000000018002f0cc     RTreeCooking.obj
 0004:000000d8       $pdata$5$??$smallSort@I$$CBU?$Less@I@shdfnd@physx@@@internal@shdfnd@physx@@YAXPEAIHHAEBU?$Less@I@12@@Z 000000018002f0d8     RTreeCooking.obj
 0004:000000e4       $pdata$6$??$smallSort@I$$CBU?$Less@I@shdfnd@physx@@@internal@shdfnd@physx@@YAXPEAIHHAEBU?$Less@I@12@@Z 000000018002f0e4     RTreeCooking.obj
 0004:000000f0       $pdata$??$smallSort@I$$CBUSortBoundsPredicate@physx@@@internal@shdfnd@physx@@YAXPEAIHHAEBUSortBoundsPredicate@2@@Z 000000018002f0f0     RTreeCooking.obj
 0004:000000fc       $pdata$6$??$smallSort@I$$CBUSortBoundsPredicate@physx@@@internal@shdfnd@physx@@YAXPEAIHHAEBUSortBoundsPredicate@2@@Z 000000018002f0fc     RTreeCooking.obj
 0004:00000108       $pdata$7$??$smallSort@I$$CBUSortBoundsPredicate@physx@@@internal@shdfnd@physx@@YAXPEAIHHAEBUSortBoundsPredicate@2@@Z 000000018002f108     RTreeCooking.obj
 0004:00000114       $pdata$??$sort@I@shdfnd@physx@@YAXPEAII@Z 000000018002f114     RTreeCooking.obj
 0004:00000120       $pdata$??$sort@IU?$Less@I@shdfnd@physx@@V?$ReflectionAllocator@I@23@@shdfnd@physx@@YAXPEAIIAEBU?$Less@I@01@AEBV?$ReflectionAllocator@I@01@I@Z 000000018002f120     RTreeCooking.obj
 0004:0000012c       $pdata$??$sort@IUSortBoundsPredicate@physx@@@shdfnd@physx@@YAXPEAIIAEBUSortBoundsPredicate@1@@Z 000000018002f12c     RTreeCooking.obj
 0004:00000138       $pdata$??$sort@IUSortBoundsPredicate@physx@@V?$ReflectionAllocator@I@shdfnd@2@@shdfnd@physx@@YAXPEAIIAEBUSortBoundsPredicate@1@AEBV?$ReflectionAllocator@I@01@I@Z 000000018002f138     RTreeCooking.obj
 0004:00000144       $pdata$??0?$Array@IV?$ReflectionAllocator@I@shdfnd@physx@@@shdfnd@physx@@QEAA@IAEBIAEBV?$ReflectionAllocator@I@12@@Z 000000018002f144     RTreeCooking.obj
 0004:00000150       $pdata$??0SubSortQuick@physx@@QEAA@PEAIPEBUPxBounds3V@1@IM@Z 000000018002f150     RTreeCooking.obj
 0004:0000015c       $pdata$??0SubSortSAH@physx@@QEAA@PEAIPEBUPxBounds3V@1@IPEBI22222M@Z 000000018002f15c     RTreeCooking.obj
 0004:00000168       $pdata$??1?$Array@IV?$ReflectionAllocator@I@shdfnd@physx@@@shdfnd@physx@@QEAA@XZ 000000018002f168     RTreeCooking.obj
 0004:00000174       $pdata$??1?$Array@UInterval@physx@@V?$InlineAllocator@$0CA@V?$ReflectionAllocator@UInterval@physx@@@shdfnd@physx@@@shdfnd@2@@shdfnd@physx@@QEAA@XZ 000000018002f174     RTreeCooking.obj
 0004:00000180       $pdata$??1?$Array@UPxBounds3V@physx@@V?$ReflectionAllocator@UPxBounds3V@physx@@@shdfnd@2@@shdfnd@physx@@QEAA@XZ 000000018002f180     RTreeCooking.obj
 0004:0000018c       $pdata$??1?$Array@URTreeNodeNQ@physx@@V?$ReflectionAllocator@URTreeNodeNQ@physx@@@shdfnd@2@@shdfnd@physx@@QEAA@XZ 000000018002f18c     RTreeCooking.obj
 0004:00000198       $pdata$??1?$Array@URTreeNodeQ@Gu@physx@@V?$ReflectionAllocator@URTreeNodeQ@Gu@physx@@@shdfnd@3@@shdfnd@physx@@QEAA@XZ 000000018002f198     RTreeCooking.obj
 0004:000001a4       $pdata$??1?$Array@VPxVec3@physx@@V?$ReflectionAllocator@VPxVec3@physx@@@shdfnd@2@@shdfnd@physx@@QEAA@XZ 000000018002f1a4     RTreeCooking.obj
 0004:000001b0       $pdata$??1?$InlineArray@UInterval@physx@@$03V?$ReflectionAllocator@UInterval@physx@@@shdfnd@2@@shdfnd@physx@@QEAA@XZ 000000018002f1b0     RTreeCooking.obj
 0004:000001bc       $pdata$??1?$Stack@V?$ReflectionAllocator@I@shdfnd@physx@@@internal@shdfnd@physx@@QEAA@XZ 000000018002f1bc     RTreeCooking.obj
 0004:000001c8       $pdata$0$??1?$Stack@V?$ReflectionAllocator@I@shdfnd@physx@@@internal@shdfnd@physx@@QEAA@XZ 000000018002f1c8     RTreeCooking.obj
 0004:000001d4       $pdata$2$??1?$Stack@V?$ReflectionAllocator@I@shdfnd@physx@@@internal@shdfnd@physx@@QEAA@XZ 000000018002f1d4     RTreeCooking.obj
 0004:000001e0       $pdata$3$??1?$Stack@V?$ReflectionAllocator@I@shdfnd@physx@@@internal@shdfnd@physx@@QEAA@XZ 000000018002f1e0     RTreeCooking.obj
 0004:000001ec       $pdata$??1SubSortQuick@physx@@QEAA@XZ 000000018002f1ec     RTreeCooking.obj
 0004:000001f8       $pdata$??1SubSortSAH@physx@@QEAA@XZ 000000018002f1f8     RTreeCooking.obj
 0004:00000204       $pdata$?PxMemCopy@physx@@YAPEAXPEIAXPEIBXI@Z 000000018002f204     RTreeCooking.obj
 0004:00000210       $pdata$?allocate@?$AlignedAllocator@$0IA@VAllocator@shdfnd@physx@@@shdfnd@physx@@QEAAPEAX_KPEBDH@Z 000000018002f210     RTreeCooking.obj
 0004:0000021c       $pdata$?allocate@?$Array@UInterval@physx@@V?$InlineAllocator@$0CA@V?$ReflectionAllocator@UInterval@physx@@@shdfnd@physx@@@shdfnd@2@@shdfnd@physx@@IEAAPEAUInterval@3@I@Z 000000018002f21c     RTreeCooking.obj
 0004:00000228       $pdata$?allocate@?$ReflectionAllocator@I@shdfnd@physx@@QEAAPEAX_KPEBDH@Z 000000018002f228     RTreeCooking.obj
 0004:00000234       $pdata$0$?allocate@?$ReflectionAllocator@I@shdfnd@physx@@QEAAPEAX_KPEBDH@Z 000000018002f234     RTreeCooking.obj
 0004:00000240       $pdata$1$?allocate@?$ReflectionAllocator@I@shdfnd@physx@@QEAAPEAX_KPEBDH@Z 000000018002f240     RTreeCooking.obj
 0004:0000024c       $pdata$?allocate@?$ReflectionAllocator@UInterval@physx@@@shdfnd@physx@@QEAAPEAX_KPEBDH@Z 000000018002f24c     RTreeCooking.obj
 0004:00000258       $pdata$0$?allocate@?$ReflectionAllocator@UInterval@physx@@@shdfnd@physx@@QEAAPEAX_KPEBDH@Z 000000018002f258     RTreeCooking.obj
 0004:00000264       $pdata$1$?allocate@?$ReflectionAllocator@UInterval@physx@@@shdfnd@physx@@QEAAPEAX_KPEBDH@Z 000000018002f264     RTreeCooking.obj
 0004:00000270       $pdata$?allocate@?$ReflectionAllocator@UPxBounds3V@physx@@@shdfnd@physx@@QEAAPEAX_KPEBDH@Z 000000018002f270     RTreeCooking.obj
 0004:0000027c       $pdata$0$?allocate@?$ReflectionAllocator@UPxBounds3V@physx@@@shdfnd@physx@@QEAAPEAX_KPEBDH@Z 000000018002f27c     RTreeCooking.obj
 0004:00000288       $pdata$1$?allocate@?$ReflectionAllocator@UPxBounds3V@physx@@@shdfnd@physx@@QEAAPEAX_KPEBDH@Z 000000018002f288     RTreeCooking.obj
 0004:00000294       $pdata$?allocate@?$ReflectionAllocator@URTreeNodeNQ@physx@@@shdfnd@physx@@QEAAPEAX_KPEBDH@Z 000000018002f294     RTreeCooking.obj
 0004:000002a0       $pdata$0$?allocate@?$ReflectionAllocator@URTreeNodeNQ@physx@@@shdfnd@physx@@QEAAPEAX_KPEBDH@Z 000000018002f2a0     RTreeCooking.obj
 0004:000002ac       $pdata$1$?allocate@?$ReflectionAllocator@URTreeNodeNQ@physx@@@shdfnd@physx@@QEAAPEAX_KPEBDH@Z 000000018002f2ac     RTreeCooking.obj
 0004:000002b8       $pdata$?allocate@?$ReflectionAllocator@URTreeNodeQ@Gu@physx@@@shdfnd@physx@@QEAAPEAX_KPEBDH@Z 000000018002f2b8     RTreeCooking.obj
 0004:000002c4       $pdata$0$?allocate@?$ReflectionAllocator@URTreeNodeQ@Gu@physx@@@shdfnd@physx@@QEAAPEAX_KPEBDH@Z 000000018002f2c4     RTreeCooking.obj
 0004:000002d0       $pdata$1$?allocate@?$ReflectionAllocator@URTreeNodeQ@Gu@physx@@@shdfnd@physx@@QEAAPEAX_KPEBDH@Z 000000018002f2d0     RTreeCooking.obj
 0004:000002dc       $pdata$?allocate@?$ReflectionAllocator@VPxVec3@physx@@@shdfnd@physx@@QEAAPEAX_KPEBDH@Z 000000018002f2dc     RTreeCooking.obj
 0004:000002e8       $pdata$0$?allocate@?$ReflectionAllocator@VPxVec3@physx@@@shdfnd@physx@@QEAAPEAX_KPEBDH@Z 000000018002f2e8     RTreeCooking.obj
 0004:000002f4       $pdata$1$?allocate@?$ReflectionAllocator@VPxVec3@physx@@@shdfnd@physx@@QEAAPEAX_KPEBDH@Z 000000018002f2f4     RTreeCooking.obj
 0004:00000300       $pdata$?copy@?$Array@URTreeNodeNQ@physx@@V?$ReflectionAllocator@URTreeNodeNQ@physx@@@shdfnd@2@@shdfnd@physx@@KAXPEAURTreeNodeNQ@3@0PEBU43@@Z 000000018002f300     RTreeCooking.obj
 0004:0000030c       $pdata$0$?copy@?$Array@URTreeNodeNQ@physx@@V?$ReflectionAllocator@URTreeNodeNQ@physx@@@shdfnd@2@@shdfnd@physx@@KAXPEAURTreeNodeNQ@3@0PEBU43@@Z 000000018002f30c     RTreeCooking.obj
 0004:00000318       $pdata$1$?copy@?$Array@URTreeNodeNQ@physx@@V?$ReflectionAllocator@URTreeNodeNQ@physx@@@shdfnd@2@@shdfnd@physx@@KAXPEAURTreeNodeNQ@3@0PEBU43@@Z 000000018002f318     RTreeCooking.obj
 0004:00000324       $pdata$?deallocate@?$Array@IV?$ReflectionAllocator@I@shdfnd@physx@@@shdfnd@physx@@IEAAXPEAX@Z 000000018002f324     RTreeCooking.obj
 0004:00000330       $pdata$?deallocate@?$Array@UInterval@physx@@V?$InlineAllocator@$0CA@V?$ReflectionAllocator@UInterval@physx@@@shdfnd@physx@@@shdfnd@2@@shdfnd@physx@@IEAAXPEAX@Z 000000018002f330     RTreeCooking.obj
 0004:0000033c       $pdata$?deallocate@?$Array@UPxBounds3V@physx@@V?$ReflectionAllocator@UPxBounds3V@physx@@@shdfnd@2@@shdfnd@physx@@IEAAXPEAX@Z 000000018002f33c     RTreeCooking.obj
 0004:00000348       $pdata$?deallocate@?$Array@URTreeNodeNQ@physx@@V?$ReflectionAllocator@URTreeNodeNQ@physx@@@shdfnd@2@@shdfnd@physx@@IEAAXPEAX@Z 000000018002f348     RTreeCooking.obj
 0004:00000354       $pdata$?deallocate@?$Array@URTreeNodeQ@Gu@physx@@V?$ReflectionAllocator@URTreeNodeQ@Gu@physx@@@shdfnd@3@@shdfnd@physx@@IEAAXPEAX@Z 000000018002f354     RTreeCooking.obj
 0004:00000360       $pdata$?deallocate@?$Array@VPxVec3@physx@@V?$ReflectionAllocator@VPxVec3@physx@@@shdfnd@2@@shdfnd@physx@@IEAAXPEAX@Z 000000018002f360     RTreeCooking.obj
 0004:0000036c       $pdata$?deallocate@?$InlineAllocator@$0CA@V?$ReflectionAllocator@UInterval@physx@@@shdfnd@physx@@@shdfnd@physx@@QEAAXPEAX@Z 000000018002f36c     RTreeCooking.obj
 0004:00000378       $pdata$?deallocate@?$ReflectionAllocator@I@shdfnd@physx@@QEAAXPEAX@Z 000000018002f378     RTreeCooking.obj
 0004:00000384       $pdata$?deallocate@?$ReflectionAllocator@UInterval@physx@@@shdfnd@physx@@QEAAXPEAX@Z 000000018002f384     RTreeCooking.obj
 0004:00000390       $pdata$?deallocate@?$ReflectionAllocator@UPxBounds3V@physx@@@shdfnd@physx@@QEAAXPEAX@Z 000000018002f390     RTreeCooking.obj
 0004:0000039c       $pdata$?deallocate@?$ReflectionAllocator@URTreeNodeNQ@physx@@@shdfnd@physx@@QEAAXPEAX@Z 000000018002f39c     RTreeCooking.obj
 0004:000003a8       $pdata$?deallocate@?$ReflectionAllocator@URTreeNodeQ@Gu@physx@@@shdfnd@physx@@QEAAXPEAX@Z 000000018002f3a8     RTreeCooking.obj
 0004:000003b4       $pdata$?deallocate@?$ReflectionAllocator@VPxVec3@physx@@@shdfnd@physx@@QEAAXPEAX@Z 000000018002f3b4     RTreeCooking.obj
 0004:000003c0       $pdata$?getName@?$ReflectionAllocator@I@shdfnd@physx@@CAPEBDXZ 000000018002f3c0     RTreeCooking.obj
 0004:000003cc       $pdata$?getName@?$ReflectionAllocator@UInterval@physx@@@shdfnd@physx@@CAPEBDXZ 000000018002f3cc     RTreeCooking.obj
 0004:000003d8       $pdata$?getName@?$ReflectionAllocator@UPxBounds3V@physx@@@shdfnd@physx@@CAPEBDXZ 000000018002f3d8     RTreeCooking.obj
 0004:000003e4       $pdata$?getName@?$ReflectionAllocator@URTreeNodeNQ@physx@@@shdfnd@physx@@CAPEBDXZ 000000018002f3e4     RTreeCooking.obj
 0004:000003f0       $pdata$?getName@?$ReflectionAllocator@URTreeNodeQ@Gu@physx@@@shdfnd@physx@@CAPEBDXZ 000000018002f3f0     RTreeCooking.obj
 0004:000003fc       $pdata$?getName@?$ReflectionAllocator@VPxVec3@physx@@@shdfnd@physx@@CAPEBDXZ 000000018002f3fc     RTreeCooking.obj
 0004:00000408       $pdata$?grow@?$Stack@V?$ReflectionAllocator@I@shdfnd@physx@@@internal@shdfnd@physx@@QEAAXXZ 000000018002f408     RTreeCooking.obj
 0004:00000414       $pdata$?growAndPushBack@?$Array@IV?$ReflectionAllocator@I@shdfnd@physx@@@shdfnd@physx@@IEAAAEAIAEBI@Z 000000018002f414     RTreeCooking.obj
 0004:00000420       $pdata$?growAndPushBack@?$Array@UInterval@physx@@V?$InlineAllocator@$0CA@V?$ReflectionAllocator@UInterval@physx@@@shdfnd@physx@@@shdfnd@2@@shdfnd@physx@@IEAAAEAUInterval@3@AEBU43@@Z 000000018002f420     RTreeCooking.obj
 0004:0000042c       $pdata$?growAndPushBack@?$Array@UPxBounds3V@physx@@V?$ReflectionAllocator@UPxBounds3V@physx@@@shdfnd@2@@shdfnd@physx@@IEAAAEAUPxBounds3V@3@AEBU43@@Z 000000018002f42c     RTreeCooking.obj
 0004:00000438       $pdata$?growAndPushBack@?$Array@URTreeNodeNQ@physx@@V?$ReflectionAllocator@URTreeNodeNQ@physx@@@shdfnd@2@@shdfnd@physx@@IEAAAEAURTreeNodeNQ@3@AEBU43@@Z 000000018002f438     RTreeCooking.obj
 0004:00000444       $pdata$?growAndPushBack@?$Array@URTreeNodeQ@Gu@physx@@V?$ReflectionAllocator@URTreeNodeQ@Gu@physx@@@shdfnd@3@@shdfnd@physx@@IEAAAEAURTreeNodeQ@Gu@3@AEBU453@@Z 000000018002f444     RTreeCooking.obj
 0004:00000450       $pdata$?growAndPushBack@?$Array@VPxVec3@physx@@V?$ReflectionAllocator@VPxVec3@physx@@@shdfnd@2@@shdfnd@physx@@IEAAAEAVPxVec3@3@AEBV43@@Z 000000018002f450     RTreeCooking.obj
 0004:0000045c       $pdata$?memCopy@intrinsics@physx@@YAPEAXPEIAXPEIBXI@Z 000000018002f45c     RTreeCooking.obj
 0004:00000468       $pdata$?push@?$Stack@V?$ReflectionAllocator@I@shdfnd@physx@@@internal@shdfnd@physx@@QEAAXHH@Z 000000018002f468     RTreeCooking.obj
 0004:00000474       $pdata$?recreate@?$Array@IV?$ReflectionAllocator@I@shdfnd@physx@@@shdfnd@physx@@IEAAXI@Z 000000018002f474     RTreeCooking.obj
 0004:00000480       $pdata$?recreate@?$Array@UPxBounds3V@physx@@V?$ReflectionAllocator@UPxBounds3V@physx@@@shdfnd@2@@shdfnd@physx@@IEAAXI@Z 000000018002f480     RTreeCooking.obj
 0004:0000048c       $pdata$?recreate@?$Array@URTreeNodeNQ@physx@@V?$ReflectionAllocator@URTreeNodeNQ@physx@@@shdfnd@2@@shdfnd@physx@@IEAAXI@Z 000000018002f48c     RTreeCooking.obj
 0004:00000498       $pdata$?recreate@?$Array@URTreeNodeQ@Gu@physx@@V?$ReflectionAllocator@URTreeNodeQ@Gu@physx@@@shdfnd@3@@shdfnd@physx@@IEAAXI@Z 000000018002f498     RTreeCooking.obj
 0004:000004a4       $pdata$?recreate@?$Array@VPxVec3@physx@@V?$ReflectionAllocator@VPxVec3@physx@@@shdfnd@2@@shdfnd@physx@@IEAAXI@Z 000000018002f4a4     RTreeCooking.obj
 0004:000004b0       $pdata$?resize@?$Array@IV?$ReflectionAllocator@I@shdfnd@physx@@@shdfnd@physx@@QEAAXIAEBI@Z 000000018002f4b0     RTreeCooking.obj
 0004:000004bc       $pdata$?resizeUninitialized@?$Array@URTreeNodeNQ@physx@@V?$ReflectionAllocator@URTreeNodeNQ@physx@@@shdfnd@2@@shdfnd@physx@@QEAAXI@Z 000000018002f4bc     RTreeCooking.obj
 0004:000004c8       $pdata$?sort4@SubSortQuick@physx@@QEAAXPEIAIIAEAV?$Array@URTreeNodeNQ@physx@@V?$ReflectionAllocator@URTreeNodeNQ@physx@@@shdfnd@2@@shdfnd@2@AEAIAEAUPxBounds3V@2@I@Z 000000018002f4c8     RTreeCooking.obj
 0004:000004d4       $pdata$?sort4@SubSortSAH@physx@@QEAAXPEAIIAEAV?$Array@URTreeNodeNQ@physx@@V?$ReflectionAllocator@URTreeNodeNQ@physx@@@shdfnd@2@@shdfnd@2@AEAIIPEAURTreeNodeNQ@2@@Z 000000018002f4d4     RTreeCooking.obj
 0004:000004e0       $pdata$?split@SubSortSAH@physx@@QEAAIPEAII@Z 000000018002f4e0     RTreeCooking.obj
 0004:000004ec       $pdata$4$?split@SubSortSAH@physx@@QEAAIPEAII@Z 000000018002f4ec     RTreeCooking.obj
 0004:000004f8       $pdata$5$?split@SubSortSAH@physx@@QEAAIPEAII@Z 000000018002f4f8     RTreeCooking.obj
 0004:00000504       $pdata$6$?split@SubSortSAH@physx@@QEAAIPEAII@Z 000000018002f504     RTreeCooking.obj
 0004:00000510       $pdata$7$?split@SubSortSAH@physx@@QEAAIPEAII@Z 000000018002f510     RTreeCooking.obj
 0004:0000051c       $pdata$?loadFromDesc@TriangleMeshBuilder@physx@@QEAA_NAEBVPxTriangleMeshDesc@2@AEBUPxCookingParams@2@_N@Z 000000018002f51c     TriangleMeshBuilder.obj
 0004:00000528       $pdata$0$?loadFromDesc@TriangleMeshBuilder@physx@@QEAA_NAEBVPxTriangleMeshDesc@2@AEBUPxCookingParams@2@_N@Z 000000018002f528     TriangleMeshBuilder.obj
 0004:00000534       $pdata$1$?loadFromDesc@TriangleMeshBuilder@physx@@QEAA_NAEBVPxTriangleMeshDesc@2@AEBUPxCookingParams@2@_N@Z 000000018002f534     TriangleMeshBuilder.obj
 0004:00000540       $pdata$2$?loadFromDesc@TriangleMeshBuilder@physx@@QEAA_NAEBVPxTriangleMeshDesc@2@AEBUPxCookingParams@2@_N@Z 000000018002f540     TriangleMeshBuilder.obj
 0004:0000054c       $pdata$3$?loadFromDesc@TriangleMeshBuilder@physx@@QEAA_NAEBVPxTriangleMeshDesc@2@AEBUPxCookingParams@2@_N@Z 000000018002f54c     TriangleMeshBuilder.obj
 0004:00000558       $pdata$4$?loadFromDesc@TriangleMeshBuilder@physx@@QEAA_NAEBVPxTriangleMeshDesc@2@AEBUPxCookingParams@2@_N@Z 000000018002f558     TriangleMeshBuilder.obj
 0004:00000564       $pdata$5$?loadFromDesc@TriangleMeshBuilder@physx@@QEAA_NAEBVPxTriangleMeshDesc@2@AEBUPxCookingParams@2@_N@Z 000000018002f564     TriangleMeshBuilder.obj
 0004:00000570       $pdata$?save@TriangleMeshBuilder@physx@@QEBA_NAEAVPxOutputStream@2@_NAEBUPxCookingParams@2@@Z 000000018002f570     TriangleMeshBuilder.obj
 0004:0000057c       $pdata$0$?save@TriangleMeshBuilder@physx@@QEBA_NAEAVPxOutputStream@2@_NAEBUPxCookingParams@2@@Z 000000018002f57c     TriangleMeshBuilder.obj
 0004:00000588       $pdata$3$?save@TriangleMeshBuilder@physx@@QEBA_NAEAVPxOutputStream@2@_NAEBUPxCookingParams@2@@Z 000000018002f588     TriangleMeshBuilder.obj
 0004:00000594       $pdata$4$?save@TriangleMeshBuilder@physx@@QEBA_NAEAVPxOutputStream@2@_NAEBUPxCookingParams@2@@Z 000000018002f594     TriangleMeshBuilder.obj
 0004:000005a0       $pdata$5$?save@TriangleMeshBuilder@physx@@QEBA_NAEAVPxOutputStream@2@_NAEBUPxCookingParams@2@@Z 000000018002f5a0     TriangleMeshBuilder.obj
 0004:000005ac       $pdata$?computeLocalBounds@TriangleMeshBuilder@physx@@IEAAXXZ 000000018002f5ac     TriangleMeshBuilder.obj
 0004:000005b8       $pdata$?importMesh@TriangleMeshBuilder@physx@@IEAA_NAEBVPxTriangleMeshDesc@2@AEBUPxCookingParams@2@_N@Z 000000018002f5b8     TriangleMeshBuilder.obj
 0004:000005c4       $pdata$??_H@YAXPEAX_KHP6APEAX0@Z@Z 000000018002f5c4     TriangleMeshBuilder.obj
 0004:000005d0       $pdata$?gatherStrided@shdfnd@physx@@YAXPEBXPEAXIII@Z 000000018002f5d0     TriangleMeshBuilder.obj
 0004:000005dc       $pdata$1$?gatherStrided@shdfnd@physx@@YAXPEBXPEAXIII@Z 000000018002f5dc     TriangleMeshBuilder.obj
 0004:000005e8       $pdata$2$?gatherStrided@shdfnd@physx@@YAXPEBXPEAXIII@Z 000000018002f5e8     TriangleMeshBuilder.obj
 0004:000005f4       $pdata$?Precompute@BigConvexDataBuilder@physx@@QEAA_NI@Z 000000018002f5f4     BigConvexDataBuilder.obj
 0004:00000600       $pdata$12$?Precompute@BigConvexDataBuilder@physx@@QEAA_NI@Z 000000018002f600     BigConvexDataBuilder.obj
 0004:0000060c       $pdata$14$?Precompute@BigConvexDataBuilder@physx@@QEAA_NI@Z 000000018002f60c     BigConvexDataBuilder.obj
 0004:00000618       $pdata$15$?Precompute@BigConvexDataBuilder@physx@@QEAA_NI@Z 000000018002f618     BigConvexDataBuilder.obj
 0004:00000624       $pdata$?Initialize@BigConvexDataBuilder@physx@@QEAA_NXZ 000000018002f624     BigConvexDataBuilder.obj
 0004:00000630       $pdata$0$?Initialize@BigConvexDataBuilder@physx@@QEAA_NXZ 000000018002f630     BigConvexDataBuilder.obj
 0004:0000063c       $pdata$1$?Initialize@BigConvexDataBuilder@physx@@QEAA_NXZ 000000018002f63c     BigConvexDataBuilder.obj
 0004:00000648       $pdata$?PrecomputeSample@BigConvexDataBuilder@physx@@QEAA_NIAEBVPxVec3@2@@Z 000000018002f648     BigConvexDataBuilder.obj
 0004:00000654       $pdata$?Save@BigConvexDataBuilder@physx@@QEBA_NAEAVPxOutputStream@2@_NIPEBUHullTriangleData@2@@Z 000000018002f654     BigConvexDataBuilder.obj
 0004:00000660       $pdata$?ComputeValencies@BigConvexDataBuilder@physx@@QEBA_NIPEBUHullTriangleData@2@@Z 000000018002f660     BigConvexDataBuilder.obj
 0004:0000066c       $pdata$?Compute@BigConvexDataBuilder@physx@@QEBA_NAEBUVALENCIESCREATE@2@@Z 000000018002f66c     BigConvexDataBuilder.obj
 0004:00000678       $pdata$?Save@BigConvexDataBuilder@physx@@QEBA_NAEAVPxOutputStream@2@_N@Z 000000018002f678     BigConvexDataBuilder.obj
 0004:00000684       $pdata$2$?Save@BigConvexDataBuilder@physx@@QEBA_NAEAVPxOutputStream@2@_N@Z 000000018002f684     BigConvexDataBuilder.obj
 0004:00000690       $pdata$3$?Save@BigConvexDataBuilder@physx@@QEBA_NAEAVPxOutputStream@2@_N@Z 000000018002f690     BigConvexDataBuilder.obj
 0004:0000069c       $pdata$?PxMemZero@physx@@YAPEAXPEIAXI@Z 000000018002f69c     BigConvexDataBuilder.obj
 0004:000006a8       $pdata$?allocate@?$ReflectionAllocator@E@shdfnd@physx@@QEAAPEAX_KPEBDH@Z 000000018002f6a8     BigConvexDataBuilder.obj
 0004:000006b4       $pdata$0$?allocate@?$ReflectionAllocator@E@shdfnd@physx@@QEAAPEAX_KPEBDH@Z 000000018002f6b4     BigConvexDataBuilder.obj
 0004:000006c0       $pdata$1$?allocate@?$ReflectionAllocator@E@shdfnd@physx@@QEAAPEAX_KPEBDH@Z 000000018002f6c0     BigConvexDataBuilder.obj
 0004:000006cc       $pdata$?allocate@?$ReflectionAllocator@G@shdfnd@physx@@QEAAPEAX_KPEBDH@Z 000000018002f6cc     BigConvexDataBuilder.obj
 0004:000006d8       $pdata$0$?allocate@?$ReflectionAllocator@G@shdfnd@physx@@QEAAPEAX_KPEBDH@Z 000000018002f6d8     BigConvexDataBuilder.obj
 0004:000006e4       $pdata$1$?allocate@?$ReflectionAllocator@G@shdfnd@physx@@QEAAPEAX_KPEBDH@Z 000000018002f6e4     BigConvexDataBuilder.obj
 0004:000006f0       $pdata$?allocate@?$ReflectionAllocator@UValency@Gu@physx@@@shdfnd@physx@@QEAAPEAX_KPEBDH@Z 000000018002f6f0     BigConvexDataBuilder.obj
 0004:000006fc       $pdata$0$?allocate@?$ReflectionAllocator@UValency@Gu@physx@@@shdfnd@physx@@QEAAPEAX_KPEBDH@Z 000000018002f6fc     BigConvexDataBuilder.obj
 0004:00000708       $pdata$1$?allocate@?$ReflectionAllocator@UValency@Gu@physx@@@shdfnd@physx@@QEAAPEAX_KPEBDH@Z 000000018002f708     BigConvexDataBuilder.obj
 0004:00000714       $pdata$?getName@?$ReflectionAllocator@E@shdfnd@physx@@CAPEBDXZ 000000018002f714     BigConvexDataBuilder.obj
 0004:00000720       $pdata$?getName@?$ReflectionAllocator@G@shdfnd@physx@@CAPEBDXZ 000000018002f720     BigConvexDataBuilder.obj
 0004:0000072c       $pdata$?getName@?$ReflectionAllocator@UValency@Gu@physx@@@shdfnd@physx@@CAPEBDXZ 000000018002f72c     BigConvexDataBuilder.obj
 0004:00000738       $pdata$?memZero@intrinsics@physx@@YAPEAXPEIAXI@Z 000000018002f738     BigConvexDataBuilder.obj
 0004:00000744       $pdata$?normalize@PxVec3@physx@@QEAAMXZ 000000018002f744     BigConvexDataBuilder.obj
 0004:00000750       $pdata$??1ConvexHullBuilder@physx@@QEAA@XZ 000000018002f750     ConvexHullBuilder.obj
 0004:0000075c       $pdata$?Init@ConvexHullBuilder@physx@@QEAA_NIPEBVPxVec3@2@IPEBIIPEBUPxHullPolygon@2@@Z 000000018002f75c     ConvexHullBuilder.obj
 0004:00000768       $pdata$1$?Init@ConvexHullBuilder@physx@@QEAA_NIPEBVPxVec3@2@IPEBIIPEBUPxHullPolygon@2@@Z 000000018002f768     ConvexHullBuilder.obj
 0004:00000774       $pdata$2$?Init@ConvexHullBuilder@physx@@QEAA_NIPEBVPxVec3@2@IPEBIIPEBUPxHullPolygon@2@@Z 000000018002f774     ConvexHullBuilder.obj
 0004:00000780       $pdata$?Save@ConvexHullBuilder@physx@@QEBA_NAEAVPxOutputStream@2@_N@Z 000000018002f780     ConvexHullBuilder.obj
 0004:0000078c       $pdata$3$?Save@ConvexHullBuilder@physx@@QEBA_NAEAVPxOutputStream@2@_N@Z 000000018002f78c     ConvexHullBuilder.obj
 0004:00000798       $pdata$4$?Save@ConvexHullBuilder@physx@@QEBA_NAEAVPxOutputStream@2@_N@Z 000000018002f798     ConvexHullBuilder.obj
 0004:000007a4       $pdata$?CreateEdgeList@ConvexHullBuilder@physx@@QEAA_NXZ 000000018002f7a4     ConvexHullBuilder.obj
 0004:000007b0       $pdata$?CreatePolygonData@ConvexHullBuilder@physx@@QEAA_NXZ 000000018002f7b0     ConvexHullBuilder.obj
 0004:000007bc       $pdata$2$?CreatePolygonData@ConvexHullBuilder@physx@@QEAA_NXZ 000000018002f7bc     ConvexHullBuilder.obj
 0004:000007c8       $pdata$3$?CreatePolygonData@ConvexHullBuilder@physx@@QEAA_NXZ 000000018002f7c8     ConvexHullBuilder.obj
 0004:000007d4       $pdata$?CheckHullPolygons@ConvexHullBuilder@physx@@QEBA_NXZ 000000018002f7d4     ConvexHullBuilder.obj
 0004:000007e0       $pdata$?CreateTrianglesFromPolygons@ConvexHullBuilder@physx@@QEAA_NXZ 000000018002f7e0     ConvexHullBuilder.obj
 0004:000007ec       $pdata$0$?CreateTrianglesFromPolygons@ConvexHullBuilder@physx@@QEAA_NXZ 000000018002f7ec     ConvexHullBuilder.obj
 0004:000007f8       $pdata$6$?CreateTrianglesFromPolygons@ConvexHullBuilder@physx@@QEAA_NXZ 000000018002f7f8     ConvexHullBuilder.obj
 0004:00000804       $pdata$7$?CreateTrianglesFromPolygons@ConvexHullBuilder@physx@@QEAA_NXZ 000000018002f804     ConvexHullBuilder.obj
 0004:00000810       $pdata$12$?CreateTrianglesFromPolygons@ConvexHullBuilder@physx@@QEAA_NXZ 000000018002f810     ConvexHullBuilder.obj
 0004:0000081c       $pdata$14$?CreateTrianglesFromPolygons@ConvexHullBuilder@physx@@QEAA_NXZ 000000018002f81c     ConvexHullBuilder.obj
 0004:00000828       $pdata$21$?CreateTrianglesFromPolygons@ConvexHullBuilder@physx@@QEAA_NXZ 000000018002f828     ConvexHullBuilder.obj
 0004:00000834       $pdata$22$?CreateTrianglesFromPolygons@ConvexHullBuilder@physx@@QEAA_NXZ 000000018002f834     ConvexHullBuilder.obj
 0004:00000840       $pdata$23$?CreateTrianglesFromPolygons@ConvexHullBuilder@physx@@QEAA_NXZ 000000018002f840     ConvexHullBuilder.obj
 0004:0000084c       $pdata$?ComputeGeomCenter@ConvexHullBuilder@physx@@QEBA_NAEAVPxVec3@2@@Z 000000018002f84c     ConvexHullBuilder.obj
 0004:00000858       $pdata$1$?ComputeGeomCenter@ConvexHullBuilder@physx@@QEBA_NAEAVPxVec3@2@@Z 000000018002f858     ConvexHullBuilder.obj
 0004:00000864       $pdata$7$?ComputeGeomCenter@ConvexHullBuilder@physx@@QEBA_NAEAVPxVec3@2@@Z 000000018002f864     ConvexHullBuilder.obj
 0004:00000870       $pdata$8$?ComputeGeomCenter@ConvexHullBuilder@physx@@QEBA_NAEAVPxVec3@2@@Z 000000018002f870     ConvexHullBuilder.obj
 0004:0000087c       $pdata$9$?ComputeGeomCenter@ConvexHullBuilder@physx@@QEBA_NAEAVPxVec3@2@@Z 000000018002f87c     ConvexHullBuilder.obj
 0004:00000888       $pdata$?CalculateVertexMapTable@ConvexHullBuilder@physx@@QEAA_NI_N@Z 000000018002f888     ConvexHullBuilder.obj
 0004:00000894       $pdata$?ComputeHullPolygons@ConvexHullBuilder@physx@@QEAA_NAEBIPEBVPxVec3@2@0PEBI@Z 000000018002f894     ConvexHullBuilder.obj
 0004:000008a0       $pdata$?inverseBuffer@@YA_NIPEAE@Z 000000018002f8a0     ConvexHullBuilder.obj
 0004:000008ac       $pdata$0$?inverseBuffer@@YA_NIPEAE@Z 000000018002f8ac     ConvexHullBuilder.obj
 0004:000008b8       $pdata$1$?inverseBuffer@@YA_NIPEAE@Z 000000018002f8b8     ConvexHullBuilder.obj
 0004:000008c4       $pdata$?findLineStrip@@YA_NAEAVContainer@Gu@physx@@AEBV123@@Z 000000018002f8c4     ConvexHullBuilder.obj
 0004:000008d0       $pdata$1$?findLineStrip@@YA_NAEAVContainer@Gu@physx@@AEBV123@@Z 000000018002f8d0     ConvexHullBuilder.obj
 0004:000008dc       $pdata$?CheckRedundantVertices@@YAXAEAIAEAVContainer@Gu@physx@@AEBVConvexHullBuilder@3@11@Z 000000018002f8dc     ConvexHullBuilder.obj
 0004:000008e8       $pdata$?ExtractHullPolygons@@YA_NAEAIAEAVContainer@Gu@physx@@AEBVConvexHullBuilder@3@PEAV123@1@Z 000000018002f8e8     ConvexHullBuilder.obj
 0004:000008f4       $pdata$?FloodFill@Local@?8??ExtractHullPolygons@@YA_NAEAIAEAVContainer@Gu@physx@@AEBVConvexHullBuilder@5@PEAV345@1@Z@SAX1PEBVAdjTriangle@5@IPEA_N@Z 000000018002f8f4     ConvexHullBuilder.obj
 0004:00000900       $pdata$?GetNeighborFace@Local@?8??ExtractHullPolygons@@YA_NAEAIAEAVContainer@Gu@physx@@AEBVConvexHullBuilder@5@PEAV345@1@Z@SA_NIIPEBVAdjTriangle@5@PEBI00@Z 000000018002f900     ConvexHullBuilder.obj
 0004:0000090c       $pdata$?CheckFloodFillFace@Local@?8??ExtractHullPolygons@@YA_NAEAIAEAVContainer@Gu@physx@@AEBVConvexHullBuilder@5@PEAV345@1@Z@SA_NIPEBVAdjTriangle@5@PEBI@Z 000000018002f90c     ConvexHullBuilder.obj
 0004:00000918       $pdata$6$?CheckFloodFillFace@Local@?8??ExtractHullPolygons@@YA_NAEAIAEAVContainer@Gu@physx@@AEBVConvexHullBuilder@5@PEAV345@1@Z@SA_NIPEBVAdjTriangle@5@PEBI@Z 000000018002f918     ConvexHullBuilder.obj
 0004:00000924       $pdata$8$?CheckFloodFillFace@Local@?8??ExtractHullPolygons@@YA_NAEAIAEAVContainer@Gu@physx@@AEBVConvexHullBuilder@5@PEAV345@1@Z@SA_NIPEBVAdjTriangle@5@PEBI@Z 000000018002f924     ConvexHullBuilder.obj
 0004:00000930       $pdata$?CheckFloodFill@Local@?8??ExtractHullPolygons@@YA_NAEAIAEAVContainer@Gu@physx@@AEBVConvexHullBuilder@5@PEAV345@1@Z@SA_N1PEAVAdjTriangle@5@PEA_NPEBI@Z 000000018002f930     ConvexHullBuilder.obj
 0004:0000093c       $pdata$?TestDuplicateTriangles@@YA_NAEAIPEAU?$TriangleT@I@Gu@physx@@_N@Z 000000018002f93c     ConvexHullBuilder.obj
 0004:00000948       $pdata$?testCulling@@YA_NAEBU?$TriangleT@I@Gu@physx@@PEBVPxVec3@3@AEBV43@@Z 000000018002f948     ConvexHullBuilder.obj
 0004:00000954       $pdata$?TestUnifiedNormals@@YA_NIPEBVPxVec3@physx@@IPEAU?$TriangleT@I@Gu@2@_N@Z 000000018002f954     ConvexHullBuilder.obj
 0004:00000960       $pdata$8$?TestUnifiedNormals@@YA_NIPEBVPxVec3@physx@@IPEAU?$TriangleT@I@Gu@2@_N@Z 000000018002f960     ConvexHullBuilder.obj
 0004:0000096c       $pdata$12$?TestUnifiedNormals@@YA_NIPEBVPxVec3@physx@@IPEAU?$TriangleT@I@Gu@2@_N@Z 000000018002f96c     ConvexHullBuilder.obj
 0004:00000978       $pdata$13$?TestUnifiedNormals@@YA_NIPEBVPxVec3@physx@@IPEAU?$TriangleT@I@Gu@2@_N@Z 000000018002f978     ConvexHullBuilder.obj
 0004:00000984       $pdata$14$?TestUnifiedNormals@@YA_NIPEBVPxVec3@physx@@IPEAU?$TriangleT@I@Gu@2@_N@Z 000000018002f984     ConvexHullBuilder.obj
 0004:00000990       $pdata$?cleanMesh@@YA_NAEAI0PEAVPxVec3@physx@@PEAU?$TriangleT@I@Gu@2@@Z 000000018002f990     ConvexHullBuilder.obj
 0004:0000099c       $pdata$?CleanHull@@YA_NAEAIPEAU?$TriangleT@I@Gu@physx@@0PEAVPxVec3@3@@Z 000000018002f99c     ConvexHullBuilder.obj
 0004:000009a8       $pdata$?CheckHull@@YA_NIPEBU?$TriangleT@I@Gu@physx@@IPEBVPxVec3@3@@Z 000000018002f9a8     ConvexHullBuilder.obj
 0004:000009b4       $pdata$?computeNewellPlane@@YA_NAEAVPxPlane@physx@@IPEBEPEBVPxVec3@2@@Z 000000018002f9b4     ConvexHullBuilder.obj
 0004:000009c0       $pdata$7$?computeNewellPlane@@YA_NAEAVPxPlane@physx@@IPEBEPEBVPxVec3@2@@Z 000000018002f9c0     ConvexHullBuilder.obj
 0004:000009cc       $pdata$10$?computeNewellPlane@@YA_NAEAVPxPlane@physx@@IPEBEPEBVPxVec3@2@@Z 000000018002f9cc     ConvexHullBuilder.obj
 0004:000009d8       $pdata$11$?computeNewellPlane@@YA_NAEAVPxPlane@physx@@IPEBEPEBVPxVec3@2@@Z 000000018002f9d8     ConvexHullBuilder.obj
 0004:000009e4       $pdata$12$?computeNewellPlane@@YA_NAEAVPxPlane@physx@@IPEBEPEBVPxVec3@2@@Z 000000018002f9e4     ConvexHullBuilder.obj
 0004:000009f0       $pdata$13$?computeNewellPlane@@YA_NAEAVPxPlane@physx@@IPEBEPEBVPxVec3@2@@Z 000000018002f9f0     ConvexHullBuilder.obj
 0004:000009fc       $pdata$??$PlaneEquation@U?$TriangleT@I@Gu@physx@@@@YA?AVPxPlane@physx@@AEBU?$TriangleT@I@Gu@1@PEBVPxVec3@1@@Z 000000018002f9fc     ConvexHullBuilder.obj
 0004:00000a08       $pdata$??0PxPlane@physx@@QEAA@AEBVPxVec3@1@00@Z 000000018002fa08     ConvexHullBuilder.obj
 0004:00000a14       $pdata$?ComputeNbPolygons@ConvexHullBuilder@physx@@QEBAIXZ 000000018002fa14     ConvexHullBuilder.obj
 0004:00000a20       $pdata$?allocate@?$ReflectionAllocator@UEdgeDescData@Gu@physx@@@shdfnd@physx@@QEAAPEAX_KPEBDH@Z 000000018002fa20     ConvexHullBuilder.obj
 0004:00000a2c       $pdata$0$?allocate@?$ReflectionAllocator@UEdgeDescData@Gu@physx@@@shdfnd@physx@@QEAAPEAX_KPEBDH@Z 000000018002fa2c     ConvexHullBuilder.obj
 0004:00000a38       $pdata$1$?allocate@?$ReflectionAllocator@UEdgeDescData@Gu@physx@@@shdfnd@physx@@QEAAPEAX_KPEBDH@Z 000000018002fa38     ConvexHullBuilder.obj
 0004:00000a44       $pdata$?allocate@?$ReflectionAllocator@UHullTriangleData@physx@@@shdfnd@physx@@QEAAPEAX_KPEBDH@Z 000000018002fa44     ConvexHullBuilder.obj
 0004:00000a50       $pdata$0$?allocate@?$ReflectionAllocator@UHullTriangleData@physx@@@shdfnd@physx@@QEAAPEAX_KPEBDH@Z 000000018002fa50     ConvexHullBuilder.obj
 0004:00000a5c       $pdata$1$?allocate@?$ReflectionAllocator@UHullTriangleData@physx@@@shdfnd@physx@@QEAAPEAX_KPEBDH@Z 000000018002fa5c     ConvexHullBuilder.obj
 0004:00000a68       $pdata$?area@?$TriangleT@I@Gu@physx@@QEBAMPEBVPxVec3@3@@Z 000000018002fa68     ConvexHullBuilder.obj
 0004:00000a74       $pdata$?getName@?$ReflectionAllocator@UEdgeDescData@Gu@physx@@@shdfnd@physx@@CAPEBDXZ 000000018002fa74     ConvexHullBuilder.obj
 0004:00000a80       $pdata$?getName@?$ReflectionAllocator@UHullTriangleData@physx@@@shdfnd@physx@@CAPEBDXZ 000000018002fa80     ConvexHullBuilder.obj
 0004:00000a8c       $pdata$?getNormalized@PxVec3@physx@@QEBA?AV12@XZ 000000018002fa8c     ConvexHullBuilder.obj
 0004:00000a98       $pdata$??0ConvexMeshBuilder@physx@@QEAA@XZ 000000018002fa98     ConvexMeshBuilder.obj
 0004:00000aa4       $pdata$??1ConvexMeshBuilder@physx@@UEAA@XZ 000000018002faa4     ConvexMeshBuilder.obj
 0004:00000ab0       $pdata$?loadFromDesc@ConvexMeshBuilder@physx@@QEAA_NAEBVPxConvexMeshDesc@2@W4Enum@PxPlatform@2@@Z 000000018002fab0     ConvexMeshBuilder.obj
 0004:00000abc       $pdata$?save@ConvexMeshBuilder@physx@@QEBA_NAEAVPxOutputStream@2@_N@Z 000000018002fabc     ConvexMeshBuilder.obj
 0004:00000ac8       $pdata$1$?save@ConvexMeshBuilder@physx@@QEBA_NAEAVPxOutputStream@2@_N@Z 000000018002fac8     ConvexMeshBuilder.obj
 0004:00000ad4       $pdata$2$?save@ConvexMeshBuilder@physx@@QEBA_NAEAVPxOutputStream@2@_N@Z 000000018002fad4     ConvexMeshBuilder.obj
 0004:00000ae0       $pdata$?loadConvexHull@ConvexMeshBuilder@physx@@QEAA_NAEBVPxConvexMeshDesc@2@@Z 000000018002fae0     ConvexMeshBuilder.obj
 0004:00000aec       $pdata$?computeHullPolygons@ConvexMeshBuilder@physx@@QEAA_NAEBIPEBVPxVec3@2@0PEBIAEAVPxAllocatorCallback@2@AEAIAEAPEAV32@4AEAPEAI4AEAPEAUPxHullPolygon@2@@Z 000000018002faec     ConvexMeshBuilder.obj
 0004:00000af8       $pdata$2$?computeHullPolygons@ConvexMeshBuilder@physx@@QEAA_NAEBIPEBVPxVec3@2@0PEBIAEAVPxAllocatorCallback@2@AEAIAEAPEAV32@4AEAPEAI4AEAPEAUPxHullPolygon@2@@Z 000000018002faf8     ConvexMeshBuilder.obj
 0004:00000b04       $pdata$3$?computeHullPolygons@ConvexMeshBuilder@physx@@QEAA_NAEBIPEBVPxVec3@2@0PEBIAEAVPxAllocatorCallback@2@AEAIAEAPEAV32@4AEAPEAI4AEAPEAUPxHullPolygon@2@@Z 000000018002fb04     ConvexMeshBuilder.obj
 0004:00000b10       $pdata$?computeGaussMaps@ConvexMeshBuilder@physx@@QEAA_NXZ 000000018002fb10     ConvexMeshBuilder.obj
 0004:00000b1c       $pdata$?computeMassInfo@ConvexMeshBuilder@physx@@QEAAXXZ 000000018002fb1c     ConvexMeshBuilder.obj
 0004:00000b28       $pdata$1$?computeMassInfo@ConvexMeshBuilder@physx@@QEAAXXZ 000000018002fb28     ConvexMeshBuilder.obj
 0004:00000b34       $pdata$2$?computeMassInfo@ConvexMeshBuilder@physx@@QEAAXXZ 000000018002fb34     ConvexMeshBuilder.obj
 0004:00000b40       $pdata$6$?computeMassInfo@ConvexMeshBuilder@physx@@QEAAXXZ 000000018002fb40     ConvexMeshBuilder.obj
 0004:00000b4c       $pdata$7$?computeMassInfo@ConvexMeshBuilder@physx@@QEAAXXZ 000000018002fb4c     ConvexMeshBuilder.obj
 0004:00000b58       $pdata$8$?computeMassInfo@ConvexMeshBuilder@physx@@QEAAXXZ 000000018002fb58     ConvexMeshBuilder.obj
 0004:00000b64       $pdata$9$?computeMassInfo@ConvexMeshBuilder@physx@@QEAAXXZ 000000018002fb64     ConvexMeshBuilder.obj
 0004:00000b70       $pdata$?computeInternalObjects@ConvexMeshBuilder@physx@@QEAAXXZ 000000018002fb70     ConvexMeshBuilder.obj
 0004:00000b7c       $pdata$?ComputeAABBNoTransform@@YAXAEAVPxVec3@physx@@0IPEBV12@@Z 000000018002fb7c     ConvexMeshBuilder.obj
 0004:00000b88       $pdata$?TestContainment@@YA_NAEBVPxVec3@physx@@QEBMIPEBUHullPolygonData@Gu@2@@Z 000000018002fb88     ConvexMeshBuilder.obj
 0004:00000b94       $pdata$??3UserAllocated@shdfnd@physx@@SAXPEAX@Z 000000018002fb94     ConvexMeshBuilder.obj
 0004:00000ba0       $pdata$??GPxMat33@physx@@QEBA?AV01@XZ 000000018002fba0     ConvexMeshBuilder.obj
 0004:00000bac       $pdata$??_GBigConvexData@physx@@QEAAPEAXI@Z 000000018002fbac     ConvexMeshBuilder.obj
 0004:00000bb8       $pdata$??_GConvexMeshBuilder@physx@@UEAAPEAXI@Z 000000018002fbb8     ConvexMeshBuilder.obj
 0004:00000bc4       $pdata$?PxIsFinite@physx@@YA_NM@Z 000000018002fbc4     ConvexMeshBuilder.obj
 0004:00000bd0       $pdata$?allocate@?$ReflectionAllocator@VBigConvexData@physx@@@shdfnd@physx@@QEAAPEAX_KPEBDH@Z 000000018002fbd0     ConvexMeshBuilder.obj
 0004:00000bdc       $pdata$0$?allocate@?$ReflectionAllocator@VBigConvexData@physx@@@shdfnd@physx@@QEAAPEAX_KPEBDH@Z 000000018002fbdc     ConvexMeshBuilder.obj
 0004:00000be8       $pdata$1$?allocate@?$ReflectionAllocator@VBigConvexData@physx@@@shdfnd@physx@@QEAAPEAX_KPEBDH@Z 000000018002fbe8     ConvexMeshBuilder.obj
 0004:00000bf4       $pdata$?getName@?$ReflectionAllocator@VBigConvexData@physx@@@shdfnd@physx@@CAPEBDXZ 000000018002fbf4     ConvexMeshBuilder.obj
 0004:00000c00       $pdata$?isFinite@PxVec3@physx@@QEBA_NXZ 000000018002fc00     ConvexMeshBuilder.obj
 0004:00000c0c       $pdata$?isFinite@intrinsics@physx@@YA_NM@Z 000000018002fc0c     ConvexMeshBuilder.obj
 0004:00000c18       $pdata$??0HullLibrary@physx@@QEAA@XZ 000000018002fc18     hulllib.obj
 0004:00000c24       $pdata$??1HullLibrary@physx@@QEAA@XZ 000000018002fc24     hulllib.obj
 0004:00000c30       $pdata$?CreateConvexHull@HullLibrary@physx@@QEAA?AW4HullError@2@AEBVHullDesc@2@AEAVHullResult@2@@Z 000000018002fc30     hulllib.obj
 0004:00000c3c       $pdata$3$?CreateConvexHull@HullLibrary@physx@@QEAA?AW4HullError@2@AEBVHullDesc@2@AEAVHullResult@2@@Z 000000018002fc3c     hulllib.obj
 0004:00000c48       $pdata$4$?CreateConvexHull@HullLibrary@physx@@QEAA?AW4HullError@2@AEBVHullDesc@2@AEAVHullResult@2@@Z 000000018002fc48     hulllib.obj
 0004:00000c54       $pdata$5$?CreateConvexHull@HullLibrary@physx@@QEAA?AW4HullError@2@AEBVHullDesc@2@AEAVHullResult@2@@Z 000000018002fc54     hulllib.obj
 0004:00000c60       $pdata$6$?CreateConvexHull@HullLibrary@physx@@QEAA?AW4HullError@2@AEBVHullDesc@2@AEAVHullResult@2@@Z 000000018002fc60     hulllib.obj
 0004:00000c6c       $pdata$?ReleaseResult@HullLibrary@physx@@QEAA?AW4HullError@2@AEAVHullResult@2@@Z 000000018002fc6c     hulllib.obj
 0004:00000c78       $pdata$?CreateTriangleMesh@HullLibrary@physx@@QEAA?AW4HullError@2@AEAVHullResult@2@PEAVConvexHullTriangleInterface@2@@Z 000000018002fc78     hulllib.obj
 0004:00000c84       $pdata$5$?CreateTriangleMesh@HullLibrary@physx@@QEAA?AW4HullError@2@AEAVHullResult@2@PEAVConvexHullTriangleInterface@2@@Z 000000018002fc84     hulllib.obj
 0004:00000c90       $pdata$6$?CreateTriangleMesh@HullLibrary@physx@@QEAA?AW4HullError@2@AEAVHullResult@2@PEAVConvexHullTriangleInterface@2@@Z 000000018002fc90     hulllib.obj
 0004:00000c9c       $pdata$?b2bfix@HullLibrary@physx@@AEAAXPEAVTri@2@0@Z 000000018002fc9c     hulllib.obj
 0004:00000ca8       $pdata$?removeb2b@HullLibrary@physx@@AEAAXPEAVTri@2@0@Z 000000018002fca8     hulllib.obj
 0004:00000cb4       $pdata$?extrude@HullLibrary@physx@@AEAAXPEAVTri@2@H@Z 000000018002fcb4     hulllib.obj
 0004:00000cc0       $pdata$?extrudable@HullLibrary@physx@@AEBAPEAVTri@2@M@Z 000000018002fcc0     hulllib.obj
 0004:00000ccc       $pdata$?calchullgen@HullLibrary@physx@@AEAA?AW4HullError@2@PEAVfloat3@2@HHM@Z 000000018002fccc     hulllib.obj
 0004:00000cd8       $pdata$6$?calchullgen@HullLibrary@physx@@AEAA?AW4HullError@2@PEAVfloat3@2@HHM@Z 000000018002fcd8     hulllib.obj
 0004:00000ce4       $pdata$11$?calchullgen@HullLibrary@physx@@AEAA?AW4HullError@2@PEAVfloat3@2@HHM@Z 000000018002fce4     hulllib.obj
 0004:00000cf0       $pdata$12$?calchullgen@HullLibrary@physx@@AEAA?AW4HullError@2@PEAVfloat3@2@HHM@Z 000000018002fcf0     hulllib.obj
 0004:00000cfc       $pdata$13$?calchullgen@HullLibrary@physx@@AEAA?AW4HullError@2@PEAVfloat3@2@HHM@Z 000000018002fcfc     hulllib.obj
 0004:00000d08       $pdata$14$?calchullgen@HullLibrary@physx@@AEAA?AW4HullError@2@PEAVfloat3@2@HHM@Z 000000018002fd08     hulllib.obj
 0004:00000d14       $pdata$15$?calchullgen@HullLibrary@physx@@AEAA?AW4HullError@2@PEAVfloat3@2@HHM@Z 000000018002fd14     hulllib.obj
 0004:00000d20       $pdata$16$?calchullgen@HullLibrary@physx@@AEAA?AW4HullError@2@PEAVfloat3@2@HHM@Z 000000018002fd20     hulllib.obj
 0004:00000d2c       $pdata$?calchull@HullLibrary@physx@@AEAA?AW4HullError@2@PEAVfloat3@2@HAEAPEAHAEAHAEAPEAV42@2HM@Z 000000018002fd2c     hulllib.obj
 0004:00000d38       $pdata$4$?calchull@HullLibrary@physx@@AEAA?AW4HullError@2@PEAVfloat3@2@HAEAPEAHAEAHAEAPEAV42@2HM@Z 000000018002fd38     hulllib.obj
 0004:00000d44       $pdata$5$?calchull@HullLibrary@physx@@AEAA?AW4HullError@2@PEAVfloat3@2@HAEAPEAHAEAHAEAPEAV42@2HM@Z 000000018002fd44     hulllib.obj
 0004:00000d50       $pdata$?expandhull@HullLibrary@physx@@AEAA?AW4HullError@2@PEAVfloat3@2@HAEAPEAV42@AEAHM@Z 000000018002fd50     hulllib.obj
 0004:00000d5c       $pdata$1$?expandhull@HullLibrary@physx@@AEAA?AW4HullError@2@PEAVfloat3@2@HAEAPEAV42@AEAHM@Z 000000018002fd5c     hulllib.obj
 0004:00000d68       $pdata$2$?expandhull@HullLibrary@physx@@AEAA?AW4HullError@2@PEAVfloat3@2@HAEAPEAV42@AEAHM@Z 000000018002fd68     hulllib.obj
 0004:00000d74       $pdata$7$?expandhull@HullLibrary@physx@@AEAA?AW4HullError@2@PEAVfloat3@2@HAEAPEAV42@AEAHM@Z 000000018002fd74     hulllib.obj
 0004:00000d80       $pdata$8$?expandhull@HullLibrary@physx@@AEAA?AW4HullError@2@PEAVfloat3@2@HAEAPEAV42@AEAHM@Z 000000018002fd80     hulllib.obj
 0004:00000d8c       $pdata$9$?expandhull@HullLibrary@physx@@AEAA?AW4HullError@2@PEAVfloat3@2@HAEAPEAV42@AEAHM@Z 000000018002fd8c     hulllib.obj
 0004:00000d98       $pdata$10$?expandhull@HullLibrary@physx@@AEAA?AW4HullError@2@PEAVfloat3@2@HAEAPEAV42@AEAHM@Z 000000018002fd98     hulllib.obj
 0004:00000da4       $pdata$11$?expandhull@HullLibrary@physx@@AEAA?AW4HullError@2@PEAVfloat3@2@HAEAPEAV42@AEAHM@Z 000000018002fda4     hulllib.obj
 0004:00000db0       $pdata$?calchullpbev@HullLibrary@physx@@AEAA?AW4HullError@2@PEAVfloat3@2@HHAEAV?$Array@VPlane@physx@@@hullLibArray@2@M@Z 000000018002fdb0     hulllib.obj
 0004:00000dbc       $pdata$14$?calchullpbev@HullLibrary@physx@@AEAA?AW4HullError@2@PEAVfloat3@2@HHAEAV?$Array@VPlane@physx@@@hullLibArray@2@M@Z 000000018002fdbc     hulllib.obj
 0004:00000dc8       $pdata$15$?calchullpbev@HullLibrary@physx@@AEAA?AW4HullError@2@PEAVfloat3@2@HHAEAV?$Array@VPlane@physx@@@hullLibArray@2@M@Z 000000018002fdc8     hulllib.obj
 0004:00000dd4       $pdata$?ComputeHull@HullLibrary@physx@@AEAA?AW4HullError@2@IPEBMAEAVPHullResult@2@IMM@Z 000000018002fdd4     hulllib.obj
 0004:00000de0       $pdata$0$?ComputeHull@HullLibrary@physx@@AEAA?AW4HullError@2@IPEBMAEAVPHullResult@2@IMM@Z 000000018002fde0     hulllib.obj
 0004:00000dec       $pdata$2$?ComputeHull@HullLibrary@physx@@AEAA?AW4HullError@2@IPEBMAEAVPHullResult@2@IMM@Z 000000018002fdec     hulllib.obj
 0004:00000df8       $pdata$3$?ComputeHull@HullLibrary@physx@@AEAA?AW4HullError@2@IPEBMAEAVPHullResult@2@IMM@Z 000000018002fdf8     hulllib.obj
 0004:00000e04       $pdata$4$?ComputeHull@HullLibrary@physx@@AEAA?AW4HullError@2@IPEBMAEAVPHullResult@2@IMM@Z 000000018002fe04     hulllib.obj
 0004:00000e10       $pdata$?overhullv@HullLibrary@physx@@AEAA?AW4HullError@2@PEAVfloat3@2@HHAEAPEAV42@AEAHAEAPEAH2MMHM@Z 000000018002fe10     hulllib.obj
 0004:00000e1c       $pdata$3$?overhullv@HullLibrary@physx@@AEAA?AW4HullError@2@PEAVfloat3@2@HHAEAPEAV42@AEAHAEAPEAH2MMHM@Z 000000018002fe1c     hulllib.obj
 0004:00000e28       $pdata$4$?overhullv@HullLibrary@physx@@AEAA?AW4HullError@2@PEAVfloat3@2@HHAEAPEAV42@AEAHAEAPEAH2MMHM@Z 000000018002fe28     hulllib.obj
 0004:00000e34       $pdata$?normalize@physx@@YA?AVfloat3@1@AEBV21@@Z 000000018002fe34     hulllib.obj
 0004:00000e40       $pdata$?Determinant@physx@@YAMAEBVfloat3x3@1@@Z 000000018002fe40     hulllib.obj
 0004:00000e4c       $pdata$?Inverse@physx@@YA?AVfloat3x3@1@AEBV21@@Z 000000018002fe4c     hulllib.obj
 0004:00000e58       $pdata$?Transpose@physx@@YA?AVfloat3x3@1@AEBV21@@Z 000000018002fe58     hulllib.obj
 0004:00000e64       $pdata$??Dphysx@@YA?AVfloat3@0@AEBV10@AEBVfloat3x3@0@@Z 000000018002fe64     hulllib.obj
 0004:00000e70       $pdata$?ThreePlaneIntersection@physx@@YA?AVfloat3@1@AEBVPlane@1@00@Z 000000018002fe70     hulllib.obj
 0004:00000e7c       $pdata$?TriNormal@physx@@YA?AVfloat3@1@AEBV21@00@Z 000000018002fe7c     hulllib.obj
 0004:00000e88       $pdata$??0ConvexH@physx@@QEAA@HHH@Z 000000018002fe88     hulllib.obj
 0004:00000e94       $pdata$?ConvexHDup@physx@@YAPEAVConvexH@1@PEAV21@@Z 000000018002fe94     hulllib.obj
 0004:00000ea0       $pdata$?AssertIntact@physx@@YAHAEAVConvexH@1@@Z 000000018002fea0     hulllib.obj
 0004:00000eac       $pdata$6$?AssertIntact@physx@@YAHAEAVConvexH@1@@Z 000000018002feac     hulllib.obj
 0004:00000eb8       $pdata$7$?AssertIntact@physx@@YAHAEAVConvexH@1@@Z 000000018002feb8     hulllib.obj
 0004:00000ec4       $pdata$8$?AssertIntact@physx@@YAHAEAVConvexH@1@@Z 000000018002fec4     hulllib.obj
 0004:00000ed0       $pdata$?test_cube@physx@@YAPEAVConvexH@1@XZ 000000018002fed0     hulllib.obj
 0004:00000edc       $pdata$?ConvexHMakeCube@physx@@YAPEAVConvexH@1@AEBVfloat3@1@0@Z 000000018002fedc     hulllib.obj
 0004:00000ee8       $pdata$?ConvexHCrop@physx@@YAPEAVConvexH@1@AEAV21@AEBVPlane@1@@Z 000000018002fee8     hulllib.obj
 0004:00000ef4       $pdata$7$?ConvexHCrop@physx@@YAPEAVConvexH@1@AEAV21@AEBVPlane@1@@Z 000000018002fef4     hulllib.obj
 0004:00000f00       $pdata$8$?ConvexHCrop@physx@@YAPEAVConvexH@1@AEAV21@AEBVPlane@1@@Z 000000018002ff00     hulllib.obj
 0004:00000f0c       $pdata$?candidateplane@physx@@YAHPEAVPlane@1@HPEAVConvexH@1@M@Z 000000018002ff0c     hulllib.obj
 0004:00000f18       $pdata$6$?candidateplane@physx@@YAHPEAVPlane@1@HPEAVConvexH@1@M@Z 000000018002ff18     hulllib.obj
 0004:00000f24       $pdata$7$?candidateplane@physx@@YAHPEAVPlane@1@HPEAVConvexH@1@M@Z 000000018002ff24     hulllib.obj
 0004:00000f30       $pdata$?orth@physx@@YA?AVfloat3@1@AEBV21@@Z 000000018002ff30     hulllib.obj
 0004:00000f3c       $pdata$?above@physx@@YAHPEAVfloat3@1@AEBVint3@1@AEBV21@M@Z 000000018002ff3c     hulllib.obj
 0004:00000f48       $pdata$?deleteTri@physx@@YAXPEAVTri@1@PEAV?$Array@PEAVTri@physx@@@hullLibArray@1@@Z 000000018002ff48     hulllib.obj
 0004:00000f54       $pdata$?neib@Tri@physx@@QEAAAEAHHH@Z 000000018002ff54     hulllib.obj
 0004:00000f60       $pdata$?hasVolume@physx@@YA_NPEAVfloat3@1@HHHH@Z 000000018002ff60     hulllib.obj
 0004:00000f6c       $pdata$2$?hasVolume@physx@@YA_NPEAVfloat3@1@HHHH@Z 000000018002ff6c     hulllib.obj
 0004:00000f78       $pdata$3$?hasVolume@physx@@YA_NPEAVfloat3@1@HHHH@Z 000000018002ff78     hulllib.obj
 0004:00000f84       $pdata$?FindSimplex@physx@@YA?AVint4@1@PEAVfloat3@1@HAEAV?$Array@H@hullLibArray@1@AEBV31@@Z 000000018002ff84     hulllib.obj
 0004:00000f90       $pdata$2$?FindSimplex@physx@@YA?AVint4@1@PEAVfloat3@1@HAEAV?$Array@H@hullLibArray@1@AEBV31@@Z 000000018002ff90     hulllib.obj
 0004:00000f9c       $pdata$3$?FindSimplex@physx@@YA?AVint4@1@PEAVfloat3@1@HAEAV?$Array@H@hullLibArray@1@AEBV31@@Z 000000018002ff9c     hulllib.obj
 0004:00000fa8       $pdata$4$?FindSimplex@physx@@YA?AVint4@1@PEAVfloat3@1@HAEAV?$Array@H@hullLibArray@1@AEBV31@@Z 000000018002ffa8     hulllib.obj
 0004:00000fb4       $pdata$5$?FindSimplex@physx@@YA?AVint4@1@PEAVfloat3@1@HAEAV?$Array@H@hullLibArray@1@AEBV31@@Z 000000018002ffb4     hulllib.obj
 0004:00000fc0       $pdata$?PlaneCheck@LocalTests@?1??expandhull@HullLibrary@physx@@AEAA?AW4HullError@4@PEAVfloat3@4@HAEAPEAV64@AEAHM@Z@SA_NPEBV64@HAEAV?$Array@UExpandPlane@physx@@@hullLibArray@4@@Z 000000018002ffc0     hulllib.obj
 0004:00000fcc       $pdata$?area2@physx@@YAMAEBVfloat3@1@00@Z 000000018002ffcc     hulllib.obj
 0004:00000fd8       $pdata$?overhull@physx@@YA?AW4HullError@1@PEAVPlane@1@HPEAVfloat3@1@HHAEAPEAV41@AEAHAEAPEAH3M@Z 000000018002ffd8     hulllib.obj
 0004:00000fe4       $pdata$3$?overhull@physx@@YA?AW4HullError@1@PEAVPlane@1@HPEAVfloat3@1@HHAEAPEAV41@AEAHAEAPEAH3M@Z 000000018002ffe4     hulllib.obj
 0004:00000ff0       $pdata$4$?overhull@physx@@YA?AW4HullError@1@PEAVPlane@1@HPEAVfloat3@1@HHAEAPEAV41@AEAHAEAPEAH3M@Z 000000018002fff0     hulllib.obj
 0004:00000ffc       $pdata$8$?overhull@physx@@YA?AW4HullError@1@PEAVPlane@1@HPEAVfloat3@1@HHAEAPEAV41@AEAHAEAPEAH3M@Z 000000018002fffc     hulllib.obj
 0004:00001008       $pdata$9$?overhull@physx@@YA?AW4HullError@1@PEAVPlane@1@HPEAVfloat3@1@HHAEAPEAV41@AEAHAEAPEAH3M@Z 0000000180030008     hulllib.obj
 0004:00001014       $pdata$10$?overhull@physx@@YA?AW4HullError@1@PEAVPlane@1@HPEAVfloat3@1@HHAEAPEAV41@AEAHAEAPEAH3M@Z 0000000180030014     hulllib.obj
 0004:00001020       $pdata$11$?overhull@physx@@YA?AW4HullError@1@PEAVPlane@1@HPEAVfloat3@1@HHAEAPEAV41@AEAHAEAPEAH3M@Z 0000000180030020     hulllib.obj
 0004:0000102c       $pdata$12$?overhull@physx@@YA?AW4HullError@1@PEAVPlane@1@HPEAVfloat3@1@HHAEAPEAV41@AEAHAEAPEAH3M@Z 000000018003002c     hulllib.obj
 0004:00001038       $pdata$?ReleaseHull@physx@@YAXAEAVPHullResult@1@@Z 0000000180030038     hulllib.obj
 0004:00001044       $pdata$?BringOutYourDead@physx@@YAXPEBMIPEAMAEAIPEAII@Z 0000000180030044     hulllib.obj
 0004:00001050       $pdata$?CleanupVertices@physx@@YA_NIPEBMIAEAIPEAMM2@Z 0000000180030050     hulllib.obj
 0004:0000105c       $pdata$5$?CleanupVertices@physx@@YA_NIPEBMIAEAIPEAMM2@Z 000000018003005c     hulllib.obj
 0004:00001068       $pdata$9$?CleanupVertices@physx@@YA_NIPEBMIAEAIPEAMM2@Z 0000000180030068     hulllib.obj
 0004:00001074       $pdata$10$?CleanupVertices@physx@@YA_NIPEBMIAEAIPEAMM2@Z 0000000180030074     hulllib.obj
 0004:00001080       $pdata$11$?CleanupVertices@physx@@YA_NIPEBMIAEAIPEAMM2@Z 0000000180030080     hulllib.obj
 0004:0000108c       $pdata$12$?CleanupVertices@physx@@YA_NIPEBMIAEAIPEAMM2@Z 000000018003008c     hulllib.obj
 0004:00001098       $pdata$13$?CleanupVertices@physx@@YA_NIPEBMIAEAIPEAMM2@Z 0000000180030098     hulllib.obj
 0004:000010a4       $pdata$15$?CleanupVertices@physx@@YA_NIPEBMIAEAIPEAMM2@Z 00000001800300a4     hulllib.obj
 0004:000010b0       $pdata$?ComputeNormal@physx@@YAMPEAMPEBM11@Z 00000001800300b0     hulllib.obj
 0004:000010bc       $pdata$?AddConvexTriangle@physx@@YAXPEAVConvexHullTriangleInterface@1@PEBM11@Z 00000001800300bc     hulllib.obj
 0004:000010c8       $pdata$??$maxdir@Vfloat3@physx@@@physx@@YAHPEBVfloat3@0@HAEBV10@@Z 00000001800300c8     hulllib.obj
 0004:000010d4       $pdata$0$??$maxdir@Vfloat3@physx@@@physx@@YAHPEBVfloat3@0@HAEBV10@@Z 00000001800300d4     hulllib.obj
 0004:000010e0       $pdata$2$??$maxdir@Vfloat3@physx@@@physx@@YAHPEBVfloat3@0@HAEBV10@@Z 00000001800300e0     hulllib.obj
 0004:000010ec       $pdata$3$??$maxdir@Vfloat3@physx@@@physx@@YAHPEBVfloat3@0@HAEBV10@@Z 00000001800300ec     hulllib.obj
 0004:000010f8       $pdata$4$??$maxdir@Vfloat3@physx@@@physx@@YAHPEBVfloat3@0@HAEBV10@@Z 00000001800300f8     hulllib.obj
 0004:00001104       $pdata$??$maxdirfiltered@Vfloat3@physx@@@physx@@YAHPEBVfloat3@0@HAEBV10@PEA_N@Z 0000000180030104     hulllib.obj
 0004:00001110       $pdata$2$??$maxdirfiltered@Vfloat3@physx@@@physx@@YAHPEBVfloat3@0@HAEBV10@PEA_N@Z 0000000180030110     hulllib.obj
 0004:0000111c       $pdata$3$??$maxdirfiltered@Vfloat3@physx@@@physx@@YAHPEBVfloat3@0@HAEBV10@PEA_N@Z 000000018003011c     hulllib.obj
 0004:00001128       $pdata$??$maxdirsterid@Vfloat3@physx@@@physx@@YAHPEBVfloat3@0@HAEBV10@AEAV?$Array@H@hullLibArray@0@@Z 0000000180030128     hulllib.obj
 0004:00001134       $pdata$??0?$Array@H@hullLibArray@physx@@QEAA@H@Z 0000000180030134     hulllib.obj
 0004:00001140       $pdata$??0?$Array@PEAVTri@physx@@@hullLibArray@physx@@QEAA@H@Z 0000000180030140     hulllib.obj
 0004:0000114c       $pdata$??0?$Array@UExpandPlane@physx@@@hullLibArray@physx@@QEAA@H@Z 000000018003014c     hulllib.obj
 0004:00001158       $pdata$??0?$Array@VHalfEdge@ConvexH@physx@@@hullLibArray@physx@@QEAA@H@Z 0000000180030158     hulllib.obj
 0004:00001164       $pdata$??0?$Array@VPlane@physx@@@hullLibArray@physx@@QEAA@H@Z 0000000180030164     hulllib.obj
 0004:00001170       $pdata$??0?$Array@Vfloat3@physx@@@hullLibArray@physx@@QEAA@H@Z 0000000180030170     hulllib.obj
 0004:0000117c       $pdata$??0?$Array@Vint3@physx@@@hullLibArray@physx@@QEAA@H@Z 000000018003017c     hulllib.obj
 0004:00001188       $pdata$??0Tri@physx@@QEAA@HHHPEAV?$Array@PEAVTri@physx@@@hullLibArray@1@@Z 0000000180030188     hulllib.obj
 0004:00001194       $pdata$??1?$Array@H@hullLibArray@physx@@QEAA@XZ 0000000180030194     hulllib.obj
 0004:000011a0       $pdata$??1?$Array@PEAVTri@physx@@@hullLibArray@physx@@QEAA@XZ 00000001800301a0     hulllib.obj
 0004:000011ac       $pdata$??1?$Array@UExpandPlane@physx@@@hullLibArray@physx@@QEAA@XZ 00000001800301ac     hulllib.obj
 0004:000011b8       $pdata$??1?$Array@VHalfEdge@ConvexH@physx@@@hullLibArray@physx@@QEAA@XZ 00000001800301b8     hulllib.obj
 0004:000011c4       $pdata$??1?$Array@VPlane@physx@@@hullLibArray@physx@@QEAA@XZ 00000001800301c4     hulllib.obj
 0004:000011d0       $pdata$??1?$Array@Vfloat3@physx@@@hullLibArray@physx@@QEAA@XZ 00000001800301d0     hulllib.obj
 0004:000011dc       $pdata$??1?$Array@Vint3@physx@@@hullLibArray@physx@@QEAA@XZ 00000001800301dc     hulllib.obj
 0004:000011e8       $pdata$??1ConvexH@physx@@QEAA@XZ 00000001800301e8     hulllib.obj
 0004:000011f4       $pdata$??_G?$Array@PEAVTri@physx@@@hullLibArray@physx@@QEAAPEAXI@Z 00000001800301f4     hulllib.obj
 0004:00001200       $pdata$??_GConvexH@physx@@QEAAPEAXI@Z 0000000180030200     hulllib.obj
 0004:0000120c       $pdata$??_GTri@physx@@IEAAPEAXI@Z 000000018003020c     hulllib.obj
 0004:00001218       $pdata$?Add@?$Array@H@hullLibArray@physx@@QEAAAEAHH@Z 0000000180030218     hulllib.obj
 0004:00001224       $pdata$?Add@?$Array@PEAVTri@physx@@@hullLibArray@physx@@QEAAAEAPEAVTri@3@PEAV43@@Z 0000000180030224     hulllib.obj
 0004:00001230       $pdata$?Add@?$Array@UExpandPlane@physx@@@hullLibArray@physx@@QEAAAEAUExpandPlane@3@U43@@Z 0000000180030230     hulllib.obj
 0004:0000123c       $pdata$?Add@?$Array@VPlane@physx@@@hullLibArray@physx@@QEAAAEAVPlane@3@V43@@Z 000000018003023c     hulllib.obj
 0004:00001248       $pdata$?Add@?$Array@Vfloat3@physx@@@hullLibArray@physx@@QEAAAEAVfloat3@3@V43@@Z 0000000180030248     hulllib.obj
 0004:00001254       $pdata$?Add@?$Array@Vint3@physx@@@hullLibArray@physx@@QEAAAEAVint3@3@V43@@Z 0000000180030254     hulllib.obj
 0004:00001260       $pdata$?PxMemSet@physx@@YAPEAXPEIAXHI@Z 0000000180030260     hulllib.obj
 0004:0000126c       $pdata$?SetSize@?$Array@PEAVTri@physx@@@hullLibArray@physx@@QEAAXH@Z 000000018003026c     hulllib.obj
 0004:00001278       $pdata$?SetSize@?$Array@Vint3@physx@@@hullLibArray@physx@@QEAAXH@Z 0000000180030278     hulllib.obj
 0004:00001284       $pdata$?allocate@?$Array@H@hullLibArray@physx@@QEAAXH@Z 0000000180030284     hulllib.obj
 0004:00001290       $pdata$?allocate@?$Array@PEAVTri@physx@@@hullLibArray@physx@@QEAAXH@Z 0000000180030290     hulllib.obj
 0004:0000129c       $pdata$?allocate@?$Array@UExpandPlane@physx@@@hullLibArray@physx@@QEAAXH@Z 000000018003029c     hulllib.obj
 0004:000012a8       $pdata$?allocate@?$Array@VHalfEdge@ConvexH@physx@@@hullLibArray@physx@@QEAAXH@Z 00000001800302a8     hulllib.obj
 0004:000012b4       $pdata$?allocate@?$Array@VPlane@physx@@@hullLibArray@physx@@QEAAXH@Z 00000001800302b4     hulllib.obj
 0004:000012c0       $pdata$?allocate@?$Array@Vfloat3@physx@@@hullLibArray@physx@@QEAAXH@Z 00000001800302c0     hulllib.obj
 0004:000012cc       $pdata$?allocate@?$Array@Vint3@physx@@@hullLibArray@physx@@QEAAXH@Z 00000001800302cc     hulllib.obj
 0004:000012d8       $pdata$?allocate@?$ReflectionAllocator@M@shdfnd@physx@@QEAAPEAX_KPEBDH@Z 00000001800302d8     hulllib.obj
 0004:000012e4       $pdata$0$?allocate@?$ReflectionAllocator@M@shdfnd@physx@@QEAAPEAX_KPEBDH@Z 00000001800302e4     hulllib.obj
 0004:000012f0       $pdata$1$?allocate@?$ReflectionAllocator@M@shdfnd@physx@@QEAAPEAX_KPEBDH@Z 00000001800302f0     hulllib.obj
 0004:000012fc       $pdata$?allocate@?$ReflectionAllocator@VConvexH@physx@@@shdfnd@physx@@QEAAPEAX_KPEBDH@Z 00000001800302fc     hulllib.obj
 0004:00001308       $pdata$0$?allocate@?$ReflectionAllocator@VConvexH@physx@@@shdfnd@physx@@QEAAPEAX_KPEBDH@Z 0000000180030308     hulllib.obj
 0004:00001314       $pdata$1$?allocate@?$ReflectionAllocator@VConvexH@physx@@@shdfnd@physx@@QEAAPEAX_KPEBDH@Z 0000000180030314     hulllib.obj
 0004:00001320       $pdata$?allocate@?$ReflectionAllocator@VTri@physx@@@shdfnd@physx@@QEAAPEAX_KPEBDH@Z 0000000180030320     hulllib.obj
 0004:0000132c       $pdata$0$?allocate@?$ReflectionAllocator@VTri@physx@@@shdfnd@physx@@QEAAPEAX_KPEBDH@Z 000000018003032c     hulllib.obj
 0004:00001338       $pdata$1$?allocate@?$ReflectionAllocator@VTri@physx@@@shdfnd@physx@@QEAAPEAX_KPEBDH@Z 0000000180030338     hulllib.obj
 0004:00001344       $pdata$?getName@?$ReflectionAllocator@M@shdfnd@physx@@CAPEBDXZ 0000000180030344     hulllib.obj
 0004:00001350       $pdata$?getName@?$ReflectionAllocator@VConvexH@physx@@@shdfnd@physx@@CAPEBDXZ 0000000180030350     hulllib.obj
 0004:0000135c       $pdata$?getName@?$ReflectionAllocator@VTri@physx@@@shdfnd@physx@@CAPEBDXZ 000000018003035c     hulllib.obj
 0004:00001368       $pdata$?memSet@intrinsics@physx@@YAPEAXPEIAXHI@Z 0000000180030368     hulllib.obj
 0004:00001374       $pdata$?computeVolumeIntegrals@physx@@YA_NAEBVPxSimpleTriangleMesh@1@MAEAUPxIntegrals@1@@Z 0000000180030374     VolumeIntegration.obj
 0004:00001380       $pdata$?computeVolumeIntegralsEberly@physx@@YA_NAEBVPxSimpleTriangleMesh@1@MAEAUPxIntegrals@1@AEBVPxVec3@1@@Z 0000000180030380     VolumeIntegration.obj
 0004:0000138c       $pdata$?computeVolumeIntegrals@VolumeIntegrator@?A0xd2749a4a@physx@@QEAA_NAEAUPxIntegrals@3@@Z 000000018003038c     VolumeIntegration.obj
 0004:00001398       $pdata$?computeInertiaTensor@VolumeIntegrator@?A0xd2749a4a@physx@@AEAAXPEAN@Z 0000000180030398     VolumeIntegration.obj
 0004:000013a4       $pdata$?computeCOMInertiaTensor@VolumeIntegrator@?A0xd2749a4a@physx@@AEAAXPEAN@Z 00000001800303a4     VolumeIntegration.obj
 0004:000013b0       $pdata$?computeFaceNormal@VolumeIntegrator@?A0xd2749a4a@physx@@AEAAXAEAUFace@123@PEAI@Z 00000001800303b0     VolumeIntegration.obj
 0004:000013bc       $pdata$?computeProjectionIntegrals@VolumeIntegrator@?A0xd2749a4a@physx@@AEAAXAEBUFace@123@@Z 00000001800303bc     VolumeIntegration.obj
 0004:000013c8       $pdata$?computeFaceIntegrals@VolumeIntegrator@?A0xd2749a4a@physx@@AEAAXAEBUFace@123@@Z 00000001800303c8     VolumeIntegration.obj
 0004:000013d4       $pdata$?computeVolumeIntegrals@VolumeIntegratorEberly@?A0xd2749a4a@physx@@QEAA_NAEAUPxIntegrals@3@AEBVPxVec3@3@@Z 00000001800303d4     VolumeIntegration.obj
 0004:000013e0       $pdata$7$?computeVolumeIntegrals@VolumeIntegratorEberly@?A0xd2749a4a@physx@@QEAA_NAEAUPxIntegrals@3@AEBVPxVec3@3@@Z 00000001800303e0     VolumeIntegration.obj
 0004:000013ec       $pdata$8$?computeVolumeIntegrals@VolumeIntegratorEberly@?A0xd2749a4a@physx@@QEAA_NAEAUPxIntegrals@3@AEBVPxVec3@3@@Z 00000001800303ec     VolumeIntegration.obj
 0004:000013f8       $pdata$??1Adjacencies@physx@@QEAA@XZ 00000001800303f8     Adjacencies.obj
 0004:00001404       $pdata$?Load@Adjacencies@physx@@QEAA_NAEAVPxInputStream@2@@Z 0000000180030404     Adjacencies.obj
 0004:00001410       $pdata$2$?Load@Adjacencies@physx@@QEAA_NAEAVPxInputStream@2@@Z 0000000180030410     Adjacencies.obj
 0004:0000141c       $pdata$3$?Load@Adjacencies@physx@@QEAA_NAEAVPxInputStream@2@@Z 000000018003041c     Adjacencies.obj
 0004:00001428       $pdata$?Walk@Adjacencies@physx@@QEAA_NP6AXAEBUCommonWalkParams@2@IIII@ZPEAX@Z 0000000180030428     Adjacencies.obj
 0004:00001434       $pdata$2$?Walk@Adjacencies@physx@@QEAA_NP6AXAEBUCommonWalkParams@2@IIII@ZPEAX@Z 0000000180030434     Adjacencies.obj
 0004:00001440       $pdata$3$?Walk@Adjacencies@physx@@QEAA_NP6AXAEBUCommonWalkParams@2@IIII@ZPEAX@Z 0000000180030440     Adjacencies.obj
 0004:0000144c       $pdata$?Walk2@Adjacencies@physx@@QEAA_NP6AXAEBUCommonWalkParams@2@IIII@ZPEAXPEBVPxVec3@2@PEBU?$TriangleT@I@Gu@2@@Z 000000018003044c     Adjacencies.obj
 0004:00001458       $pdata$4$?Walk2@Adjacencies@physx@@QEAA_NP6AXAEBUCommonWalkParams@2@IIII@ZPEAXPEBVPxVec3@2@PEBU?$TriangleT@I@Gu@2@@Z 0000000180030458     Adjacencies.obj
 0004:00001464       $pdata$5$?Walk2@Adjacencies@physx@@QEAA_NP6AXAEBUCommonWalkParams@2@IIII@ZPEAXPEBVPxVec3@2@PEBU?$TriangleT@I@Gu@2@@Z 0000000180030464     Adjacencies.obj
 0004:00001470       $pdata$?GetBoundaryVertices@Adjacencies@physx@@QEBA_NIPEA_NPEBU?$TriangleT@I@Gu@2@@Z 0000000180030470     Adjacencies.obj
 0004:0000147c       $pdata$?MakeLastRef@Adjacencies@physx@@QEAA_NAEAVAdjTriangle@2@IPEAU?$TriangleT@I@Gu@2@@Z 000000018003047c     Adjacencies.obj
 0004:00001488       $pdata$1$?MakeLastRef@Adjacencies@physx@@QEAA_NAEAVAdjTriangle@2@IPEAU?$TriangleT@I@Gu@2@@Z 0000000180030488     Adjacencies.obj
 0004:00001494       $pdata$3$?MakeLastRef@Adjacencies@physx@@QEAA_NAEAVAdjTriangle@2@IPEAU?$TriangleT@I@Gu@2@@Z 0000000180030494     Adjacencies.obj
 0004:000014a0       $pdata$4$?MakeLastRef@Adjacencies@physx@@QEAA_NAEAVAdjTriangle@2@IPEAU?$TriangleT@I@Gu@2@@Z 00000001800304a0     Adjacencies.obj
 0004:000014ac       $pdata$5$?MakeLastRef@Adjacencies@physx@@QEAA_NAEAVAdjTriangle@2@IPEAU?$TriangleT@I@Gu@2@@Z 00000001800304ac     Adjacencies.obj
 0004:000014b8       $pdata$7$?MakeLastRef@Adjacencies@physx@@QEAA_NAEAVAdjTriangle@2@IPEAU?$TriangleT@I@Gu@2@@Z 00000001800304b8     Adjacencies.obj
 0004:000014c4       $pdata$??1AdjacenciesBuilder@physx@@QEAA@XZ 00000001800304c4     Adjacencies.obj
 0004:000014d0       $pdata$?Init@AdjacenciesBuilder@physx@@QEAA_NAEBUADJACENCIESCREATE@2@@Z 00000001800304d0     Adjacencies.obj
 0004:000014dc       $pdata$2$?Init@AdjacenciesBuilder@physx@@QEAA_NAEBUADJACENCIESCREATE@2@@Z 00000001800304dc     Adjacencies.obj
 0004:000014e8       $pdata$3$?Init@AdjacenciesBuilder@physx@@QEAA_NAEBUADJACENCIESCREATE@2@@Z 00000001800304e8     Adjacencies.obj
 0004:000014f4       $pdata$5$?Init@AdjacenciesBuilder@physx@@QEAA_NAEBUADJACENCIESCREATE@2@@Z 00000001800304f4     Adjacencies.obj
 0004:00001500       $pdata$6$?Init@AdjacenciesBuilder@physx@@QEAA_NAEBUADJACENCIESCREATE@2@@Z 0000000180030500     Adjacencies.obj
 0004:0000150c       $pdata$7$?Init@AdjacenciesBuilder@physx@@QEAA_NAEBUADJACENCIESCREATE@2@@Z 000000018003050c     Adjacencies.obj
 0004:00001518       $pdata$8$?Init@AdjacenciesBuilder@physx@@QEAA_NAEBUADJACENCIESCREATE@2@@Z 0000000180030518     Adjacencies.obj
 0004:00001524       $pdata$?_WalkFace@Local@?1??Walk@Adjacencies@physx@@QEAA_NP6AXAEBUCommonWalkParams@4@IIII@ZPEAX@Z@SAXAEAUPrivateWalkParams@?1??234@QEAA_N12@Z@IIII@Z 0000000180030524     Adjacencies.obj
 0004:00001530       $pdata$1$?_WalkFace@Local@?1??Walk@Adjacencies@physx@@QEAA_NP6AXAEBUCommonWalkParams@4@IIII@ZPEAX@Z@SAXAEAUPrivateWalkParams@?1??234@QEAA_N12@Z@IIII@Z 0000000180030530     Adjacencies.obj
 0004:0000153c       $pdata$2$?_WalkFace@Local@?1??Walk@Adjacencies@physx@@QEAA_NP6AXAEBUCommonWalkParams@4@IIII@ZPEAX@Z@SAXAEAUPrivateWalkParams@?1??234@QEAA_N12@Z@IIII@Z 000000018003053c     Adjacencies.obj
 0004:00001548       $pdata$?_WalkFace@Local@?1??Walk2@Adjacencies@physx@@QEAA_NP6AXAEBUCommonWalkParams@4@IIII@ZPEAXPEBVPxVec3@4@PEBU?$TriangleT@I@Gu@4@@Z@SAXAEAUPrivateWalkParams@?1??234@QEAA_N1234@Z@IIII@Z 0000000180030548     Adjacencies.obj
 0004:00001554       $pdata$2$?_WalkFace@Local@?1??Walk2@Adjacencies@physx@@QEAA_NP6AXAEBUCommonWalkParams@4@IIII@ZPEAXPEBVPxVec3@4@PEBU?$TriangleT@I@Gu@4@@Z@SAXAEAUPrivateWalkParams@?1??234@QEAA_N1234@Z@IIII@Z 0000000180030554     Adjacencies.obj
 0004:00001560       $pdata$3$?_WalkFace@Local@?1??Walk2@Adjacencies@physx@@QEAA_NP6AXAEBUCommonWalkParams@4@IIII@ZPEAXPEBVPxVec3@4@PEBU?$TriangleT@I@Gu@4@@Z@SAXAEAUPrivateWalkParams@?1??234@QEAA_N1234@Z@IIII@Z 0000000180030560     Adjacencies.obj
 0004:0000156c       $pdata$4$?_WalkFace@Local@?1??Walk2@Adjacencies@physx@@QEAA_NP6AXAEBUCommonWalkParams@4@IIII@ZPEAXPEBVPxVec3@4@PEBU?$TriangleT@I@Gu@4@@Z@SAXAEAUPrivateWalkParams@?1??234@QEAA_N1234@Z@IIII@Z 000000018003056c     Adjacencies.obj
 0004:00001578       $pdata$5$?_WalkFace@Local@?1??Walk2@Adjacencies@physx@@QEAA_NP6AXAEBUCommonWalkParams@4@IIII@ZPEAXPEBVPxVec3@4@PEBU?$TriangleT@I@Gu@4@@Z@SAXAEAUPrivateWalkParams@?1??234@QEAA_N1234@Z@IIII@Z 0000000180030578     Adjacencies.obj
 0004:00001584       $pdata$6$?_WalkFace@Local@?1??Walk2@Adjacencies@physx@@QEAA_NP6AXAEBUCommonWalkParams@4@IIII@ZPEAXPEBVPxVec3@4@PEBU?$TriangleT@I@Gu@4@@Z@SAXAEAUPrivateWalkParams@?1??234@QEAA_N1234@Z@IIII@Z 0000000180030584     Adjacencies.obj
 0004:00001590       $pdata$?AddTriangle@@YAXIIIIPEAVAdjTriangle@physx@@AEAIPEAVAdjEdge@@@Z 0000000180030590     Adjacencies.obj
 0004:0000159c       $pdata$?UpdateLink@@YA_NIIIIPEAVAdjTriangle@physx@@AEBUADJACENCIESCREATE@2@@Z 000000018003059c     Adjacencies.obj
 0004:000015a8       $pdata$3$?UpdateLink@@YA_NIIIIPEAVAdjTriangle@physx@@AEBUADJACENCIESCREATE@2@@Z 00000001800305a8     Adjacencies.obj
 0004:000015b4       $pdata$5$?UpdateLink@@YA_NIIIIPEAVAdjTriangle@physx@@AEBUADJACENCIESCREATE@2@@Z 00000001800305b4     Adjacencies.obj
 0004:000015c0       $pdata$6$?UpdateLink@@YA_NIIIIPEAVAdjTriangle@physx@@AEBUADJACENCIESCREATE@2@@Z 00000001800305c0     Adjacencies.obj
 0004:000015cc       $pdata$7$?UpdateLink@@YA_NIIIIPEAVAdjTriangle@physx@@AEBUADJACENCIESCREATE@2@@Z 00000001800305cc     Adjacencies.obj
 0004:000015d8       $pdata$8$?UpdateLink@@YA_NIIIIPEAVAdjTriangle@physx@@AEBUADJACENCIESCREATE@2@@Z 00000001800305d8     Adjacencies.obj
 0004:000015e4       $pdata$?CreateDatabase@@YA_NPEAVAdjTriangle@physx@@IPEBVAdjEdge@@AEBUADJACENCIESCREATE@2@@Z 00000001800305e4     Adjacencies.obj
 0004:000015f0       $pdata$??_EAdjEdge@@QEAAPEAXI@Z 00000001800305f0     Adjacencies.obj
 0004:000015fc       $pdata$??_EAdjTriangle@physx@@QEAAPEAXI@Z 00000001800305fc     Adjacencies.obj
 0004:00001608       $pdata$??_I@YAXPEAX_KHP6AX0@Z@Z 0000000180030608     Adjacencies.obj
 0004:00001614       $pdata$??_VUserAllocated@shdfnd@physx@@SAXPEAX@Z 0000000180030614     Adjacencies.obj
 0004:00001620       $pdata$?allocate@?$ReflectionAllocator@VAdjEdge@@@shdfnd@physx@@QEAAPEAX_KPEBDH@Z 0000000180030620     Adjacencies.obj
 0004:0000162c       $pdata$0$?allocate@?$ReflectionAllocator@VAdjEdge@@@shdfnd@physx@@QEAAPEAX_KPEBDH@Z 000000018003062c     Adjacencies.obj
 0004:00001638       $pdata$1$?allocate@?$ReflectionAllocator@VAdjEdge@@@shdfnd@physx@@QEAAPEAX_KPEBDH@Z 0000000180030638     Adjacencies.obj
 0004:00001644       $pdata$?allocate@?$ReflectionAllocator@VAdjTriangle@physx@@@shdfnd@physx@@QEAAPEAX_KPEBDH@Z 0000000180030644     Adjacencies.obj
 0004:00001650       $pdata$0$?allocate@?$ReflectionAllocator@VAdjTriangle@physx@@@shdfnd@physx@@QEAAPEAX_KPEBDH@Z 0000000180030650     Adjacencies.obj
 0004:0000165c       $pdata$1$?allocate@?$ReflectionAllocator@VAdjTriangle@physx@@@shdfnd@physx@@QEAAPEAX_KPEBDH@Z 000000018003065c     Adjacencies.obj
 0004:00001668       $pdata$?getName@?$ReflectionAllocator@VAdjEdge@@@shdfnd@physx@@CAPEBDXZ 0000000180030668     Adjacencies.obj
 0004:00001674       $pdata$?getName@?$ReflectionAllocator@VAdjTriangle@physx@@@shdfnd@physx@@CAPEBDXZ 0000000180030674     Adjacencies.obj
 0004:00001680       $pdata$PxCreateCooking     0000000180030680     Cooking.obj
 0004:0000168c       $pdata$?release@Cooking@physx@@UEAAXXZ 000000018003068c     Cooking.obj
 0004:00001698       $pdata$?cookTriangleMesh@Cooking@physx@@UEAA_NAEBVPxTriangleMeshDesc@2@AEAVPxOutputStream@2@@Z 0000000180030698     Cooking.obj
 0004:000016a4       $pdata$?createTriangleMesh@Cooking@physx@@UEAAPEAVPxTriangleMesh@2@AEBVPxTriangleMeshDesc@2@AEAVPxPhysicsInsertionCallback@2@@Z 00000001800306a4     Cooking.obj
 0004:000016b0       $pdata$?validateTriangleMesh@Cooking@physx@@UEAA_NAEBVPxTriangleMeshDesc@2@@Z 00000001800306b0     Cooking.obj
 0004:000016bc       $pdata$?cookConvexMesh@Cooking@physx@@UEAA_NAEBVPxConvexMeshDesc@2@AEAVPxOutputStream@2@PEAW4Enum@PxConvexMeshCookingResult@2@@Z 00000001800306bc     Cooking.obj
 0004:000016c8       $pdata$?computeHullPolygons@Cooking@physx@@UEAA_NAEBVPxSimpleTriangleMesh@2@AEAVPxAllocatorCallback@2@AEAIAEAPEAVPxVec3@2@2AEAPEAI2AEAPEAUPxHullPolygon@2@@Z 00000001800306c8     Cooking.obj
 0004:000016d4       $pdata$?cookHeightField@Cooking@physx@@UEAA_NAEBVPxHeightFieldDesc@2@AEAVPxOutputStream@2@@Z 00000001800306d4     Cooking.obj
 0004:000016e0       $pdata$?createHeightField@Cooking@physx@@UEAAPEAVPxHeightField@2@AEBVPxHeightFieldDesc@2@AEAVPxPhysicsInsertionCallback@2@@Z 00000001800306e0     Cooking.obj
 0004:000016ec       $pdata$?loadTriangleMeshDesc@Cooking@physx@@AEAA_NAEBVPxTriangleMeshDesc@2@AEAVTriangleMeshBuilder@2@@Z 00000001800306ec     Cooking.obj
 0004:000016f8       $pdata$??0TriangleMeshBuilder@physx@@QEAA@XZ 00000001800306f8     Cooking.obj
 0004:00001704       $pdata$??_GCooking@physx@@UEAAPEAXI@Z 0000000180030704     Cooking.obj
 0004:00001710       $pdata$??_GPxCooking@physx@@MEAAPEAXI@Z 0000000180030710     Cooking.obj
 0004:0000171c       $pdata$??_GTriangleMeshBuilder@physx@@UEAAPEAXI@Z 000000018003071c     Cooking.obj
 0004:00001728       $pdata$?allocate@?$ReflectionAllocator@VCooking@physx@@@shdfnd@physx@@QEAAPEAX_KPEBDH@Z 0000000180030728     Cooking.obj
 0004:00001734       $pdata$0$?allocate@?$ReflectionAllocator@VCooking@physx@@@shdfnd@physx@@QEAAPEAX_KPEBDH@Z 0000000180030734     Cooking.obj
 0004:00001740       $pdata$1$?allocate@?$ReflectionAllocator@VCooking@physx@@@shdfnd@physx@@QEAAPEAX_KPEBDH@Z 0000000180030740     Cooking.obj
 0004:0000174c       $pdata$?allocate@?$ReflectionAllocator@VHeightField@Gu@physx@@@shdfnd@physx@@QEAAPEAX_KPEBDH@Z 000000018003074c     Cooking.obj
 0004:00001758       $pdata$0$?allocate@?$ReflectionAllocator@VHeightField@Gu@physx@@@shdfnd@physx@@QEAAPEAX_KPEBDH@Z 0000000180030758     Cooking.obj
 0004:00001764       $pdata$1$?allocate@?$ReflectionAllocator@VHeightField@Gu@physx@@@shdfnd@physx@@QEAAPEAX_KPEBDH@Z 0000000180030764     Cooking.obj
 0004:00001770       $pdata$?allocate@?$ReflectionAllocator@VTriangleMeshBuilder@physx@@@shdfnd@physx@@QEAAPEAX_KPEBDH@Z 0000000180030770     Cooking.obj
 0004:0000177c       $pdata$0$?allocate@?$ReflectionAllocator@VTriangleMeshBuilder@physx@@@shdfnd@physx@@QEAAPEAX_KPEBDH@Z 000000018003077c     Cooking.obj
 0004:00001788       $pdata$1$?allocate@?$ReflectionAllocator@VTriangleMeshBuilder@physx@@@shdfnd@physx@@QEAAPEAX_KPEBDH@Z 0000000180030788     Cooking.obj
 0004:00001794       $pdata$?getName@?$ReflectionAllocator@VCooking@physx@@@shdfnd@physx@@CAPEBDXZ 0000000180030794     Cooking.obj
 0004:000017a0       $pdata$?getName@?$ReflectionAllocator@VHeightField@Gu@physx@@@shdfnd@physx@@CAPEBDXZ 00000001800307a0     Cooking.obj
 0004:000017ac       $pdata$?getName@?$ReflectionAllocator@VTriangleMeshBuilder@physx@@@shdfnd@physx@@CAPEBDXZ 00000001800307ac     Cooking.obj
 0004:000017b8       $pdata$??1ReducedVertexCloud@physx@@QEAA@XZ 00000001800307b8     CookingUtils.obj
 0004:000017c4       $pdata$?Clean@ReducedVertexCloud@physx@@QEAAAEAV12@XZ 00000001800307c4     CookingUtils.obj
 0004:000017d0       $pdata$?Reduce@ReducedVertexCloud@physx@@QEAA_NPEAUREDUCEDCLOUD@2@@Z 00000001800307d0     CookingUtils.obj
 0004:000017dc       $pdata$1$?Reduce@ReducedVertexCloud@physx@@QEAA_NPEAUREDUCEDCLOUD@2@@Z 00000001800307dc     CookingUtils.obj
 0004:000017e8       $pdata$3$?Reduce@ReducedVertexCloud@physx@@QEAA_NPEAUREDUCEDCLOUD@2@@Z 00000001800307e8     CookingUtils.obj
 0004:000017f4       $pdata$4$?Reduce@ReducedVertexCloud@physx@@QEAA_NPEAUREDUCEDCLOUD@2@@Z 00000001800307f4     CookingUtils.obj
 0004:00001800       $pdata$5$?Reduce@ReducedVertexCloud@physx@@QEAA_NPEAUREDUCEDCLOUD@2@@Z 0000000180030800     CookingUtils.obj
 0004:0000180c       $pdata$6$?Reduce@ReducedVertexCloud@physx@@QEAA_NPEAUREDUCEDCLOUD@2@@Z 000000018003080c     CookingUtils.obj
 0004:00001818       $pdata$??1EdgeList@Gu@physx@@QEAA@XZ 0000000180030818     EdgeList.obj
 0004:00001824       $pdata$?Load@EdgeList@Gu@physx@@QEAA_NAEAVPxInputStream@3@@Z 0000000180030824     EdgeList.obj
 0004:00001830       $pdata$?Init@EdgeListBuilder@Gu@physx@@QEAA_NAEBUEDGELISTCREATE@23@@Z 0000000180030830     EdgeList.obj
 0004:0000183c       $pdata$?CreateFacesToEdges@EdgeListBuilder@Gu@physx@@AEAA_NIPEBIPEBG@Z 000000018003083c     EdgeList.obj
 0004:00001848       $pdata$4$?CreateFacesToEdges@EdgeListBuilder@Gu@physx@@AEAA_NIPEBIPEBG@Z 0000000180030848     EdgeList.obj
 0004:00001854       $pdata$5$?CreateFacesToEdges@EdgeListBuilder@Gu@physx@@AEAA_NIPEBIPEBG@Z 0000000180030854     EdgeList.obj
 0004:00001860       $pdata$?CreateEdgesToFaces@EdgeListBuilder@Gu@physx@@AEAA_NIPEBIPEBG@Z 0000000180030860     EdgeList.obj
 0004:0000186c       $pdata$?ComputeActiveEdges@EdgeListBuilder@Gu@physx@@AEAA_NIPEBIPEBGPEBVPxVec3@3@M@Z 000000018003086c     EdgeList.obj
 0004:00001878       $pdata$0$?ComputeActiveEdges@EdgeListBuilder@Gu@physx@@AEAA_NIPEBIPEBGPEBVPxVec3@3@M@Z 0000000180030878     EdgeList.obj
 0004:00001884       $pdata$3$?ComputeActiveEdges@EdgeListBuilder@Gu@physx@@AEAA_NIPEBIPEBGPEBVPxVec3@3@M@Z 0000000180030884     EdgeList.obj
 0004:00001890       $pdata$5$?ComputeActiveEdges@EdgeListBuilder@Gu@physx@@AEAA_NIPEBIPEBGPEBVPxVec3@3@M@Z 0000000180030890     EdgeList.obj
 0004:0000189c       $pdata$15$?ComputeActiveEdges@EdgeListBuilder@Gu@physx@@AEAA_NIPEBIPEBGPEBVPxVec3@3@M@Z 000000018003089c     EdgeList.obj
 0004:000018a8       $pdata$16$?ComputeActiveEdges@EdgeListBuilder@Gu@physx@@AEAA_NIPEBIPEBGPEBVPxVec3@3@M@Z 00000001800308a8     EdgeList.obj
 0004:000018b4       $pdata$17$?ComputeActiveEdges@EdgeListBuilder@Gu@physx@@AEAA_NIPEBIPEBGPEBVPxVec3@3@M@Z 00000001800308b4     EdgeList.obj
 0004:000018c0       $pdata$18$?ComputeActiveEdges@EdgeListBuilder@Gu@physx@@AEAA_NIPEBIPEBGPEBVPxVec3@3@M@Z 00000001800308c0     EdgeList.obj
 0004:000018cc       $pdata$?allocate@?$ReflectionAllocator@UEdgeData@Gu@physx@@@shdfnd@physx@@QEAAPEAX_KPEBDH@Z 00000001800308cc     EdgeList.obj
 0004:000018d8       $pdata$0$?allocate@?$ReflectionAllocator@UEdgeData@Gu@physx@@@shdfnd@physx@@QEAAPEAX_KPEBDH@Z 00000001800308d8     EdgeList.obj
 0004:000018e4       $pdata$1$?allocate@?$ReflectionAllocator@UEdgeData@Gu@physx@@@shdfnd@physx@@QEAAPEAX_KPEBDH@Z 00000001800308e4     EdgeList.obj
 0004:000018f0       $pdata$?allocate@?$ReflectionAllocator@UEdgeTriangleData@Gu@physx@@@shdfnd@physx@@QEAAPEAX_KPEBDH@Z 00000001800308f0     EdgeList.obj
 0004:000018fc       $pdata$0$?allocate@?$ReflectionAllocator@UEdgeTriangleData@Gu@physx@@@shdfnd@physx@@QEAAPEAX_KPEBDH@Z 00000001800308fc     EdgeList.obj
 0004:00001908       $pdata$1$?allocate@?$ReflectionAllocator@UEdgeTriangleData@Gu@physx@@@shdfnd@physx@@QEAAPEAX_KPEBDH@Z 0000000180030908     EdgeList.obj
 0004:00001914       $pdata$?angle@shdfnd@physx@@YAMAEBVPxVec3@2@0@Z 0000000180030914     EdgeList.obj
 0004:00001920       $pdata$?getName@?$ReflectionAllocator@UEdgeData@Gu@physx@@@shdfnd@physx@@CAPEBDXZ 0000000180030920     EdgeList.obj
 0004:0000192c       $pdata$?getName@?$ReflectionAllocator@UEdgeTriangleData@Gu@physx@@@shdfnd@physx@@CAPEBDXZ 000000018003092c     EdgeList.obj
 0004:00001938       $pdata$?normal@PxTriangle@physx@@QEBAXAEAVPxVec3@2@@Z 0000000180030938     EdgeList.obj
 0004:00001944       $pdata$??1InternalTriangleMeshBuilder@physx@@QEAA@XZ 0000000180030944     InternalTriangleMeshBuilder.obj
 0004:00001950       $pdata$?cleanMesh@InternalTriangleMeshBuilder@physx@@QEAA_N_N@Z 0000000180030950     InternalTriangleMeshBuilder.obj
 0004:0000195c       $pdata$0$?cleanMesh@InternalTriangleMeshBuilder@physx@@QEAA_N_N@Z 000000018003095c     InternalTriangleMeshBuilder.obj
 0004:00001968       $pdata$1$?cleanMesh@InternalTriangleMeshBuilder@physx@@QEAA_N_N@Z 0000000180030968     InternalTriangleMeshBuilder.obj
 0004:00001974       $pdata$2$?cleanMesh@InternalTriangleMeshBuilder@physx@@QEAA_N_N@Z 0000000180030974     InternalTriangleMeshBuilder.obj
 0004:00001980       $pdata$5$?cleanMesh@InternalTriangleMeshBuilder@physx@@QEAA_N_N@Z 0000000180030980     InternalTriangleMeshBuilder.obj
 0004:0000198c       $pdata$6$?cleanMesh@InternalTriangleMeshBuilder@physx@@QEAA_N_N@Z 000000018003098c     InternalTriangleMeshBuilder.obj
 0004:00001998       $pdata$7$?cleanMesh@InternalTriangleMeshBuilder@physx@@QEAA_N_N@Z 0000000180030998     InternalTriangleMeshBuilder.obj
 0004:000019a4       $pdata$8$?cleanMesh@InternalTriangleMeshBuilder@physx@@QEAA_N_N@Z 00000001800309a4     InternalTriangleMeshBuilder.obj
 0004:000019b0       $pdata$9$?cleanMesh@InternalTriangleMeshBuilder@physx@@QEAA_N_N@Z 00000001800309b0     InternalTriangleMeshBuilder.obj
 0004:000019bc       $pdata$?fillRemapTable@InternalTriangleMeshBuilder@physx@@QEAAXXZ 00000001800309bc     InternalTriangleMeshBuilder.obj
 0004:000019c8       $pdata$0$?fillRemapTable@InternalTriangleMeshBuilder@physx@@QEAAXXZ 00000001800309c8     InternalTriangleMeshBuilder.obj
 0004:000019d4       $pdata$1$?fillRemapTable@InternalTriangleMeshBuilder@physx@@QEAAXXZ 00000001800309d4     InternalTriangleMeshBuilder.obj
 0004:000019e0       $pdata$2$?fillRemapTable@InternalTriangleMeshBuilder@physx@@QEAAXXZ 00000001800309e0     InternalTriangleMeshBuilder.obj
 0004:000019ec       $pdata$3$?fillRemapTable@InternalTriangleMeshBuilder@physx@@QEAAXXZ 00000001800309ec     InternalTriangleMeshBuilder.obj
 0004:000019f8       $pdata$?remapTopology@InternalTriangleMeshBuilder@physx@@QEAAXPEBI@Z 00000001800309f8     InternalTriangleMeshBuilder.obj
 0004:00001a04       $pdata$3$?remapTopology@InternalTriangleMeshBuilder@physx@@QEAAXPEBI@Z 0000000180030a04     InternalTriangleMeshBuilder.obj
 0004:00001a10       $pdata$4$?remapTopology@InternalTriangleMeshBuilder@physx@@QEAAXPEBI@Z 0000000180030a10     InternalTriangleMeshBuilder.obj
 0004:00001a1c       $pdata$?createRTree@InternalTriangleMeshBuilder@physx@@QEAA_NXZ 0000000180030a1c     InternalTriangleMeshBuilder.obj
 0004:00001a28       $pdata$?createSharedEdgeData@InternalTriangleMeshBuilder@physx@@QEAAX_N0@Z 0000000180030a28     InternalTriangleMeshBuilder.obj
 0004:00001a34       $pdata$?releaseEdgeList@InternalTriangleMeshBuilder@physx@@AEAAXXZ 0000000180030a34     InternalTriangleMeshBuilder.obj
 0004:00001a40       $pdata$?createEdgeList@InternalTriangleMeshBuilder@physx@@AEAAXXZ 0000000180030a40     InternalTriangleMeshBuilder.obj
 0004:00001a4c       $pdata$??_GEdgeListBuilder@Gu@physx@@QEAAPEAXI@Z 0000000180030a4c     InternalTriangleMeshBuilder.obj
 0004:00001a58       $pdata$??_GRTreeCookerRemap@@UEAAPEAXI@Z 0000000180030a58     InternalTriangleMeshBuilder.obj
 0004:00001a64       $pdata$??_GRemapCallback@RTreeCooker@physx@@UEAAPEAXI@Z 0000000180030a64     InternalTriangleMeshBuilder.obj
 0004:00001a70       $pdata$?allocate@?$ReflectionAllocator@VEdgeListBuilder@Gu@physx@@@shdfnd@physx@@QEAAPEAX_KPEBDH@Z 0000000180030a70     InternalTriangleMeshBuilder.obj
 0004:00001a7c       $pdata$0$?allocate@?$ReflectionAllocator@VEdgeListBuilder@Gu@physx@@@shdfnd@physx@@QEAAPEAX_KPEBDH@Z 0000000180030a7c     InternalTriangleMeshBuilder.obj
 0004:00001a88       $pdata$1$?allocate@?$ReflectionAllocator@VEdgeListBuilder@Gu@physx@@@shdfnd@physx@@QEAAPEAX_KPEBDH@Z 0000000180030a88     InternalTriangleMeshBuilder.obj
 0004:00001a94       $pdata$?getName@?$ReflectionAllocator@VEdgeListBuilder@Gu@physx@@@shdfnd@physx@@CAPEBDXZ 0000000180030a94     InternalTriangleMeshBuilder.obj
 0004:00001aa0       $pdata$??0MeshCleaner@physx@@QEAA@IPEBVPxVec3@1@IPEBIM@Z 0000000180030aa0     MeshCleaner.obj
 0004:00001aac       $pdata$3$??0MeshCleaner@physx@@QEAA@IPEBVPxVec3@1@IPEBIM@Z 0000000180030aac     MeshCleaner.obj
 0004:00001ab8       $pdata$5$??0MeshCleaner@physx@@QEAA@IPEBVPxVec3@1@IPEBIM@Z 0000000180030ab8     MeshCleaner.obj
 0004:00001ac4       $pdata$7$??0MeshCleaner@physx@@QEAA@IPEBVPxVec3@1@IPEBIM@Z 0000000180030ac4     MeshCleaner.obj
 0004:00001ad0       $pdata$8$??0MeshCleaner@physx@@QEAA@IPEBVPxVec3@1@IPEBIM@Z 0000000180030ad0     MeshCleaner.obj
 0004:00001adc       $pdata$9$??0MeshCleaner@physx@@QEAA@IPEBVPxVec3@1@IPEBIM@Z 0000000180030adc     MeshCleaner.obj
 0004:00001ae8       $pdata$10$??0MeshCleaner@physx@@QEAA@IPEBVPxVec3@1@IPEBIM@Z 0000000180030ae8     MeshCleaner.obj
 0004:00001af4       $pdata$11$??0MeshCleaner@physx@@QEAA@IPEBVPxVec3@1@IPEBIM@Z 0000000180030af4     MeshCleaner.obj
 0004:00001b00       $pdata$12$??0MeshCleaner@physx@@QEAA@IPEBVPxVec3@1@IPEBIM@Z 0000000180030b00     MeshCleaner.obj
 0004:00001b0c       $pdata$13$??0MeshCleaner@physx@@QEAA@IPEBVPxVec3@1@IPEBIM@Z 0000000180030b0c     MeshCleaner.obj
 0004:00001b18       $pdata$14$??0MeshCleaner@physx@@QEAA@IPEBVPxVec3@1@IPEBIM@Z 0000000180030b18     MeshCleaner.obj
 0004:00001b24       $pdata$??1MeshCleaner@physx@@QEAA@XZ 0000000180030b24     MeshCleaner.obj
 0004:00001b3c       $pdata$?PiddFromDllName@@YAPEBUImgDelayDescr@@PEBD@Z 0000000180030b3c     delayimp:delayhlp.obj
 0004:00001b48       $pdata$__FUnloadDelayLoadedDLL2 0000000180030b48     delayimp:delayhlp.obj
 0004:00001b54       $pdata$__HrLoadAllImportsForDll 0000000180030b54     delayimp:delayhlp.obj
 0004:00001b60       $pdata$__delayLoadHelper2  0000000180030b60     delayimp:delayhlp.obj
 0004:00001b78       $pdata$??_Etype_info@@UEAAPEAXI@Z 0000000180030b78     MSVCRT:ti_inst.obj
 0004:00001b84       $pdata$pre_c_init          0000000180030b84     MSVCRT:crtdll.obj
 0004:00001b90       $pdata$_CRT_INIT           0000000180030b90     MSVCRT:crtdll.obj
 0004:00001b9c       $pdata$_DllMainCRTStartup  0000000180030b9c     MSVCRT:crtdll.obj
 0004:00001ba8       $pdata$__DllMainCRTStartup 0000000180030ba8     MSVCRT:crtdll.obj
 0004:00001bb4       $pdata$??_M@YAXPEAX_KHP6AX0@Z@Z 0000000180030bb4     MSVCRT:ehvecdtr.obj
 0004:00001bc0       $pdata$?ArrayUnwindFilter@@YAHPEAU_EXCEPTION_POINTERS@@@Z 0000000180030bc0     MSVCRT:ehvecdtr.obj
 0004:00001bcc       $pdata$?__ArrayUnwind@@YAXPEAX_KHP6AX0@Z@Z 0000000180030bcc     MSVCRT:ehvecdtr.obj
 0004:00001bd8       $pdata$_IsNonwritableInCurrentImage 0000000180030bd8     MSVCRT:pesect.obj
 0004:00001be4       $pdata$__atonexitinit      0000000180030be4     MSVCRT:atonexit.obj
 0004:00001bf0       $pdata$_onexit             0000000180030bf0     MSVCRT:atonexit.obj
 0004:00001bfc       $pdata$atexit              0000000180030bfc     MSVCRT:atonexit.obj
 0004:00001c08       $pdata$__security_init_cookie 0000000180030c08     MSVCRT:gs_support.obj
 0004:00001c14       $pdata$DllMain             0000000180030c14     MSVCRT:dllmain.obj
 0004:00001c20       $pdata$_RTC_Initialize     0000000180030c20     MSVCRT:initsect.obj
 0004:00001c2c       $pdata$_RTC_Terminate      0000000180030c2c     MSVCRT:initsect.obj
 0004:00001c38       $pdata$__DllMainCRTStartup$filt$0 0000000180030c38     MSVCRT:crtdll.obj
 0004:00001c44       $pdata$__DllMainCRTStartup$fin$1 0000000180030c44     MSVCRT:crtdll.obj
 0004:00001c50       $pdata$?fin$0@?0???_M@YAXPEAX_KHP6AX0@Z@Z@4HA 0000000180030c50     MSVCRT:ehvecdtr.obj
 0004:00001c5c       $pdata$?filt$0@?0??__ArrayUnwind@@YAXPEAX_KHP6AX0@Z@Z@4HA 0000000180030c5c     MSVCRT:ehvecdtr.obj
 0004:00001c68       $pdata$_IsNonwritableInCurrentImage$filt$0 0000000180030c68     MSVCRT:pesect.obj
 0004:00001c74       $pdata$_onexit$fin$0       0000000180030c74     MSVCRT:atonexit.obj
 0005:00000060       $R000000                   0000000180031060     * linker generated manifest res *
